 d2hackmap

 Timestamp is 627f84d4 (Sat May 14 18:30:44 2022)

 Preferred load address is 10000000

 Start         Length     Name                   Class
 0001:00000000 00007380H .text$di                CODE
 0001:00007380 000284b0H .text$mn                CODE
 0001:0002f821 00000000H .text$x                 CODE
 0001:0002f830 0000001fH .text$yd                CODE
 0002:00000000 000001acH .idata$5                DATA
 0002:000001ac 00000004H .00cfg                  DATA
 0002:000001b0 00000004H .CRT$XCA                DATA
 0002:000001b4 0000027cH .CRT$XCU                DATA
 0002:00000430 00000004H .CRT$XCZ                DATA
 0002:00000434 00000004H .CRT$XIA                DATA
 0002:00000438 00000010H .CRT$XIC                DATA
 0002:00000448 00000004H .CRT$XIZ                DATA
 0002:0000044c 00000004H .CRT$XLA                DATA
 0002:00000450 00000004H .CRT$XLZ                DATA
 0002:00000454 00000004H .CRT$XPA                DATA
 0002:00000458 00000008H .CRT$XPX                DATA
 0002:00000460 00000004H .CRT$XPXA               DATA
 0002:00000464 00000004H .CRT$XPZ                DATA
 0002:00000468 00000004H .CRT$XTA                DATA
 0002:0000046c 00000004H .CRT$XTZ                DATA
 0002:00000470 00000000H .gfids$y                DATA
 0002:00000470 00008d90H .rdata                  DATA
 0002:00009200 00000000H .rdata$CastGuardVftablesA DATA
 0002:00009200 00000000H .rdata$CastGuardVftablesC DATA
 0002:00009200 00000018H .rdata$T                DATA
 0002:00009218 0000012cH .rdata$r                DATA
 0002:00009344 00000008H .rdata$sxdata           DATA
 0002:0000934c 00000398H .rdata$zzzdbg           DATA
 0002:000096e4 00000004H .rtc$IAA                DATA
 0002:000096e8 00000004H .rtc$IZZ                DATA
 0002:000096ec 00000004H .rtc$TAA                DATA
 0002:000096f0 00000004H .rtc$TZZ                DATA
 0002:000096f4 00000004H .tls                    DATA
 0002:000096f8 00000004H .tls$                   DATA
 0002:000096fc 00000004H .tls$ZZZ                DATA
 0002:00009700 00000530H .xdata$x                DATA
 0002:00009c30 00000050H .edata                  DATA
 0002:00009c80 00000064H .idata$2                DATA
 0002:00009ce4 00000014H .idata$3                DATA
 0002:00009cf8 000001acH .idata$4                DATA
 0002:00009ea4 00000750H .idata$6                DATA
 0003:00000000 00003cc0H .data                   DATA
 0003:00003cc0 00000060H .data$r                 DATA
 0003:00003d20 00000018H .data$rs                DATA
 0003:00003d38 0a8a0cfcH .bss                    DATA
 0004:00000000 00000060H .rsrc$01                DATA
 0004:00000060 00000180H .rsrc$02                DATA

  Address         Publics by Value              Rva+Base       Lib:Object

 0000:00000000       ___guard_iat_count         00000000     <absolute>
 0000:00000000       ___volatile_metadata       00000000     <absolute>
 0000:00000000       ___arm64x_extra_rfe_table  00000000     <absolute>
 0000:00000000       ___guard_eh_cont_table     00000000     <absolute>
 0000:00000000       ___arm64x_redirection_metadata 00000000     <absolute>
 0000:00000000       ___guard_eh_cont_count     00000000     <absolute>
 0000:00000000       __except_list              00000000     <absolute>
 0000:00000000       ___x64_code_ranges_to_entry_points_count 00000000     <absolute>
 0000:00000000       ___arm64x_native_entrypoint 00000000     <absolute>
 0000:00000000       ___hybrid_code_map_count   00000000     <absolute>
 0000:00000000       ___x64_code_ranges_to_entry_points 00000000     <absolute>
 0000:00000000       ___guard_iat_table         00000000     <absolute>
 0000:00000000       ___guard_longjmp_table     00000000     <absolute>
 0000:00000000       ___hybrid_code_map         00000000     <absolute>
 0000:00000000       ___arm64x_extra_rfe_table_size 00000000     <absolute>
 0000:00000000       ___guard_longjmp_count     00000000     <absolute>
 0000:00000000       ___guard_check_icall_a64n_fptr 00000000     <absolute>
 0000:00000000       ___arm64x_redirection_metadata_count 00000000     <absolute>
 0000:00000000       ___guard_fids_count        00000000     <absolute>
 0000:00000000       ___hybrid_auxiliary_iat    00000000     <absolute>
 0000:00000000       ___dynamic_value_reloc_table 00000000     <absolute>
 0000:00000000       ___AbsoluteZero            00000000     <absolute>
 0000:00000000       ___enclave_config          00000000     <absolute>
 0000:00000000       ___guard_fids_table        00000000     <absolute>
 0000:00000000       ___hybrid_auxiliary_iat_copy 00000000     <absolute>
 0000:00000002       ___safe_se_handler_count   00000002     <absolute>
 0000:0000002c       __tls_array                0000002c     <absolute>
 0000:00000100       ___guard_flags             00000100     <absolute>
 0000:00000000       ___ImageBase               10000000     <linker-defined>
 0001:00007380       ?strrchr@@YAPADQADH@Z      10008380 f i DllMain.obj
 0001:000073a0       ??0id@locale@std@@QAE@I@Z  100083a0 f i DllMain.obj
 0001:000073c0       ??0WSInit@detail@httplib@@QAE@XZ 100083c0 f i DllMain.obj
 0001:00007400       ??1WSInit@detail@httplib@@QAE@XZ 10008400 f i DllMain.obj
 0001:00007420       ?ReleaseMem@@YAXXZ         10008420 f   DllMain.obj
 0001:00007430       _DllMain@12                10008430 f   DllMain.obj
 0001:000074b0       _QueryInterface@0          100084b0 f   DllMain.obj
 0001:00007500       ?GetDllOffset@@YAKPADH@Z   10008500 f   HelpFunc.obj
 0001:00007550       ?GetDllOffset@@YAKH@Z      10008550 f   HelpFunc.obj
 0001:00007580       ?VirtualProtect@@YAKKKK@Z  10008580 f   HelpFunc.obj
 0001:000075b0       ?WriteLocalBYTES@@YAXKPAXH@Z 100085b0 f   HelpFunc.obj
 0001:00007600       ?ReadLocalBYTES@@YAXKPAXH@Z 10008600 f   HelpFunc.obj
 0001:00007620       ?FillLocalBYTES@@YAXKEH@Z  10008620 f   HelpFunc.obj
 0001:00007680       ?InterceptLocalCode2@@YAXEKKH@Z 10008680 f   HelpFunc.obj
 0001:00007700       ?InterceptLocalCode@@YAXEKKH@Z 10008700 f   HelpFunc.obj
 0001:00007730       ?PatchCALL@@YAXKKK@Z       10008730 f   HelpFunc.obj
 0001:00007750       ?PatchJMP@@YAXKKK@Z        10008750 f   HelpFunc.obj
 0001:00007770       ?PatchFILL@@YAXKKK@Z       10008770 f   HelpFunc.obj
 0001:00007790       ?PatchVALUE@@YAXKKK@Z      10008790 f   HelpFunc.obj
 0001:000077b0       ?OpenFileNew@@YAPAXPAD@Z   100087b0 f   HelpFunc.obj
 0001:000077e0       ?OpenFileRead@@YAPAXPAD@Z  100087e0 f   HelpFunc.obj
 0001:00007810       ?OpenFileWrite@@YAPAXPAD@Z 10008810 f   HelpFunc.obj
 0001:00007840       ?WriteFile@@YAKPAX0K@Z     10008840 f   HelpFunc.obj
 0001:00007870       ?ReadFile@@YAKPAX0K@Z      10008870 f   HelpFunc.obj
 0001:000078a0       ?AllocReadFile@@YAPAEPAD@Z 100088a0 f   HelpFunc.obj
 0001:00007910       ?ReadFileLine@@YAPADPADHPAX@Z 10008910 f   HelpFunc.obj
 0001:00007990       ?SwapInt@@YAXAAH0@Z        10008990 f   HelpFunc.obj
 0001:000079c0       ?memcpy2@@YAPAXPAXPBXI@Z   100089c0 f   HelpFunc.obj
 0001:000079e0       ?wcscpy2@@YAXPA_WPAD@Z     100089e0 f   HelpFunc.obj
 0001:00007a20       ?wcsrcat@@YAPA_WPA_W0@Z    10008a20 f   HelpFunc.obj
 0001:00007af0       ?wscolorcpy@@YAPA_WPA_W0E@Z 10008af0 f   HelpFunc.obj
 0001:00007bb0       ?trimspaces@@YAXPA_W@Z     10008bb0 f   HelpFunc.obj
 0001:00007c70       ?DblToStr@@YAPADNHPAD@Z    10008c70 f   HelpFunc.obj
 0001:00007d70       ?wsprintfW2@@YAPA_WPA_WPADZZ 10008d70 f   HelpFunc.obj
 0001:00007dd0       ?AllocStrN@@YAPADPADH@Z    10008dd0 f   HelpFunc.obj
 0001:00007e20       ?ColourD2String@@YIPA_WPA_WK@Z 10008e20 f   HelpFunc.obj
 0001:00007ec0       ?wsprintfW2Colour@@YAPA_WPA_WHPADZZ 10008ec0 f   HelpFunc.obj
 0001:00007f60       ?ConvertToColorString@@YAXPAEPADH@Z 10008f60 f   HelpFunc.obj
 0001:00008100       ?UnicodeFix2@@YAXPA_W@Z    10009100 f   HelpFunc.obj
 0001:00008190       ?MyMultiByteToWideChar@@YAHIKPBDHPA_WH@Z 10009190 f   HelpFunc.obj
 0001:000081d0       ?GB2GBK@@YAXPAD@Z          100091d0 f   HelpFunc.obj
 0001:00008350       ?RelocD2Ptrs@@YAHXZ        10009350 f   Install.obj
 0001:000083b0       ?InstallD2Patchs@@YAHPAUPatch_t@@0@Z 100093b0 f   Install.obj
 0001:00008480       ?RemoveD2Patchs@@YAXPAUPatch_t@@0@Z 10009480 f   Install.obj
 0001:000084f0       ?RelocD2Ptrs2@@YAHXZ       100094f0 f   Install.obj
 0001:00008550       ?InstallPatchAfterLoad@@YAXXZ 10009550 f   Install.obj
 0001:00008580       ?InstallPatchAfterLoad_ASM@@YAXXZ 10009580 f   Install.obj
 0001:000085a0       ?InstallPatchs@@YAHXZ      100095a0 f   Install.obj
 0001:000085d0       ?RemovePatchs@@YAXXZ       100095d0 f   Install.obj
 0001:00008620       ?InitCellFiles@@YAXXZ      10009620 f   Install.obj
 0001:00008800       ?DeleteCellFiles@@YAXXZ    10009800 f   Install.obj
 0001:000088e0       ?Install@@YAHXZ            100098e0 f   Install.obj
 0001:00008980       ?Uninstall@@YAXXZ          10009980 f   Install.obj
 0001:000089a0       ?ReloadConfig@@YAXXZ       100099a0 f   Install.obj
 0001:000089e0       ?CalcFuncOffset_X@@YAKKKH@Z 100099e0 f   Install.obj
 0001:00008a10       ?GetD2Version@@YAKPBX@Z    10009a10 f   Install.obj
 0001:00008ad0       ?GetD2Version@@YAKPAD@Z    10009ad0 f   Install.obj
 0001:00008b70       ?Map_D2Version@@YAKXZ      10009b70 f   Install.obj
 0001:00008c70       ?strstr@@YAPADQADQBD@Z     10009c70 f i Install.obj
 0001:00008c90       ___local_stdio_printf_options 10009c90 f i Install.obj
 0001:00008ca0       __vsnprintf_l              10009ca0 f i Install.obj
 0001:00008cf0       __vsprintf_l               10009cf0 f i Install.obj
 0001:00008d10       _sprintf                   10009d10 f i Install.obj
 0001:00008d50       ?InitValues@@YAXXZ         10009d50 f   LoadConfig.obj
 0001:00008f70       ?FixValues@@YAXXZ          10009f70 f   LoadConfig.obj
 0001:00009410       ?InitKeyEvent@@YAXXZ       1000a410 f   LoadConfig.obj
 0001:000094f0       ?AddMinimapConfig@@YAXKGEE@Z 1000a4f0 f   LoadConfig.obj
 0001:000095a0       ?AddWarningMessage@@YAXPADH@Z 1000a5a0 f   LoadConfig.obj
 0001:00009650       ?ShowWarningMessage@@YAXXZ 1000a650 f   LoadConfig.obj
 0001:000096c0       ?OpenFileReadHelper@@YAPAXPAD@Z 1000a6c0 f   LoadConfig.obj
 0001:000097a0       ?DeleteTree@@YAXAAPAUTreeNode@@@Z 1000a7a0 f   LoadConfig.obj
 0001:00009840       ?SearchTree@@YAAAPAUTreeNode@@AAPAU1@PAD@Z 1000a840 f   LoadConfig.obj
 0001:000098b0       ?isquote@@YADD@Z           1000a8b0 f   LoadConfig.obj
 0001:000098e0       ?FilterSpace@@YAXPAD0@Z    1000a8e0 f   LoadConfig.obj
 0001:000099a0       ?SplitLine@@YAXPAD00@Z     1000a9a0 f   LoadConfig.obj
 0001:00009bb0       ?ReplaceByVcb@@YAXPAD@Z    1000abb0 f   LoadConfig.obj
 0001:00009df0       ?ConvertToD2String@@YAXPA_WPADH@Z 1000adf0 f   LoadConfig.obj
 0001:00009f70       ?strtol2@@YAHAAHAAPADH@Z   1000af70 f   LoadConfig.obj
 0001:00009fc0       ?StoreArrayConfig@@YAHPAUConfigVar@@HHPAD1@Z 1000afc0 f   LoadConfig.obj
 0001:0000a390       ?StoreConfig@@YAXPAUConfigVar@@PAD1@Z 1000b390 f   LoadConfig.obj
 0001:0000ad30       ?LoadConfig@@YAHXZ         1000bd30 f   LoadConfig.obj
 0001:0000b1c0       ?D2SetAutomapParty@@YIXK@Z 1000c1c0 f   D2CallStub.obj
 0001:0000b1d0       ?D2SetAutomapNames@@YIXK@Z 1000c1d0 f   D2CallStub.obj
 0001:0000b1e0       ?D2GetSkillsDescTxt@@YIPAUSkillDescBIN@@K@Z 1000c1e0 f   D2CallStub.obj
 0001:0000b210       ?D2GetSkillsTxt@@YIPAUSkillsTxt@@K@Z 1000c210 f   D2CallStub.obj
 0001:0000b240       ?D2ChatInput@@YIKPAUD2MSG@@@Z 1000c240 f   D2CallStub.obj
 0001:0000b250       ?D2CheckUiStatus@@YIKK@Z   1000c250 f   D2CallStub.obj
 0001:0000b260       ?D2InitAutomapLayer@@YIPAUAutomapLayer@@K@Z 1000c260 f   D2CallStub.obj
 0001:0000b270       ?D2GetUniqueItemTxt@@YIPAUUniqueItemTxt@@K@Z 1000c270 f   D2CallStub.obj
 0001:0000b2a0       ?D2GetPropertiesTxt@@YIPAUPropertiesTxt@@K@Z 1000c2a0 f   D2CallStub.obj
 0001:0000b2d0       ?D2GetSetItemTxt@@YIPAUSetItemTxt@@K@Z 1000c2d0 f   D2CallStub.obj
 0001:0000b300       ?D2GetItemTypeTxt@@YIPAUItemTypeTxt@@K@Z 1000c300 f   D2CallStub.obj
 0001:0000b330       ?D2GetRuneWordTxt@@YIPAURuneWordTxt@@K@Z 1000c330 f   D2CallStub.obj
 0001:0000b360       ?D2GetRuneWordTxtIndex@@YIKK@Z 1000c360 f   D2CallStub.obj
 0001:0000b3a0       ?D2LoadUiImage@@YIPAUCellFile@@PAD@Z 1000c3a0 f   D2CallStub.obj
 0001:0000b3b0       ?SetCenterAlertMsg@@YAXHPA_W@Z 1000c3b0 f   D2HelpFunc.obj
 0001:0000b410       ?DrawCenterAlertMsg@@YAXXZ 1000c410 f   D2HelpFunc.obj
 0001:0000b450       ?ShowGameMessage@@YAXPAD@Z 1000c450 f   D2HelpFunc.obj
 0001:0000b4a0       ?GetAreaLevel@@YAGXZ       1000c4a0 f   D2HelpFunc.obj
 0001:0000b500       ?TestPvpFlag@@YAEKK@Z      1000c500 f   D2HelpFunc.obj
 0001:0000b5f0       ?GetUnitDistanceInSubtiles@@YINPAUUnitAny@@0@Z 1000c5f0 f   D2HelpFunc.obj
 0001:0000b700       ?GetUnitMagicStat@@YAKPAUUnitAny@@K@Z 1000c700 f   D2HelpFunc.obj
 0001:0000b750       ?GetUnitResist@@YAHPAUUnitAny@@K@Z 1000c750 f   D2HelpFunc.obj
 0001:0000b7a0       ?CheckUnitSelect@@YAHPAUUnitAny@@@Z 1000c7a0 f   D2HelpFunc.obj
 0001:0000b8d0       ?GetItemILvlAfterCube@@YAHHHH@Z 1000c8d0 f   D2HelpFunc.obj
 0001:0000b980       ?GetItemAlvl@@YAHHHH@Z     1000c980 f   D2HelpFunc.obj
 0001:0000ba00       ?TestMonsterOnScreen@@YAHPAUUnitAny@@0@Z 1000ca00 f   D2HelpFunc.obj
 0001:0000ba80       ?PreparePosForDraw@@YAXPAUtagPOINT@@HH@Z 1000ca80 f   D2HelpFunc.obj
 0001:0000baf0       ?MapToAbsScreen@@YAXPAUtagPOINT@@HH@Z 1000caf0 f   D2HelpFunc.obj
 0001:0000bb20       ?LoadBmpCellFile@@YAPAUCellFile@@PAEHH@Z 1000cb20 f   D2HelpFunc.obj
 0001:0000bd50       ?LoadBmpCellFile@@YAPAUCellFile@@PAD@Z 1000cd50 f   D2HelpFunc.obj
 0001:0000bdf0       ?InitCellFile@@YAPAUCellFile@@PAU1@@Z 1000cdf0 f   D2HelpFunc.obj
 0001:0000be20       ?DeleteCellFile@@YAXPAUCellFile@@@Z 1000ce20 f   D2HelpFunc.obj
 0001:0000be50       ?GetTextWidth@@YAKPA_W@Z   1000ce50 f   D2HelpFunc.obj
 0001:0000be70       ?DrawD2Text@@YAXKPA_WHHKK@Z 1000ce70 f   D2HelpFunc.obj
 0001:0000beb0       ?DrawCenterText@@YAXKPA_WHHKHK@Z 1000ceb0 f   D2HelpFunc.obj
 0001:0000bf00       ?DrawDefaultFontText@@YAXPA_WHHKHK@Z 1000cf00 f   D2HelpFunc.obj
 0001:0000bf30       ?ExitGame@@YAXXZ           1000cf30 f   D2HelpFunc.obj
 0001:0000bf60       ?DrawAutomapCell@@YAXPAUCellFile@@HHE@Z 1000cf60 f   D2HelpFunc.obj
 0001:0000c160       ?GetGameLanguage@@YAHXZ    1000d160 f   D2HelpFunc.obj
 0001:0000c220       ?GameLoopPatch@@YAXXZ      1000d220 f   GameMainLoop.obj
 0001:0000c4f0       ?GameEndPatch@@YAXXZ       1000d4f0 f   GameMainLoop.obj
 0001:0000c620       ?GameLoopPatch_ASM@@YAXXZ  1000d620 f   GameMainLoop.obj
 0001:0000c630       ?GameEndPatch_ASM@@YAXXZ   1000d630 f   GameMainLoop.obj
 0001:0000c640       ?KeydownPatch@@YIXEE@Z     1000d640 f   KeyEventControl.obj
 0001:0000c940       ?KeydownPatch_ASM@@YAXXZ   1000d940 f   KeyEventControl.obj
 0001:0000c960       ?KeyupPatch_ASM@@YAXXZ     1000d960 f   KeyEventControl.obj
 0001:0000c980       ?MButtonDownPatch_ASM@@YAXXZ 1000d980 f   KeyEventControl.obj
 0001:0000c9a0       ?WeatherPatch_ASM@@YAXXZ   1000d9a0 f   Environment.obj
 0001:0000c9b0       ?LightingPatch_ASM@@YAXXZ  1000d9b0 f   Environment.obj
 0001:0000c9e0       ?ShakeScreenPatch@@YGXPAK0@Z 1000d9e0 f   Environment.obj
 0001:0000ca60       ?InfravisionPatch@@YIKPAUUnitAny@@@Z 1000da60 f   Environment.obj
 0001:0000cb70       ?InfravisionPatch_ASM@@YAXXZ 1000db70 f   Environment.obj
 0001:0000cb90       ?ShowGameCount@@YAXXZ      1000db90 f   GameCount.obj
 0001:0000cda0       ?SetKills@@YIXK@Z          1000dda0 f   GameCount.obj
 0001:0000cde0       ?KillCountPatch_ASM@@YAXXZ 1000dde0 f   GameCount.obj
 0001:0000ce00       ?UnitModeChangePatch_ASM@@YAXXZ 1000de00 f   GameCount.obj
 0001:0000ce40       ?DrawMonitorInfo@@YAXXZ    1000de40 f   GameMonitor.obj
 0001:0000cfd0       ?ResetMonitor@@YAXXZ       1000dfd0 f   GameMonitor.obj
 0001:0000d020       ?SetState@@YGXKH@Z         1000e020 f   GameMonitor.obj
 0001:0000d0a0       ?RecvCommand_A7_Patch_ASM@@YAXXZ 1000e0a0 f   GameMonitor.obj
 0001:0000d0d0       ?RecvCommand_A8_Patch_ASM@@YAXXZ 1000e0d0 f   GameMonitor.obj
 0001:0000d100       ?RecvCommand_A9_Patch_ASM@@YAXXZ 1000e100 f   GameMonitor.obj
 0001:0000d130       ?LogMessage@@YIXPA_W@Z     1000e130 f   MessageLog.obj
 0001:0000d500       ?MessageLogPatch1_ASM@@YAXXZ 1000e500 f   MessageLog.obj
 0001:0000d520       ?MessageLogPatch2_ASM@@YAXXZ 1000e520 f   MessageLog.obj
 0001:0000d540       ?LogExitMessage@@YAXXZ     1000e540 f   MessageLog.obj
 0001:0000d790       ?DrawPetHeadPath@@YIXHPAUUnitAny@@@Z 1000e790 f   PartyInfo.obj
 0001:0000d810       ?DrawPetHeadPath_ASM@@YAXXZ 1000e810 f   PartyInfo.obj
 0001:0000d820       ?DrawPartyHeadPath@@YIXHPAURosterUnit@@@Z 1000e820 f   PartyInfo.obj
 0001:0000d8e0       ?DrawPartyHeadPath_ASM@@YAXXZ 1000e8e0 f   PartyInfo.obj
 0001:0000d900       ?SetTickCount@@YAXXZ       1000e900 f   RoomInfo.obj
 0001:0000d910       ?DrawGameVersionPatch@@YAXPAD@Z 1000e910 f   RoomInfo.obj
 0001:0000d960       ?DrawGameVersionPatch_ASM@@YAXXZ 1000e960 f   RoomInfo.obj
 0001:0000d970       ?DrawGameInfoPatch@@YIXK@Z 1000e970 f   RoomInfo.obj
 0001:0000dd20       ?UpdateExp@@YAXXZ          1000ed20 f   ScreenHook.obj
 0001:0000dfa0       ?InitExp@@YAXXZ            1000efa0 f   ScreenHook.obj
 0001:0000dfd0       ?UpdateExp_ASM@@YAXXZ      1000efd0 f   ScreenHook.obj
 0001:0000dff0       ?InitScreenHook@@YAXXZ     1000eff0 f   ScreenHook.obj
 0001:0000e1d0       ?DrawClientPatch@@YAXXZ    1000f1d0 f   ScreenHook.obj
 0001:0000e340       ?DrawClientPatch_ASM@@YAXXZ 1000f340 f   ScreenHook.obj
 0001:0000e350       ?ShowLifeWithMyPattern@@YGKKHH@Z 1000f350 f   ShowOrbs.obj
 0001:0000e3d0       ?ShowManaWithMyPattern@@YGKKHH@Z 1000f3d0 f   ShowOrbs.obj
 0001:0000e460       ?ShowLifePatch_ASM@@YAXXZ  1000f460 f   ShowOrbs.obj
 0001:0000e480       ?ShowManaPatch_ASM@@YAXXZ  1000f480 f   ShowOrbs.obj
 0001:0000e4a0       ?SetLifeManaShow@@YAXXZ    1000f4a0 f   ShowOrbs.obj
 0001:0000e4f0       ?GetItemIndex@@YAHH@Z      1000f4f0 f   ItemDefine.obj
 0001:0000e560       ?GetItemColour@@YAEPAUUnitAny@@K@Z 1000f560 f   ItemDefine.obj
 0001:0000e720       ?SwitchItemMode@@YAXXZ     1000f720 f   ItemDefine.obj
 0001:0000e7b0       ?ItemDescPath@@YIXPA_WHHHH@Z 1000f7b0 f   ItemDesc.obj
 0001:0000e8e0       ?SocketViewCallRoutine@@YIXPAUUnitAny@@KP6GX0K@Z@Z 1000f8e0 f   ItemDesc.obj
 0001:0000e8f0       ?ItemSocketViewPatch@@YGXP6GXPAUUnitAny@@K@Z0K@Z 1000f8f0 f   ItemDesc.obj
 0001:0000e9b0       ?ItemSocketViewPatch_ASM@@YAXXZ 1000f9b0 f   ItemDesc.obj
 0001:0000e9c0       ?SocketItemStatViewPatch_ASM@@YAXXZ 1000f9c0 f   ItemDesc.obj
 0001:0000e9e0       ?GetItemExtStatListPatch@@YGPAUStatList@@PAUUnitAny@@KK@Z 1000f9e0 f   ItemDesc.obj
 0001:0000ea10       ?ItemBasicStatPatch_ASM@@YAXXZ 1000fa10 f   ItemDesc.obj
 0001:0000ea40       ?LoadExtInfo@@YAXXZ        1000fa40 f   ItemExtInfo.obj
 0001:0000f780       ?UnLoadExtInfo@@YAXXZ      10010780 f   ItemExtInfo.obj
 0001:0000f950       ?SetExtInfoPos@@YAXHHKK@Z  10010950 f   ItemExtInfo.obj
 0001:0000fa40       ?ShowItemExtInfo@@YAXXZ    10010a40 f   ItemExtInfo.obj
 0001:0000fda0       ?DrawHoverPatch_ASM@@YAXXZ 10010da0 f   ItemExtInfo.obj
 0001:0000fdb0       ?CheckItemVisible@@YAHPAUUnitAny@@@Z 10010db0 f   ItemInGround.obj
 0001:0000fe60       ?GetItemPicks@@YAEPAUUnitAny@@K@Z 10010e60 f   ItemInGround.obj
 0001:0000ff30       ?GetDistance@@YAKJJJJ@Z    10010f30 f   ItemInGround.obj
 0001:0000ff70       ?GetItemMapDistanceFrom@@YAKPAUUnitAny@@@Z 10010f70 f   ItemInGround.obj
 0001:0000ffb0       ?EnumStorageDirectBag@@YAPAUUnitAny@@KKPAE@Z 10010fb0 f   ItemInGround.obj
 0001:00010140       ?GoToEntity@@YAHPAUUnitAny@@H@Z 10011140 f   ItemInGround.obj
 0001:000101a0       ?PickGroundItem@@YAHPAUUnitAny@@H@Z 100111a0 f   ItemInGround.obj
 0001:00010250       ?PickLoop@@YAXXZ           10011250 f   ItemInGround.obj
 0001:00010300       ?Deal9C@@YIXPAUUnitAny@@@Z 10011300 f   ItemInGround.obj
 0001:00010950       ?ITEMBAG_GetFreeSlot@@YGHPAUStatList2@@K@Z 10011950 f   ItemInGround.obj
 0001:000109b0       ?RecvCommand_PickUp_Patch_ASM@@YAXXZ 100119b0 f   ItemInGround.obj
 0001:000109c0       ?ItemHaveLevel@@YAHE@Z     100119c0 f   ItemName.obj
 0001:00010a20       ?ItemNamePatch@@YIXPA_WPAUUnitAny@@PAUItemTxt@@@Z 10011a20 f   ItemName.obj
 0001:00011d40       ?ItemNamePatch_ASM@@YAXXZ  10012d40 f   ItemName.obj
 0001:00011d60       ?OpenCubeStringPatch@@YIPA_WPA_WK@Z 10012d60 f   ItemName.obj
 0001:00011df0       ?OpenCubeStringPatch_ASM@@YAXXZ 10012df0 f   ItemName.obj
 0001:00011e00       ?SetPropInfo@@YAXHHHPAUItemProp@@@Z 10012e00 f   ItemVariableProp.obj
 0001:00012340       ?GetStatRange@@YAPA_WPA_WKK@Z 10013340 f   ItemVariableProp.obj
 0001:00012ce0       ?GetItemPropStringPatch@@YIKPA_WPAUStatEx@@K@Z 10013ce0 f   ItemVariableProp.obj
 0001:00012dc0       ?GetItemPropStringPatch_ASM@@YAXXZ 10013dc0 f   ItemVariableProp.obj
 0001:00012de0       ?StrcatItemPropStringPatch@@YIXPA_W0K@Z 10013de0 f   ItemVariableProp.obj
 0001:00012f00       ?StrcatItemPropStringPatch_ASM@@YAXXZ 10013f00 f   ItemVariableProp.obj
 0001:00012f10       ?StrcatSocketStringPatch@@YIPA_WPA_W@Z 10013f10 f   ItemVariableProp.obj
 0001:00012f40       ?StrcatSocketStringPatch_ASM@@YAXXZ 10013f40 f   ItemVariableProp.obj
 0001:00012f50       ?StrcatDefenseStringPatch@@YIPA_WPA_W@Z 10013f50 f   ItemVariableProp.obj
 0001:000131e0       ?StrcatDefenseStringPatch_ASM@@YAXXZ 100141e0 f   ItemVariableProp.obj
 0001:000131f0       ?StrcatDamageStringPatch@@YIPA_WPA_W@Z 100141f0 f   ItemVariableProp.obj
 0001:00013380       ?StrcatDamageStringPatch_ASM1@@YAXXZ 10014380 f   ItemVariableProp.obj
 0001:00013390       ?StrcatDamageStringPatch_ASM2@@YAXXZ 10014390 f   ItemVariableProp.obj
 0001:000133b0       ?ProtectAction@@YAXPA_WHE@Z 100143b0 f   CheckDangerous.obj
 0001:00013580       ?ChickenLife@@YAXXZ        10014580 f   CheckDangerous.obj
 0001:00013740       ?CheckDangerousPlayer@@YAXPAUUnitAny@@@Z 10014740 f   CheckDangerous.obj
 0001:00013830       ?CheckDangerousMonster@@YAXPAUUnitAny@@@Z 10014830 f   CheckDangerous.obj
 0001:00013950       ?ToggleIMEInput@@YAXH@Z    10014950 f   IMEProtect.obj
 0001:000139b0       ?ShowSocketProtectInfo@@YAXXZ 100149b0 f   ItemSocketProtect.obj
 0001:000139d0       ?SocketProtectPatch_ASM@@YAXXZ 100149d0 f   ItemSocketProtect.obj
 0001:000139f0       ?SocketProtectPatch1_ASM@@YAXXZ 100149f0 f   ItemSocketProtect.obj
 0001:00013a10       ?SocketProtectPatch2_ASM@@YAXXZ 10014a10 f   ItemSocketProtect.obj
 0001:00013a30       ?ReSetTimer@@YAXXZ         10014a30 f   QuestProtect.obj
 0001:00013a70       ?InitBugInfo@@YAXXZ        10014a70 f   QuestProtect.obj
 0001:00013bc0       ?SetBugQuestStatus@@YAXXZ  10014bc0 f   QuestProtect.obj
 0001:00013d50       ?ShowBugInfo@@YAXXZ        10014d50 f   QuestProtect.obj
 0001:00013f00       ?BugKDProtect@@YIXK@Z      10014f00 f   QuestProtect.obj
 0001:00013f60       ?RecvCommand_89_Patch_ASM@@YAXXZ 10014f60 f   QuestProtect.obj
 0001:00013f80       ?BugKBProtect@@YIXPAE@Z    10014f80 f   QuestProtect.obj
 0001:00014010       ?RecvCommand_5D_Patch_ASM@@YAXXZ 10015010 f   QuestProtect.obj
 0001:00014020       ?CheckUnitKM@@YAXXZ        10015020 f   QuestProtect.obj
 0001:00014100       ?DrawQuestPagePatch@@YIXHH@Z 10015100 f   QuestProtect.obj
 0001:000141d0       ?DrawQuestPagePatch_ASM@@YAXXZ 100151d0 f   QuestProtect.obj
 0001:000141e0       ?UnicodeFix@@YAXPA_WPAK@Z  100151e0 f   UnicodeSupport.obj
 0001:000143e0       ?D2Lang_Unicode2WinPatch@@YIPBDPADPA_WK@Z 100153e0 f   UnicodeSupport.obj
 0001:00014420       ?D2Lang_Win2UnicodePatch@@YIPA_WPA_WPBDK@Z 10015420 f   UnicodeSupport.obj
 0001:00014450       ?EditDeleteSelect@@YAXPAUD2EditBox@@@Z 10015450 f   UnicodeSupport.obj
 0001:00014580       ?ChannelEnterCharPatch@@YIKPAUD2EditBox@@E@Z 10015580 f   UnicodeSupport.obj
 0001:000148d0       ?UnicodeToUTF_8@@YAXPADPA_W@Z 100158d0 f   UnicodeSupport.obj
 0001:00014970       ?MultiByteFix@@YGXPAD@Z    10015970 f   UnicodeSupport.obj
 0001:00014b70       ?MultiByteFixPatch_ASM@@YAXXZ 10015b70 f   UnicodeSupport.obj
 0001:00014b80       ?IsPritableCharacterPatch_ASM@@YAXXZ 10015b80 f   UnicodeSupport.obj
 0001:00014ba0       ?ResetMonsterColours@@YAXXZ 10015ba0 f   MonsterColour.obj
 0001:00017dc0       ?MonsterDeathPatch_ASM@@YAXXZ 10018dc0 f   MonsterDeath.obj
 0001:00017de0       ?MonsterNamePatch@@YIJPA_WJPAUUnitAny@@JJ@Z 10018de0 f   MonsterLifeBar.obj
 0001:000184d0       ?MonsterNamePatch_ASM@@YAXXZ 100194d0 f   MonsterLifeBar.obj
 0001:000184f0       ?MonsterDescCommaPatch1_ASM@@YAXXZ 100194f0 f   MonsterLifeBar.obj
 0001:00018500       ?MonsterDescCommaPatch2_ASM@@YAXXZ 10019500 f   MonsterLifeBar.obj
 0001:00018510       ?MonsterDescCommaPatch3@@YIXPA_WPAUMonsterTxt@@@Z 10019510 f   MonsterLifeBar.obj
 0001:000185a0       ?MonsterDescCommaPatch3_ASM@@YAXXZ 100195a0 f   MonsterLifeBar.obj
 0001:000185b0       ?LifeBarPatch_ASM@@YAXXZ   100195b0 f   MonsterLifeBar.obj
 0001:000185d0       ?CalculateHighestTC@@YAXHG@Z 100195d0 f   MonsterTC.obj
 0001:00018820       ?InitTCList@@YAXXZ         10019820 f   MonsterTC.obj
 0001:000188a0       ?GetPlayerHpPercent@@YAHPAUUnitAny@@@Z 100198a0 f   PlayerLifeBar.obj
 0001:000188e0       ?PlayerNamePatch@@YIXPA_WPAUUnitAny@@@Z 100198e0 f   PlayerLifeBar.obj
 0001:00018a50       ?PlayerNamePatch_ASM@@YAXXZ 10019a50 f   PlayerLifeBar.obj
 0001:00018a70       ?GetViewEquUnit@@YAPAUUnitAny@@XZ 10019a70 f   ViewTargetUnitInfo.obj
 0001:00018aa0       ?GetViewStatUnit@@YAPAUUnitAny@@XZ 10019aa0 f   ViewTargetUnitInfo.obj
 0001:00018ad0       ?SetViewUnit@@YAXXZ        10019ad0 f   ViewTargetUnitInfo.obj
 0001:00018ba0       ?ViewUnit@@YAXH@Z          10019ba0 f   ViewTargetUnitInfo.obj
 0001:00018c30       ?GetViewingStatsPlayerPatch1_ASM@@YAXXZ 10019c30 f   ViewTargetUnitInfo.obj
 0001:00018c40       ?GetViewingStatsPlayerPatch2_ASM@@YAXXZ 10019c40 f   ViewTargetUnitInfo.obj
 0001:00018c50       ?GetUnitDrawEquipItemPatch_ASM@@YAXXZ 10019c50 f   ViewTargetUnitInfo.obj
 0001:00018c60       ?GetUnitDrawItemDescPath_ASM@@YAXXZ 10019c60 f   ViewTargetUnitInfo.obj
 0001:00018c70       ?GetUnitTestHasItem_ASM@@YAXXZ 10019c70 f   ViewTargetUnitInfo.obj
 0001:00018c90       ?GetUnitText@@YIPA_WPA_WPAUUnitAny@@@Z 10019c90 f   ViewTargetUnitInfo.obj
 0001:00018d20       ?ViewDrawInvItemPatch@@YAPAUUnitAny@@XZ 10019d20 f   ViewTargetUnitInfo.obj
 0001:00018da0       ?GetUnitDrawInvItemPatch_ASM@@YAXXZ 10019da0 f   ViewTargetUnitInfo.obj
 0001:00018db0       ?GetUnitProtectClickEquipPatch_ASM@@YAXXZ 10019db0 f   ViewTargetUnitInfo.obj
 0001:00018df0       ?GetUnitProtectClickInvPatch_ASM@@YAXXZ 10019df0 f   ViewTargetUnitInfo.obj
 0001:00018e20       ?SwitchStatPage@@YAXH@Z    10019e20 f   ViewUnitStat.obj
 0001:00018e70       ?DrawUnitStat@@YAXHHHHPAD00KHH@Z 10019e70 f   ViewUnitStat.obj
 0001:00018f70       ?DrawUnitStat@@YAXHHHHPAD0PA_WKHH@Z 10019f70 f   ViewUnitStat.obj
 0001:00019070       ?ViewUnitStatPatch@@YIXPAUUnitAny@@@Z 1001a070 f   ViewUnitStat.obj
 0001:00019d20       ?ViewUnitStatPatch_ASM@@YAXXZ 1001ad20 f   ViewUnitStat.obj
 0001:00019d40       ?ViewPetStatPatch@@YIXPAUUnitAny@@@Z 1001ad40 f   ViewUnitStat.obj
 0001:00019fe0       ?ViewPetStatPatch_ASM@@YAXXZ 1001afe0 f   ViewUnitStat.obj
 0001:0001a000       ?ResetMapStatus@@YAXXZ     1001b000 f   AutoMap.obj
 0001:0001a040       ?InitAutomapLayer@@YAXK@Z  1001b040 f   AutoMap.obj
 0001:0001a060       ?RevealAutomapRoom@@YAXPAUDrlgRoom2@@@Z 1001b060 f   AutoMap.obj
 0001:0001a090       ?RevealAutomapLevel@@YAXPAUDrlgLevel@@@Z 1001b090 f   AutoMap.obj
 0001:0001a1d0       ?RevealLevelPlayerIn@@YAXXZ 1001b1d0 f   AutoMap.obj
 0001:0001a210       ?InitDrlgLevelInfo@@YAXPAUDrlgMisc@@@Z 1001b210 f   AutoMap.obj
 0001:0001a2d0       ?RevealAutomap@@YAXXZ      1001b2d0 f   AutoMap.obj
 0001:0001a3b0       ?ShowAutoMap@@YAXXZ        1001b3b0 f   AutoMap.obj
 0001:0001a3d0       ?DrawAutomapBlob@@YIXHHKPAUUnitAny@@@Z 1001b3d0 f   AutoMapBlob.obj
 0001:0001a5a0       ?ForceDrawBlob_ASM@@YAXXZ  1001b5a0 f   AutoMapBlob.obj
 0001:0001a5b0       ?DrawBlobPath_ASM@@YAXXZ   1001b5b0 f   AutoMapBlob.obj
 0001:0001a5c0       ?DrawPartyPlayerBlobPatch_ASM@@YAXXZ 1001b5c0 f   AutoMapBlob.obj
 0001:0001a5d0       ?HostilePlayerPatch@@YIEPAUUnitAny@@@Z 1001b5d0 f   AutoMapBlob.obj
 0001:0001a610       ?HostilePlayerColor_ASM@@YAXXZ 1001b610 f   AutoMapBlob.obj
 0001:0001a620       ?DrawPlayerTextPatch@@YIEPAUUnitAny@@@Z 1001b620 f   AutoMapBlob.obj
 0001:0001a690       ?DrawPlayerTextPatch_ASM@@YAXXZ 1001b690 f   AutoMapBlob.obj
 0001:0001a6b0       ?MonsterBlobDesc@@YIXPAUUnitAny@@@Z 1001b6b0 f   AutoMapBlob.obj
 0001:0001aa70       ?MonsterBlobDescPatch_ASM@@YAXXZ 1001ba70 f   AutoMapBlob.obj
 0001:0001aa90       ?MonsterBlobCol@@YIEPAUUnitAny@@@Z 1001ba90 f   AutoMapBlob.obj
 0001:0001abe0       ?CorpseBlobCol@@YIEPAUUnitAny@@@Z 1001bbe0 f   AutoMapBlob.obj
 0001:0001aca0       ?ObjectBlobCol@@YIEPAUUnitAny@@@Z 1001bca0 f   AutoMapBlob.obj
 0001:0001ae80       ?MissileBlobCol@@YIEPAUUnitAny@@@Z 1001be80 f   AutoMapBlob.obj
 0001:0001af90       ?MixedBlobColPatch@@YIEPAUUnitAny@@@Z 1001bf90 f   AutoMapBlob.obj
 0001:0001b040       ?MixedBlobColPatch_ASM@@YAXXZ 1001c040 f   AutoMapBlob.obj
 0001:0001b060       ?RemoveAutomapCell@@YAXPAUAutomapCell@@@Z 1001c060 f   AutoMapCell.obj
 0001:0001b0d0       ?RemoveMyAutomapCells@@YAXXZ 1001c0d0 f   AutoMapCell.obj
 0001:0001b130       ?AddAutoMapCell@@YAXPAUDrlgRoom2@@@Z 1001c130 f   AutoMapCell.obj
 0001:0001b580       ?DrawAutomapCellPatch@@YGXPAUCellContext@@KKPAUtagRECT@@K@Z 1001c580 f   AutoMapCell.obj
 0001:0001b8f0       ?AddShrinePatch_ASM@@YAXXZ 1001c8f0 f   AutoMapCell.obj
 0001:0001b920       ?OverrideShrinePatch@@YIXPAUAutomapCell@@0@Z 1001c920 f   AutoMapCell.obj
 0001:0001b980       ?OverrideShrinePatch_ASM@@YAXXZ 1001c980 f   AutoMapCell.obj
 0001:0001b9a0       ?AddMinimapCell@@YAXPAUDrlgLevel@@FFF@Z 1001c9a0 f   MinimapPoint.obj
 0001:0001baf0       ?ResetMiniCells@@YAXXZ     1001caf0 f   MinimapPoint.obj
 0001:0001bb40       ?BuildMiniMapPoint@@YAXK@Z 1001cb40 f   MinimapPoint.obj
 0001:0001bd40       ?ComputePos@@YAXPAUtagPOINT@@HH@Z 1001cd40 f   RoomArea.obj
 0001:0001bd80       ?ScreenToAutomapRelative@@YAXPAUtagPOINT@@HH@Z 1001cd80 f   RoomArea.obj
 0001:0001bdc0       ?DrawRoom2@@YAXPAUDrlgRoom2@@K@Z 1001cdc0 f   RoomArea.obj
 0001:0001bec0       ?RoomPatch@@YAXXZ          1001cec0 f   RoomArea.obj
 0001:0001c070       ?RoomPatch_ASM@@YAXXZ      1001d070 f   RoomArea.obj
 0001:0001c080       ?AutoEnchantLoop@@YAXPAUUnitAny@@@Z 1001d080 f   AutoEnchant.obj
 0001:0001c210       ?AutoEnchant@@YAXPAUUnitAny@@@Z 1001d210 f   AutoEnchant.obj
 0001:0001c250       ?SendChatMessage@@YAXPAD@Z 1001d250 f   GameChat.obj
 0001:0001c2f0       ?WisperPatch@@YAXXZ        1001d2f0 f   GameChat.obj
 0001:0001c310       ?WisperPatch_ASM@@YAXXZ    1001d310 f   GameChat.obj
 0001:0001c320       ?CheckD2WinEditBox@@YAXXZ  1001d320 f   GameChat.obj
 0001:0001c380       ?InputLinePatch@@YAHE@Z    1001d380 f   GameChat.obj
 0001:0001c410       ?InputLinePatch1_ASM@@YAXXZ 1001d410 f   GameChat.obj
 0001:0001c430       ?EditBoxCallBack@@YGHPAUD2EditBox@@KPAD@Z 1001d430 f   GameChat.obj
 0001:0001c430       ?Filterbox_InputHandler@@YGHPAUD2EditBox@@KPAD@Z 1001d430 f   GameFilter.obj
 0001:0001c440       ?InitD2EditBox@@YAHXZ      1001d440 f   GameChat.obj
 0001:0001c510       ?InputLinePatch2_ASM@@YAXXZ 1001d510 f   GameChat.obj
 0001:0001c530       ?SelectTextPatch1@@YGHPAD@Z 1001d530 f   GameChat.obj
 0001:0001c610       ?SelectTextPatch1_ASM@@YAXXZ 1001d610 f   GameChat.obj
 0001:0001c630       ?SelectTextPatch2@@YGHPAD@Z 1001d630 f   GameChat.obj
 0001:0001c6e0       ?SelectTextPatch2_ASM@@YAXXZ 1001d6e0 f   GameChat.obj
 0001:0001c700       ?ResetGameList@@YAXXZ      1001d700 f   GameFilter.obj
 0001:0001c730       ?D2MCPPacketHandler_05_Patch@@YIHPAE@Z 1001d730 f   GameFilter.obj
 0001:0001c880       ?D2MCPPacketHandler_05_Patch_ASM@@YAXXZ 1001d880 f   GameFilter.obj
 0001:0001c8a0       ?Filterbox_ReturnHandler@@YGHPA_W@Z 1001d8a0 f   GameFilter.obj
 0001:0001c920       ?CreateFilterBox@@YAXXZ    1001d920 f   GameFilter.obj
 0001:0001c9a0       ?CreateGameBoxPatch_ASM@@YAXXZ 1001d9a0 f   GameFilter.obj
 0001:0001c9b0       ?DestroyGamelistPatch@@YGXPAUD2EditBox@@@Z 1001d9b0 f   GameFilter.obj
 0001:0001c9f0       ?GameListRefreshTimePatch_ASM@@YAXXZ 1001d9f0 f   GameFilter.obj
 0001:0001ca30       ?DrawGameListPatch@@YAXXZ  1001da30 f   GameFilter.obj
 0001:0001cbc0       ?DrawGameListPatch_ASM@@YAXXZ 1001dbc0 f   GameFilter.obj
 0001:0001cbd0       ?IsFullWindow@@YAHXZ       1001dbd0 f   GameWindow.obj
 0001:0001ccd0       ?KeepWindowPatch@@YAXXZ    1001dcd0 f   GameWindow.obj
 0001:0001cd30       ?RemoveKeepWindowPatch@@YAXXZ 1001dd30 f   GameWindow.obj
 0001:0001cd60       ?NoHidePatch_ASM@@YAXXZ    1001dd60 f   GameWindow.obj
 0001:0001cd90       ?strchr@@YAPADQADH@Z       1001dd90 f i GameWindow.obj
 0001:0001cdb0       ?NsPassingActBugFixPatch_ASM@@YAXXZ 1001ddb0 f   NsPassBugFix.obj
 0001:0001cdc0       ?OutTownSelectPatch@@YIHPAUUnitAny@@@Z 1001ddc0 f   OutTownSelect.obj
 0001:0001ce00       ?OutTownSelectPatch_ASM1@@YAXXZ 1001de00 f   OutTownSelect.obj
 0001:0001ce30       ?CheckOutTownSelected@@YGHPAUUnitAny@@@Z 1001de30 f   OutTownSelect.obj
 0001:0001ce90       ?OutTownSelectPatch_ASM2@@YAXXZ 1001de90 f   OutTownSelect.obj
 0001:0001ceb0       ?ResponseInvite@@YAXXZ     1001deb0 f   PartyHelp.obj
 0001:0001cf60       ?CheckInvite@@YAHXZ        1001df60 f   PartyHelp.obj
 0001:0001cfb0       ?InviteAll@@YAXXZ          1001dfb0 f   PartyHelp.obj
 0001:0001d040       ?PermitAll@@YAXXZ          1001e040 f   PartyHelp.obj
 0001:0001d0c0       ?AutoParty@@YGXPAE@Z       1001e0c0 f   PartyHelp.obj
 0001:0001d1c0       ?RecvCommand_5A_Patch_ASM@@YAXXZ 1001e1c0 f   PartyHelp.obj
 0001:0001d1d0       ?AutoInvite@@YGXPAE@Z      1001e1d0 f   PartyHelp.obj
 0001:0001d380       ?RecvCommand_5B_Patch_ASM@@YAXXZ 1001e380 f   PartyHelp.obj
 0001:0001d3a0       ?PermShowItemsPatch1@@YAHXZ 1001e3a0 f   PermShowItem.obj
 0001:0001d3e0       ?PermShowItemsPatch2@@YAHXZ 1001e3e0 f   PermShowItem.obj
 0001:0001d450       ?PermShowItemsPatch3@@YAHXZ 1001e450 f   PermShowItem.obj
 0001:0001d4e0       ?PermShowItemsPatch1_ASM@@YAXXZ 1001e4e0 f   PermShowItem.obj
 0001:0001d4f0       ?PermShowItemsPatch2_ASM@@YAXXZ 1001e4f0 f   PermShowItem.obj
 0001:0001d510       ?PermShowItemsPatch3_ASM@@YAXXZ 1001e510 f   PermShowItem.obj
 0001:0001d530       ?PermShowItemsPatch4_ASM@@YAXXZ 1001e530 f   PermShowItem.obj
 0001:0001d540       ?CalSrollOfTownportal@@YAKXZ 1001e540 f   QuickBackTown.obj
 0001:0001d5a0       ?BackToTown@@YAXXZ         1001e5a0 f   QuickBackTown.obj
 0001:0001d660       ?AutoBackToTown@@YIXPAE@Z  1001e660 f   QuickBackTown.obj
 0001:0001d770       ?RecvCommand_60_Patch_ASM@@YAXXZ 1001e770 f   QuickBackTown.obj
 0001:0001d780       ?SaveGameName@@YAXXZ       1001e780 f   QuickGame.obj
 0001:0001d7e0       ?QuickExitGame@@YAXXZ      1001e7e0 f   QuickGame.obj
 0001:0001d800       ?QuickNextGame@@YAXH@Z     1001e800 f   QuickGame.obj
 0001:0001d990       ?NextGameNamePatch@@YIXPAUD2EditBox@@P6GH0KPAD@Z@Z 1001e990 f   QuickGame.obj
 0001:0001d9d0       ?NextGamePasswordPatch@@YIXPAUD2EditBox@@P6GH0KPAD@Z@Z 1001e9d0 f   QuickGame.obj
 0001:0001da10       ?MoveItem@@YAXPAUD2MSG@@@Z 1001ea10 f   QuickSwapItem.obj
 0001:0001df80       ?RButtonUpHandlerPatch@@YGXPAUD2MSG@@@Z 1001ef80 f   QuickSwapItem.obj
 0001:0001dfc0       ?RButtonUpHandlerPatch_ASM@@YAXXZ 1001efc0 f   QuickSwapItem.obj
 0001:0001dfe0       ?RButtonInTradePatch_ASM@@YAXXZ 1001efe0 f   QuickSwapItem.obj
 0001:0001e000       ?DealCtrlClick@@YAXXZ      1001f000 f   QuickSwapItem.obj
 0001:0001e080       ?CtrlClickHandlerPatch_ASM@@YAXXZ 1001f080 f   QuickSwapItem.obj
 0001:0001e0c0       ?LButtonUpHandlerPatch@@YGXPAUD2MSG@@@Z 1001f0c0 f   QuickSwapItem.obj
 0001:0001e120       ?LButtonUpHandlerPatch_ASM@@YAXXZ 1001f120 f   QuickSwapItem.obj
 0001:0001e140       ?SetScrollMapPos@@YAXDD@Z  1001f140 f   ScrollLock.obj
 0001:0001e250       ?CenterMap@@YAXXZ          1001f250 f   ScrollLock.obj
 0001:0001e270       ?SetMapShake@@YAXXZ        1001f270 f   ScrollLock.obj
 0001:0001e310       ?ScrollMap@@YAXH@Z         1001f310 f   ScrollLock.obj
 0001:0001e3b0       ?InitScrollLock@@YAXH@Z    1001f3b0 f   ScrollLock.obj
 0001:0001e510       ?DrawScollOffset@@YAXPA_WH@Z 1001f510 f   ScrollLock.obj
 0001:0001e5a0       ?NPCMessageLoopPatch_ASM@@YAXXZ 1001f5a0 f   SkipNpcMessage.obj
 0001:0001e5e0       ?NPCQuestMessageStartPatch_ASM@@YAXXZ 1001f5e0 f   SkipNpcMessage.obj
 0001:0001e600       ?NPCQuestMessageEndPatch1_ASM@@YAXXZ 1001f600 f   SkipNpcMessage.obj
 0001:0001e620       ?NPCQuestMessageEndPatch2_ASM@@YAXXZ 1001f620 f   SkipNpcMessage.obj
 0001:0001e630       ?FixSocketTimeOut_ASM@@YAXXZ 1001f630 f   Socket.obj
 0001:0001e640       ?FixSocketErrRet_ASM@@YAXXZ 1001f640 f   Socket.obj
 0001:0001e660       ?SetGoldPatch@@YIHH@Z      1001f660 f   TransGoldHelp.obj
 0001:0001e6e0       ?SetGoldPatch_ASM@@YAXXZ   1001f6e0 f   TransGoldHelp.obj
 0001:0001e6f0       ?SetDefaultGoldPatch_ASM@@YAXXZ 1001f6f0 f   TransGoldHelp.obj
 0001:0001e700       ?ULCPatch_ASM@@YAXXZ       1001f700 f   ULCPath.obj
 0001:0001e720       @__security_check_cookie@4 1001f720 f   LIBCMT:secchk.obj
 0001:0001e775       ___scrt_acquire_startup_lock 1001f775 f   LIBCMT:utility.obj
 0001:0001e7a7       ___scrt_dllmain_after_initialize_c 1001f7a7 f   LIBCMT:utility.obj
 0001:0001e7d2       ___scrt_dllmain_before_initialize_c 1001f7d2 f   LIBCMT:utility.obj
 0001:0001e7e0       ___scrt_dllmain_crt_thread_attach 1001f7e0 f   LIBCMT:utility.obj
 0001:0001e7ff       ___scrt_dllmain_crt_thread_detach 1001f7ff f   LIBCMT:utility.obj
 0001:0001e80c       ___scrt_dllmain_exception_filter 1001f80c f   LIBCMT:utility.obj
 0001:0001e840       ___scrt_dllmain_uninitialize_c 1001f840 f   LIBCMT:utility.obj
 0001:0001e863       ___scrt_dllmain_uninitialize_critical 1001f863 f   LIBCMT:utility.obj
 0001:0001e870       ___scrt_initialize_crt     1001f870 f   LIBCMT:utility.obj
 0001:0001e8a9       ___scrt_initialize_onexit_tables 1001f8a9 f   LIBCMT:utility.obj
 0001:0001e930       ___scrt_is_nonwritable_in_current_image 1001f930 f   LIBCMT:utility.obj
 0001:0001e9c4       ___scrt_release_startup_lock 1001f9c4 f   LIBCMT:utility.obj
 0001:0001e9e1       ___scrt_uninitialize_crt   1001f9e1 f   LIBCMT:utility.obj
 0001:0001ea09       __onexit                   1001fa09 f   LIBCMT:utility.obj
 0001:0001ea36       _atexit                    1001fa36 f   LIBCMT:utility.obj
 0001:0001ea4b       ??_U@YAPAXI@Z              1001fa4b f   LIBCMT:new_array.obj
 0001:0001ea54       ??3@YAXPAXI@Z              1001fa54 f   LIBCMT:delete_scalar_size.obj
 0001:0001ea62       ??_V@YAXPAX@Z              1001fa62 f   LIBCMT:delete_array.obj
 0001:0001ea67       ??2@YAPAXI@Z               1001fa67 f   LIBCMT:new_scalar.obj
 0001:0001ea97       ___raise_securityfailure   1001fa97 f   LIBCMT:gs_report.obj
 0001:0001eabf       ___report_gsfailure        1001fabf f   LIBCMT:gs_report.obj
 0001:0001ebb9       ___report_rangecheckfailure 1001fbb9 f   LIBCMT:gs_report.obj
 0001:0001ebc5       ___report_securityfailure  1001fbc5 f   LIBCMT:gs_report.obj
 0001:0001ed59       __Init_thread_footer       1001fd59 f   LIBCMT:thread_safe_statics.obj
 0001:0001eda3       __Init_thread_header       1001fda3 f   LIBCMT:thread_safe_statics.obj
 0001:0001edf5       __Init_thread_notify       1001fdf5 f   LIBCMT:thread_safe_statics.obj
 0001:0001ee2b       __Init_thread_wait         1001fe2b f   LIBCMT:thread_safe_statics.obj
 0001:0001f1b9       __DllMainCRTStartup@12     100201b9 f   LIBCMT:dll_dllmain.obj
 0001:0001f1dc       ___isa_available_init      100201dc f   LIBCMT:cpu_disp.obj
 0001:0001f3ad       __get_startup_argv_mode    100203ad f   LIBCMT:argv_mode.obj
 0001:0001f3b1       ___scrt_is_ucrt_dll_in_use 100203b1 f   LIBCMT:ucrt_detection.obj
 0001:0001f3bd       ___scrt_fastfail           100203bd f   LIBCMT:utility_desktop.obj
 0001:0001f4d8       __crt_debugger_hook        100204d8 f   LIBCMT:utility_desktop.obj
 0001:0001f4e0       __SEH_prolog4              100204e0 f   LIBCMT:sehprolg4.obj
 0001:0001f526       @_guard_check_icall_nop@4  10020526 f i LIBCMT:guard_support.obj
 0001:0001f529       ??3@YAXPAX@Z               10020529 f   LIBCMT:delete_scalar.obj
 0001:0001f52e       ??0bad_alloc@std@@QAE@ABV01@@Z 1002052e f i LIBCMT:throw_bad_alloc.obj
 0001:0001f549       ??0bad_alloc@std@@QAE@XZ   10020549 f i LIBCMT:throw_bad_alloc.obj
 0001:0001f561       ??0bad_array_new_length@std@@QAE@ABV01@@Z 10020561 f i LIBCMT:throw_bad_alloc.obj
 0001:0001f57c       ??0bad_array_new_length@std@@QAE@XZ 1002057c f i LIBCMT:throw_bad_alloc.obj
 0001:0001f594       ??0exception@std@@QAE@ABV01@@Z 10020594 f i LIBCMT:throw_bad_alloc.obj
 0001:0001f5c0       ??1bad_alloc@std@@UAE@XZ   100205c0 f i LIBCMT:throw_bad_alloc.obj
 0001:0001f5c0       ??1bad_array_new_length@std@@UAE@XZ 100205c0 f i LIBCMT:throw_bad_alloc.obj
 0001:0001f5d1       ??_Gbad_array_new_length@std@@UAEPAXI@Z 100205d1 f i LIBCMT:throw_bad_alloc.obj
 0001:0001f5d1       ??_Gbad_alloc@std@@UAEPAXI@Z 100205d1 f i LIBCMT:throw_bad_alloc.obj
 0001:0001f5d1       ??_Ebad_alloc@std@@UAEPAXI@Z 100205d1 f i LIBCMT:throw_bad_alloc.obj
 0001:0001f5d1       ??_Eexception@std@@UAEPAXI@Z 100205d1 f i LIBCMT:throw_bad_alloc.obj
 0001:0001f5d1       ??_Gexception@std@@UAEPAXI@Z 100205d1 f i LIBCMT:throw_bad_alloc.obj
 0001:0001f5d1       ??_Ebad_array_new_length@std@@UAEPAXI@Z 100205d1 f i LIBCMT:throw_bad_alloc.obj
 0001:0001f5fe       ?__scrt_throw_std_bad_alloc@@YAXXZ 100205fe f   LIBCMT:throw_bad_alloc.obj
 0001:0001f61b       ?__scrt_throw_std_bad_array_new_length@@YAXXZ 1002061b f   LIBCMT:throw_bad_alloc.obj
 0001:0001f638       ?what@exception@std@@UBEPBDXZ 10020638 f i LIBCMT:throw_bad_alloc.obj
 0001:0001f692       ___security_init_cookie    10020692 f   LIBCMT:gs_support.obj
 0001:0001f6dd       ?__scrt_initialize_type_info@@YAXXZ 100206dd f   LIBCMT:tncleanup.obj
 0001:0001f6e9       ?__scrt_uninitialize_type_info@@YAXXZ 100206e9 f   LIBCMT:tncleanup.obj
 0001:0001f6f5       ___local_stdio_scanf_options 100206f5 f i LIBCMT:default_local_stdio_options.obj
 0001:0001f6fb       ___scrt_initialize_default_local_stdio_options 100206fb f   LIBCMT:default_local_stdio_options.obj
 0001:0001f718       ___scrt_get_dyn_tls_init_callback 10020718 f   LIBCMT:dyn_tls_init.obj
 0001:0001f71e       __RTC_Initialize           1002071e f   LIBCMT:initsect.obj
 0001:0001f74a       __RTC_Terminate            1002074a f   LIBCMT:initsect.obj
 0001:0001f776       ??_Gtype_info@@UAEPAXI@Z   10020776 f i LIBCMT:std_type_info_static.obj
 0001:0001f776       ??_Etype_info@@UAEPAXI@Z   10020776 f i LIBCMT:std_type_info_static.obj
 0001:0001f799       ___DestructExceptionObject 10020799 f   libvcruntime:ehhelpers.obj
 0001:0001f83a       ?_CallMemberFunction0@@YGXQAX0@Z 1002083a f i libvcruntime:ehhelpers.obj
 0001:0001f8a0       _strrchr                   100208a0 f   libvcruntime:strrchr.obj
 0001:0001fa20       __except_handler4          10020a20 f   libvcruntime:chandler4.obj
 0001:0001fb80       _strstr                    10020b80 f   libvcruntime:strstr.obj
 0001:0001fdf0       _strchr                    10020df0 f   libvcruntime:strchr.obj
 0001:0001fe5e       ___from_strstr_to_strchr   10020e5e     libvcruntime:strchr.obj
 0001:0001ff1b       ___vcrt_initialize         10020f1b f   libvcruntime:initialization.obj
 0001:0001ff3a       ___vcrt_thread_attach      10020f3a f   libvcruntime:initialization.obj
 0001:0001ff45       ___vcrt_thread_detach      10020f45 f   libvcruntime:initialization.obj
 0001:0001ff50       ___vcrt_uninitialize       10020f50 f   libvcruntime:initialization.obj
 0001:0001ff67       ___vcrt_uninitialize_critical 10020f67 f   libvcruntime:initialization.obj
 0001:0001ff70       _memset                    10020f70 f   libvcruntime:memset.obj
 0001:000200ca       ___std_exception_copy      100210ca f   libvcruntime:std_exception.obj
 0001:0002012d       ___std_exception_destroy   1002112d f   libvcruntime:std_exception.obj
 0001:0002014c       __CxxThrowException@8      1002114c f   libvcruntime:throw.obj
 0001:000201b8       ___std_type_info_destroy_list 100211b8 f   libvcruntime:std_type_info.obj
 0001:000201db       ___vcrt_freefls@4          100211db f   libvcruntime:per_thread_data.obj
 0001:000201f7       ___vcrt_freeptd            100211f7 f   libvcruntime:per_thread_data.obj
 0001:0002022d       ___vcrt_getptd             1002122d f   libvcruntime:per_thread_data.obj
 0001:0002023b       ___vcrt_getptd_noexit      1002123b f   libvcruntime:per_thread_data.obj
 0001:000202cd       ___vcrt_initialize_ptd     100212cd f   libvcruntime:per_thread_data.obj
 0001:00020300       ___vcrt_uninitialize_ptd   10021300 f   libvcruntime:per_thread_data.obj
 0001:00020320       ___except_validate_context_record 10021320 f   libvcruntime:jbcxrval.obj
 0001:00020350       __local_unwind4            10021350 f   libvcruntime:exsup4.obj
 0001:00020440       @_EH4_CallFilterFunc@8     10021440 f   libvcruntime:exsup4.obj
 0001:00020460       @_EH4_TransferToHandler@8  10021460 f   libvcruntime:exsup4.obj
 0001:00020480       @_EH4_GlobalUnwind2@8      10021480 f   libvcruntime:exsup4.obj
 0001:000204a0       @_EH4_LocalUnwind@16       100214a0 f   libvcruntime:exsup4.obj
 0001:000204b7       ___vcrt_initialize_locks   100214b7 f   libvcruntime:locks.obj
 0001:000204f3       ___vcrt_uninitialize_locks 100214f3 f   libvcruntime:locks.obj
 0001:00020605       ___vcrt_FlsAlloc           10021605 f   libvcruntime:winapi_downlevel.obj
 0001:00020640       ___vcrt_FlsFree            10021640 f   libvcruntime:winapi_downlevel.obj
 0001:0002067b       ___vcrt_FlsGetValue        1002167b f   libvcruntime:winapi_downlevel.obj
 0001:000206b6       ___vcrt_FlsSetValue        100216b6 f   libvcruntime:winapi_downlevel.obj
 0001:000206f4       ___vcrt_InitializeCriticalSectionEx 100216f4 f   libvcruntime:winapi_downlevel.obj
 0001:00020740       _memcpy                    10021740 f   libvcruntime:memcpy.obj
 0001:00020740       _memmove                   10021740 f   libvcruntime:memmove.obj
 0001:00020cc0       __NLG_Notify               10021cc0 f   libvcruntime:exsup.obj
 0001:00020cd7       __NLG_Dispatch2            10021cd7     libvcruntime:exsup.obj
 0001:00020cd7       __NLG_Dispatch             10021cd7     libvcruntime:exsup.obj
 0001:00020ce0       __NLG_Call                 10021ce0 f   libvcruntime:exsup.obj
 0001:00020ce2       __NLG_Return2              10021ce2     libvcruntime:exsup.obj
 0001:00020cf0       ___acrt_locale_get_ctype_array_value 10021cf0 f i libucrt:_ctype.obj
 0001:00020d20       _isalnum                   10021d20 f   libucrt:_ctype.obj
 0001:00020db0       _isalpha                   10021db0 f   libucrt:_ctype.obj
 0001:00020e40       _isdigit                   10021e40 f   libucrt:_ctype.obj
 0001:00020ed0       _isspace                   10021ed0 f   libucrt:_ctype.obj
 0001:00020f54       ??0_LocaleUpdate@@QAE@QAU__crt_locale_pointers@@@Z 10021f54 f i libucrt:_wctype.obj
 0001:00020fd7       __isleadbyte_l             10021fd7 f i libucrt:_wctype.obj
 0001:00021011       _iswdigit                  10022011 f i libucrt:_wctype.obj
 0001:00021024       _iswspace                  10022024 f i libucrt:_wctype.obj
 0001:000210e4       __ecvt                     100220e4 f   libucrt:fcvt.obj
 0001:0002112d       __ecvt_s                   1002212d f   libucrt:fcvt.obj
 0001:0002120b       __toupper_l                1002220b f   libucrt:tolower_toupper.obj
 0001:00021310       _toupper                   10022310 f   libucrt:tolower_toupper.obj
 0001:00021340       ??$is_overflow_condition@K@__crt_strtox@@YA_NIK@Z 10022340 f i libucrt:strtox.obj
 0001:00021371       ??$make_c_string_character_source@DPAPAD@__crt_strtox@@YA?AV?$c_string_character_source@D@0@QBDQAPAD@Z 10022371 f i libucrt:strtox.obj
 0001:00021371       ??$make_c_string_character_source@_WPAPA_W@__crt_strtox@@YA?AV?$c_string_character_source@_W@0@QB_WQAPA_W@Z 10022371 f i libucrt:strtox.obj
 0001:0002138c       ??$parse_integer@KV?$c_string_character_source@D@__crt_strtox@@@__crt_strtox@@YAKQAU__crt_locale_pointers@@V?$c_string_character_source@D@0@H_N@Z 1002238c f i libucrt:strtox.obj
 0001:000215af       ??$parse_integer@KV?$c_string_character_source@_W@__crt_strtox@@@__crt_strtox@@YAKQAU__crt_locale_pointers@@V?$c_string_character_source@_W@0@H_N@Z 100225af f i libucrt:strtox.obj
 0001:00021bb7       ?unget@?$c_string_character_source@D@__crt_strtox@@QAEXD@Z 10022bb7 f i libucrt:strtox.obj
 0001:00021be0       ?unget@?$c_string_character_source@_W@__crt_strtox@@QAEX_W@Z 10022be0 f i libucrt:strtox.obj
 0001:00021c0e       ?validate@?$c_string_character_source@_W@__crt_strtox@@QBE_NXZ 10022c0e f i libucrt:strtox.obj
 0001:00021c0e       ?validate@?$c_string_character_source@D@__crt_strtox@@QBE_NXZ 10022c0e f i libucrt:strtox.obj
 0001:00021c0e       ?validate@?$string_output_adapter@D@__crt_stdio_output@@QBE_NXZ 10022c0e f i libucrt:output.obj
 0001:00021c29       __ischartype_l             10022c29 f i libucrt:strtox.obj
 0001:00021c7d       _strtol                    10022c7d f   libucrt:strtox.obj
 0001:00021ca7       _strtoul                   10022ca7 f   libucrt:strtox.obj
 0001:00021cd1       _wcstol                    10022cd1 f   libucrt:strtox.obj
 0001:00021d00       _strncpy                   10022d00 f   libucrt:strncpy.obj
 0001:00021fa2       ??$count@D@formatting_buffer@__crt_stdio_output@@QBEIXZ 10022fa2 f i libucrt:output.obj
 0001:00021fba       ??$ensure_buffer_is_big_enough@D@formatting_buffer@__crt_stdio_output@@QAE_NI@Z 10022fba f i libucrt:output.obj
 0001:00022037       ??$is_wide_character_specifier@D@__crt_stdio_output@@YA_N_KDW4length_modifier@0@@Z 10023037 f i libucrt:output.obj
 0001:00022068       ??$scratch_data@D@formatting_buffer@__crt_stdio_output@@QAEPADXZ 10023068 f i libucrt:output.obj
 0001:00022086       ??$type_case_integer_parse_into_buffer@I@?$output_processor@DV?$string_output_adapter@D@__crt_stdio_output@@V?$standard_base@DV?$string_output_adapter@D@__crt_stdio_output@@@2@@__crt_stdio_output@@AAEXII_N@Z 10023086 f i libucrt:output.obj
 0001:000220f9       ??$type_case_integer_parse_into_buffer@_K@?$output_processor@DV?$string_output_adapter@D@__crt_stdio_output@@V?$standard_base@DV?$string_output_adapter@D@__crt_stdio_output@@@2@@__crt_stdio_output@@AAEX_KI_N@Z 100230f9 f i libucrt:output.obj
 0001:00022187       ??$write_multiple_characters@V?$string_output_adapter@D@__crt_stdio_output@@D@__crt_stdio_output@@YAXABV?$string_output_adapter@D@0@DHQAH@Z 10023187 f i libucrt:output.obj
 0001:000221b3       ??0?$common_data@D@__crt_stdio_output@@IAE@XZ 100231b3 f i libucrt:output.obj
 0001:000221f8       ??0?$output_adapter_data@DV?$string_output_adapter@D@__crt_stdio_output@@@__crt_stdio_output@@IAE@ABV?$string_output_adapter@D@1@_KQBDQAU__crt_locale_pointers@@QAD@Z 100231f8 f i libucrt:output.obj
 0001:00022234       ??1formatting_buffer@__crt_stdio_output@@QAE@XZ 10023234 f i libucrt:output.obj
 0001:0002224e       ??4?$__crt_unique_heap_ptr@DU__crt_internal_free_policy@@@@QAEAAV0@$$QAV0@@Z 1002324e f i libucrt:output.obj
 0001:00022280       ?crop_zeroes@__crt_stdio_output@@YAXPADQAU__crt_locale_pointers@@@Z 10023280 f i libucrt:output.obj
 0001:00022301       ?find_next_state@?$output_processor@DV?$string_output_adapter@D@__crt_stdio_output@@V?$standard_base@DV?$string_output_adapter@D@__crt_stdio_output@@@2@@__crt_stdio_output@@ABE?AW4state@2@DW432@@Z 10023301 f i libucrt:output.obj
 0001:00022340       ?force_decimal_point@__crt_stdio_output@@YAXPADQAU__crt_locale_pointers@@@Z 10023340 f i libucrt:output.obj
 0001:000223a5       ?parse_int_from_format_string@?$output_processor@DV?$string_output_adapter@D@__crt_stdio_output@@V?$standard_base@DV?$string_output_adapter@D@__crt_stdio_output@@@2@@__crt_stdio_output@@AAE_NQAH@Z 100233a5 f i libucrt:output.obj
 0001:00022419       ?process@?$output_processor@DV?$string_output_adapter@D@__crt_stdio_output@@V?$standard_base@DV?$string_output_adapter@D@__crt_stdio_output@@@2@@__crt_stdio_output@@QAEHXZ 10023419 f i libucrt:output.obj
 0001:0002252d       ?state_case_flag@?$output_processor@DV?$string_output_adapter@D@__crt_stdio_output@@V?$standard_base@DV?$string_output_adapter@D@__crt_stdio_output@@@2@@__crt_stdio_output@@AAE_NXZ 1002352d f i libucrt:output.obj
 0001:0002256a       ?state_case_normal@?$output_processor@DV?$string_output_adapter@D@__crt_stdio_output@@V?$standard_base@DV?$string_output_adapter@D@__crt_stdio_output@@@2@@__crt_stdio_output@@AAE_NXZ 1002356a f i libucrt:output.obj
 0001:00022589       ?state_case_normal_common@?$output_processor@DV?$string_output_adapter@D@__crt_stdio_output@@V?$standard_base@DV?$string_output_adapter@D@__crt_stdio_output@@@2@@__crt_stdio_output@@AAE_NXZ 10023589 f i libucrt:output.obj
 0001:000225b3       ?state_case_normal_tchar@?$output_processor@DV?$string_output_adapter@D@__crt_stdio_output@@V?$standard_base@DV?$string_output_adapter@D@__crt_stdio_output@@@2@@__crt_stdio_output@@AAE_ND@Z 100235b3 f i libucrt:output.obj
 0001:00022617       ?state_case_precision@?$output_processor@DV?$string_output_adapter@D@__crt_stdio_output@@V?$standard_base@DV?$string_output_adapter@D@__crt_stdio_output@@@2@@__crt_stdio_output@@AAE_NXZ 10023617 f i libucrt:output.obj
 0001:0002263d       ?state_case_size@?$output_processor@DV?$string_output_adapter@D@__crt_stdio_output@@V?$standard_base@DV?$string_output_adapter@D@__crt_stdio_output@@@2@@__crt_stdio_output@@AAE_NXZ 1002363d f i libucrt:output.obj
 0001:0002278b       ?state_case_type@?$output_processor@DV?$string_output_adapter@D@__crt_stdio_output@@V?$standard_base@DV?$string_output_adapter@D@__crt_stdio_output@@@2@@__crt_stdio_output@@AAE_NXZ 1002378b f i libucrt:output.obj
 0001:000229bd       ?state_case_width@?$output_processor@DV?$string_output_adapter@D@__crt_stdio_output@@V?$standard_base@DV?$string_output_adapter@D@__crt_stdio_output@@@2@@__crt_stdio_output@@AAE_NXZ 100239bd f i libucrt:output.obj
 0001:000229f0       ?to_integer_size@__crt_stdio_output@@YAIW4length_modifier@1@@Z 100239f0 f i libucrt:output.obj
 0001:00022a4c       ?type_case_Z@?$output_processor@DV?$string_output_adapter@D@__crt_stdio_output@@V?$standard_base@DV?$string_output_adapter@D@__crt_stdio_output@@@2@@__crt_stdio_output@@AAE_NXZ 10023a4c f i libucrt:output.obj
 0001:00022aa6       ?type_case_a@?$output_processor@DV?$string_output_adapter@D@__crt_stdio_output@@V?$standard_base@DV?$string_output_adapter@D@__crt_stdio_output@@@2@@__crt_stdio_output@@AAE_NXZ 10023aa6 f i libucrt:output.obj
 0001:00022bf7       ?type_case_c_tchar@?$output_processor@DV?$string_output_adapter@D@__crt_stdio_output@@V?$standard_base@DV?$string_output_adapter@D@__crt_stdio_output@@@2@@__crt_stdio_output@@AAE_ND@Z 10023bf7 f i libucrt:output.obj
 0001:00022c8a       ?type_case_integer@?$output_processor@DV?$string_output_adapter@D@__crt_stdio_output@@V?$standard_base@DV?$string_output_adapter@D@__crt_stdio_output@@@2@@__crt_stdio_output@@AAE_NI_N@Z 10023c8a f i libucrt:output.obj
 0001:00022ddb       ?type_case_n@?$output_processor@DV?$string_output_adapter@D@__crt_stdio_output@@V?$standard_base@DV?$string_output_adapter@D@__crt_stdio_output@@@2@@__crt_stdio_output@@AAE_NXZ 10023ddb f i libucrt:output.obj
 0001:00022e4f       ?type_case_o@?$output_processor@DV?$string_output_adapter@D@__crt_stdio_output@@V?$standard_base@DV?$string_output_adapter@D@__crt_stdio_output@@@2@@__crt_stdio_output@@AAE_NXZ 10023e4f f i libucrt:output.obj
 0001:00022e6e       ?type_case_p@?$output_processor@DV?$string_output_adapter@D@__crt_stdio_output@@V?$standard_base@DV?$string_output_adapter@D@__crt_stdio_output@@@2@@__crt_stdio_output@@AAE_NXZ 10023e6e f i libucrt:output.obj
 0001:00022e86       ?type_case_s@?$output_processor@DV?$string_output_adapter@D@__crt_stdio_output@@V?$standard_base@DV?$string_output_adapter@D@__crt_stdio_output@@@2@@__crt_stdio_output@@AAE_NXZ 10023e86 f i libucrt:output.obj
 0001:00022ef7       ?write_character@?$string_output_adapter@D@__crt_stdio_output@@QBE_NDQAH@Z 10023ef7 f i libucrt:output.obj
 0001:00022f39       ?write_stored_string_tchar@?$output_processor@DV?$string_output_adapter@D@__crt_stdio_output@@V?$standard_base@DV?$string_output_adapter@D@__crt_stdio_output@@@2@@__crt_stdio_output@@AAE_ND@Z 10023f39 f i libucrt:output.obj
 0001:00022fde       ?write_string@?$string_output_adapter@D@__crt_stdio_output@@QBEXQBDHQAHAAV__crt_deferred_errno_cache@@@Z 10023fde f i libucrt:output.obj
 0001:00023045       ___stdio_common_vsprintf   10024045 f   libucrt:output.obj
 0001:00023069       ___ascii_stricmp           10024069 f   libucrt:stricmp.obj
 0001:000230a2       __stricmp                  100240a2 f   libucrt:stricmp.obj
 0001:000230eb       __stricmp_l                100240eb f   libucrt:stricmp.obj
 0001:00023179       _strtok                    10024179 f   libucrt:strtok.obj
 0001:00023249       ??$__acrt_mbs_to_wcs_cp@U__crt_win32_buffer_internal_dynamic_resizing@@@@YAHQBDAAV?$__crt_win32_buffer@_WU__crt_win32_buffer_internal_dynamic_resizing@@@@I@Z 10024249 f i libucrt:rename.obj
 0001:00023266       ?__acrt_get_utf8_acp_compatibility_codepage@@YAIXZ 10024266 f i libucrt:rename.obj
 0001:000232a5       ?_deallocate@?$__crt_win32_buffer@DU__crt_win32_buffer_internal_dynamic_resizing@@@@AAEXXZ 100242a5 f i libucrt:argv_wildcards.obj
 0001:000232a5       ?_deallocate@?$__crt_win32_buffer@_WU__crt_win32_buffer_internal_dynamic_resizing@@@@AAEXXZ 100242a5 f i libucrt:rename.obj
 0001:000232bf       ?allocate@?$__crt_win32_buffer@_WU__crt_win32_buffer_internal_dynamic_resizing@@@@QAEHI@Z 100242bf f i libucrt:rename.obj
 0001:000232fe       ?allocate@__crt_win32_buffer_internal_dynamic_resizing@@SAHQAPAXIABV__crt_win32_buffer_empty_debug_info@@@Z 100242fe f i libucrt:rename.obj
 0001:0002331d       _rename                    1002431d f   libucrt:rename.obj
 0001:00023537       __freea_crt                10024537 f i libucrt:strupr.obj
 0001:00023557       __strupr                   10024557 f   libucrt:strupr.obj
 0001:000235b3       __strupr_s_l               100245b3 f   libucrt:strupr.obj
 0001:000235ea       __seh_filter_dll           100245ea f   libucrt:exception_filter.obj
 0001:0002360a       __seh_filter_exe           1002460a f   libucrt:exception_filter.obj
 0001:000239d8       ___acrt_initialize_thread_local_exit_callback 100249d8 f   libucrt:exit.obj
 0001:000239e7       __cexit                    100249e7 f   libucrt:exit.obj
 0001:000239f6       __exit                     100249f6 f   libucrt:exit.obj
 0001:00023a0c       __is_c_termination_complete 10024a0c f   libucrt:exit.obj
 0001:00023cbd       ___acrt_allocate_buffer_for_argv 10024cbd f   libucrt:argv_parsing.obj
 0001:00023d0c       __configure_narrow_argv    10024d0c f   libucrt:argv_parsing.obj
 0001:00023e69       ??$uninitialize@A6AXAAPAPAD@Z@?$dual_state_global@PAPAD@__crt_state_management@@QAEXA6AXAAPAPAD@Z@Z 10024e69 f i libucrt:environment_initialization.obj
 0001:00023e69       ??$uninitialize@A6AXAAPAPA_W@Z@?$dual_state_global@PAPA_W@__crt_state_management@@QAEXA6AXAAPAPA_W@Z@Z 10024e69 f i libucrt:environment_initialization.obj
 0001:00023ec8       ___dcrt_uninitialize_environments_nolock 10024ec8 f   libucrt:environment_initialization.obj
 0001:00023eff       __initialize_narrow_environment 10024eff f   libucrt:environment_initialization.obj
 0001:00023fba       ??$__crt_fast_encode_pointer@PAP6AXXZ@@YAPAP6AXXZQAP6AXXZ@Z 10024fba f i libucrt:onexit.obj
 0001:00023fba       ??$__crt_fast_encode_pointer@PAX@@YAPAXQAX@Z 10024fba f i libucrt:initialization.obj
 0001:00023fba       ??$__crt_fast_encode_pointer@P6AHXZ@@YAP6AHXZQ6AHXZ@Z 10024fba f i libucrt:onexit.obj
 0001:000241dc       __crt_atexit               100251dc f   libucrt:onexit.obj
 0001:000241f2       __execute_onexit_table     100251f2 f   libucrt:onexit.obj
 0001:0002421f       __initialize_onexit_table  1002521f f   libucrt:onexit.obj
 0001:00024248       __register_onexit_function 10025248 f   libucrt:onexit.obj
 0001:000242a2       ___acrt_uninitialize_command_line 100252a2 f   libucrt:argv_data.obj
 0001:00024379       ___acrt_initialize         10025379 f   libucrt:initialization.obj
 0001:0002438b       ___acrt_thread_attach      1002538b f   libucrt:initialization.obj
 0001:00024396       ___acrt_thread_detach      10025396 f   libucrt:initialization.obj
 0001:0002439e       ___acrt_uninitialize       1002539e f   libucrt:initialization.obj
 0001:000243ce       ___acrt_uninitialize_critical 100253ce f   libucrt:initialization.obj
 0001:000243e0       ___acrt_initialize_new_handler 100253e0 f   libucrt:new_handler.obj
 0001:000243ef       __callnewh                 100253ef f   libucrt:new_handler.obj
 0001:0002441c       __query_new_handler        1002541c f   libucrt:new_handler.obj
 0001:00024478       _malloc                    10025478 f   libucrt:malloc.obj
 0001:00024483       __initterm                 10025483 f   libucrt:initterm.obj
 0001:000244c8       __initterm_e               100254c8 f   libucrt:initterm.obj
 0001:000244f6       _terminate                 100254f6 f   libucrt:terminate.obj
 0001:00024532       _free                      10025532 f   libucrt:free.obj
 0001:0002454d       _abort                     1002554d f   libucrt:abort.obj
 0001:00024591       _strcpy_s                  10025591 f   libucrt:strcpy_s.obj
 0001:000245eb       _calloc                    100255eb f   libucrt:calloc.obj
 0001:00024600       _strncmp                   10025600 f   libucrt:strncmp.obj
 0001:00024678       _wcsncmp                   10025678 f   libucrt:wcsncmp.obj
 0001:000246b2       __isctype_l                100256b2 f   libucrt:isctype.obj
 0001:00024abb       ___acrt_freeptd            10025abb f   libucrt:per_thread_data.obj
 0001:00024ae7       ___acrt_getptd             10025ae7 f   libucrt:per_thread_data.obj
 0001:00024ba4       ___acrt_getptd_head        10025ba4 f   libucrt:per_thread_data.obj
 0001:00024c3e       ___acrt_getptd_noexit      10025c3e f   libucrt:per_thread_data.obj
 0001:00024cf3       ___acrt_initialize_ptd     10025cf3 f   libucrt:per_thread_data.obj
 0001:00024d1f       ___acrt_uninitialize_ptd   10025d1f f   libucrt:per_thread_data.obj
 0001:00024d39       ___acrt_update_locale_info 10025d39 f   libucrt:locale_update.obj
 0001:00024d66       ___acrt_update_multibyte_info 10025d66 f   libucrt:locale_update.obj
 0001:00024e01       ___acrt_set_locale_changed 10025e01 f   libucrt:wsetlocale.obj
 0001:00024e0c       ___acrt_uninitialize_locale 10025e0c f   libucrt:wsetlocale.obj
 0001:00024e33       _iswctype                  10025e33 f   libucrt:iswctype.obj
 0001:00024e9c       ___acrt_call_reportfault   10025e9c f   libucrt:invalid_parameter.obj
 0001:00024fd5       ___acrt_initialize_invalid_parameter_handler 10025fd5 f   libucrt:invalid_parameter.obj
 0001:00024fe4       __invalid_parameter        10025fe4 f   libucrt:invalid_parameter.obj
 0001:00025048       __invalid_parameter_noinfo 10026048 f   libucrt:invalid_parameter.obj
 0001:00025058       __invoke_watson            10026058 f   libucrt:invalid_parameter.obj
 0001:0002508c       ___acrt_errno_from_os_error 1002608c f   libucrt:errno.obj
 0001:000250cf       ___acrt_errno_map_os_error 100260cf f   libucrt:errno.obj
 0001:000250f2       ___doserrno                100260f2 f   libucrt:errno.obj
 0001:00025105       __errno                    10026105 f   libucrt:errno.obj
 0001:00025118       __free_base                10026118 f   libucrt:free_base.obj
 0001:00025152       __malloc_base              10026152 f   libucrt:malloc_base.obj
 0001:0002521a       ___acrt_fp_strflt_to_string 1002621a f   libucrt:_fptostr.obj
 0001:000252f6       ?__acrt_fp_classify@@YA?AW4__acrt_fp_class@@ABN@Z 100262f6 f i libucrt:cfout.obj
 0001:00025360       ?divide@__crt_strtox@@YA_KAAUbig_integer@1@ABU21@@Z 10026360 f i libucrt:cfout.obj
 0001:000257f8       ___acrt_fltout             100267f8 f   libucrt:cfout.obj
 0001:00026f6a       ___acrt_LCMapStringA       10027f6a f   libucrt:lcmapstringa.obj
 0001:00026fb3       ___pctype_func             10027fb3 f   libucrt:ctype.obj
 0001:00026fd7       __mbtowc_l                 10027fd7 f   libucrt:mbtowc.obj
 0001:00027119       _mbtowc                    10028119 f   libucrt:mbtowc.obj
 0001:00027133       __wctomb_s_l               10028133 f   libucrt:wctomb.obj
 0001:0002728e       _strnlen                   1002828e f   libucrt:strnlen.obj
 0001:000273b0       _wcsnlen                   100283b0 f   libucrt:strnlen.obj
 0001:00027eb1       ___acrt_fp_format          10028eb1 f   libucrt:cvt.obj
 0001:0002800d       __fileno                   1002900d f   libucrt:fileno.obj
 0001:00028034       ___acrt_initialize_stdio   10029034 f   libucrt:_file.obj
 0001:000280fc       ___acrt_uninitialize_stdio 100290fc f   libucrt:_file.obj
 0001:00028148       __lock_file                10029148 f   libucrt:_file.obj
 0001:0002815c       __unlock_file              1002915c f   libucrt:_file.obj
 0001:00028170       __get_printf_count_output  10029170 f   libucrt:printf_count_output.obj
 0001:000282ef       ___acrt_initialize_lowio   100292ef f   libucrt:ioinit.obj
 0001:0002834f       ___acrt_uninitialize_lowio 1002934f f   libucrt:ioinit.obj
 0001:0002837b       ___acrt_strtok_s_novalidation 1002937b f   libucrt:strtok_s.obj
 0001:00028467       ___acrt_MultiByteToWideChar 10029467 f   libucrt:multibytetowidechar.obj
 0001:0002867b       ___acrt_AppPolicyGetProcessTerminationMethodInternal@4 1002967b f   libucrt:winapi_thunks.obj
 0001:000286bb       ___acrt_AreFileApisANSI@0  100296bb f   libucrt:winapi_thunks.obj
 0001:000286da       ___acrt_FlsAlloc@4         100296da f   libucrt:winapi_thunks.obj
 0001:00028719       ___acrt_FlsFree@4          10029719 f   libucrt:winapi_thunks.obj
 0001:00028758       ___acrt_FlsGetValue@4      10029758 f   libucrt:winapi_thunks.obj
 0001:00028797       ___acrt_FlsSetValue@8      10029797 f   libucrt:winapi_thunks.obj
 0001:000287d9       ___acrt_InitializeCriticalSectionEx@12 100297d9 f   libucrt:winapi_thunks.obj
 0001:00028824       ___acrt_LCMapStringEx@36   10029824 f   libucrt:winapi_thunks.obj
 0001:00028881       ___acrt_LocaleNameToLCID@8 10029881 f   libucrt:winapi_thunks.obj
 0001:000288b2       ___acrt_initialize_winapi_thunks 100298b2 f   libucrt:winapi_thunks.obj
 0001:000288dd       ___acrt_uninitialize_winapi_thunks 100298dd f   libucrt:winapi_thunks.obj
 0001:00028913       __wrename                  10029913 f   libucrt:wrename.obj
 0001:00028940       ___acrt_initialize_locks   10029940 f   libucrt:locks.obj
 0001:00028981       ___acrt_lock               10029981 f   libucrt:locks.obj
 0001:00028998       ___acrt_uninitialize_locks 10029998 f   libucrt:locks.obj
 0001:000289c9       ___acrt_unlock             100299c9 f   libucrt:locks.obj
 0001:000289e0       ___acrt_get_process_end_policy 100299e0 f   libucrt:win_policies.obj
 0001:00028a11       __calloc_base              10029a11 f   libucrt:calloc_base.obj
 0001:0002904c       ?allocate@?$__crt_win32_buffer@DU__crt_win32_buffer_internal_dynamic_resizing@@@@QAEHI@Z 1002a04c f i libucrt:argv_wildcards.obj
 0001:0002910f       ___acrt_expand_narrow_argv_wildcards 1002a10f f   libucrt:argv_wildcards.obj
 0001:000291e1       ?allocate@?$__crt_win32_buffer@DU__crt_win32_buffer_no_resizing@@@@QAEHI@Z 1002a1e1 f i libucrt:getmodulefilenamea.obj
 0001:00029208       ?set_to_nullptr@?$__crt_win32_buffer@DU__crt_win32_buffer_no_resizing@@@@QAEXXZ 1002a208 f i libucrt:getmodulefilenamea.obj
 0001:0002921c       ___acrt_GetModuleFileNameA 1002a21c f   libucrt:getmodulefilenamea.obj
 0001:000297d5       ___acrt_initialize_multibyte 1002a7d5 f   libucrt:mbctype.obj
 0001:0002981d       ___acrt_update_thread_multibyte_data 1002a81d f   libucrt:mbctype.obj
 0001:00029830       __setmbcp_nolock           1002a830 f   libucrt:mbctype.obj
 0001:00029a7a       __ismbblead                1002aa7a f   libucrt:ismbbyte.obj
 0001:00029a92       ___acrt_initialize_command_line 1002aa92 f   libucrt:argv_data.obj
 0001:00029aab       ___acrt_WideCharToMultiByte 1002aaab f   libucrt:widechartomultibyte.obj
 0001:00029b99       ___dcrt_get_narrow_environment_from_os 1002ab99 f   libucrt:get_environment_from_os.obj
 0001:00029c1d       __recalloc_base            1002ac1d f   libucrt:recalloc.obj
 0001:00029c8a       ___acrt_initialize_heap    1002ac8a f   libucrt:heap_handle.obj
 0001:00029c9b       ___acrt_uninitialize_heap  1002ac9b f   libucrt:heap_handle.obj
 0001:00029ca5       ___acrt_execute_initializers 1002aca5 f   libucrt:shared_initialization.obj
 0001:00029d0d       ___acrt_execute_uninitializers 1002ad0d f   libucrt:shared_initialization.obj
 0001:00029e0c       ___acrt_get_sigabrt_handler 1002ae0c f   libucrt:signal.obj
 0001:00029e33       ___acrt_initialize_signal_handlers 1002ae33 f   libucrt:signal.obj
 0001:00029e51       _raise                     1002ae51 f   libucrt:signal.obj
 0001:0002a044       ___acrt_has_user_matherr   1002b044 f   libucrt:matherr.obj
 0001:0002a05c       ___acrt_initialize_user_matherr 1002b05c f   libucrt:matherr.obj
 0001:0002a06b       ___acrt_invoke_user_matherr 1002b06b f   libucrt:matherr.obj
 0001:0002a27a       ___acrt_stdio_flush_nolock 1002b27a f   libucrt:fflush.obj
 0001:0002a2df       __fflush_nolock            1002b2df f   libucrt:fflush.obj
 0001:0002a327       __flushall                 1002b327 f   libucrt:fflush.obj
 0001:0002a330       ___acrt_GetStringTypeA     1002b330 f   libucrt:getstringtypea.obj
 0001:0002a433       ___acrt_add_locale_ref     1002b433 f   libucrt:locale_refcounting.obj
 0001:0002a4b0       ___acrt_free_locale        1002b4b0 f   libucrt:locale_refcounting.obj
 0001:0002a5f8       ___acrt_locale_add_lc_time_reference 1002b5f8 f   libucrt:locale_refcounting.obj
 0001:0002a621       ___acrt_locale_free_lc_time_if_unreferenced 1002b621 f   libucrt:locale_refcounting.obj
 0001:0002a652       ___acrt_locale_release_lc_time_reference 1002b652 f   libucrt:locale_refcounting.obj
 0001:0002a67b       ___acrt_release_locale_ref 1002b67b f   libucrt:locale_refcounting.obj
 0001:0002a6fc       ___acrt_update_thread_locale_data 1002b6fc f   libucrt:locale_refcounting.obj
 0001:0002a77d       __updatetlocinfoEx_nolock  1002b77d f   libucrt:locale_refcounting.obj
 0001:0002a7cd       ___acrt_locale_free_monetary 1002b7cd f   libucrt:initmon.obj
 0001:0002a8cb       ___acrt_locale_free_numeric 1002b8cb f   libucrt:initnum.obj
 0001:0002a96c       ___acrt_locale_free_time   1002b96c f   libucrt:inittime.obj
 0001:0002aa50       ___acrt_GetStringTypeW     1002ba50 f   libucrt:getstringtypew.obj
 0001:0002aa69       __query_new_mode           1002ba69 f   libucrt:new_mode.obj
 0001:0002aa70       _fegetround                1002ba70 f   libucrt:fegetround.obj
 0001:0002aa7d       __controlfp_s              1002ba7d f   libucrt:contrlfp.obj
 0001:0002aadc       _fegetenv                  1002badc f   libucrt:fegetenv.obj
 0001:0002aaf9       _fesetenv                  1002baf9 f   libucrt:fesetenv.obj
 0001:0002ab44       _feholdexcept              1002bb44 f   libucrt:feholdexcept.obj
 0001:0002aba0       __CIlog10                  1002bba0 f   libucrt:log10_impl.obj
 0001:0002abdb       __CIlog10_default          1002bbdb f   libucrt:log10_impl.obj
 0001:0002abef       __log10_default            1002bbef     libucrt:log10_impl.obj
 0001:0002acb0       _ceil                      1002bcb0 f   libucrt:ceil_pentium4.obj
 0001:0002acf0       __ceil_pentium4            1002bcf0 f   libucrt:ceil_pentium4.obj
 0001:0002adcd       ___strncnt                 1002bdcd f   libucrt:strncnt.obj
 0001:0002ae15       ?__mbrtowc_utf8@__crt_mbstring@@YAIPA_WPBDIPAU_Mbstatet@@@Z 1002be15 f   libucrt:mbrtowc.obj
 0001:0002ae55       ?__mbsrtowcs_utf8@__crt_mbstring@@YAIPA_WPAPBDIPAU_Mbstatet@@@Z 1002be55 f   libucrt:mbrtowc.obj
 0001:0002af50       ?__c32rtomb_utf8@__crt_mbstring@@YAIPAD_UPAU_Mbstatet@@@Z 1002bf50 f   libucrt:c32rtomb.obj
 0001:0002affb       ?return_illegal_sequence@__crt_mbstring@@YAIPAU_Mbstatet@@@Z 1002bffb f i libucrt:c32rtomb.obj
 0001:0002b01a       __fcloseall                1002c01a f   libucrt:closeall.obj
 0001:0002b0c5       ___acrt_stdio_free_buffer_nolock 1002c0c5 f   libucrt:_freebuf.obj
 0001:0002b105       __isatty                   1002c105 f   libucrt:isatty.obj
 0001:0002b15b       ___acrt_lowio_create_handle_array 1002c15b f   libucrt:osfinfo.obj
 0001:0002b1d6       ___acrt_lowio_destroy_handle_array 1002c1d6 f   libucrt:osfinfo.obj
 0001:0002b20b       ___acrt_lowio_ensure_fh_exists 1002c20b f   libucrt:osfinfo.obj
 0001:0002b2a9       ___acrt_lowio_lock_fh      1002c2a9 f   libucrt:osfinfo.obj
 0001:0002b2cc       ___acrt_lowio_unlock_fh    1002c2cc f   libucrt:osfinfo.obj
 0001:0002b2ef       __free_osfhnd              1002c2ef f   libucrt:osfinfo.obj
 0001:0002b380       __get_osfhandle            1002c380 f   libucrt:osfinfo.obj
 0001:0002b43a       ___acrt_DownlevelLocaleNameToLCID 1002c43a f   libucrt:lcidtoname_downlevel.obj
 0001:0002b470       _qsort                     1002c470 f   libucrt:qsort.obj
 0001:0002ba11       _strncpy_s                 1002ca11 f   libucrt:strncpy_s.obj
 0001:0002ba20       _strpbrk                   1002ca20 f   libucrt:strpbrk.obj
 0001:0002ba60       __mbsdec                   1002ca60 f   libucrt:mbsdec.obj
 0001:0002ba77       __mbsdec_l                 1002ca77 f   libucrt:mbsdec.obj
 0001:0002bb13       __msize_base               1002cb13 f   libucrt:msize.obj
 0001:0002bb46       __realloc_base             1002cb46 f   libucrt:realloc_base.obj
 0001:0002bc51       __commit                   1002cc51 f   libucrt:commit.obj
 0001:0002c449       __write                    1002d449 f   libucrt:write.obj
 0001:0002c53b       __write_nolock             1002d53b f   libucrt:write.obj
 0001:0002c715       ___ascii_wcsnicmp          1002d715 f   libucrt:wcsnicmp.obj
 0001:0002ca81       ___acrt_fenv_get_common_round_control 1002da81 f   libucrt:_fenvutils.obj
 0001:0002caa3       ___acrt_fenv_get_control   1002daa3 f   libucrt:_fenvutils.obj
 0001:0002cb23       ___acrt_fenv_get_status    1002db23 f   libucrt:_fenvutils.obj
 0001:0002cbdb       ___acrt_fenv_set_control   1002dbdb f   libucrt:_fenvutils.obj
 0001:0002cc43       ___acrt_fenv_set_status    1002dc43 f   libucrt:_fenvutils.obj
 0001:0002cde1       __clearfp                  1002dde1 f   libucrt:ieee87.obj
 0001:0002cebf       __control87                1002debf f   libucrt:ieee87.obj
 0001:0002d25e       ___acrt_initialize_sse2    1002e25e f   libucrt:mathfcns.obj
 0001:0002d270       __CIlog10_pentium4         1002e270 f   libucrt:log10_pentium4.obj
 0001:0002d288       __log10_pentium4           1002e288     libucrt:log10_pentium4.obj
 0001:0002d520       __fFEXP                    1002e520 f   libucrt:87tran.obj
 0001:0002d577       __rtinfpopse               1002e577     libucrt:87tran.obj
 0001:0002d579       __rtinfnpopse              1002e579     libucrt:87tran.obj
 0001:0002d589       __fFLN                     1002e589     libucrt:87tran.obj
 0001:0002d63e       __rtinfpop                 1002e63e     libucrt:87tran.obj
 0001:0002d640       __rtinfnpop                1002e640     libucrt:87tran.obj
 0001:0002d650       __rtforexpinf              1002e650 f   libucrt:87tran.obj
 0001:0002d65d       __ffexpm1                  1002e65d     libucrt:87tran.obj
 0001:0002d710       __trandisp1                1002e710 f   libucrt:87disp.obj
 0001:0002d785       __trandisp2                1002e785 f   libucrt:87disp.obj
 0001:0002d81f       __rttospopde               1002e81f     libucrt:87disp.obj
 0001:0002d824       __rttospop                 1002e824     libucrt:87disp.obj
 0001:0002d830       __rtnospop                 1002e830 f   libucrt:87disp.obj
 0001:0002d840       __rttosnpop                1002e840 f   libucrt:87disp.obj
 0001:0002d841       __rtnospopde               1002e841     libucrt:87disp.obj
 0001:0002d848       __rtzeropop                1002e848     libucrt:87disp.obj
 0001:0002d84a       __rtzeronpop               1002e84a     libucrt:87disp.obj
 0001:0002d850       __rtzerospop               1002e850 f   libucrt:87disp.obj
 0001:0002d85d       __rtonepop                 1002e85d     libucrt:87disp.obj
 0001:0002d860       __rtonenpop                1002e860 f   libucrt:87disp.obj
 0001:0002d870       __tosnan1                  1002e870 f   libucrt:87disp.obj
 0001:0002d8a0       __nosnan2                  1002e8a0 f   libucrt:87disp.obj
 0001:0002d8b0       __tosnan2                  1002e8b0 f   libucrt:87disp.obj
 0001:0002d8e0       __nan2                     1002e8e0 f   libucrt:87disp.obj
 0001:0002d920       __rtindfpop                1002e920 f   libucrt:87disp.obj
 0001:0002d922       __rtindfnpop               1002e922     libucrt:87disp.obj
 0001:0002d933       __rttosnpopde              1002e933     libucrt:87disp.obj
 0001:0002d940       __rtatan2inf               1002e940 f   libucrt:87disp.obj
 0001:0002d95d       __rtchsifneg               1002e95d     libucrt:87disp.obj
 0001:0002d970       __twoToTOS                 1002e970 f   libucrt:common.obj
 0001:0002d985       __load_CW                  1002e985 f   libucrt:common.obj
 0001:0002d99c       __convertTOStoQNaN         1002e99c f   libucrt:common.obj
 0001:0002d9b5       __fload_withFB             1002e9b5 f   libucrt:common.obj
 0001:0002d9f8       __checkTOS_withFB          1002e9f8 f   libucrt:common.obj
 0001:0002da0e       __fast_exit                1002ea0e f   libucrt:common.obj
 0001:0002da1b       __math_exit                1002ea1b f   libucrt:common.obj
 0001:0002da45       __check_overflow_exit      1002ea45 f   libucrt:common.obj
 0001:0002da59       __check_range_exit         1002ea59 f   libucrt:common.obj
 0001:0002db00       __startTwoArgErrorHandling 1002eb00 f   libucrt:genexcep.obj
 0001:0002db17       __startOneArgErrorHandling 1002eb17 f   libucrt:genexcep.obj
 0001:0002db53       ___libm_error_support      1002eb53 f   libucrt:libm_error.obj
 0001:0002dd47       __ceil_default             1002ed47 f   libucrt:ceil.obj
 0001:0002ddfc       ?__mbrtoc32_utf8@__crt_mbstring@@YAIPA_UPBDIPAU_Mbstatet@@@Z 1002edfc f   libucrt:mbrtoc32.obj
 0001:0002e01f       __lseeki64_nolock          1002f01f f   libucrt:lseek.obj
 0001:0002e03a       __fclose_nolock            1002f03a f   libucrt:fclose.obj
 0001:0002e0b1       _fclose                    1002f0b1 f   libucrt:fclose.obj
 0001:0002e135       __query_app_type           1002f135 f   libucrt:report_runtime_error.obj
 0001:0002e13b       __putwch_nolock            1002f13b f   libucrt:putwch.obj
 0001:0002e16d       ___set_fpsr_sse2           1002f16d f   libucrt:fpctrl.obj
 0001:0002e1ed       __clrfp                    1002f1ed f   libucrt:fpctrl.obj
 0001:0002e1fe       __ctrlfp                   1002f1fe f   libucrt:fpctrl.obj
 0001:0002e228       __set_statfp               1002f228 f   libucrt:fpctrl.obj
 0001:0002e281       __statfp                   1002f281 f   libucrt:fpctrl.obj
 0001:0002e291       __d_inttype                1002f291 f   libucrt:powhlp.obj
 0001:0002e2f9       __powhlp                   1002f2f9 f   libucrt:powhlp.obj
 0001:0002e424       __87except                 1002f424 f   libucrt:87except.obj
 0001:0002e52e       __frnd                     1002f52e f   libucrt:frnd.obj
 0001:0002e542       __errcode                  1002f542 f   libucrt:fpexcept.obj
 0001:0002e576       __except1                  1002f576 f   libucrt:fpexcept.obj
 0001:0002e644       __handle_exc               1002f644 f   libucrt:fpexcept.obj
 0001:0002e82f       __raise_exc                1002f82f f   libucrt:fpexcept.obj
 0001:0002e852       __raise_exc_ex             1002f852 f   libucrt:fpexcept.obj
 0001:0002eb48       __set_errno_from_matherr   1002fb48 f   libucrt:fpexcept.obj
 0001:0002eb77       __umatherr                 1002fb77 f   libucrt:fpexcept.obj
 0001:0002ec17       __decomp                   1002fc17 f   libucrt:util.obj
 0001:0002ece9       __set_exp                  1002fce9 f   libucrt:util.obj
 0001:0002ed16       __sptype                   1002fd16 f   libucrt:util.obj
 0001:0002ee00       __close                    1002fe00 f   libucrt:close.obj
 0001:0002ee8d       __close_nolock             1002fe8d f   libucrt:close.obj
 0001:0002ef29       ?__acrt_stdio_free_stream@@YAXV__crt_stdio_stream@@@Z 1002ff29 f   libucrt:stream.obj
 0001:0002ef70       ___ascii_strnicmp          1002ff70 f   libucrt:_strnicm.obj
 0001:0002eff0       ___dcrt_lowio_ensure_console_output_initialized 1002fff0 f   libucrt:initcon.obj
 0001:0002f00f       ___dcrt_terminate_console_output 1003000f f   libucrt:initcon.obj
 0001:0002f026       ___dcrt_write_console      10030026 f   libucrt:initcon.obj
 0001:0002f07b       __fpclass                  1003007b f   libucrt:ieeemisc.obj
 0001:0002f120       __FindPESection            10030120 f   LIBCMT:pesect.obj
 0001:0002f170       __IsNonwritableInCurrentImage 10030170 f   LIBCMT:pesect.obj
 0001:0002f230       __ValidateImageBase        10030230 f   LIBCMT:pesect.obj
 0001:0002f270       __aulldvrm                 10030270 f   LIBCMT:ulldvrm.obj
 0001:0002f310       __allmul                   10030310 f   LIBCMT:llmul.obj
 0001:0002f350       __alloca_probe_16          10030350 f   LIBCMT:alloca16.obj
 0001:0002f366       __alloca_probe_8           10030366     LIBCMT:alloca16.obj
 0001:0002f380       __allshl                   10030380 f   LIBCMT:llshl.obj
 0001:0002f3a0       __ftol2_sse                100303a0 f   LIBCMT:ftol2.obj
 0001:0002f3b0       __ftoi2                    100303b0 f   LIBCMT:ftol2.obj
 0001:0002f430       __alldvrm                  10030430 f   LIBCMT:lldvrm.obj
 0001:0002f510       __aullshr                  10030510 f   LIBCMT:ullshr.obj
 0001:0002f530       __chkstk                   10030530 f   LIBCMT:chkstk.obj
 0001:0002f530       __alloca_probe             10030530 f   LIBCMT:chkstk.obj
 0001:0002f55d       __filter_x86_sse2_floating_point_exception_default 1003055d f   LIBCMT:x86_exception_filter.obj
 0001:0002f55d       __filter_x86_sse2_floating_point_exception 1003055d f   LIBCMT:x86_exception_filter.obj
 0001:0002f5e0       __dtoui3                   100305e0 f   LIBCMT:ftol3.obj
 0001:0002f660       __libm_sse2_sqrt_precise   10030660 f   libucrt:sqrt_sse2_precise.obj
 0001:0002f760       _sqrt                      10030760 f   libucrt:sqrt.obj
 0001:0002f770       __CIsqrt                   10030770 f   libucrt:sqrt_impl.obj
 0001:0002f784       __sqrt_common              10030784     libucrt:sqrt_impl.obj
 0002:00000000       __imp__ImmAssociateContext@8 10031000     imm32:IMM32.dll
 0002:00000004       \177IMM32_NULL_THUNK_DATA  10031004     imm32:IMM32.dll
 0002:00000008       __imp__LoadLibraryA@4      10031008     kernel32:KERNEL32.dll
 0002:0000000c       __imp__GetModuleHandleA@4  1003100c     kernel32:KERNEL32.dll
 0002:00000010       __imp__GetProcAddress@8    10031010     kernel32:KERNEL32.dll
 0002:00000014       __imp__VirtualProtect@16   10031014     kernel32:KERNEL32.dll
 0002:00000018       __imp__WriteProcessMemory@20 10031018     kernel32:KERNEL32.dll
 0002:0000001c       __imp__GetCurrentProcess@0 1003101c     kernel32:KERNEL32.dll
 0002:00000020       __imp__ReadProcessMemory@20 10031020     kernel32:KERNEL32.dll
 0002:00000024       __imp__CreateFileA@28      10031024     kernel32:KERNEL32.dll
 0002:00000028       __imp__WriteFile@20        10031028     kernel32:KERNEL32.dll
 0002:0000002c       __imp__ReadFile@20         1003102c     kernel32:KERNEL32.dll
 0002:00000030       __imp__GetFileSize@8       10031030     kernel32:KERNEL32.dll
 0002:00000034       __imp__CloseHandle@4       10031034     kernel32:KERNEL32.dll
 0002:00000038       __imp__MultiByteToWideChar@24 10031038     kernel32:KERNEL32.dll
 0002:0000003c       __imp__LCMapStringA@24     1003103c     kernel32:KERNEL32.dll
 0002:00000040       __imp__GetTickCount@0      10031040     kernel32:KERNEL32.dll
 0002:00000044       __imp__WideCharToMultiByte@32 10031044     kernel32:KERNEL32.dll
 0002:00000048       __imp__GetLocalTime@4      10031048     kernel32:KERNEL32.dll
 0002:0000004c       __imp__GetCurrentProcessId@0 1003104c     kernel32:KERNEL32.dll
 0002:00000050       __imp__SetFilePointer@16   10031050     kernel32:KERNEL32.dll
 0002:00000054       __imp__GlobalAlloc@8       10031054     kernel32:KERNEL32.dll
 0002:00000058       __imp__DisableThreadLibraryCalls@4 10031058     kernel32:KERNEL32.dll
 0002:0000005c       __imp__GlobalUnlock@4      1003105c     kernel32:KERNEL32.dll
 0002:00000060       __imp__GlobalFree@4        10031060     kernel32:KERNEL32.dll
 0002:00000064       __imp__GetCommandLineA@0   10031064     kernel32:KERNEL32.dll
 0002:00000068       __imp__CreateFileW@28      10031068     kernel32:KERNEL32.dll
 0002:0000006c       __imp__DecodePointer@4     1003106c     kernel32:KERNEL32.dll
 0002:00000070       __imp__GetConsoleMode@8    10031070     kernel32:KERNEL32.dll
 0002:00000074       __imp__GetConsoleOutputCP@0 10031074     kernel32:KERNEL32.dll
 0002:00000078       __imp__FlushFileBuffers@4  10031078     kernel32:KERNEL32.dll
 0002:0000007c       __imp__HeapReAlloc@16      1003107c     kernel32:KERNEL32.dll
 0002:00000080       __imp__HeapSize@12         10031080     kernel32:KERNEL32.dll
 0002:00000084       __imp__SetStdHandle@8      10031084     kernel32:KERNEL32.dll
 0002:00000088       __imp__SetFilePointerEx@20 10031088     kernel32:KERNEL32.dll
 0002:0000008c       __imp__GetStringTypeW@16   1003108c     kernel32:KERNEL32.dll
 0002:00000090       __imp__GetProcessHeap@0    10031090     kernel32:KERNEL32.dll
 0002:00000094       __imp__FreeEnvironmentStringsW@4 10031094     kernel32:KERNEL32.dll
 0002:00000098       __imp__GetEnvironmentStringsW@0 10031098     kernel32:KERNEL32.dll
 0002:0000009c       __imp__GlobalLock@4        1003109c     kernel32:KERNEL32.dll
 0002:000000a0       __imp__GetModuleFileNameA@12 100310a0     kernel32:KERNEL32.dll
 0002:000000a4       __imp__UnhandledExceptionFilter@4 100310a4     kernel32:KERNEL32.dll
 0002:000000a8       __imp__SetUnhandledExceptionFilter@4 100310a8     kernel32:KERNEL32.dll
 0002:000000ac       __imp__TerminateProcess@8  100310ac     kernel32:KERNEL32.dll
 0002:000000b0       __imp__IsProcessorFeaturePresent@4 100310b0     kernel32:KERNEL32.dll
 0002:000000b4       __imp__EnterCriticalSection@4 100310b4     kernel32:KERNEL32.dll
 0002:000000b8       __imp__LeaveCriticalSection@4 100310b8     kernel32:KERNEL32.dll
 0002:000000bc       __imp__InitializeCriticalSectionAndSpinCount@8 100310bc     kernel32:KERNEL32.dll
 0002:000000c0       __imp__DeleteCriticalSection@4 100310c0     kernel32:KERNEL32.dll
 0002:000000c4       __imp__SetEvent@4          100310c4     kernel32:KERNEL32.dll
 0002:000000c8       __imp__ResetEvent@4        100310c8     kernel32:KERNEL32.dll
 0002:000000cc       __imp__WaitForSingleObjectEx@12 100310cc     kernel32:KERNEL32.dll
 0002:000000d0       __imp__CreateEventW@16     100310d0     kernel32:KERNEL32.dll
 0002:000000d4       __imp__GetModuleHandleW@4  100310d4     kernel32:KERNEL32.dll
 0002:000000d8       __imp__IsDebuggerPresent@0 100310d8     kernel32:KERNEL32.dll
 0002:000000dc       __imp__GetStartupInfoW@4   100310dc     kernel32:KERNEL32.dll
 0002:000000e0       __imp__QueryPerformanceCounter@4 100310e0     kernel32:KERNEL32.dll
 0002:000000e4       __imp__GetCurrentThreadId@0 100310e4     kernel32:KERNEL32.dll
 0002:000000e8       __imp__GetSystemTimeAsFileTime@4 100310e8     kernel32:KERNEL32.dll
 0002:000000ec       __imp__InitializeSListHead@4 100310ec     kernel32:KERNEL32.dll
 0002:000000f0       __imp__RtlUnwind@16        100310f0     kernel32:KERNEL32.dll
 0002:000000f4       __imp__RaiseException@16   100310f4     kernel32:KERNEL32.dll
 0002:000000f8       __imp__InterlockedFlushSList@4 100310f8     kernel32:KERNEL32.dll
 0002:000000fc       __imp__GetLastError@0      100310fc     kernel32:KERNEL32.dll
 0002:00000100       __imp__SetLastError@4      10031100     kernel32:KERNEL32.dll
 0002:00000104       __imp__TlsAlloc@0          10031104     kernel32:KERNEL32.dll
 0002:00000108       __imp__TlsGetValue@4       10031108     kernel32:KERNEL32.dll
 0002:0000010c       __imp__TlsSetValue@8       1003110c     kernel32:KERNEL32.dll
 0002:00000110       __imp__TlsFree@4           10031110     kernel32:KERNEL32.dll
 0002:00000114       __imp__FreeLibrary@4       10031114     kernel32:KERNEL32.dll
 0002:00000118       __imp__LoadLibraryExW@12   10031118     kernel32:KERNEL32.dll
 0002:0000011c       __imp__ExitProcess@4       1003111c     kernel32:KERNEL32.dll
 0002:00000120       __imp__GetModuleHandleExW@12 10031120     kernel32:KERNEL32.dll
 0002:00000124       __imp__GetModuleFileNameW@12 10031124     kernel32:KERNEL32.dll
 0002:00000128       __imp__HeapFree@12         10031128     kernel32:KERNEL32.dll
 0002:0000012c       __imp__HeapAlloc@12        1003112c     kernel32:KERNEL32.dll
 0002:00000130       __imp__GetStdHandle@4      10031130     kernel32:KERNEL32.dll
 0002:00000134       __imp__GetFileType@4       10031134     kernel32:KERNEL32.dll
 0002:00000138       __imp__LCMapStringW@24     10031138     kernel32:KERNEL32.dll
 0002:0000013c       __imp__MoveFileExW@12      1003113c     kernel32:KERNEL32.dll
 0002:00000140       __imp__FindClose@4         10031140     kernel32:KERNEL32.dll
 0002:00000144       __imp__FindFirstFileExW@24 10031144     kernel32:KERNEL32.dll
 0002:00000148       __imp__FindNextFileW@8     10031148     kernel32:KERNEL32.dll
 0002:0000014c       __imp__IsValidCodePage@4   1003114c     kernel32:KERNEL32.dll
 0002:00000150       __imp__GetACP@0            10031150     kernel32:KERNEL32.dll
 0002:00000154       __imp__GetOEMCP@0          10031154     kernel32:KERNEL32.dll
 0002:00000158       __imp__GetCPInfo@8         10031158     kernel32:KERNEL32.dll
 0002:0000015c       __imp__GetCommandLineW@0   1003115c     kernel32:KERNEL32.dll
 0002:00000160       __imp__WriteConsoleW@20    10031160     kernel32:KERNEL32.dll
 0002:00000164       \177KERNEL32_NULL_THUNK_DATA 10031164     kernel32:KERNEL32.dll
 0002:00000168       __imp__wvsprintfA@12       10031168     user32:USER32.dll
 0002:0000016c       __imp__wsprintfW           1003116c     user32:USER32.dll
 0002:00000170       __imp__SendMessageA@16     10031170     user32:USER32.dll
 0002:00000174       __imp__MessageBeep@4       10031174     user32:USER32.dll
 0002:00000178       __imp__OpenClipboard@4     10031178     user32:USER32.dll
 0002:0000017c       __imp__EmptyClipboard@0    1003117c     user32:USER32.dll
 0002:00000180       __imp__GetWindowInfo@8     10031180     user32:USER32.dll
 0002:00000184       __imp__CloseClipboard@0    10031184     user32:USER32.dll
 0002:00000188       __imp__SetClipboardData@8  10031188     user32:USER32.dll
 0002:0000018c       \177USER32_NULL_THUNK_DATA 1003118c     user32:USER32.dll
 0002:00000190       __imp__GetFileVersionInfoSizeA@8 10031190     Version:VERSION.dll
 0002:00000194       __imp__VerQueryValueA@16   10031194     Version:VERSION.dll
 0002:00000198       __imp__GetFileVersionInfoA@16 10031198     Version:VERSION.dll
 0002:0000019c       \177VERSION_NULL_THUNK_DATA 1003119c     Version:VERSION.dll
 0002:000001a0       __imp__WSACleanup@0        100311a0     ws2_32:WS2_32.dll
 0002:000001a4       __imp__WSAStartup@8        100311a4     ws2_32:WS2_32.dll
 0002:000001a8       \177WS2_32_NULL_THUNK_DATA 100311a8     ws2_32:WS2_32.dll
 0002:000001ac       ___guard_check_icall_fptr  100311ac     LIBCMT:guard_support.obj
 0002:000001b0       ___xc_a                    100311b0     LIBCMT:initializers.obj
 0002:00000430       ___xc_z                    10031430     LIBCMT:initializers.obj
 0002:00000434       ___xi_a                    10031434     LIBCMT:initializers.obj
 0002:0000043c       ___acrt_stdio_initializer  1003143c     libucrt:stdio_initializer.obj
 0002:00000440       ___acrt_multibyte_initializer 10031440     libucrt:multibyte_initializer.obj
 0002:00000444       ___acrt_tran_sse2_initializer 10031444     libucrt:sse2_initializer.obj
 0002:00000448       ___xi_z                    10031448     LIBCMT:initializers.obj
 0002:0000044c       ___xl_a                    1003144c     LIBCMT:tlssup.obj
 0002:00000450       ___xl_z                    10031450     LIBCMT:tlssup.obj
 0002:00000454       ___xp_a                    10031454     LIBCMT:initializers.obj
 0002:00000458       ___acrt_locale_terminator  10031458     libucrt:locale_initializer.obj
 0002:0000045c       ___dcrt_console_output_terminator 1003145c     libucrt:console_output_initializer.obj
 0002:00000460       ___acrt_stdio_terminator   10031460     libucrt:stdio_initializer.obj
 0002:00000464       ___xp_z                    10031464     LIBCMT:initializers.obj
 0002:00000468       ___xt_a                    10031468     LIBCMT:initializers.obj
 0002:0000046c       ___xt_z                    1003146c     LIBCMT:initializers.obj
 0002:00000478       ??_C@_1EC@JIJBPKFM@?$AAa?$AAp?$AAi?$AA?9?$AAm?$AAs?$AA?9?$AAw?$AAi?$AAn?$AA?9?$AAc?$AAo?$AAr?$AAe@ 10031478     LIBCMT:thread_safe_statics.obj
 0002:000004bc       ??_C@_1BK@MGMFAEKH@?$AAk?$AAe?$AAr?$AAn?$AAe?$AAl?$AA3?$AA2?$AA?4?$AAd?$AAl?$AAl@ 100314bc     LIBCMT:thread_safe_statics.obj
 0002:000004d8       ??_C@_0BJ@JEBJOJFJ@SleepConditionVariableCS@ 100314d8     LIBCMT:thread_safe_statics.obj
 0002:000004f4       ??_C@_0BJ@PGPPEPCC@WakeAllConditionVariable@ 100314f4     LIBCMT:thread_safe_statics.obj
 0002:00000510       __pRawDllMain              10031510     LIBCMT:dll_dllmain.obj
 0002:00000510       __pDefaultRawDllMain       10031510     LIBCMT:dll_dllmain.obj
 0002:00000518       ??_7exception@std@@6B@     10031518     LIBCMT:throw_bad_alloc.obj
 0002:00000520       ??_C@_0BC@EOODALEL@Unknown?5exception@ 10031520     LIBCMT:throw_bad_alloc.obj
 0002:00000538       ??_7bad_alloc@std@@6B@     10031538     LIBCMT:throw_bad_alloc.obj
 0002:00000540       ??_C@_0P@GHFPNOJB@bad?5allocation@ 10031540     LIBCMT:throw_bad_alloc.obj
 0002:00000554       ??_7bad_array_new_length@std@@6B@ 10031554     LIBCMT:throw_bad_alloc.obj
 0002:0000055c       ??_C@_0BF@KINCDENJ@bad?5array?5new?5length@ 1003155c     LIBCMT:throw_bad_alloc.obj
 0002:00000578       ??_7type_info@@6B@         10031578     LIBCMT:std_type_info_static.obj
 0002:0000057c       __pDestructExceptionObject 1003157c     libvcruntime:ehhelpers.obj
 0002:00000900       ??_C@_08EHJDFFNH@__based?$CI@ 10031900     libvcruntime:undname.obj
 0002:0000090c       ??_C@_07KOLFKCDI@__cdecl@  1003190c     libvcruntime:undname.obj
 0002:00000914       ??_C@_08GHMPAG@__pascal@   10031914     libvcruntime:undname.obj
 0002:00000920       ??_C@_09IFJBGAPI@__stdcall@ 10031920     libvcruntime:undname.obj
 0002:0000092c       ??_C@_0L@NPHFGOKO@__thiscall@ 1003192c     libvcruntime:undname.obj
 0002:00000938       ??_C@_0L@JMKHOMEK@__fastcall@ 10031938     libvcruntime:undname.obj
 0002:00000944       ??_C@_0N@BCKKPABJ@__vectorcall@ 10031944     libvcruntime:undname.obj
 0002:00000954       ??_C@_09HIJEGCPM@__clrcall@ 10031954     libvcruntime:undname.obj
 0002:00000960       ??_C@_06GHPCKEAG@__eabi@   10031960     libvcruntime:undname.obj
 0002:00000968       ??_C@_09IOPIDJLG@__swift_1@ 10031968     libvcruntime:undname.obj
 0002:00000974       ??_C@_09KFNFGKHF@__swift_2@ 10031974     libvcruntime:undname.obj
 0002:00000980       ??_C@_07JOMMBBKO@__ptr64@  10031980     libvcruntime:undname.obj
 0002:00000988       ??_C@_0L@PILCLIHE@__restrict@ 10031988     libvcruntime:undname.obj
 0002:00000994       ??_C@_0M@GFIIJFMG@__unaligned@ 10031994     libvcruntime:undname.obj
 0002:000009a0       ??_C@_09DHDLOLLB@restrict?$CI@ 100319a0     libvcruntime:undname.obj
 0002:000009aa       ??_C@_00CNPNBAHC@@         100319aa     libvcruntime:undname.obj
 0002:000009ac       ??_C@_04NIHEBCM@?5new@     100319ac     libvcruntime:undname.obj
 0002:000009b4       ??_C@_07FPCDHGMM@?5delete@ 100319b4     libvcruntime:undname.obj
 0002:000009bc       ??_C@_01NEMOKFLO@?$DN@     100319bc     libvcruntime:undname.obj
 0002:000009c0       ??_C@_02GPIOPFAK@?$DO?$DO@ 100319c0     libvcruntime:undname.obj
 0002:000009c4       ??_C@_02FODMEDOG@?$DM?$DM@ 100319c4     libvcruntime:undname.obj
 0002:000009c8       ??_C@_01DCLJPIOD@?$CB@     100319c8     libvcruntime:undname.obj
 0002:000009cc       ??_C@_02EGOFBIJA@?$DN?$DN@ 100319cc     libvcruntime:undname.obj
 0002:000009d0       ??_C@_02FDNJECIE@?$CB?$DN@ 100319d0     libvcruntime:undname.obj
 0002:000009d4       ??_C@_02GPECMEKF@?$FL?$FN@ 100319d4     libvcruntime:undname.obj
 0002:000009d8       ??_C@_08LHJFAFGD@operator@ 100319d8     libvcruntime:undname.obj
 0002:000009e4       ??_C@_02HBOOOICD@?9?$DO@   100319e4     libvcruntime:undname.obj
 0002:000009e8       ??_C@_01NBENCBCI@?$CK@     100319e8     libvcruntime:undname.obj
 0002:000009ec       ??_C@_02ECNGHCIF@?$CL?$CL@ 100319ec     libvcruntime:undname.obj
 0002:000009f0       ??_C@_02BAABKJLB@?9?9@     100319f0     libvcruntime:undname.obj
 0002:000009f4       ??_C@_01JOAMLHOP@?9@       100319f4     libvcruntime:undname.obj
 0002:000009f8       ??_C@_01MIFGBAGJ@?$CL@     100319f8     libvcruntime:undname.obj
 0002:000009fc       ??_C@_01HNPIGOCE@?$CG@     100319fc     libvcruntime:undname.obj
 0002:00000a00       ??_C@_03MNHNFDLC@?9?$DO?$CK@ 10031a00     libvcruntime:undname.obj
 0002:00000a04       ??_C@_01KMDKNFGN@?1@       10031a04     libvcruntime:undname.obj
 0002:00000a08       ??_C@_01FGNFDNOH@?$CF@     10031a08     libvcruntime:undname.obj
 0002:00000a0c       ??_C@_01MNNFJEPP@?$DM@     10031a0c     libvcruntime:undname.obj
 0002:00000a10       ??_C@_02EHCHHCKH@?$DM?$DN@ 10031a10     libvcruntime:undname.obj
 0002:00000a14       ??_C@_01PPODPGHN@?$DO@     10031a14     libvcruntime:undname.obj
 0002:00000a18       ??_C@_02EEKDKGMJ@?$DO?$DN@ 10031a18     libvcruntime:undname.obj
 0002:00000a1c       ??_C@_01IHBHIGKO@?0@       10031a1c     libvcruntime:undname.obj
 0002:00000a20       ??_C@_02HCKGKOFO@?$CI?$CJ@ 10031a20     libvcruntime:undname.obj
 0002:00000a24       ??_C@_01PJKLJHI@?$HO@      10031a24     libvcruntime:undname.obj
 0002:00000a28       ??_C@_01JKBOJNNK@?$FO@     10031a28     libvcruntime:undname.obj
 0002:00000a2c       ??_C@_01DNKMNLPK@?$HM@     10031a2c     libvcruntime:undname.obj
 0002:00000a30       ??_C@_02PPKAJPJL@?$CG?$CG@ 10031a30     libvcruntime:undname.obj
 0002:00000a34       ??_C@_02NONPIBCD@?$HM?$HM@ 10031a34     libvcruntime:undname.obj
 0002:00000a38       ??_C@_02FPIMKNGF@?$CK?$DN@ 10031a38     libvcruntime:undname.obj
 0002:00000a3c       ??_C@_02FOEOMHFC@?$CL?$DN@ 10031a3c     libvcruntime:undname.obj
 0002:00000a40       ??_C@_02FKMDLLOA@?9?$DN@   10031a40     libvcruntime:undname.obj
 0002:00000a44       ??_C@_02FJEHGPIO@?1?$DN@   10031a44     libvcruntime:undname.obj
 0002:00000a48       ??_C@_02FENAOKFI@?$CF?$DN@ 10031a48     libvcruntime:undname.obj
 0002:00000a4c       ??_C@_03IKFCCPFF@?$DO?$DO?$DN@ 10031a4c     libvcruntime:undname.obj
 0002:00000a50       ??_C@_03CDNPDDLA@?$DM?$DM?$DN@ 10031a50     libvcruntime:undname.obj
 0002:00000a54       ??_C@_02FGJGFEAB@?$CG?$DN@ 10031a54     libvcruntime:undname.obj
 0002:00000a58       ??_C@_02DHLNPPGH@?$HM?$DN@ 10031a58     libvcruntime:undname.obj
 0002:00000a5c       ??_C@_02MHEGNOJ@?$FO?$DN@  10031a5c     libvcruntime:undname.obj
 0002:00000a60       ??_C@_09IFPLHPGF@?$GAvftable?8@ 10031a60     libvcruntime:undname.obj
 0002:00000a6c       ??_C@_09BLBHBJP@?$GAvbtable?8@ 10031a6c     libvcruntime:undname.obj
 0002:00000a78       ??_C@_07FEEIOKP@?$GAvcall?8@ 10031a78     libvcruntime:undname.obj
 0002:00000a80       ??_C@_08LLFFHHDJ@?$GAtypeof?8@ 10031a80     libvcruntime:undname.obj
 0002:00000a8c       ??_C@_0BF@KDPPACIK@?$GAlocal?5static?5guard?8@ 10031a8c     libvcruntime:undname.obj
 0002:00000aa4       ??_C@_08OBABFOLI@?$GAstring?8@ 10031aa4     libvcruntime:undname.obj
 0002:00000ab0       ??_C@_0BD@JDLKDPAB@?$GAvbase?5destructor?8@ 10031ab0     libvcruntime:undname.obj
 0002:00000ac4       ??_C@_0BN@DEGPLNFK@?$GAvector?5deleting?5destructor?8@ 10031ac4     libvcruntime:undname.obj
 0002:00000ae4       ??_C@_0BO@OBMKPJIG@?$GAdefault?5constructor?5closure?8@ 10031ae4     libvcruntime:undname.obj
 0002:00000b04       ??_C@_0BN@IMDCHIKM@?$GAscalar?5deleting?5destructor?8@ 10031b04     libvcruntime:undname.obj
 0002:00000b24       ??_C@_0BO@PFGOCPJJ@?$GAvector?5constructor?5iterator?8@ 10031b24     libvcruntime:undname.obj
 0002:00000b44       ??_C@_0BN@LFPFMEDL@?$GAvector?5destructor?5iterator?8@ 10031b44     libvcruntime:undname.obj
 0002:00000b64       ??_C@_0CE@IKBNEHA@?$GAvector?5vbase?5constructor?5itera@ 10031b64     libvcruntime:undname.obj
 0002:00000b88       ??_C@_0BL@NILFHHPC@?$GAvirtual?5displacement?5map?8@ 10031b88     libvcruntime:undname.obj
 0002:00000ba4       ??_C@_0CB@JONCMFFK@?$GAeh?5vector?5constructor?5iterator@ 10031ba4     libvcruntime:undname.obj
 0002:00000bc8       ??_C@_0CA@GCEOPDGL@?$GAeh?5vector?5destructor?5iterator?8@ 10031bc8     libvcruntime:undname.obj
 0002:00000be8       ??_C@_0CH@OOJPLCPH@?$GAeh?5vector?5vbase?5constructor?5it@ 10031be8     libvcruntime:undname.obj
 0002:00000c10       ??_C@_0BL@LLKPOHJI@?$GAcopy?5constructor?5closure?8@ 10031c10     libvcruntime:undname.obj
 0002:00000c2c       ??_C@_0BA@KBCDOMBN@?$GAudt?5returning?8@ 10031c2c     libvcruntime:undname.obj
 0002:00000c3c       ??_C@_03KLGMFNMG@?$GAEH@   10031c3c     libvcruntime:undname.obj
 0002:00000c40       ??_C@_05KHLCHHI@?$GARTTI@  10031c40     libvcruntime:undname.obj
 0002:00000c48       ??_C@_0BA@KKLDJDLB@?$GAlocal?5vftable?8@ 10031c48     libvcruntime:undname.obj
 0002:00000c58       ??_C@_0CE@IIHCMGGL@?$GAlocal?5vftable?5constructor?5clos@ 10031c58     libvcruntime:undname.obj
 0002:00000c7c       ??_C@_06FHBGPFGH@?5new?$FL?$FN@ 10031c7c     libvcruntime:undname.obj
 0002:00000c84       ??_C@_09LBNFPBCA@?5delete?$FL?$FN@ 10031c84     libvcruntime:undname.obj
 0002:00000c90       ??_C@_0P@HJKNJFNN@?$GAomni?5callsig?8@ 10031c90     libvcruntime:undname.obj
 0002:00000ca0       ??_C@_0BL@CNOONJFP@?$GAplacement?5delete?5closure?8@ 10031ca0     libvcruntime:undname.obj
 0002:00000cbc       ??_C@_0BN@CKNJLHMB@?$GAplacement?5delete?$FL?$FN?5closure?8@ 10031cbc     libvcruntime:undname.obj
 0002:00000cdc       ??_C@_0CG@CFDHKGGD@?$GAmanaged?5vector?5constructor?5ite@ 10031cdc     libvcruntime:undname.obj
 0002:00000d04       ??_C@_0CF@IMGKMJNO@?$GAmanaged?5vector?5destructor?5iter@ 10031d04     libvcruntime:undname.obj
 0002:00000d2c       ??_C@_0CG@HLDDJMAG@?$GAeh?5vector?5copy?5constructor?5ite@ 10031d2c     libvcruntime:undname.obj
 0002:00000d54       ??_C@_0CM@FCBBDIGB@?$GAeh?5vector?5vbase?5copy?5construct@ 10031d54     libvcruntime:undname.obj
 0002:00000d80       ??_C@_0BL@CLIPGLGB@?$GAdynamic?5initializer?5for?5?8@ 10031d80     libvcruntime:undname.obj
 0002:00000d9c       ??_C@_0CB@PDBIFEP@?$GAdynamic?5atexit?5destructor?5for?5@ 10031d9c     libvcruntime:undname.obj
 0002:00000dc0       ??_C@_0CD@CGAJBKEJ@?$GAvector?5copy?5constructor?5iterat@ 10031dc0     libvcruntime:undname.obj
 0002:00000de4       ??_C@_0CJ@GJELGAMM@?$GAvector?5vbase?5copy?5constructor?5@ 10031de4     libvcruntime:undname.obj
 0002:00000e10       ??_C@_0CL@FGIJHLCE@?$GAmanaged?5vector?5copy?5constructo@ 10031e10     libvcruntime:undname.obj
 0002:00000e3c       ??_C@_0BM@PMGGMLDN@?$GAlocal?5static?5thread?5guard?8@ 10031e3c     libvcruntime:undname.obj
 0002:00000e58       ??_C@_0N@BDNMDMOL@operator?5?$CC?$CC?5@ 10031e58     libvcruntime:undname.obj
 0002:00000e68       ??_C@_0BC@GGEBGALA@operator?5co_await@ 10031e68     libvcruntime:undname.obj
 0002:00000e7c       ??_C@_0M@GAAIMMOH@operator?$DM?$DN?$DO@ 10031e7c     libvcruntime:undname.obj
 0002:00000e88       ??_C@_0BC@DAFEJGAK@?5Type?5Descriptor?8@ 10031e88     libvcruntime:undname.obj
 0002:00000e9c       ??_C@_0BM@LDKODKLH@?5Base?5Class?5Descriptor?5at?5?$CI@ 10031e9c     libvcruntime:undname.obj
 0002:00000eb8       ??_C@_0BD@LGICGFMM@?5Base?5Class?5Array?8@ 10031eb8     libvcruntime:undname.obj
 0002:00000ecc       ??_C@_0BN@MECKDCOJ@?5Class?5Hierarchy?5Descriptor?8@ 10031ecc     libvcruntime:undname.obj
 0002:00000eec       ??_C@_0BK@CFCOFLF@?5Complete?5Object?5Locator?8@ 10031eec     libvcruntime:undname.obj
 0002:00000f08       ??_C@_0BG@JNJLAMPM@?$GAanonymous?5namespace?8@ 10031f08     libvcruntime:undname.obj
 0002:00000f2c       ??_C@_1DM@KHCHBNEB@?$AAa?$AAp?$AAi?$AA?9?$AAm?$AAs?$AA?9?$AAw?$AAi?$AAn?$AA?9?$AAc?$AAo?$AAr?$AAe@ 10031f2c     libvcruntime:winapi_downlevel.obj
 0002:00000f68       ??_C@_1DK@LPPGFMPP@?$AAa?$AAp?$AAi?$AA?9?$AAm?$AAs?$AA?9?$AAw?$AAi?$AAn?$AA?9?$AAc?$AAo?$AAr?$AAe@ 10031f68     libvcruntime:winapi_downlevel.obj
 0002:00000fa4       ??_C@_1BC@GDMECMAK@?$AAk?$AAe?$AAr?$AAn?$AAe?$AAl?$AA3?$AA2@ 10031fa4     libvcruntime:winapi_downlevel.obj
 0002:00000fb8       ??_C@_1BA@PFFKHIOG@?$AAa?$AAp?$AAi?$AA?9?$AAm?$AAs?$AA?9@ 10031fb8     libvcruntime:winapi_downlevel.obj
 0002:00000fd0       ??_C@_08KNHFBNJ@FlsAlloc@  10031fd0     libvcruntime:winapi_downlevel.obj
 0002:00000fe4       ??_C@_07PEJMOBNF@FlsFree@  10031fe4     libvcruntime:winapi_downlevel.obj
 0002:00000ff4       ??_C@_0M@GDNOONDI@FlsGetValue@ 10031ff4     libvcruntime:winapi_downlevel.obj
 0002:00001008       ??_C@_0M@JCPCPOEF@FlsSetValue@ 10032008     libvcruntime:winapi_downlevel.obj
 0002:0000101c       ??_C@_0BM@HCFOFFN@InitializeCriticalSectionEx@ 1003201c     libvcruntime:winapi_downlevel.obj
 0002:00001038       ?standard_lookup_table_spectre@__crt_stdio_output@@3V?$spectre_mitigated_lookup_table@Ustate_transition_pair@__crt_stdio_output@@$0IA@@1@B 10032038     libucrt:output.obj
 0002:00001438       ??_C@_1O@CEDCILHN@?$AA?$CI?$AAn?$AAu?$AAl?$AAl?$AA?$CJ@ 10032438     libucrt:output.obj
 0002:00001448       ??_C@_06OJHGLDPL@?$CInull?$CJ@ 10032448     libucrt:output.obj
 0002:00001450       ___acrt_exception_action_table 10032450     libucrt:exception_filter.obj
 0002:000014e0       ___acrt_signal_action_table_count 100324e0     libucrt:exception_filter.obj
 0002:000014e4       ___acrt_signal_action_first_fpe_index 100324e4     libucrt:exception_filter.obj
 0002:000014e8       ___acrt_signal_action_fpe_count 100324e8     libucrt:exception_filter.obj
 0002:000014ec       ??_C@_1BI@BGOHAHKC@?$AAm?$AAs?$AAc?$AAo?$AAr?$AAe?$AAe?$AA?4?$AAd?$AAl?$AAl@ 100324ec     libucrt:exit.obj
 0002:00001504       ??_C@_0P@MIGLKIOC@CorExitProcess@ 10032504     libucrt:exit.obj
 0002:00001598       ___lc_time_c               10032598     libucrt:nlsdata.obj
 0002:000016fc       ??_C@_03KOEHGMDN@Sun@      100326fc     libucrt:nlsdata.obj
 0002:00001700       ??_C@_03PDAGKDH@Mon@       10032700     libucrt:nlsdata.obj
 0002:00001704       ??_C@_03NAGEINEP@Tue@      10032704     libucrt:nlsdata.obj
 0002:00001708       ??_C@_03MHOMLAJA@Wed@      10032708     libucrt:nlsdata.obj
 0002:0000170c       ??_C@_03IOFIKPDN@Thu@      1003270c     libucrt:nlsdata.obj
 0002:00001710       ??_C@_03IDIOELNC@Fri@      10032710     libucrt:nlsdata.obj
 0002:00001714       ??_C@_03FEFJNEK@Sat@       10032714     libucrt:nlsdata.obj
 0002:00001718       ??_C@_06OOPIFAJ@Sunday@    10032718     libucrt:nlsdata.obj
 0002:00001720       ??_C@_06JLEDEDGH@Monday@   10032720     libucrt:nlsdata.obj
 0002:00001728       ??_C@_07BAAGCFCM@Tuesday@  10032728     libucrt:nlsdata.obj
 0002:00001730       ??_C@_09DLIGFAKA@Wednesday@ 10032730     libucrt:nlsdata.obj
 0002:0000173c       ??_C@_08HACCIKIA@Thursday@ 1003273c     libucrt:nlsdata.obj
 0002:00001748       ??_C@_06JECMNKMI@Friday@   10032748     libucrt:nlsdata.obj
 0002:00001750       ??_C@_08INBOOONO@Saturday@ 10032750     libucrt:nlsdata.obj
 0002:0000175c       ??_C@_03JIHJHPIE@Jan@      1003275c     libucrt:nlsdata.obj
 0002:00001760       ??_C@_03HJBDCHOM@Feb@      10032760     libucrt:nlsdata.obj
 0002:00001764       ??_C@_03ODNJBKGA@Mar@      10032764     libucrt:nlsdata.obj
 0002:00001768       ??_C@_03LEOLGMJP@Apr@      10032768     libucrt:nlsdata.obj
 0002:0000176c       ??_C@_03CNMDKL@May@        1003276c     libucrt:nlsdata.obj
 0002:00001770       ??_C@_03IDFGHECI@Jun@      10032770     libucrt:nlsdata.obj
 0002:00001774       ??_C@_03LBGABGKK@Jul@      10032774     libucrt:nlsdata.obj
 0002:00001778       ??_C@_03IFJFEIGA@Aug@      10032778     libucrt:nlsdata.obj
 0002:0000177c       ??_C@_03GGCAPAJC@Sep@      1003277c     libucrt:nlsdata.obj
 0002:00001780       ??_C@_03BMAOKBAD@Oct@      10032780     libucrt:nlsdata.obj
 0002:00001784       ??_C@_03JPJOFNIA@Nov@      10032784     libucrt:nlsdata.obj
 0002:00001788       ??_C@_03MKABNOCG@Dec@      10032788     libucrt:nlsdata.obj
 0002:0000178c       ??_C@_07CGJPFGJA@January@  1003278c     libucrt:nlsdata.obj
 0002:00001794       ??_C@_08GNJGEPFN@February@ 10032794     libucrt:nlsdata.obj
 0002:000017a0       ??_C@_05HPCKOFNC@March@    100327a0     libucrt:nlsdata.obj
 0002:000017a8       ??_C@_05DMJDNLEJ@April@    100327a8     libucrt:nlsdata.obj
 0002:000017b0       ??_C@_04CNLMGBGM@June@     100327b0     libucrt:nlsdata.obj
 0002:000017b8       ??_C@_04MIEPOIFP@July@     100327b8     libucrt:nlsdata.obj
 0002:000017c0       ??_C@_06LBBHFDDG@August@   100327c0     libucrt:nlsdata.obj
 0002:000017c8       ??_C@_09BHHEALKD@September@ 100327c8     libucrt:nlsdata.obj
 0002:000017d4       ??_C@_07JJNFCEND@October@  100327d4     libucrt:nlsdata.obj
 0002:000017dc       ??_C@_08HCHEGEOA@November@ 100327dc     libucrt:nlsdata.obj
 0002:000017e8       ??_C@_08EDHMEBNP@December@ 100327e8     libucrt:nlsdata.obj
 0002:000017f4       ??_C@_02DEDBPAFC@AM@       100327f4     libucrt:nlsdata.obj
 0002:000017f8       ??_C@_02CJNFDJBF@PM@       100327f8     libucrt:nlsdata.obj
 0002:000017fc       ??_C@_08BPBNCDIB@MM?1dd?1yy@ 100327fc     libucrt:nlsdata.obj
 0002:00001808       ??_C@_0BE@CKGJFCPC@dddd?0?5MMMM?5dd?0?5yyyy@ 10032808     libucrt:nlsdata.obj
 0002:0000181c       ??_C@_08JCCMCCIL@HH?3mm?3ss@ 1003281c     libucrt:nlsdata.obj
 0002:00001828       ??_C@_17MBGCMIPB@?$AAS?$AAu?$AAn@ 10032828     libucrt:nlsdata.obj
 0002:00001830       ??_C@_17KBOMKBF@?$AAM?$AAo?$AAn@ 10032830     libucrt:nlsdata.obj
 0002:00001838       ??_C@_17BMKGEGOJ@?$AAT?$AAu?$AAe@ 10032838     libucrt:nlsdata.obj
 0002:00001840       ??_C@_17CJEDCEPE@?$AAW?$AAe?$AAd@ 10032840     libucrt:nlsdata.obj
 0002:00001848       ??_C@_17PDPHAADD@?$AAT?$AAh?$AAu@ 10032848     libucrt:nlsdata.obj
 0002:00001850       ??_C@_17HFOLPPLP@?$AAF?$AAr?$AAi@ 10032850     libucrt:nlsdata.obj
 0002:00001858       ??_C@_17GGIBDPIH@?$AAS?$AAa?$AAt@ 10032858     libucrt:nlsdata.obj
 0002:00001860       ??_C@_1O@IHNHDHPB@?$AAS?$AAu?$AAn?$AAd?$AAa?$AAy@ 10032860     libucrt:nlsdata.obj
 0002:00001870       ??_C@_1O@MMNBFLIA@?$AAM?$AAo?$AAn?$AAd?$AAa?$AAy@ 10032870     libucrt:nlsdata.obj
 0002:00001880       ??_C@_1BA@ENFBFFEK@?$AAT?$AAu?$AAe?$AAs?$AAd?$AAa?$AAy@ 10032880     libucrt:nlsdata.obj
 0002:00001890       ??_C@_1BE@EBOGMDOH@?$AAW?$AAe?$AAd?$AAn?$AAe?$AAs?$AAd?$AAa?$AAy@ 10032890     libucrt:nlsdata.obj
 0002:000018a4       ??_C@_1BC@HHMNLIHE@?$AAT?$AAh?$AAu?$AAr?$AAs?$AAd?$AAa?$AAy@ 100328a4     libucrt:nlsdata.obj
 0002:000018b8       ??_C@_1O@PDICJHAG@?$AAF?$AAr?$AAi?$AAd?$AAa?$AAy@ 100328b8     libucrt:nlsdata.obj
 0002:000018c8       ??_C@_1BC@ENMNNPAJ@?$AAS?$AAa?$AAt?$AAu?$AAr?$AAd?$AAa?$AAy@ 100328c8     libucrt:nlsdata.obj
 0002:000018dc       ??_C@_17DKNBKCHM@?$AAJ?$AAa?$AAn@ 100328dc     libucrt:nlsdata.obj
 0002:000018e4       ??_C@_17LMDJEKJN@?$AAF?$AAe?$AAb@ 100328e4     libucrt:nlsdata.obj
 0002:000018ec       ??_C@_17CKNLEDEC@?$AAM?$AAa?$AAr@ 100328ec     libucrt:nlsdata.obj
 0002:000018f4       ??_C@_17LFPOIHDD@?$AAA?$AAp?$AAr@ 100328f4     libucrt:nlsdata.obj
 0002:000018fc       ??_C@_17PNNKMEED@?$AAM?$AAa?$AAy@ 100328fc     libucrt:nlsdata.obj
 0002:00001904       ??_C@_17KCJGOCPB@?$AAJ?$AAu?$AAn@ 10032904     libucrt:nlsdata.obj
 0002:0000190c       ??_C@_17IJPCKHK@?$AAJ?$AAu?$AAl@ 1003290c     libucrt:nlsdata.obj
 0002:00001914       ??_C@_17ICPELBCN@?$AAA?$AAu?$AAg@ 10032914     libucrt:nlsdata.obj
 0002:0000191c       ??_C@_17HCHCOKMG@?$AAS?$AAe?$AAp@ 1003291c     libucrt:nlsdata.obj
 0002:00001924       ??_C@_17FNLKOI@?$AAO?$AAc?$AAt@ 10032924     libucrt:nlsdata.obj
 0002:0000192c       ??_C@_17BBDMLCIG@?$AAN?$AAo?$AAv@ 1003292c     libucrt:nlsdata.obj
 0002:00001934       ??_C@_17EGKACKIF@?$AAD?$AAe?$AAc@ 10032934     libucrt:nlsdata.obj
 0002:0000193c       ??_C@_1BA@EFMEIEBA@?$AAJ?$AAa?$AAn?$AAu?$AAa?$AAr?$AAy@ 1003293c     libucrt:nlsdata.obj
 0002:0000194c       ??_C@_1BC@JGDDFFAM@?$AAF?$AAe?$AAb?$AAr?$AAu?$AAa?$AAr?$AAy@ 1003294c     libucrt:nlsdata.obj
 0002:00001960       ??_C@_1M@IKEENEDF@?$AAM?$AAa?$AAr?$AAc?$AAh@ 10032960     libucrt:nlsdata.obj
 0002:0000196c       ??_C@_1M@GJNLMHFD@?$AAA?$AAp?$AAr?$AAi?$AAl@ 1003296c     libucrt:nlsdata.obj
 0002:00001978       ??_C@_19EPFLPGAP@?$AAJ?$AAu?$AAn?$AAe@ 10032978     libucrt:nlsdata.obj
 0002:00001984       ??_C@_19BIFMLPCD@?$AAJ?$AAu?$AAl?$AAy@ 10032984     libucrt:nlsdata.obj
 0002:00001990       ??_C@_1O@PAHLKOAC@?$AAA?$AAu?$AAg?$AAu?$AAs?$AAt@ 10032990     libucrt:nlsdata.obj
 0002:000019a0       ??_C@_1BE@DKAAMBJL@?$AAS?$AAe?$AAp?$AAt?$AAe?$AAm?$AAb?$AAe?$AAr@ 100329a0     libucrt:nlsdata.obj
 0002:000019b4       ??_C@_1BA@EPANDLNG@?$AAO?$AAc?$AAt?$AAo?$AAb?$AAe?$AAr@ 100329b4     libucrt:nlsdata.obj
 0002:000019c4       ??_C@_1BC@BGLIFPF@?$AAN?$AAo?$AAv?$AAe?$AAm?$AAb?$AAe?$AAr@ 100329c4     libucrt:nlsdata.obj
 0002:000019d8       ??_C@_1BC@FEMKIFH@?$AAD?$AAe?$AAc?$AAe?$AAm?$AAb?$AAe?$AAr@ 100329d8     libucrt:nlsdata.obj
 0002:000019ec       ??_C@_15ODEHAHHF@?$AAA?$AAM@ 100329ec     libucrt:nlsdata.obj
 0002:000019f4       ??_C@_15CLMNNGEL@?$AAP?$AAM@ 100329f4     libucrt:nlsdata.obj
 0002:000019fc       ??_C@_1BC@IEBCMHCM@?$AAM?$AAM?$AA?1?$AAd?$AAd?$AA?1?$AAy?$AAy@ 100329fc     libucrt:nlsdata.obj
 0002:00001a10       ??_C@_1CI@KNAKOEBC@?$AAd?$AAd?$AAd?$AAd?$AA?0?$AA?5?$AAM?$AAM?$AAM?$AAM?$AA?5?$AAd?$AAd?$AA?0?$AA?5@ 10032a10     libucrt:nlsdata.obj
 0002:00001a38       ??_C@_1BC@GDGBMEMK@?$AAH?$AAH?$AA?3?$AAm?$AAm?$AA?3?$AAs?$AAs@ 10032a38     libucrt:nlsdata.obj
 0002:00001a4c       ??_C@_1M@BMHNFIME@?$AAe?$AAn?$AA?9?$AAU?$AAS@ 10032a4c     libucrt:nlsdata.obj
 0002:00001bc0       ?large_power_data@?1??multiply_by_power_of_ten@__crt_strtox@@YA_NAAUbig_integer@2@I@Z@4QBIB 10032bc0     libucrt:cfout.obj
 0002:000024c8       ?large_power_indices@?1??multiply_by_power_of_ten@__crt_strtox@@YA_NAAUbig_integer@2@I@Z@4QBUunpack_index@?1??12@YA_N0I@Z@B 100334c8     libucrt:cfout.obj
 0002:00002560       ?small_powers_of_ten@?1??multiply_by_power_of_ten@__crt_strtox@@YA_NAAUbig_integer@2@I@Z@4QBIB 10033560     libucrt:cfout.obj
 0002:00002584       ??_C@_01GBGANLPD@0@        10033584     libucrt:cfout.obj
 0002:00002588       ??_C@_05DNEBIAHO@1?$CDINF@ 10033588     libucrt:cfout.obj
 0002:00002590       ??_C@_06IMKFLFPG@1?$CDQNAN@ 10033590     libucrt:cfout.obj
 0002:00002598       ??_C@_06PGGFOGJG@1?$CDSNAN@ 10033598     libucrt:cfout.obj
 0002:000025a0       ??_C@_05PHHOCPM@1?$CDIND@  100335a0     libucrt:cfout.obj
 0002:000025a8       ___newctype                100335a8     libucrt:ctype.obj
 0002:000028a8       ___newclmap                100338a8     libucrt:ctype.obj
 0002:00002a28       ___newcumap                10033a28     libucrt:ctype.obj
 0002:00002ba8       __wctype                   10033ba8     libucrt:ctype.obj
 0002:00002df0       ??_C@_03OEIAHPBN@INF@      10033df0     libucrt:cvt.obj
 0002:00002df4       ??_C@_03OJHLLCGB@inf@      10033df4     libucrt:cvt.obj
 0002:00002df8       ??_C@_03LKNCIKJB@NAN@      10033df8     libucrt:cvt.obj
 0002:00002dfc       ??_C@_03LHCJEHON@nan@      10033dfc     libucrt:cvt.obj
 0002:00002e00       ??_C@_09OFJJIMPC@NAN?$CISNAN?$CJ@ 10033e00     libucrt:cvt.obj
 0002:00002e0c       ??_C@_09IPFBKMDL@nan?$CIsnan?$CJ@ 10033e0c     libucrt:cvt.obj
 0002:00002e18       ??_C@_08IKHNHAJ@NAN?$CIIND?$CJ@ 10033e18     libucrt:cvt.obj
 0002:00002e24       ??_C@_08OFCDMILK@nan?$CIind?$CJ@ 10033e24     libucrt:cvt.obj
 0002:00002e30       ??_C@_05KLBDPFGC@e?$CL000@ 10033e30     libucrt:cvt.obj
 0002:00002e88       ??_C@_1EA@JGEFHKEI@?$AAa?$AAp?$AAi?$AA?9?$AAm?$AAs?$AA?9?$AAw?$AAi?$AAn?$AA?9?$AAc?$AAo?$AAr?$AAe@ 10033e88     libucrt:winapi_thunks.obj
 0002:00002ec8       ??_C@_1DI@IJCEHOCB@?$AAa?$AAp?$AAi?$AA?9?$AAm?$AAs?$AA?9?$AAw?$AAi?$AAn?$AA?9?$AAc?$AAo?$AAr?$AAe@ 10033ec8     libucrt:winapi_thunks.obj
 0002:00002f00       ??_C@_1EI@MPIAOHOC@?$AAa?$AAp?$AAi?$AA?9?$AAm?$AAs?$AA?9?$AAw?$AAi?$AAn?$AA?9?$AAc?$AAo?$AAr?$AAe@ 10033f00     libucrt:winapi_thunks.obj
 0002:00002f48       ??_C@_1FK@FPHCKFIE@?$AAa?$AAp?$AAi?$AA?9?$AAm?$AAs?$AA?9?$AAw?$AAi?$AAn?$AA?9?$AAc?$AAo?$AAr?$AAe@ 10033f48     libucrt:winapi_thunks.obj
 0002:00002fa8       ??_C@_1EM@DILCGIIO@?$AAa?$AAp?$AAi?$AA?9?$AAm?$AAs?$AA?9?$AAw?$AAi?$AAn?$AA?9?$AAc?$AAo?$AAr?$AAe@ 10033fa8     libucrt:winapi_thunks.obj
 0002:00002ff4       ??_C@_1DM@LNCGDDPN@?$AAa?$AAp?$AAi?$AA?9?$AAm?$AAs?$AA?9?$AAw?$AAi?$AAn?$AA?9?$AAc?$AAo?$AAr?$AAe@ 10033ff4     libucrt:winapi_thunks.obj
 0002:00003030       ??_C@_1DO@FPAPJEMD@?$AAa?$AAp?$AAi?$AA?9?$AAm?$AAs?$AA?9?$AAw?$AAi?$AAn?$AA?9?$AAc?$AAo?$AAr?$AAe@ 10034030     libucrt:winapi_thunks.obj
 0002:00003070       ??_C@_1DK@NDHNAHIO@?$AAa?$AAp?$AAi?$AA?9?$AAm?$AAs?$AA?9?$AAw?$AAi?$AAn?$AA?9?$AAc?$AAo?$AAr?$AAe@ 10034070     libucrt:winapi_thunks.obj
 0002:000030ac       ??_C@_1DM@KGHDGBCM@?$AAa?$AAp?$AAi?$AA?9?$AAm?$AAs?$AA?9?$AAw?$AAi?$AAn?$AA?9?$AAc?$AAo?$AAr?$AAe@ 100340ac     libucrt:winapi_thunks.obj
 0002:000030e8       ??_C@_1EO@IJIOEFOH@?$AAa?$AAp?$AAi?$AA?9?$AAm?$AAs?$AA?9?$AAw?$AAi?$AAn?$AA?9?$AAr?$AAt?$AAc?$AAo@ 100340e8     libucrt:winapi_thunks.obj
 0002:00003138       ??_C@_1FG@HHGEKANL@?$AAa?$AAp?$AAi?$AA?9?$AAm?$AAs?$AA?9?$AAw?$AAi?$AAn?$AA?9?$AAs?$AAe?$AAc?$AAu@ 10034138     libucrt:winapi_thunks.obj
 0002:00003190       ??_C@_1EG@DBIOJECG@?$AAe?$AAx?$AAt?$AA?9?$AAm?$AAs?$AA?9?$AAw?$AAi?$AAn?$AA?9?$AAn?$AAt?$AAu?$AAs@ 10034190     libucrt:winapi_thunks.obj
 0002:000031d8       ??_C@_1EO@FIHMJCLF@?$AAe?$AAx?$AAt?$AA?9?$AAm?$AAs?$AA?9?$AAw?$AAi?$AAn?$AA?9?$AAn?$AAt?$AAu?$AAs@ 100341d8     libucrt:winapi_thunks.obj
 0002:00003228       ??_C@_1BC@DNHGCMLG@?$AAa?$AAd?$AAv?$AAa?$AAp?$AAi?$AA3?$AA2@ 10034228     libucrt:winapi_thunks.obj
 0002:0000323c       ??_C@_1M@OAIMIKLP@?$AAn?$AAt?$AAd?$AAl?$AAl@ 1003423c     libucrt:winapi_thunks.obj
 0002:00003248       ??_C@_1EG@DPGNFKGC@?$AAa?$AAp?$AAi?$AA?9?$AAm?$AAs?$AA?9?$AAw?$AAi?$AAn?$AA?9?$AAa?$AAp?$AAp?$AAm@ 10034248     libucrt:winapi_thunks.obj
 0002:00003290       ??_C@_1O@BCCLBEOE@?$AAu?$AAs?$AAe?$AAr?$AA3?$AA2@ 10034290     libucrt:winapi_thunks.obj
 0002:000032a0       ??_C@_1BA@IAIFMGEF@?$AAe?$AAx?$AAt?$AA?9?$AAm?$AAs?$AA?9@ 100342a0     libucrt:winapi_thunks.obj
 0002:000032b4       ??_C@_0BA@FHFNEAED@AreFileApisANSI@ 100342b4     libucrt:winapi_thunks.obj
 0002:000032f4       ??_C@_0O@KKBNKAPF@LCMapStringEx@ 100342f4     libucrt:winapi_thunks.obj
 0002:0000330c       ??_C@_0BB@HBDEELFH@LocaleNameToLCID@ 1003430c     libucrt:winapi_thunks.obj
 0002:00003324       ??_C@_0CF@OJOFEIGO@AppPolicyGetProcessTerminationM@ 10034324     libucrt:winapi_thunks.obj
 0002:0000335c       ??_C@_1M@HPNHIDJI@?$AAj?$AAa?$AA?9?$AAJ?$AAP@ 1003435c     libucrt:mbctype.obj
 0002:00003368       ??_C@_1M@BIBDDEMK@?$AAz?$AAh?$AA?9?$AAC?$AAN@ 10034368     libucrt:mbctype.obj
 0002:00003374       ??_C@_1M@JLOOOEGK@?$AAk?$AAo?$AA?9?$AAK?$AAR@ 10034374     libucrt:mbctype.obj
 0002:00003380       ??_C@_1M@CLNBBOPM@?$AAz?$AAh?$AA?9?$AAT?$AAW@ 10034380     libucrt:mbctype.obj
 0002:0000338c       ??_C@_15PJPFLCCM@?$AAu?$AAk@ 1003438c     libucrt:get_qualified_locale.obj
 0002:00003b18       ??_C@_15EMKDOKLE@?$AAa?$AAr@ 10034b18     libucrt:lcidtoname_downlevel.obj
 0002:00003b20       ??_C@_15KNPADPLH@?$AAb?$AAg@ 10034b20     libucrt:lcidtoname_downlevel.obj
 0002:00003b28       ??_C@_15EDMHLDMO@?$AAc?$AAa@ 10034b28     libucrt:lcidtoname_downlevel.obj
 0002:00003b30       ??_C@_1O@BPEAJADD@?$AAz?$AAh?$AA?9?$AAC?$AAH?$AAS@ 10034b30     libucrt:lcidtoname_downlevel.obj
 0002:00003b40       ??_C@_15LJNHCMNK@?$AAc?$AAs@ 10034b40     libucrt:lcidtoname_downlevel.obj
 0002:00003b48       ??_C@_15FOMCIDHG@?$AAd?$AAa@ 10034b48     libucrt:lcidtoname_downlevel.obj
 0002:00003b50       ??_C@_15NBKABECB@?$AAd?$AAe@ 10034b50     libucrt:lcidtoname_downlevel.obj
 0002:00003b58       ??_C@_15GHPEIIAO@?$AAe?$AAl@ 10034b58     libucrt:lcidtoname_downlevel.obj
 0002:00003b60       ??_C@_15MNPNEAIF@?$AAe?$AAn@ 10034b60     libucrt:lcidtoname_downlevel.obj
 0002:00003b68       ??_C@_15GPIOMPMH@?$AAe?$AAs@ 10034b68     libucrt:lcidtoname_downlevel.obj
 0002:00003b70       ??_C@_15NGLOAKJC@?$AAf?$AAi@ 10034b70     libucrt:lcidtoname_downlevel.obj
 0002:00003b78       ??_C@_15FBKGNKAM@?$AAf?$AAr@ 10034b78     libucrt:lcidtoname_downlevel.obj
 0002:00003b80       ??_C@_15KGGCNEFK@?$AAh?$AAe@ 10034b80     libucrt:lcidtoname_downlevel.obj
 0002:00003b88       ??_C@_15PGHLIDMF@?$AAh?$AAu@ 10034b88     libucrt:lcidtoname_downlevel.obj
 0002:00003b90       ??_C@_15BIEMAPLM@?$AAi?$AAs@ 10034b90     libucrt:lcidtoname_downlevel.obj
 0002:00003b98       ??_C@_15IFJLDHAF@?$AAi?$AAt@ 10034b98     libucrt:lcidtoname_downlevel.obj
 0002:00003ba0       ??_C@_15GEMIOCAG@?$AAj?$AAa@ 10034ba0     libucrt:lcidtoname_downlevel.obj
 0002:00003ba8       ??_C@_15EPELEGJA@?$AAk?$AAo@ 10034ba8     libucrt:lcidtoname_downlevel.obj
 0002:00003bb0       ??_C@_15NDDHIMN@?$AAn?$AAl@ 10034bb0     libucrt:lcidtoname_downlevel.obj
 0002:00003bb8       ??_C@_15BPIGNHCD@?$AAn?$AAo@ 10034bb8     libucrt:lcidtoname_downlevel.obj
 0002:00003bc0       ??_C@_15DEOPBLCG@?$AAp?$AAl@ 10034bc0     libucrt:lcidtoname_downlevel.obj
 0002:00003bc8       ??_C@_15KBECGEFG@?$AAp?$AAt@ 10034bc8     libucrt:lcidtoname_downlevel.obj
 0002:00003bd0       ??_C@_15GLJCBFMD@?$AAr?$AAo@ 10034bd0     libucrt:lcidtoname_downlevel.obj
 0002:00003bd8       ??_C@_15FEDGKCDI@?$AAr?$AAu@ 10034bd8     libucrt:lcidtoname_downlevel.obj
 0002:00003be0       ??_C@_15GLKMLLHM@?$AAh?$AAr@ 10034be0     libucrt:lcidtoname_downlevel.obj
 0002:00003be8       ??_C@_15CPKMFBDB@?$AAs?$AAk@ 10034be8     libucrt:lcidtoname_downlevel.obj
 0002:00003bf0       ??_C@_15BAAIOGMK@?$AAs?$AAq@ 10034bf0     libucrt:lcidtoname_downlevel.obj
 0002:00003bf8       ??_C@_15INNPNOHD@?$AAs?$AAv@ 10034bf8     libucrt:lcidtoname_downlevel.obj
 0002:00003c00       ??_C@_15CABMMOGH@?$AAt?$AAh@ 10034c00     libucrt:lcidtoname_downlevel.obj
 0002:00003c08       ??_C@_15BPLIHJJM@?$AAt?$AAr@ 10034c08     libucrt:lcidtoname_downlevel.obj
 0002:00003c10       ??_C@_15NEOEKKDJ@?$AAu?$AAr@ 10034c10     libucrt:lcidtoname_downlevel.obj
 0002:00003c18       ??_C@_15NFICGAJK@?$AAi?$AAd@ 10034c18     libucrt:lcidtoname_downlevel.obj
 0002:00003c20       ??_C@_15HPJPHDM@?$AAb?$AAe@ 10034c20     libucrt:lcidtoname_downlevel.obj
 0002:00003c28       ??_C@_15LCHLGJII@?$AAs?$AAl@ 10034c28     libucrt:lcidtoname_downlevel.obj
 0002:00003c30       ??_C@_15PCFJPHHO@?$AAe?$AAt@ 10034c30     libucrt:lcidtoname_downlevel.obj
 0002:00003c38       ??_C@_15HPFPGODN@?$AAl?$AAv@ 10034c38     libucrt:lcidtoname_downlevel.obj
 0002:00003c40       ??_C@_15NFFGKGLG@?$AAl?$AAt@ 10034c40     libucrt:lcidtoname_downlevel.obj
 0002:00003c48       ??_C@_15BDAKCCHN@?$AAf?$AAa@ 10034c48     libucrt:lcidtoname_downlevel.obj
 0002:00003c50       ??_C@_15NFGIAIAJ@?$AAv?$AAi@ 10034c50     libucrt:lcidtoname_downlevel.obj
 0002:00003c58       ??_C@_15LMKNDMHN@?$AAh?$AAy@ 10034c58     libucrt:lcidtoname_downlevel.obj
 0002:00003c60       ??_C@_15IJBHMCFL@?$AAa?$AAz@ 10034c60     libucrt:lcidtoname_downlevel.obj
 0002:00003c68       ??_C@_15EKOFJABL@?$AAe?$AAu@ 10034c68     libucrt:lcidtoname_downlevel.obj
 0002:00003c70       ??_C@_15BGHADCNK@?$AAm?$AAk@ 10034c70     libucrt:lcidtoname_downlevel.obj
 0002:00003c78       ??_C@_15JDNICKHM@?$AAa?$AAf@ 10034c78     libucrt:lcidtoname_downlevel.obj
 0002:00003c80       ??_C@_15KPJEDBKD@?$AAk?$AAa@ 10034c80     libucrt:lcidtoname_downlevel.obj
 0002:00003c88       ??_C@_15PDNFFFEO@?$AAf?$AAo@ 10034c88     libucrt:lcidtoname_downlevel.obj
 0002:00003c90       ??_C@_15OMLEGLOC@?$AAh?$AAi@ 10034c90     libucrt:lcidtoname_downlevel.obj
 0002:00003c98       ??_C@_15IDNNENKK@?$AAm?$AAs@ 10034c98     libucrt:lcidtoname_downlevel.obj
 0002:00003ca0       ??_C@_15MACJNBMH@?$AAk?$AAk@ 10034ca0     libucrt:lcidtoname_downlevel.obj
 0002:00003ca8       ??_C@_15DKDJEOND@?$AAk?$AAy@ 10034ca8     libucrt:lcidtoname_downlevel.obj
 0002:00003cb0       ??_C@_15DFGDLJBG@?$AAs?$AAw@ 10034cb0     libucrt:lcidtoname_downlevel.obj
 0002:00003cb8       ??_C@_15BBFAICNG@?$AAu?$AAz@ 10034cb8     libucrt:lcidtoname_downlevel.obj
 0002:00003cc0       ??_C@_15DKNDCGEA@?$AAt?$AAt@ 10034cc0     libucrt:lcidtoname_downlevel.obj
 0002:00003cc8       ??_C@_15MGIFMDPL@?$AAp?$AAa@ 10034cc8     libucrt:lcidtoname_downlevel.obj
 0002:00003cd0       ??_C@_15HCNDBBA@?$AAg?$AAu@ 10034cd0     libucrt:lcidtoname_downlevel.obj
 0002:00003cd8       ??_C@_15FNBEIBON@?$AAt?$AAa@ 10034cd8     libucrt:lcidtoname_downlevel.obj
 0002:00003ce0       ??_C@_15NCHGBGLK@?$AAt?$AAe@ 10034ce0     libucrt:lcidtoname_downlevel.obj
 0002:00003ce8       ??_C@_15PHPHCBPF@?$AAk?$AAn@ 10034ce8     libucrt:lcidtoname_downlevel.obj
 0002:00003cf0       ??_C@_15DLGBCKMP@?$AAm?$AAr@ 10034cf0     libucrt:lcidtoname_downlevel.obj
 0002:00003cf8       ??_C@_15EABBLBFF@?$AAs?$AAa@ 10034cf8     libucrt:lcidtoname_downlevel.obj
 0002:00003d00       ??_C@_15CBKOMCOI@?$AAm?$AAn@ 10034d00     libucrt:lcidtoname_downlevel.obj
 0002:00003d08       ??_C@_15CKDMCJAF@?$AAg?$AAl@ 10034d08     libucrt:lcidtoname_downlevel.obj
 0002:00003d10       ??_C@_17CNJFBPG@?$AAk?$AAo?$AAk@ 10034d10     libucrt:lcidtoname_downlevel.obj
 0002:00003d18       ??_C@_17FFBJICPL@?$AAs?$AAy?$AAr@ 10034d18     libucrt:lcidtoname_downlevel.obj
 0002:00003d20       ??_C@_17KPNDCPAF@?$AAd?$AAi?$AAv@ 10034d20     libucrt:lcidtoname_downlevel.obj
 0002:00003d28       ??_C@_11LOCGONAA@@         10034d28     libucrt:lcidtoname_downlevel.obj
 0002:00003d2c       ??_C@_1M@OKAHONE@?$AAa?$AAr?$AA?9?$AAS?$AAA@ 10034d2c     libucrt:lcidtoname_downlevel.obj
 0002:00003d38       ??_C@_1M@FFFIGIGK@?$AAb?$AAg?$AA?9?$AAB?$AAG@ 10034d38     libucrt:lcidtoname_downlevel.obj
 0002:00003d44       ??_C@_1M@BJNKEDC@?$AAc?$AAa?$AA?9?$AAE?$AAS@ 10034d44     libucrt:lcidtoname_downlevel.obj
 0002:00003d50       ??_C@_1M@IJJHFJHA@?$AAc?$AAs?$AA?9?$AAC?$AAZ@ 10034d50     libucrt:lcidtoname_downlevel.obj
 0002:00003d5c       ??_C@_1M@CLPEOBGI@?$AAd?$AAa?$AA?9?$AAD?$AAK@ 10034d5c     libucrt:lcidtoname_downlevel.obj
 0002:00003d68       ??_C@_1M@MCMADGCB@?$AAd?$AAe?$AA?9?$AAD?$AAE@ 10034d68     libucrt:lcidtoname_downlevel.obj
 0002:00003d74       ??_C@_1M@OOCKEMAM@?$AAe?$AAl?$AA?9?$AAG?$AAR@ 10034d74     libucrt:lcidtoname_downlevel.obj
 0002:00003d80       ??_C@_1M@DDNJFGID@?$AAf?$AAi?$AA?9?$AAF?$AAI@ 10034d80     libucrt:lcidtoname_downlevel.obj
 0002:00003d8c       ??_C@_1M@GLIPPMAC@?$AAf?$AAr?$AA?9?$AAF?$AAR@ 10034d8c     libucrt:lcidtoname_downlevel.obj
 0002:00003d98       ??_C@_1M@GFMCHPE@?$AAh?$AAe?$AA?9?$AAI?$AAL@ 10034d98     libucrt:lcidtoname_downlevel.obj
 0002:00003da4       ??_C@_1M@MHLPGNKM@?$AAh?$AAu?$AA?9?$AAH?$AAU@ 10034da4     libucrt:lcidtoname_downlevel.obj
 0002:00003db0       ??_C@_1M@LPDDNNPN@?$AAi?$AAs?$AA?9?$AAI?$AAS@ 10034db0     libucrt:lcidtoname_downlevel.obj
 0002:00003dbc       ??_C@_1M@MADIPODN@?$AAi?$AAt?$AA?9?$AAI?$AAT@ 10034dbc     libucrt:lcidtoname_downlevel.obj
 0002:00003dc8       ??_C@_1M@IHBJJGG@?$AAn?$AAl?$AA?9?$AAN?$AAL@ 10034dc8     libucrt:lcidtoname_downlevel.obj
 0002:00003dd4       ??_C@_1M@EANAGDL@?$AAn?$AAb?$AA?9?$AAN?$AAO@ 10034dd4     libucrt:lcidtoname_downlevel.obj
 0002:00003de0       ??_C@_1M@NEIEMEGP@?$AAp?$AAl?$AA?9?$AAP?$AAL@ 10034de0     libucrt:lcidtoname_downlevel.obj
 0002:00003dec       ??_C@_1M@BOCFIGEP@?$AAp?$AAt?$AA?9?$AAB?$AAR@ 10034dec     libucrt:lcidtoname_downlevel.obj
 0002:00003df8       ??_C@_1M@IMPFOPBG@?$AAr?$AAo?$AA?9?$AAR?$AAO@ 10034df8     libucrt:lcidtoname_downlevel.obj
 0002:00003e04       ??_C@_1M@IDNNEJMM@?$AAr?$AAu?$AA?9?$AAR?$AAU@ 10034e04     libucrt:lcidtoname_downlevel.obj
 0002:00003e10       ??_C@_1M@LILEEOGM@?$AAh?$AAr?$AA?9?$AAH?$AAR@ 10034e10     libucrt:lcidtoname_downlevel.obj
 0002:00003e1c       ??_C@_1M@FKIFEHPB@?$AAs?$AAk?$AA?9?$AAS?$AAK@ 10034e1c     libucrt:lcidtoname_downlevel.obj
 0002:00003e28       ??_C@_1M@LJMAMNPJ@?$AAs?$AAq?$AA?9?$AAA?$AAL@ 10034e28     libucrt:lcidtoname_downlevel.obj
 0002:00003e34       ??_C@_1M@GIAKDKJK@?$AAs?$AAv?$AA?9?$AAS?$AAE@ 10034e34     libucrt:lcidtoname_downlevel.obj
 0002:00003e40       ??_C@_1M@MKJKIKCL@?$AAt?$AAh?$AA?9?$AAT?$AAH@ 10034e40     libucrt:lcidtoname_downlevel.obj
 0002:00003e4c       ??_C@_1M@MFLCCMPB@?$AAt?$AAr?$AA?9?$AAT?$AAR@ 10034e4c     libucrt:lcidtoname_downlevel.obj
 0002:00003e58       ??_C@_1M@OIJHDKJN@?$AAu?$AAr?$AA?9?$AAP?$AAK@ 10034e58     libucrt:lcidtoname_downlevel.obj
 0002:00003e64       ??_C@_1M@LHIPCIEK@?$AAi?$AAd?$AA?9?$AAI?$AAD@ 10034e64     libucrt:lcidtoname_downlevel.obj
 0002:00003e70       ??_C@_1M@MFMOBGI@?$AAu?$AAk?$AA?9?$AAU?$AAA@ 10034e70     libucrt:lcidtoname_downlevel.obj
 0002:00003e7c       ??_C@_1M@OBGLJIPL@?$AAb?$AAe?$AA?9?$AAB?$AAY@ 10034e7c     libucrt:lcidtoname_downlevel.obj
 0002:00003e88       ??_C@_1M@BCFAJEAD@?$AAs?$AAl?$AA?9?$AAS?$AAI@ 10034e88     libucrt:lcidtoname_downlevel.obj
 0002:00003e94       ??_C@_1M@FKFFEDDN@?$AAe?$AAt?$AA?9?$AAE?$AAE@ 10034e94     libucrt:lcidtoname_downlevel.obj
 0002:00003ea0       ??_C@_1M@KGKKAACI@?$AAl?$AAv?$AA?9?$AAL?$AAV@ 10034ea0     libucrt:lcidtoname_downlevel.obj
 0002:00003eac       ??_C@_1M@IFGBIJO@?$AAl?$AAt?$AA?9?$AAL?$AAT@ 10034eac     libucrt:lcidtoname_downlevel.obj
 0002:00003eb8       ??_C@_1M@FGEAHEDM@?$AAf?$AAa?$AA?9?$AAI?$AAR@ 10034eb8     libucrt:lcidtoname_downlevel.obj
 0002:00003ec4       ??_C@_1M@KBMAIBFN@?$AAv?$AAi?$AA?9?$AAV?$AAN@ 10034ec4     libucrt:lcidtoname_downlevel.obj
 0002:00003ed0       ??_C@_1M@GPCBKDJK@?$AAh?$AAy?$AA?9?$AAA?$AAM@ 10034ed0     libucrt:lcidtoname_downlevel.obj
 0002:00003edc       ??_C@_1BG@BECMDDJB@?$AAa?$AAz?$AA?9?$AAA?$AAZ?$AA?9?$AAL?$AAa?$AAt?$AAn@ 10034edc     libucrt:lcidtoname_downlevel.obj
 0002:00003ef4       ??_C@_1M@MAOFCAEA@?$AAe?$AAu?$AA?9?$AAE?$AAS@ 10034ef4     libucrt:lcidtoname_downlevel.obj
 0002:00003f00       ??_C@_1M@IGHABKPI@?$AAm?$AAk?$AA?9?$AAM?$AAK@ 10034f00     libucrt:lcidtoname_downlevel.obj
 0002:00003f0c       ??_C@_1M@IAIGNEJG@?$AAt?$AAn?$AA?9?$AAZ?$AAA@ 10034f0c     libucrt:lcidtoname_downlevel.obj
 0002:00003f18       ??_C@_1M@IIJCOJFA@?$AAx?$AAh?$AA?9?$AAZ?$AAA@ 10034f18     libucrt:lcidtoname_downlevel.obj
 0002:00003f24       ??_C@_1M@LGPJHNJH@?$AAz?$AAu?$AA?9?$AAZ?$AAA@ 10034f24     libucrt:lcidtoname_downlevel.obj
 0002:00003f30       ??_C@_1M@HOKAOIO@?$AAa?$AAf?$AA?9?$AAZ?$AAA@ 10034f30     libucrt:lcidtoname_downlevel.obj
 0002:00003f3c       ??_C@_1M@DPCLHLIE@?$AAk?$AAa?$AA?9?$AAG?$AAE@ 10034f3c     libucrt:lcidtoname_downlevel.obj
 0002:00003f48       ??_C@_1M@BLKMHJBI@?$AAf?$AAo?$AA?9?$AAF?$AAO@ 10034f48     libucrt:lcidtoname_downlevel.obj
 0002:00003f54       ??_C@_1M@LGGJAPPB@?$AAh?$AAi?$AA?9?$AAI?$AAN@ 10034f54     libucrt:lcidtoname_downlevel.obj
 0002:00003f60       ??_C@_1M@FIKPIHFE@?$AAm?$AAt?$AA?9?$AAM?$AAT@ 10034f60     libucrt:lcidtoname_downlevel.obj
 0002:00003f6c       ??_C@_1M@HEGGPBFA@?$AAs?$AAe?$AA?9?$AAN?$AAO@ 10034f6c     libucrt:lcidtoname_downlevel.obj
 0002:00003f78       ??_C@_1M@EIBJEEPA@?$AAm?$AAs?$AA?9?$AAM?$AAY@ 10034f78     libucrt:lcidtoname_downlevel.obj
 0002:00003f84       ??_C@_1M@FHLBGMPP@?$AAk?$AAk?$AA?9?$AAK?$AAZ@ 10034f84     libucrt:lcidtoname_downlevel.obj
 0002:00003f90       ??_C@_1M@NGJJLCGI@?$AAk?$AAy?$AA?9?$AAK?$AAG@ 10034f90     libucrt:lcidtoname_downlevel.obj
 0002:00003f9c       ??_C@_1M@GIENNBFC@?$AAs?$AAw?$AA?9?$AAK?$AAE@ 10034f9c     libucrt:lcidtoname_downlevel.obj
 0002:00003fa8       ??_C@_1BG@NDGMJIMJ@?$AAu?$AAz?$AA?9?$AAU?$AAZ?$AA?9?$AAL?$AAa?$AAt?$AAn@ 10034fa8     libucrt:lcidtoname_downlevel.obj
 0002:00003fc0       ??_C@_1M@IDCCIHBC@?$AAt?$AAt?$AA?9?$AAR?$AAU@ 10034fc0     libucrt:lcidtoname_downlevel.obj
 0002:00003fcc       ??_C@_1M@LOICPMOJ@?$AAb?$AAn?$AA?9?$AAI?$AAN@ 10034fcc     libucrt:lcidtoname_downlevel.obj
 0002:00003fd8       ??_C@_1M@KPKKNEAH@?$AAp?$AAa?$AA?9?$AAI?$AAN@ 10034fd8     libucrt:lcidtoname_downlevel.obj
 0002:00003fe4       ??_C@_1M@PJGPPBOG@?$AAg?$AAu?$AA?9?$AAI?$AAN@ 10034fe4     libucrt:lcidtoname_downlevel.obj
 0002:00003ff0       ??_C@_1M@KMKMOPHI@?$AAt?$AAa?$AA?9?$AAI?$AAN@ 10034ff0     libucrt:lcidtoname_downlevel.obj
 0002:00003ffc       ??_C@_1M@KFEHEPAC@?$AAt?$AAe?$AA?9?$AAI?$AAN@ 10034ffc     libucrt:lcidtoname_downlevel.obj
 0002:00004008       ??_C@_1M@CDCLMGHI@?$AAk?$AAn?$AA?9?$AAI?$AAN@ 10035008     libucrt:lcidtoname_downlevel.obj
 0002:00004014       ??_C@_1M@MIODLDKF@?$AAm?$AAl?$AA?9?$AAI?$AAN@ 10035014     libucrt:lcidtoname_downlevel.obj
 0002:00004020       ??_C@_1M@PBIEACPO@?$AAm?$AAr?$AA?9?$AAI?$AAN@ 10035020     libucrt:lcidtoname_downlevel.obj
 0002:0000402c       ??_C@_1M@NIDEAGPH@?$AAs?$AAa?$AA?9?$AAI?$AAN@ 1003502c     libucrt:lcidtoname_downlevel.obj
 0002:00004038       ??_C@_1M@FHIHCBIO@?$AAm?$AAn?$AA?9?$AAM?$AAN@ 10035038     libucrt:lcidtoname_downlevel.obj
 0002:00004044       ??_C@_1M@JAIJPENP@?$AAc?$AAy?$AA?9?$AAG?$AAB@ 10035044     libucrt:lcidtoname_downlevel.obj
 0002:00004050       ??_C@_1M@PHGFBEPN@?$AAg?$AAl?$AA?9?$AAE?$AAS@ 10035050     libucrt:lcidtoname_downlevel.obj
 0002:0000405c       ??_C@_1O@KPIPDNCP@?$AAk?$AAo?$AAk?$AA?9?$AAI?$AAN@ 1003505c     libucrt:lcidtoname_downlevel.obj
 0002:0000406c       ??_C@_1O@KNHJLDJA@?$AAs?$AAy?$AAr?$AA?9?$AAS?$AAY@ 1003506c     libucrt:lcidtoname_downlevel.obj
 0002:0000407c       ??_C@_1O@MKEKBLAH@?$AAd?$AAi?$AAv?$AA?9?$AAM?$AAV@ 1003507c     libucrt:lcidtoname_downlevel.obj
 0002:0000408c       ??_C@_1O@OHDCKDDF@?$AAq?$AAu?$AAz?$AA?9?$AAB?$AAO@ 1003508c     libucrt:lcidtoname_downlevel.obj
 0002:0000409c       ??_C@_1M@LEPJNLFD@?$AAn?$AAs?$AA?9?$AAZ?$AAA@ 1003509c     libucrt:lcidtoname_downlevel.obj
 0002:000040a8       ??_C@_1M@OMLEIIJB@?$AAm?$AAi?$AA?9?$AAN?$AAZ@ 100350a8     libucrt:lcidtoname_downlevel.obj
 0002:000040b4       ??_C@_1M@PMPEAILG@?$AAa?$AAr?$AA?9?$AAI?$AAQ@ 100350b4     libucrt:lcidtoname_downlevel.obj
 0002:000040c0       ??_C@_1M@CNKPNOEE@?$AAd?$AAe?$AA?9?$AAC?$AAH@ 100350c0     libucrt:lcidtoname_downlevel.obj
 0002:000040cc       ??_C@_1M@LKMGMLKO@?$AAe?$AAn?$AA?9?$AAG?$AAB@ 100350cc     libucrt:lcidtoname_downlevel.obj
 0002:000040d8       ??_C@_1M@PGKJFFGL@?$AAe?$AAs?$AA?9?$AAM?$AAX@ 100350d8     libucrt:lcidtoname_downlevel.obj
 0002:000040e4       ??_C@_1M@DNNANBDC@?$AAf?$AAr?$AA?9?$AAB?$AAE@ 100350e4     libucrt:lcidtoname_downlevel.obj
 0002:000040f0       ??_C@_1M@HLGMDFHM@?$AAi?$AAt?$AA?9?$AAC?$AAH@ 100350f0     libucrt:lcidtoname_downlevel.obj
 0002:000040fc       ??_C@_1M@CLLBGJH@?$AAn?$AAl?$AA?9?$AAB?$AAE@ 100350fc     libucrt:lcidtoname_downlevel.obj
 0002:00004108       ??_C@_1M@BODBOGLF@?$AAn?$AAn?$AA?9?$AAN?$AAO@ 10035108     libucrt:lcidtoname_downlevel.obj
 0002:00004114       ??_C@_1M@HFFAHKAD@?$AAp?$AAt?$AA?9?$AAP?$AAT@ 10035114     libucrt:lcidtoname_downlevel.obj
 0002:00004120       ??_C@_1BG@LNOAKHIE@?$AAs?$AAr?$AA?9?$AAS?$AAP?$AA?9?$AAL?$AAa?$AAt?$AAn@ 10035120     libucrt:lcidtoname_downlevel.obj
 0002:00004138       ??_C@_1M@HBMHBGAK@?$AAs?$AAv?$AA?9?$AAF?$AAI@ 10035138     libucrt:lcidtoname_downlevel.obj
 0002:00004144       ??_C@_1BG@DGCJGJBE@?$AAa?$AAz?$AA?9?$AAA?$AAZ?$AA?9?$AAC?$AAy?$AAr?$AAl@ 10035144     libucrt:lcidtoname_downlevel.obj
 0002:0000415c       ??_C@_1M@KEJDAAHB@?$AAs?$AAe?$AA?9?$AAS?$AAE@ 1003515c     libucrt:lcidtoname_downlevel.obj
 0002:00004168       ??_C@_1M@HEIBJJAD@?$AAm?$AAs?$AA?9?$AAB?$AAN@ 10035168     libucrt:lcidtoname_downlevel.obj
 0002:00004174       ??_C@_1BG@PBGJMCEM@?$AAu?$AAz?$AA?9?$AAU?$AAZ?$AA?9?$AAC?$AAy?$AAr?$AAl@ 10035174     libucrt:lcidtoname_downlevel.obj
 0002:0000418c       ??_C@_1O@LAOBCMDF@?$AAq?$AAu?$AAz?$AA?9?$AAE?$AAC@ 1003518c     libucrt:lcidtoname_downlevel.obj
 0002:0000419c       ??_C@_1M@POEEMAIO@?$AAa?$AAr?$AA?9?$AAE?$AAG@ 1003519c     libucrt:lcidtoname_downlevel.obj
 0002:000041a8       ??_C@_1M@EFAKDEDL@?$AAz?$AAh?$AA?9?$AAH?$AAK@ 100351a8     libucrt:lcidtoname_downlevel.obj
 0002:000041b4       ??_C@_1M@HKKIJHGI@?$AAd?$AAe?$AA?9?$AAA?$AAT@ 100351b4     libucrt:lcidtoname_downlevel.obj
 0002:000041c0       ??_C@_1M@KBFBEHJF@?$AAe?$AAn?$AA?9?$AAA?$AAU@ 100351c0     libucrt:lcidtoname_downlevel.obj
 0002:000041cc       ??_C@_1M@MNPLFAAH@?$AAe?$AAs?$AA?9?$AAE?$AAS@ 100351cc     libucrt:lcidtoname_downlevel.obj
 0002:000041d8       ??_C@_1M@HJOOJFMA@?$AAf?$AAr?$AA?9?$AAC?$AAA@ 100351d8     libucrt:lcidtoname_downlevel.obj
 0002:000041e4       ??_C@_1BG@JPOFPNAB@?$AAs?$AAr?$AA?9?$AAS?$AAP?$AA?9?$AAC?$AAy?$AAr?$AAl@ 100351e4     libucrt:lcidtoname_downlevel.obj
 0002:000041fc       ??_C@_1M@LNFOCMOB@?$AAs?$AAe?$AA?9?$AAF?$AAI@ 100351fc     libucrt:lcidtoname_downlevel.obj
 0002:00004208       ??_C@_1O@MGJBOAMB@?$AAq?$AAu?$AAz?$AA?9?$AAP?$AAE@ 10035208     libucrt:lcidtoname_downlevel.obj
 0002:00004218       ??_C@_1M@GJINLBOK@?$AAa?$AAr?$AA?9?$AAL?$AAY@ 10035218     libucrt:lcidtoname_downlevel.obj
 0002:00004224       ??_C@_1M@GGMNHJNL@?$AAz?$AAh?$AA?9?$AAS?$AAG@ 10035224     libucrt:lcidtoname_downlevel.obj
 0002:00004230       ??_C@_1M@HOIKODND@?$AAd?$AAe?$AA?9?$AAL?$AAU@ 10035230     libucrt:lcidtoname_downlevel.obj
 0002:0000423c       ??_C@_1M@DDOCCGFG@?$AAe?$AAn?$AA?9?$AAC?$AAA@ 1003523c     libucrt:lcidtoname_downlevel.obj
 0002:00004248       ??_C@_1M@BNOEMJLF@?$AAe?$AAs?$AA?9?$AAG?$AAT@ 10035248     libucrt:lcidtoname_downlevel.obj
 0002:00004254       ??_C@_1M@EOGNKEK@?$AAf?$AAr?$AA?9?$AAC?$AAH@ 10035254     libucrt:lcidtoname_downlevel.obj
 0002:00004260       ??_C@_1M@FLIDJFHL@?$AAh?$AAr?$AA?9?$AAB?$AAA@ 10035260     libucrt:lcidtoname_downlevel.obj
 0002:0000426c       ??_C@_1O@FMCELNAJ@?$AAs?$AAm?$AAj?$AA?9?$AAN?$AAO@ 1003526c     libucrt:lcidtoname_downlevel.obj
 0002:0000427c       ??_C@_1M@JHGLJMGJ@?$AAa?$AAr?$AA?9?$AAD?$AAZ@ 1003527c     libucrt:lcidtoname_downlevel.obj
 0002:00004288       ??_C@_1M@JKKFDCNP@?$AAz?$AAh?$AA?9?$AAM?$AAO@ 10035288     libucrt:lcidtoname_downlevel.obj
 0002:00004294       ??_C@_1M@GEEFALPE@?$AAd?$AAe?$AA?9?$AAL?$AAI@ 10035294     libucrt:lcidtoname_downlevel.obj
 0002:000042a0       ??_C@_1M@IGEOFBG@?$AAe?$AAn?$AA?9?$AAN?$AAZ@ 100352a0     libucrt:lcidtoname_downlevel.obj
 0002:000042ac       ??_C@_1M@KDBONEHP@?$AAe?$AAs?$AA?9?$AAC?$AAR@ 100352ac     libucrt:lcidtoname_downlevel.obj
 0002:000042b8       ??_C@_1M@FHMDOHNN@?$AAf?$AAr?$AA?9?$AAL?$AAU@ 100352b8     libucrt:lcidtoname_downlevel.obj
 0002:000042c4       ??_C@_1BG@NFKKMAFG@?$AAb?$AAs?$AA?9?$AAB?$AAA?$AA?9?$AAL?$AAa?$AAt?$AAn@ 100352c4     libucrt:lcidtoname_downlevel.obj
 0002:000042dc       ??_C@_1O@IMNBEMCI@?$AAs?$AAm?$AAj?$AA?9?$AAS?$AAE@ 100352dc     libucrt:lcidtoname_downlevel.obj
 0002:000042ec       ??_C@_1M@DHHMBNDP@?$AAa?$AAr?$AA?9?$AAM?$AAA@ 100352ec     libucrt:lcidtoname_downlevel.obj
 0002:000042f8       ??_C@_1M@BNBLJCGH@?$AAe?$AAn?$AA?9?$AAI?$AAE@ 100352f8     libucrt:lcidtoname_downlevel.obj
 0002:00004304       ??_C@_1M@GEPAFMDL@?$AAe?$AAs?$AA?9?$AAP?$AAA@ 10035304     libucrt:lcidtoname_downlevel.obj
 0002:00004310       ??_C@_1M@OJONDMDL@?$AAf?$AAr?$AA?9?$AAM?$AAC@ 10035310     libucrt:lcidtoname_downlevel.obj
 0002:0000431c       ??_C@_1BG@OBCNFJB@?$AAs?$AAr?$AA?9?$AAB?$AAA?$AA?9?$AAL?$AAa?$AAt?$AAn@ 1003531c     libucrt:lcidtoname_downlevel.obj
 0002:00004334       ??_C@_1O@KEMEEGPO@?$AAs?$AAm?$AAa?$AA?9?$AAN?$AAO@ 10035334     libucrt:lcidtoname_downlevel.obj
 0002:00004344       ??_C@_1M@ELMGFODK@?$AAa?$AAr?$AA?9?$AAT?$AAN@ 10035344     libucrt:lcidtoname_downlevel.obj
 0002:00004350       ??_C@_1M@BHDLHFAF@?$AAe?$AAn?$AA?9?$AAZ?$AAA@ 10035350     libucrt:lcidtoname_downlevel.obj
 0002:0000435c       ??_C@_1M@BMGIGLIF@?$AAe?$AAs?$AA?9?$AAD?$AAO@ 1003535c     libucrt:lcidtoname_downlevel.obj
 0002:00004368       ??_C@_1BG@CMBHIPBE@?$AAs?$AAr?$AA?9?$AAB?$AAA?$AA?9?$AAC?$AAy?$AAr?$AAl@ 10035368     libucrt:lcidtoname_downlevel.obj
 0002:00004380       ??_C@_1O@HEDBLHNP@?$AAs?$AAm?$AAa?$AA?9?$AAS?$AAE@ 10035380     libucrt:lcidtoname_downlevel.obj
 0002:00004390       ??_C@_1M@DAGCADIM@?$AAa?$AAr?$AA?9?$AAO?$AAM@ 10035390     libucrt:lcidtoname_downlevel.obj
 0002:0000439c       ??_C@_1M@FODLMICG@?$AAe?$AAn?$AA?9?$AAJ?$AAM@ 1003539c     libucrt:lcidtoname_downlevel.obj
 0002:000043a8       ??_C@_1M@DNMLCIHB@?$AAe?$AAs?$AA?9?$AAV?$AAE@ 100353a8     libucrt:lcidtoname_downlevel.obj
 0002:000043b4       ??_C@_1O@EOKHMKJK@?$AAs?$AAm?$AAs?$AA?9?$AAF?$AAI@ 100353b4     libucrt:lcidtoname_downlevel.obj
 0002:000043c4       ??_C@_1M@CAFJMKOF@?$AAa?$AAr?$AA?9?$AAY?$AAE@ 100353c4     libucrt:lcidtoname_downlevel.obj
 0002:000043d0       ??_C@_1M@CBFHIJLI@?$AAe?$AAn?$AA?9?$AAC?$AAB@ 100353d0     libucrt:lcidtoname_downlevel.obj
 0002:000043dc       ??_C@_1M@BGNFLDN@?$AAe?$AAs?$AA?9?$AAC?$AAO@ 100353dc     libucrt:lcidtoname_downlevel.obj
 0002:000043e8       ??_C@_1O@JMPHMAMC@?$AAs?$AAm?$AAn?$AA?9?$AAF?$AAI@ 100353e8     libucrt:lcidtoname_downlevel.obj
 0002:000043f8       ??_C@_1M@JLANABKE@?$AAa?$AAr?$AA?9?$AAS?$AAY@ 100353f8     libucrt:lcidtoname_downlevel.obj
 0002:00004404       ??_C@_1M@HPKGCFGN@?$AAe?$AAn?$AA?9?$AAB?$AAZ@ 10035404     libucrt:lcidtoname_downlevel.obj
 0002:00004410       ??_C@_1M@OLJCMLGM@?$AAe?$AAs?$AA?9?$AAP?$AAE@ 10035410     libucrt:lcidtoname_downlevel.obj
 0002:0000441c       ??_C@_1M@MKKGFKLE@?$AAa?$AAr?$AA?9?$AAJ?$AAO@ 1003541c     libucrt:lcidtoname_downlevel.obj
 0002:00004428       ??_C@_1M@EKPGLDNI@?$AAe?$AAn?$AA?9?$AAT?$AAT@ 10035428     libucrt:lcidtoname_downlevel.obj
 0002:00004434       ??_C@_1M@OONGHFHE@?$AAe?$AAs?$AA?9?$AAA?$AAR@ 10035434     libucrt:lcidtoname_downlevel.obj
 0002:00004440       ??_C@_1M@OOJFGBHE@?$AAa?$AAr?$AA?9?$AAL?$AAB@ 10035440     libucrt:lcidtoname_downlevel.obj
 0002:0000444c       ??_C@_1M@GCEJHNEG@?$AAe?$AAn?$AA?9?$AAZ?$AAW@ 1003544c     libucrt:lcidtoname_downlevel.obj
 0002:00004458       ??_C@_1M@JNOCAHJI@?$AAe?$AAs?$AA?9?$AAE?$AAC@ 10035458     libucrt:lcidtoname_downlevel.obj
 0002:00004464       ??_C@_1M@JEFHPGGB@?$AAa?$AAr?$AA?9?$AAK?$AAW@ 10035464     libucrt:lcidtoname_downlevel.obj
 0002:00004470       ??_C@_1M@MLKIBJOJ@?$AAe?$AAn?$AA?9?$AAP?$AAH@ 10035470     libucrt:lcidtoname_downlevel.obj
 0002:0000447c       ??_C@_1M@BDNIPEND@?$AAe?$AAs?$AA?9?$AAC?$AAL@ 1003547c     libucrt:lcidtoname_downlevel.obj
 0002:00004488       ??_C@_1M@MPNMEKBD@?$AAa?$AAr?$AA?9?$AAA?$AAE@ 10035488     libucrt:lcidtoname_downlevel.obj
 0002:00004494       ??_C@_1M@KBJALCPI@?$AAe?$AAs?$AA?9?$AAU?$AAY@ 10035494     libucrt:lcidtoname_downlevel.obj
 0002:000044a0       ??_C@_1M@LLCCOAGA@?$AAa?$AAr?$AA?9?$AAB?$AAH@ 100354a0     libucrt:lcidtoname_downlevel.obj
 0002:000044ac       ??_C@_1M@PBFNCDEL@?$AAe?$AAs?$AA?9?$AAP?$AAY@ 100354ac     libucrt:lcidtoname_downlevel.obj
 0002:000044b8       ??_C@_1M@EDGINPNP@?$AAa?$AAr?$AA?9?$AAQ?$AAA@ 100354b8     libucrt:lcidtoname_downlevel.obj
 0002:000044c4       ??_C@_1M@MKDBIIJI@?$AAe?$AAs?$AA?9?$AAB?$AAO@ 100354c4     libucrt:lcidtoname_downlevel.obj
 0002:000044d0       ??_C@_1M@CPKKEBLD@?$AAe?$AAs?$AA?9?$AAS?$AAV@ 100354d0     libucrt:lcidtoname_downlevel.obj
 0002:000044dc       ??_C@_1M@NDBGMMJL@?$AAe?$AAs?$AA?9?$AAH?$AAN@ 100354dc     libucrt:lcidtoname_downlevel.obj
 0002:000044e8       ??_C@_1M@JIJIBHDP@?$AAe?$AAs?$AA?9?$AAN?$AAI@ 100354e8     libucrt:lcidtoname_downlevel.obj
 0002:000044f4       ??_C@_1M@CGFMKEEK@?$AAe?$AAs?$AA?9?$AAP?$AAR@ 100354f4     libucrt:lcidtoname_downlevel.obj
 0002:00004500       ??_C@_1O@ICJHKIIK@?$AAz?$AAh?$AA?9?$AAC?$AAH?$AAT@ 10035500     libucrt:lcidtoname_downlevel.obj
 0002:00004510       ??_C@_15CLNEJCE@?$AAs?$AAr@ 10035510     libucrt:lcidtoname_downlevel.obj
 0002:00004c38       ??_C@_1M@KAHEKEIG@?$AAa?$AAf?$AA?9?$AAz?$AAa@ 10035c38     libucrt:lcidtoname_downlevel.obj
 0002:00004c44       ??_C@_1M@GIECOABL@?$AAa?$AAr?$AA?9?$AAa?$AAe@ 10035c44     libucrt:lcidtoname_downlevel.obj
 0002:00004c50       ??_C@_1M@BMLMEKGI@?$AAa?$AAr?$AA?9?$AAb?$AAh@ 10035c50     libucrt:lcidtoname_downlevel.obj
 0002:00004c5c       ??_C@_1M@DAPFDGGB@?$AAa?$AAr?$AA?9?$AAd?$AAz@ 10035c5c     libucrt:lcidtoname_downlevel.obj
 0002:00004c68       ??_C@_1M@FJNKGKIG@?$AAa?$AAr?$AA?9?$AAe?$AAg@ 10035c68     libucrt:lcidtoname_downlevel.obj
 0002:00004c74       ??_C@_1M@FLGKKCLO@?$AAa?$AAr?$AA?9?$AAi?$AAq@ 10035c74     libucrt:lcidtoname_downlevel.obj
 0002:00004c80       ??_C@_1M@GNDIPALM@?$AAa?$AAr?$AA?9?$AAj?$AAo@ 10035c80     libucrt:lcidtoname_downlevel.obj
 0002:00004c8c       ??_C@_1M@DDMJFMGJ@?$AAa?$AAr?$AA?9?$AAk?$AAw@ 10035c8c     libucrt:lcidtoname_downlevel.obj
 0002:00004c98       ??_C@_1M@EJALMLHM@?$AAa?$AAr?$AA?9?$AAl?$AAb@ 10035c98     libucrt:lcidtoname_downlevel.obj
 0002:00004ca4       ??_C@_1M@MOBDBLOC@?$AAa?$AAr?$AA?9?$AAl?$AAy@ 10035ca4     libucrt:lcidtoname_downlevel.obj
 0002:00004cb0       ??_C@_1M@JAOCLHDH@?$AAa?$AAr?$AA?9?$AAm?$AAa@ 10035cb0     libucrt:lcidtoname_downlevel.obj
 0002:00004cbc       ??_C@_1M@JHPMKJIE@?$AAa?$AAr?$AA?9?$AAo?$AAm@ 10035cbc     libucrt:lcidtoname_downlevel.obj
 0002:00004cc8       ??_C@_1M@OEPGHFNH@?$AAa?$AAr?$AA?9?$AAq?$AAa@ 10035cc8     libucrt:lcidtoname_downlevel.obj
 0002:00004cd4       ??_C@_1M@KJDONENM@?$AAa?$AAr?$AA?9?$AAs?$AAa@ 10035cd4     libucrt:lcidtoname_downlevel.obj
 0002:00004ce0       ??_C@_1M@DMJDKLKM@?$AAa?$AAr?$AA?9?$AAs?$AAy@ 10035ce0     libucrt:lcidtoname_downlevel.obj
 0002:00004cec       ??_C@_1M@OMFIPEDC@?$AAa?$AAr?$AA?9?$AAt?$AAn@ 10035cec     libucrt:lcidtoname_downlevel.obj
 0002:00004cf8       ??_C@_1M@IHMHGAON@?$AAa?$AAr?$AA?9?$AAy?$AAe@ 10035cf8     libucrt:lcidtoname_downlevel.obj
 0002:00004d04       ??_C@_1BG@KDCPGJGB@?$AAa?$AAz?$AA?9?$AAa?$AAz?$AA?9?$AAc?$AAy?$AAr?$AAl@ 10035d04     libucrt:lcidtoname_downlevel.obj
 0002:00004d1c       ??_C@_1BG@IBCKDDOE@?$AAa?$AAz?$AA?9?$AAa?$AAz?$AA?9?$AAl?$AAa?$AAt?$AAn@ 10035d1c     libucrt:lcidtoname_downlevel.obj
 0002:00004d34       ??_C@_1M@EGPFDCPD@?$AAb?$AAe?$AA?9?$AAb?$AAy@ 10035d34     libucrt:lcidtoname_downlevel.obj
 0002:00004d40       ??_C@_1M@PCMGMCGC@?$AAb?$AAg?$AA?9?$AAb?$AAg@ 10035d40     libucrt:lcidtoname_downlevel.obj
 0002:00004d4c       ??_C@_1M@BJBMFGOB@?$AAb?$AAn?$AA?9?$AAi?$AAn@ 10035d4c     libucrt:lcidtoname_downlevel.obj
 0002:00004d58       ??_C@_1BG@EAKMMACD@?$AAb?$AAs?$AA?9?$AAb?$AAa?$AA?9?$AAl?$AAa?$AAt?$AAn@ 10035d58     libucrt:lcidtoname_downlevel.obj
 0002:00004d70       ??_C@_1M@KGADAODK@?$AAc?$AAa?$AA?9?$AAe?$AAs@ 10035d70     libucrt:lcidtoname_downlevel.obj
 0002:00004d7c       ??_C@_1M@COAJPDHI@?$AAc?$AAs?$AA?9?$AAc?$AAz@ 10035d7c     libucrt:lcidtoname_downlevel.obj
 0002:00004d88       ??_C@_1M@DHBHFONH@?$AAc?$AAy?$AA?9?$AAg?$AAb@ 10035d88     libucrt:lcidtoname_downlevel.obj
 0002:00004d94       ??_C@_1M@IMGKELGA@?$AAd?$AAa?$AA?9?$AAd?$AAk@ 10035d94     libucrt:lcidtoname_downlevel.obj
 0002:00004da0       ??_C@_1M@NNDGDNGA@?$AAd?$AAe?$AA?9?$AAa?$AAt@ 10035da0     libucrt:lcidtoname_downlevel.obj
 0002:00004dac       ??_C@_1M@IKDBHEEM@?$AAd?$AAe?$AA?9?$AAc?$AAh@ 10035dac     libucrt:lcidtoname_downlevel.obj
 0002:00004db8       ??_C@_1M@GFFOJMCJ@?$AAd?$AAe?$AA?9?$AAd?$AAe@ 10035db8     libucrt:lcidtoname_downlevel.obj
 0002:00004dc4       ??_C@_1M@MDNLKBPM@?$AAd?$AAe?$AA?9?$AAl?$AAi@ 10035dc4     libucrt:lcidtoname_downlevel.obj
 0002:00004dd0       ??_C@_1M@NJBEEJNL@?$AAd?$AAe?$AA?9?$AAl?$AAu@ 10035dd0     libucrt:lcidtoname_downlevel.obj
 0002:00004ddc       ??_C@_1O@GNNELBAP@?$AAd?$AAi?$AAv?$AA?9?$AAm?$AAv@ 10035ddc     libucrt:lcidtoname_downlevel.obj
 0002:00004dec       ??_C@_1M@EJLEOGAE@?$AAe?$AAl?$AA?9?$AAg?$AAr@ 10035dec     libucrt:lcidtoname_downlevel.obj
 0002:00004df8       ??_C@_1M@GMPONJN@?$AAe?$AAn?$AA?9?$AAa?$AAu@ 10035df8     libucrt:lcidtoname_downlevel.obj
 0002:00004e04       ??_C@_1M@NIDIIPGF@?$AAe?$AAn?$AA?9?$AAb?$AAz@ 10035e04     libucrt:lcidtoname_downlevel.obj
 0002:00004e10       ??_C@_1M@JEHMIMFO@?$AAe?$AAn?$AA?9?$AAc?$AAa@ 10035e10     libucrt:lcidtoname_downlevel.obj
 0002:00004e1c       ??_C@_1M@IGMJCDLA@?$AAe?$AAn?$AA?9?$AAc?$AAb@ 10035e1c     libucrt:lcidtoname_downlevel.obj
 0002:00004e28       ??_C@_1M@BNFIGBKG@?$AAe?$AAn?$AA?9?$AAg?$AAb@ 10035e28     libucrt:lcidtoname_downlevel.obj
 0002:00004e34       ??_C@_1M@LKIFDIGP@?$AAe?$AAn?$AA?9?$AAi?$AAe@ 10035e34     libucrt:lcidtoname_downlevel.obj
 0002:00004e40       ??_C@_1M@PJKFGCCO@?$AAe?$AAn?$AA?9?$AAj?$AAm@ 10035e40     libucrt:lcidtoname_downlevel.obj
 0002:00004e4c       ??_C@_1M@KPPKEPBO@?$AAe?$AAn?$AA?9?$AAn?$AAz@ 10035e4c     libucrt:lcidtoname_downlevel.obj
 0002:00004e58       ??_C@_1M@GMDGLDOB@?$AAe?$AAn?$AA?9?$AAp?$AAh@ 10035e58     libucrt:lcidtoname_downlevel.obj
 0002:00004e64       ??_C@_1M@ONGIBJNA@?$AAe?$AAn?$AA?9?$AAt?$AAt@ 10035e64     libucrt:lcidtoname_downlevel.obj
 0002:00004e70       ??_C@_1M@LLODPCMM@?$AAe?$AAn?$AA?9?$AAu?$AAs@ 10035e70     libucrt:lcidtoname_downlevel.obj
 0002:00004e7c       ??_C@_1M@LAKFNPAN@?$AAe?$AAn?$AA?9?$AAz?$AAa@ 10035e7c     libucrt:lcidtoname_downlevel.obj
 0002:00004e88       ??_C@_1M@MFNHNHEO@?$AAe?$AAn?$AA?9?$AAz?$AAw@ 10035e88     libucrt:lcidtoname_downlevel.obj
 0002:00004e94       ??_C@_1M@EJEINPHM@?$AAe?$AAs?$AA?9?$AAa?$AAr@ 10035e94     libucrt:lcidtoname_downlevel.obj
 0002:00004ea0       ??_C@_1M@GNKPCCJA@?$AAe?$AAs?$AA?9?$AAb?$AAo@ 10035ea0     libucrt:lcidtoname_downlevel.obj
 0002:00004eac       ??_C@_1M@LEEGFONL@?$AAe?$AAs?$AA?9?$AAc?$AAl@ 10035eac     libucrt:lcidtoname_downlevel.obj
 0002:00004eb8       ??_C@_1M@KGPDPBDF@?$AAe?$AAs?$AA?9?$AAc?$AAo@ 10035eb8     libucrt:lcidtoname_downlevel.obj
 0002:00004ec4       ??_C@_1M@EIAHOHH@?$AAe?$AAs?$AA?9?$AAc?$AAr@ 10035ec4     libucrt:lcidtoname_downlevel.obj
 0002:00004ed0       ??_C@_1M@LLPGMBIN@?$AAe?$AAs?$AA?9?$AAd?$AAo@ 10035ed0     libucrt:lcidtoname_downlevel.obj
 0002:00004edc       ??_C@_1M@DKHMKNJA@?$AAe?$AAs?$AA?9?$AAe?$AAc@ 10035edc     libucrt:lcidtoname_downlevel.obj
 0002:00004ee8       ??_C@_1M@GKGFPKAP@?$AAe?$AAs?$AA?9?$AAe?$AAs@ 10035ee8     libucrt:lcidtoname_downlevel.obj
 0002:00004ef4       ??_C@_1M@LKHKGDLN@?$AAe?$AAs?$AA?9?$AAg?$AAt@ 10035ef4     libucrt:lcidtoname_downlevel.obj
 0002:00004f00       ??_C@_1M@HEIIGGJD@?$AAe?$AAs?$AA?9?$AAh?$AAn@ 10035f00     libucrt:lcidtoname_downlevel.obj
 0002:00004f0c       ??_C@_1M@FBDHPPGD@?$AAe?$AAs?$AA?9?$AAm?$AAx@ 10035f0c     libucrt:lcidtoname_downlevel.obj
 0002:00004f18       ??_C@_1M@DPAGLNDH@?$AAe?$AAs?$AA?9?$AAn?$AAi@ 10035f18     libucrt:lcidtoname_downlevel.obj
 0002:00004f24       ??_C@_1M@MDGOPGDD@?$AAe?$AAs?$AA?9?$AAp?$AAa@ 10035f24     libucrt:lcidtoname_downlevel.obj
 0002:00004f30       ??_C@_1M@EMAMGBGE@?$AAe?$AAs?$AA?9?$AAp?$AAe@ 10035f30     libucrt:lcidtoname_downlevel.obj
 0002:00004f3c       ??_C@_1M@IBMCAOEC@?$AAe?$AAs?$AA?9?$AAp?$AAr@ 10035f3c     libucrt:lcidtoname_downlevel.obj
 0002:00004f48       ??_C@_1M@FGMDIJED@?$AAe?$AAs?$AA?9?$AAp?$AAy@ 10035f48     libucrt:lcidtoname_downlevel.obj
 0002:00004f54       ??_C@_1M@IIDEOLLL@?$AAe?$AAs?$AA?9?$AAs?$AAv@ 10035f54     libucrt:lcidtoname_downlevel.obj
 0002:00004f60       ??_C@_1M@GAOBIPA@?$AAe?$AAs?$AA?9?$AAu?$AAy@ 10035f60     libucrt:lcidtoname_downlevel.obj
 0002:00004f6c       ??_C@_1M@JKFFICHJ@?$AAe?$AAs?$AA?9?$AAv?$AAe@ 10035f6c     libucrt:lcidtoname_downlevel.obj
 0002:00004f78       ??_C@_1M@PNMLOJDF@?$AAe?$AAt?$AA?9?$AAe?$AAe@ 10035f78     libucrt:lcidtoname_downlevel.obj
 0002:00004f84       ??_C@_1M@GHHLIKEI@?$AAe?$AAu?$AA?9?$AAe?$AAs@ 10035f84     libucrt:lcidtoname_downlevel.obj
 0002:00004f90       ??_C@_1M@PBNONODE@?$AAf?$AAa?$AA?9?$AAi?$AAr@ 10035f90     libucrt:lcidtoname_downlevel.obj
 0002:00004f9c       ??_C@_1M@JEEHPMIL@?$AAf?$AAi?$AA?9?$AAf?$AAi@ 10035f9c     libucrt:lcidtoname_downlevel.obj
 0002:00004fa8       ??_C@_1M@LMDCNDBA@?$AAf?$AAo?$AA?9?$AAf?$AAo@ 10035fa8     libucrt:lcidtoname_downlevel.obj
 0002:00004fb4       ??_C@_1M@JKEOHLDK@?$AAf?$AAr?$AA?9?$AAb?$AAe@ 10035fb4     libucrt:lcidtoname_downlevel.obj
 0002:00004fc0       ??_C@_1M@NOHADPMI@?$AAf?$AAr?$AA?9?$AAc?$AAa@ 10035fc0     libucrt:lcidtoname_downlevel.obj
 0002:00004fcc       ??_C@_1M@KDHIHAEC@?$AAf?$AAr?$AA?9?$AAc?$AAh@ 10035fcc     libucrt:lcidtoname_downlevel.obj
 0002:00004fd8       ??_C@_1M@MMBBFGAK@?$AAf?$AAr?$AA?9?$AAf?$AAr@ 10035fd8     libucrt:lcidtoname_downlevel.obj
 0002:00004fe4       ??_C@_1M@PAFNENNF@?$AAf?$AAr?$AA?9?$AAl?$AAu@ 10035fe4     libucrt:lcidtoname_downlevel.obj
 0002:00004ff0       ??_C@_1M@EOHDJGDD@?$AAf?$AAr?$AA?9?$AAm?$AAc@ 10035ff0     libucrt:lcidtoname_downlevel.obj
 0002:00004ffc       ??_C@_1M@FAPLLOPF@?$AAg?$AAl?$AA?9?$AAe?$AAs@ 10035ffc     libucrt:lcidtoname_downlevel.obj
 0002:00005008       ??_C@_1M@FOPBFLOO@?$AAg?$AAu?$AA?9?$AAi?$AAn@ 10036008     libucrt:lcidtoname_downlevel.obj
 0002:00005014       ??_C@_1M@KBMCINPM@?$AAh?$AAe?$AA?9?$AAi?$AAl@ 10036014     libucrt:lcidtoname_downlevel.obj
 0002:00005020       ??_C@_1M@BBPHKFPJ@?$AAh?$AAi?$AA?9?$AAi?$AAn@ 10036020     libucrt:lcidtoname_downlevel.obj
 0002:0000502c       ??_C@_1M@PMBNDPHD@?$AAh?$AAr?$AA?9?$AAb?$AAa@ 1003602c     libucrt:lcidtoname_downlevel.obj
 0002:00005038       ??_C@_1M@BPCKOEGE@?$AAh?$AAr?$AA?9?$AAh?$AAr@ 10036038     libucrt:lcidtoname_downlevel.obj
 0002:00005044       ??_C@_1M@GACBMHKE@?$AAh?$AAu?$AA?9?$AAh?$AAu@ 10036044     libucrt:lcidtoname_downlevel.obj
 0002:00005050       ??_C@_1M@MILPAJJC@?$AAh?$AAy?$AA?9?$AAa?$AAm@ 10036050     libucrt:lcidtoname_downlevel.obj
 0002:0000505c       ??_C@_1M@BABBICEC@?$AAi?$AAd?$AA?9?$AAi?$AAd@ 1003605c     libucrt:lcidtoname_downlevel.obj
 0002:00005068       ??_C@_1M@BIKNHHPF@?$AAi?$AAs?$AA?9?$AAi?$AAs@ 10036068     libucrt:lcidtoname_downlevel.obj
 0002:00005074       ??_C@_1M@NMPCJPHE@?$AAi?$AAt?$AA?9?$AAc?$AAh@ 10036074     libucrt:lcidtoname_downlevel.obj
 0002:00005080       ??_C@_1M@GHKGFEDF@?$AAi?$AAt?$AA?9?$AAi?$AAt@ 10036080     libucrt:lcidtoname_downlevel.obj
 0002:0000508c       ??_C@_1M@NIEJCJJA@?$AAj?$AAa?$AA?9?$AAj?$AAp@ 1003608c     libucrt:lcidtoname_downlevel.obj
 0002:00005098       ??_C@_1M@JILFNBIM@?$AAk?$AAa?$AA?9?$AAg?$AAe@ 10036098     libucrt:lcidtoname_downlevel.obj
 0002:000050a4       ??_C@_1M@PACPMGPH@?$AAk?$AAk?$AA?9?$AAk?$AAz@ 100360a4     libucrt:lcidtoname_downlevel.obj
 0002:000050b0       ??_C@_1M@IELFGMHA@?$AAk?$AAn?$AA?9?$AAi?$AAn@ 100360b0     libucrt:lcidtoname_downlevel.obj
 0002:000050bc       ??_C@_1O@IBBJHCH@?$AAk?$AAo?$AAk?$AA?9?$AAi?$AAn@ 100360bc     libucrt:lcidtoname_downlevel.obj
 0002:000050cc       ??_C@_1M@DMHAEOGC@?$AAk?$AAo?$AA?9?$AAk?$AAr@ 100360cc     libucrt:lcidtoname_downlevel.obj
 0002:000050d8       ??_C@_1M@HBAHBIGA@?$AAk?$AAy?$AA?9?$AAk?$AAg@ 100360d8     libucrt:lcidtoname_downlevel.obj
 0002:000050e4       ??_C@_1M@KPMILCJG@?$AAl?$AAt?$AA?9?$AAl?$AAt@ 100360e4     libucrt:lcidtoname_downlevel.obj
 0002:000050f0       ??_C@_1M@BDEKKCA@?$AAl?$AAv?$AA?9?$AAl?$AAv@ 100360f0     libucrt:lcidtoname_downlevel.obj
 0002:000050fc       ??_C@_1M@ELCKCCJJ@?$AAm?$AAi?$AA?9?$AAn?$AAz@ 100360fc     libucrt:lcidtoname_downlevel.obj
 0002:00005108       ??_C@_1M@CBOOLAPA@?$AAm?$AAk?$AA?9?$AAm?$AAk@ 10036108     libucrt:lcidtoname_downlevel.obj
 0002:00005114       ??_C@_1M@GPHNBJKN@?$AAm?$AAl?$AA?9?$AAi?$AAn@ 10036114     libucrt:lcidtoname_downlevel.obj
 0002:00005120       ??_C@_1M@PABJILIG@?$AAm?$AAn?$AA?9?$AAm?$AAn@ 10036120     libucrt:lcidtoname_downlevel.obj
 0002:0000512c       ??_C@_1M@FGBKKIPG@?$AAm?$AAr?$AA?9?$AAi?$AAn@ 1003612c     libucrt:lcidtoname_downlevel.obj
 0002:00005138       ??_C@_1M@NDBPDDAL@?$AAm?$AAs?$AA?9?$AAb?$AAn@ 10036138     libucrt:lcidtoname_downlevel.obj
 0002:00005144       ??_C@_1M@OPIHOOPI@?$AAm?$AAs?$AA?9?$AAm?$AAy@ 10036144     libucrt:lcidtoname_downlevel.obj
 0002:00005150       ??_C@_1M@PPDBCNFM@?$AAm?$AAt?$AA?9?$AAm?$AAt@ 10036150     libucrt:lcidtoname_downlevel.obj
 0002:0000515c       ??_C@_1M@KDJDKMDD@?$AAn?$AAb?$AA?9?$AAn?$AAo@ 1003615c     libucrt:lcidtoname_downlevel.obj
 0002:00005168       ??_C@_1M@KFCFLMJP@?$AAn?$AAl?$AA?9?$AAb?$AAe@ 10036168     libucrt:lcidtoname_downlevel.obj
 0002:00005174       ??_C@_1M@KPOPDDGO@?$AAn?$AAl?$AA?9?$AAn?$AAl@ 10036174     libucrt:lcidtoname_downlevel.obj
 0002:00005180       ??_C@_1M@LJKPEMLN@?$AAn?$AAn?$AA?9?$AAn?$AAo@ 10036180     libucrt:lcidtoname_downlevel.obj
 0002:0000518c       ??_C@_1M@BDGHHBFL@?$AAn?$AAs?$AA?9?$AAz?$AAa@ 1003618c     libucrt:lcidtoname_downlevel.obj
 0002:00005198       ??_C@_1M@IDEHOAP@?$AAp?$AAa?$AA?9?$AAi?$AAn@ 10036198     libucrt:lcidtoname_downlevel.obj
 0002:000051a4       ??_C@_1M@HDBKGOGH@?$AAp?$AAl?$AA?9?$AAp?$AAl@ 100361a4     libucrt:lcidtoname_downlevel.obj
 0002:000051b0       ??_C@_1M@LJLLCMEH@?$AAp?$AAt?$AA?9?$AAb?$AAr@ 100361b0     libucrt:lcidtoname_downlevel.obj
 0002:000051bc       ??_C@_1M@NCMONAAL@?$AAp?$AAt?$AA?9?$AAp?$AAt@ 100361bc     libucrt:lcidtoname_downlevel.obj
 0002:000051c8       ??_C@_1O@EAKMAJDN@?$AAq?$AAu?$AAz?$AA?9?$AAb?$AAo@ 100361c8     libucrt:lcidtoname_downlevel.obj
 0002:000051d8       ??_C@_1O@BHHPIGDN@?$AAq?$AAu?$AAz?$AA?9?$AAe?$AAc@ 100361d8     libucrt:lcidtoname_downlevel.obj
 0002:000051e8       ??_C@_1O@GBAPEKMJ@?$AAq?$AAu?$AAz?$AA?9?$AAp?$AAe@ 100361e8     libucrt:lcidtoname_downlevel.obj
 0002:000051f8       ??_C@_1M@CLGLEFBO@?$AAr?$AAo?$AA?9?$AAr?$AAo@ 100361f8     libucrt:lcidtoname_downlevel.obj
 0002:00005204       ??_C@_1M@CEEDODME@?$AAr?$AAu?$AA?9?$AAr?$AAu@ 10036204     libucrt:lcidtoname_downlevel.obj
 0002:00005210       ??_C@_1M@HPKKKMPP@?$AAs?$AAa?$AA?9?$AAi?$AAn@ 10036210     libucrt:lcidtoname_downlevel.obj
 0002:0000521c       ??_C@_1M@BKMAIGOJ@?$AAs?$AAe?$AA?9?$AAf?$AAi@ 1003621c     libucrt:lcidtoname_downlevel.obj
 0002:00005228       ??_C@_1M@NDPIFLFI@?$AAs?$AAe?$AA?9?$AAn?$AAo@ 10036228     libucrt:lcidtoname_downlevel.obj
 0002:00005234       ??_C@_1M@DANKKHJ@?$AAs?$AAe?$AA?9?$AAs?$AAe@ 10036234     libucrt:lcidtoname_downlevel.obj
 0002:00005240       ??_C@_1M@PNBLONPJ@?$AAs?$AAk?$AA?9?$AAs?$AAk@ 10036240     libucrt:lcidtoname_downlevel.obj
 0002:0000524c       ??_C@_1M@LFMODOAL@?$AAs?$AAl?$AA?9?$AAs?$AAi@ 1003624c     libucrt:lcidtoname_downlevel.obj
 0002:00005258       ??_C@_1O@DFKOMPG@?$AAs?$AAm?$AAa?$AA?9?$AAn?$AAo@ 10036258     libucrt:lcidtoname_downlevel.obj
 0002:00005268       ??_C@_1O@NDKPBNNH@?$AAs?$AAm?$AAa?$AA?9?$AAs?$AAe@ 10036268     libucrt:lcidtoname_downlevel.obj
 0002:00005278       ??_C@_1O@PLLKBHAB@?$AAs?$AAm?$AAj?$AA?9?$AAn?$AAo@ 10036278     libucrt:lcidtoname_downlevel.obj
 0002:00005288       ??_C@_1O@CLEPOGCA@?$AAs?$AAm?$AAj?$AA?9?$AAs?$AAe@ 10036288     libucrt:lcidtoname_downlevel.obj
 0002:00005298       ??_C@_1O@DLGJGKMK@?$AAs?$AAm?$AAn?$AA?9?$AAf?$AAi@ 10036298     libucrt:lcidtoname_downlevel.obj
 0002:000052a8       ??_C@_1O@OJDJGAJC@?$AAs?$AAm?$AAs?$AA?9?$AAf?$AAi@ 100362a8     libucrt:lcidtoname_downlevel.obj
 0002:000052b8       ??_C@_1M@BOFOGHPB@?$AAs?$AAq?$AA?9?$AAa?$AAl@ 100362b8     libucrt:lcidtoname_downlevel.obj
 0002:000052c4       ??_C@_1BG@LJBBIPGB@?$AAs?$AAr?$AA?9?$AAb?$AAa?$AA?9?$AAc?$AAy?$AAr?$AAl@ 100362c4     libucrt:lcidtoname_downlevel.obj
 0002:000052dc       ??_C@_1BG@JLBENFOE@?$AAs?$AAr?$AA?9?$AAb?$AAa?$AA?9?$AAl?$AAa?$AAt?$AAn@ 100362dc     libucrt:lcidtoname_downlevel.obj
 0002:000052f4       ??_C@_1BG@KODPNHE@?$AAs?$AAr?$AA?9?$AAs?$AAp?$AA?9?$AAc?$AAy?$AAr?$AAl@ 100362f4     libucrt:lcidtoname_downlevel.obj
 0002:0000530c       ??_C@_1BG@CIOGKHPB@?$AAs?$AAr?$AA?9?$AAs?$AAp?$AA?9?$AAl?$AAa?$AAt?$AAn@ 1003630c     libucrt:lcidtoname_downlevel.obj
 0002:00005324       ??_C@_1M@NGFJLMAC@?$AAs?$AAv?$AA?9?$AAf?$AAi@ 10036324     libucrt:lcidtoname_downlevel.obj
 0002:00005330       ??_C@_1M@MPJEJAJC@?$AAs?$AAv?$AA?9?$AAs?$AAe@ 10036330     libucrt:lcidtoname_downlevel.obj
 0002:0000533c       ??_C@_1M@MPNDHLFK@?$AAs?$AAw?$AA?9?$AAk?$AAe@ 1003633c     libucrt:lcidtoname_downlevel.obj
 0002:00005348       ??_C@_1O@KOHBJJI@?$AAs?$AAy?$AAr?$AA?9?$AAs?$AAy@ 10036348     libucrt:lcidtoname_downlevel.obj
 0002:00005358       ??_C@_1M@LDCEFHA@?$AAt?$AAa?$AA?9?$AAi?$AAn@ 10036358     libucrt:lcidtoname_downlevel.obj
 0002:00005364       ??_C@_1M@CNJOFAK@?$AAt?$AAe?$AA?9?$AAi?$AAn@ 10036364     libucrt:lcidtoname_downlevel.obj
 0002:00005370       ??_C@_1M@GNAECACD@?$AAt?$AAh?$AA?9?$AAt?$AAh@ 10036370     libucrt:lcidtoname_downlevel.obj
 0002:0000537c       ??_C@_1M@CHBIHOJO@?$AAt?$AAn?$AA?9?$AAz?$AAa@ 1003637c     libucrt:lcidtoname_downlevel.obj
 0002:00005388       ??_C@_1M@GCCMIGPJ@?$AAt?$AAr?$AA?9?$AAt?$AAr@ 10036388     libucrt:lcidtoname_downlevel.obj
 0002:00005394       ??_C@_1M@CELMCNBK@?$AAt?$AAt?$AA?9?$AAr?$AAu@ 10036394     libucrt:lcidtoname_downlevel.obj
 0002:000053a0       ??_C@_1M@KLMCELGA@?$AAu?$AAk?$AA?9?$AAu?$AAa@ 100363a0     libucrt:lcidtoname_downlevel.obj
 0002:000053ac       ??_C@_1M@EPAJJAJF@?$AAu?$AAr?$AA?9?$AAp?$AAk@ 100363ac     libucrt:lcidtoname_downlevel.obj
 0002:000053b8       ??_C@_1BG@GEGPMCDJ@?$AAu?$AAz?$AA?9?$AAu?$AAz?$AA?9?$AAc?$AAy?$AAr?$AAl@ 100363b8     libucrt:lcidtoname_downlevel.obj
 0002:000053d0       ??_C@_1BG@EGGKJILM@?$AAu?$AAz?$AA?9?$AAu?$AAz?$AA?9?$AAl?$AAa?$AAt?$AAn@ 100363d0     libucrt:lcidtoname_downlevel.obj
 0002:000053e8       ??_C@_1M@GFOCLFF@?$AAv?$AAi?$AA?9?$AAv?$AAn@ 100363e8     libucrt:lcidtoname_downlevel.obj
 0002:000053f4       ??_C@_1M@CPAMEDFI@?$AAx?$AAh?$AA?9?$AAz?$AAa@ 100363f4     libucrt:lcidtoname_downlevel.obj
 0002:00005400       ??_C@_1O@EBKIFIGN@?$AAz?$AAh?$AA?9?$AAc?$AAh?$AAs@ 10036400     libucrt:lcidtoname_downlevel.obj
 0002:00005410       ??_C@_1O@NMHPGANE@?$AAz?$AAh?$AA?9?$AAc?$AAh?$AAt@ 10036410     libucrt:lcidtoname_downlevel.obj
 0002:00005420       ??_C@_1M@LPINJOMC@?$AAz?$AAh?$AA?9?$AAc?$AAn@ 10036420     libucrt:lcidtoname_downlevel.obj
 0002:0000542c       ??_C@_1M@OCJEJODD@?$AAz?$AAh?$AA?9?$AAh?$AAk@ 1003642c     libucrt:lcidtoname_downlevel.obj
 0002:00005438       ??_C@_1M@DNDLJINH@?$AAz?$AAh?$AA?9?$AAm?$AAo@ 10036438     libucrt:lcidtoname_downlevel.obj
 0002:00005444       ??_C@_1M@MBFDNDND@?$AAz?$AAh?$AA?9?$AAs?$AAg@ 10036444     libucrt:lcidtoname_downlevel.obj
 0002:00005450       ??_C@_1M@IMEPLEPE@?$AAz?$AAh?$AA?9?$AAt?$AAw@ 10036450     libucrt:lcidtoname_downlevel.obj
 0002:0000545c       ??_C@_1M@BBGHNHJP@?$AAz?$AAu?$AA?9?$AAz?$AAa@ 1003645c     libucrt:lcidtoname_downlevel.obj
 0002:00005570       __infinity                 10036570     libucrt:87tran.obj
 0002:0000557a       __minfinity                1003657a     libucrt:87tran.obj
 0002:00005584       __logemax                  10036584     libucrt:87tran.obj
 0002:000055aa       __OP_EXPjmptab             100365aa     libucrt:87tran.obj
 0002:000055d0       __indefinite               100365d0     libucrt:87disp.obj
 0002:000055da       __piby2                    100365da     libucrt:87disp.obj
 0002:000055e4       __piby4                    100365e4     libucrt:87disp.obj
 0002:00005618       __DEFAULT_CW_in_mem        10036618     libucrt:common.obj
 0002:0000561a       __pi_by_2_to_61            1003661a     libucrt:common.obj
 0002:00005654       ??_C@_03MGHMBJCF@log@      10036654     libucrt:libm_error.obj
 0002:00005658       ??_C@_05HGHHAHAP@log10@    10036658     libucrt:libm_error.obj
 0002:00005660       ??_C@_03KHJOGHMM@exp@      10036660     libucrt:libm_error.obj
 0002:00005664       ??_C@_03JGHBODFD@pow@      10036664     libucrt:libm_error.obj
 0002:00005668       ??_C@_04FIHNOPOL@asin@     10036668     libucrt:libm_error.obj
 0002:00005670       ??_C@_04PDIFKINK@acos@     10036670     libucrt:libm_error.obj
 0002:00005678       ??_C@_04EIAKFFMI@sqrt@     10036678     libucrt:libm_error.obj
 0002:00005680       __real@3ff0000000000000    10036680     libucrt:libm_error.obj
 0002:000056a0       ___acrt_log10_table_t      100366a0     libucrt:log10_tables.obj
 0002:00005ab0       ___acrt_log10_table_cb     10036ab0     libucrt:log10_tables.obj
 0002:00005ec0       __real@3fe0000000000000    10036ec0     libucrt:powhlp.obj
 0002:00005fb0       ??_C@_04COOMCNPB@sinh@     10036fb0     libucrt:fpexcept.obj
 0002:00005fb8       ??_C@_04HPJJNFIM@cosh@     10036fb8     libucrt:fpexcept.obj
 0002:00005fc0       ??_C@_04FJHINJAO@tanh@     10036fc0     libucrt:fpexcept.obj
 0002:00005fc8       ??_C@_04MLLJIGOK@atan@     10036fc8     libucrt:fpexcept.obj
 0002:00005fd0       ??_C@_05KNGEOGJB@atan2@    10036fd0     libucrt:fpexcept.obj
 0002:00005fd8       ??_C@_03BLEJJJBH@sin@      10036fd8     libucrt:fpexcept.obj
 0002:00005fdc       ??_C@_03LALBNOCG@cos@      10036fdc     libucrt:fpexcept.obj
 0002:00005fe0       ??_C@_03IIINPABG@tan@      10036fe0     libucrt:fpexcept.obj
 0002:00005fe4       ??_C@_04GFPJNGEK@ceil@     10036fe4     libucrt:fpexcept.obj
 0002:00005fec       ??_C@_05PBJFFIGL@floor@    10036fec     libucrt:fpexcept.obj
 0002:00005ff4       ??_C@_04ODHECPBC@fabs@     10036ff4     libucrt:fpexcept.obj
 0002:00005ffc       ??_C@_04EHEDPDJG@modf@     10036ffc     libucrt:fpexcept.obj
 0002:00006004       ??_C@_05CEJMAHNP@ldexp@    10037004     libucrt:fpexcept.obj
 0002:0000600c       ??_C@_05KBKMEMPO@_cabs@    1003700c     libucrt:fpexcept.obj
 0002:00006014       ??_C@_06MEIMCGCF@_hypot@   10037014     libucrt:fpexcept.obj
 0002:0000601c       ??_C@_04KEPJIHGP@fmod@     1003701c     libucrt:fpexcept.obj
 0002:00006024       ??_C@_05GKKHEGJL@frexp@    10037024     libucrt:fpexcept.obj
 0002:0000602c       ??_C@_03MJLDFKDL@_y0@      1003702c     libucrt:fpexcept.obj
 0002:00006030       ??_C@_03NAKIGLHK@_y1@      10037030     libucrt:fpexcept.obj
 0002:00006034       ??_C@_03ONILCKOB@_yn@      10037034     libucrt:fpexcept.obj
 0002:00006038       ??_C@_05JGDBENOH@_logb@    10037038     libucrt:fpexcept.obj
 0002:00006040       ??_C@_0L@KDOEJCKC@_nextafter@ 10037040     libucrt:fpexcept.obj
 0002:00006050       __d_inf                    10037050     libucrt:util.obj
 0002:00006058       __d_max                    10037058     libucrt:util.obj
 0002:00006060       __d_mzero                  10037060     libucrt:util.obj
 0002:00006068       ??_C@_1BA@BALFACEM@?$AAC?$AAO?$AAN?$AAO?$AAU?$AAT?$AA$@ 10037068     libucrt:initcon.obj
 0002:00009070       __real@3fd999999999999a    1003a070     D2HelpFunc.obj
 0002:00009078       __real@3ff8000000000000    1003a078     ItemVariableProp.obj
 0002:00009080       __real@4000000000000000    1003a080     D2HelpFunc.obj
 0002:00009088       __real@4008000000000000    1003a088     D2HelpFunc.obj
 0002:00009090       __real@4060000000000000    1003a090     ViewUnitStat.obj
 0002:00009098       __real@4070000000000000    1003a098     ViewUnitStat.obj
 0002:000090a0       __real@40a0000000000000    1003a0a0     ItemName.obj
 0002:000090a8       __real@42c80000            1003a0a8     ScreenHook.obj
 0002:000090b0       __xmm@41f00000000000000000000000000000 1003a0b0     D2HelpFunc.obj
 0002:00009140       __load_config_used         1003a140     LIBCMT:loadcfg.obj
 0002:00009200       __tls_used                 1003a200     LIBCMT:tlssup.obj
 0002:00009218       ??_R4exception@std@@6B@    1003a218     LIBCMT:throw_bad_alloc.obj
 0002:0000922c       ??_R3exception@std@@8      1003a22c     LIBCMT:throw_bad_alloc.obj
 0002:0000923c       ??_R2exception@std@@8      1003a23c     LIBCMT:throw_bad_alloc.obj
 0002:00009244       ??_R1A@?0A@EA@exception@std@@8 1003a244     LIBCMT:throw_bad_alloc.obj
 0002:00009260       ??_R4bad_alloc@std@@6B@    1003a260     LIBCMT:throw_bad_alloc.obj
 0002:00009274       ??_R3bad_alloc@std@@8      1003a274     LIBCMT:throw_bad_alloc.obj
 0002:00009284       ??_R2bad_alloc@std@@8      1003a284     LIBCMT:throw_bad_alloc.obj
 0002:00009290       ??_R1A@?0A@EA@bad_alloc@std@@8 1003a290     LIBCMT:throw_bad_alloc.obj
 0002:000092ac       ??_R4bad_array_new_length@std@@6B@ 1003a2ac     LIBCMT:throw_bad_alloc.obj
 0002:000092c0       ??_R3bad_array_new_length@std@@8 1003a2c0     LIBCMT:throw_bad_alloc.obj
 0002:000092d0       ??_R2bad_array_new_length@std@@8 1003a2d0     LIBCMT:throw_bad_alloc.obj
 0002:000092e0       ??_R1A@?0A@EA@bad_array_new_length@std@@8 1003a2e0     LIBCMT:throw_bad_alloc.obj
 0002:000092fc       ??_R4type_info@@6B@        1003a2fc     LIBCMT:std_type_info_static.obj
 0002:00009310       ??_R3type_info@@8          1003a310     LIBCMT:std_type_info_static.obj
 0002:00009320       ??_R2type_info@@8          1003a320     LIBCMT:std_type_info_static.obj
 0002:00009328       ??_R1A@?0A@EA@type_info@@8 1003a328     LIBCMT:std_type_info_static.obj
 0002:00009344       ___safe_se_handler_table   1003a344     <linker-defined>
 0002:000096e4       ___rtc_iaa                 1003a6e4     LIBCMT:initsect.obj
 0002:000096e8       ___rtc_izz                 1003a6e8     LIBCMT:initsect.obj
 0002:000096ec       ___rtc_taa                 1003a6ec     LIBCMT:initsect.obj
 0002:000096f0       ___rtc_tzz                 1003a6f0     LIBCMT:initsect.obj
 0002:000096f4       __tls_start                1003a6f4     LIBCMT:tlssup.obj
 0002:000096f8       __Init_thread_epoch        1003a6f8     LIBCMT:thread_safe_statics.obj
 0002:000096fc       __tls_end                  1003a6fc     LIBCMT:tlssup.obj
 0002:0000981c       __TI2?AVbad_alloc@std@@    1003a81c     LIBCMT:throw_bad_alloc.obj
 0002:0000982c       __CTA2?AVbad_alloc@std@@   1003a82c     LIBCMT:throw_bad_alloc.obj
 0002:00009838       __CT??_R0?AVbad_alloc@std@@@8??0bad_alloc@std@@QAE@ABV01@@Z12 1003a838     LIBCMT:throw_bad_alloc.obj
 0002:00009854       __CT??_R0?AVexception@std@@@8??0exception@std@@QAE@ABV01@@Z12 1003a854     LIBCMT:throw_bad_alloc.obj
 0002:00009870       __TI3?AVbad_array_new_length@std@@ 1003a870     LIBCMT:throw_bad_alloc.obj
 0002:00009880       __CTA3?AVbad_array_new_length@std@@ 1003a880     LIBCMT:throw_bad_alloc.obj
 0002:00009890       __CT??_R0?AVbad_array_new_length@std@@@8??0bad_array_new_length@std@@QAE@ABV01@@Z12 1003a890     LIBCMT:throw_bad_alloc.obj
 0002:00009c80       __IMPORT_DESCRIPTOR_KERNEL32 1003ac80     kernel32:KERNEL32.dll
 0002:00009c94       __IMPORT_DESCRIPTOR_USER32 1003ac94     user32:USER32.dll
 0002:00009ca8       __IMPORT_DESCRIPTOR_WS2_32 1003aca8     ws2_32:WS2_32.dll
 0002:00009cbc       __IMPORT_DESCRIPTOR_VERSION 1003acbc     Version:VERSION.dll
 0002:00009cd0       __IMPORT_DESCRIPTOR_IMM32  1003acd0     imm32:IMM32.dll
 0002:00009ce4       __NULL_IMPORT_DESCRIPTOR   1003ace4     kernel32:KERNEL32.dll
 0003:00000000       ___scrt_native_dllmain_reason 1003c000     LIBCMT:utility.obj
 0003:00000004       __Init_global_epoch        1003c004     LIBCMT:thread_safe_statics.obj
 0003:00000008       ___security_cookie_complement 1003c008     LIBCMT:gs_cookie.obj
 0003:0000000c       ___security_cookie         1003c00c     LIBCMT:gs_cookie.obj
 0003:00000010       ___isa_enabled             1003c010     LIBCMT:cpu_disp.obj
 0003:00000030       __NLG_Destination          1003c030     libvcruntime:exsup.obj
 0003:00000040       ___abort_behavior          1003c040     libucrt:abort.obj
 0003:00000058       ___acrt_initial_locale_data 1003c058     libucrt:nlsdata.obj
 0003:00000110       ___acrt_initial_locale_pointers 1003c110     libucrt:nlsdata.obj
 0003:00000118       ___acrt_wide_c_locale_string 1003c118     libucrt:nlsdata.obj
 0003:00000124       __pwctype                  1003c124     libucrt:ctype.obj
 0003:00000128       __iob                      1003c128     libucrt:_file.obj
 0003:000001d0       ___acrt_initial_multibyte_data 1003c1d0     libucrt:mbctype.obj
 0003:000006f0       ___globallocalestatus      1003c6f0     libucrt:glstatus.obj
 0003:000006f8       ___acrt_lconv_c            1003c6f8     libucrt:localeconv.obj
 0003:00000748       ___acrt_lconv_static_decimal 1003c748     libucrt:localeconv.obj
 0003:0000074c       ___acrt_lconv_static_W_decimal 1003c74c     libucrt:localeconv.obj
 0003:00000750       __lookuptrailbytes         1003c750     libucrt:read.obj
 0003:00000870       __fltused                  1003c870     LIBCMT:fltused.obj
 0003:00000880       ?tNoHide@@3UToggleVar@@A   1003c880     GlobalVariable.obj
 0003:00000894       ?tKeepGameWindow@@3UToggleVar@@A 1003c894     GlobalVariable.obj
 0003:000008a8       ?fFixSocketError@@3HA      1003c8a8     GlobalVariable.obj
 0003:000008ac       ?dwSocketTimeOut@@3KA      1003c8ac     GlobalVariable.obj
 0003:000008b0       ?dwSocketTimeOutSec@@3KA   1003c8b0     GlobalVariable.obj
 0003:000008b4       ?tUseCustomFont@@3UToggleVar@@A 1003c8b4     GlobalVariable.obj
 0003:000008c8       ?tInputLine@@3UToggleVar@@A 1003c8c8     GlobalVariable.obj
 0003:000008dc       ?tWisperNotice@@3UToggleVar@@A 1003c8dc     GlobalVariable.obj
 0003:000008f0       ?tSocketProtect@@3UToggleVar@@A 1003c8f0     GlobalVariable.obj
 0003:00000904       ?tAlertNoBug@@3UToggleVar@@A 1003c904     GlobalVariable.obj
 0003:00000918       ?dwBugAlertTimes@@3KA      1003c918     GlobalVariable.obj
 0003:0000091c       ?tBugAutoQuit@@3UToggleVar@@A 1003c91c     GlobalVariable.obj
 0003:00000930       ?tBugKB@@3UToggleVar@@A    1003c930     GlobalVariable.obj
 0003:00000944       ?tBugKD@@3UToggleVar@@A    1003c944     GlobalVariable.obj
 0003:00000958       ?tBugKM@@3UToggleVar@@A    1003c958     GlobalVariable.obj
 0003:0000096c       ?nDangerousMonsterAction@@3KA 1003c96c     GlobalVariable.obj
 0003:00000970       ?tChickenDangerousMonster@@3UToggleVar@@A 1003c970     GlobalVariable.obj
 0003:00000984       ?tChickenHostileNearby@@3UToggleVar@@A 1003c984     GlobalVariable.obj
 0003:00000998       ?tChickenHostile@@3UToggleVar@@A 1003c998     GlobalVariable.obj
 0003:000009ac       ?tChickenLife@@3UToggleVar@@A 1003c9ac     GlobalVariable.obj
 0003:000009c0       ?nChickenLifeAction@@3KA   1003c9c0     GlobalVariable.obj
 0003:000009c4       ?tPlayerHPPercent@@3UToggleVar@@A 1003c9c4     GlobalVariable.obj
 0003:000009d8       ?tPlayerDistance@@3UToggleVar@@A 1003c9d8     GlobalVariable.obj
 0003:000009ec       ?tPlayerLevel@@3UToggleVar@@A 1003c9ec     GlobalVariable.obj
 0003:00000a00       ?nLifeBarColour@@3EA       1003ca00     GlobalVariable.obj
 0003:00000a01       ?nLifeBarTrans@@3EA        1003ca01     GlobalVariable.obj
 0003:00000a02       ?nDefaultExtInfoColour@@3EA 1003ca02     GlobalVariable.obj
 0003:00000a03       ?nQuestItemColour@@3EA     1003ca03     GlobalVariable.obj
 0003:00000a04       ?tMonsterID@@3UToggleVar@@A 1003ca04     GlobalVariable.obj
 0003:00000a18       ?tMonsterDistance@@3UToggleVar@@A 1003ca18     GlobalVariable.obj
 0003:00000a2c       ?tMonsterHPPercent@@3UToggleVar@@A 1003ca2c     GlobalVariable.obj
 0003:00000a40       ?tMonsterResists@@3UToggleVar@@A 1003ca40     GlobalVariable.obj
 0003:00000a54       ?tMonsterRuneTC@@3UToggleVar@@A 1003ca54     GlobalVariable.obj
 0003:00000a68       ?tMonsterTC@@3UToggleVar@@A 1003ca68     GlobalVariable.obj
 0003:00000a7c       ?tMonsterLevel@@3UToggleVar@@A 1003ca7c     GlobalVariable.obj
 0003:00000a90       ?tViewPlayerStatsKey@@3UToggleVar@@A 1003ca90     GlobalVariable.obj
 0003:00000aa4       ?tViewEquipmentKey@@3UToggleVar@@A 1003caa4     GlobalVariable.obj
 0003:00000ab8       ?tPrevPlayerStat@@3UToggleVar@@A 1003cab8     GlobalVariable.obj
 0003:00000acc       ?tNextPlayerStat@@3UToggleVar@@A 1003cacc     GlobalVariable.obj
 0003:00000ae0       ?tFirstPlayerStat@@3UToggleVar@@A 1003cae0     GlobalVariable.obj
 0003:00000af4       ?tShowBaseStat@@3UToggleVar@@A 1003caf4     GlobalVariable.obj
 0003:00000b08       ?tItemExtInfo@@3UToggleVar@@A 1003cb08     GlobalVariable.obj
 0003:00000b1c       ?tVariableAffix@@3UToggleVar@@A 1003cb1c     GlobalVariable.obj
 0003:00000b30       ?tVariableLvl@@3UToggleVar@@A 1003cb30     GlobalVariable.obj
 0003:00000b44       ?tShowItemVariableProp@@3UToggleVar@@A 1003cb44     GlobalVariable.obj
 0003:00000b58       ?tLeftView@@3UToggleVar@@A 1003cb58     GlobalVariable.obj
 0003:00000b6c       ?tViewSocketBase@@3UToggleVar@@A 1003cb6c     GlobalVariable.obj
 0003:00000b80       ?tViewSocketable@@3UToggleVar@@A 1003cb80     GlobalVariable.obj
 0003:00000b94       ?tItemBasicStat@@3UToggleVar@@A 1003cb94     GlobalVariable.obj
 0003:00000ba8       ?tLockAltToggle@@3UToggleVar@@A 1003cba8     GlobalVariable.obj
 0003:00000bbc       ?tPermShowItems@@3UToggleVar@@A 1003cbbc     GlobalVariable.obj
 0003:00000bd0       ?tAutoPickItems@@3UToggleVar@@A 1003cbd0     GlobalVariable.obj
 0003:00000be4       ?tHiddenItems@@3UToggleVar@@A 1003cbe4     GlobalVariable.obj
 0003:00000bf8       ?tShowIdentifiedItem@@3UToggleVar@@A 1003cbf8     GlobalVariable.obj
 0003:00000c0c       ?tShowBaseED@@3UToggleVar@@A 1003cc0c     GlobalVariable.obj
 0003:00000c20       ?dwItemValueNpc@@3PAKA     1003cc20     GlobalVariable.obj
 0003:00000c34       ?tItemStatShow@@3UToggleVar@@A 1003cc34     GlobalVariable.obj
 0003:00000c48       ?tLifePerLevel@@3UToggleVar@@A 1003cc48     GlobalVariable.obj
 0003:00000c5c       ?tAfterCube@@3UToggleVar@@A 1003cc5c     GlobalVariable.obj
 0003:00000c70       ?tItemALevel@@3UToggleVar@@A 1003cc70     GlobalVariable.obj
 0003:00000c84       ?tItemMLevel@@3UToggleVar@@A 1003cc84     GlobalVariable.obj
 0003:00000c98       ?tItemQLevel@@3UToggleVar@@A 1003cc98     GlobalVariable.obj
 0003:00000cac       ?tUnitNumber@@3UToggleVar@@A 1003ccac     GlobalVariable.obj
 0003:00000cc0       ?tItemFileIndex@@3UToggleVar@@A 1003ccc0     GlobalVariable.obj
 0003:00000cd4       ?tItemIndex@@3UToggleVar@@A 1003ccd4     GlobalVariable.obj
 0003:00000ce8       ?tItemValue@@3UToggleVar@@A 1003cce8     GlobalVariable.obj
 0003:00000cfc       ?tItemLevel@@3UToggleVar@@A 1003ccfc     GlobalVariable.obj
 0003:00000d10       ?tSocketNumbers@@3UToggleVar@@A 1003cd10     GlobalVariable.obj
 0003:00000d24       ?tRuneNumbers@@3UToggleVar@@A 1003cd24     GlobalVariable.obj
 0003:00000d38       ?nItemShowMode@@3KA        1003cd38     GlobalVariable.obj
 0003:00000d3c       ?tSwitchItemMode@@3UToggleVar@@A 1003cd3c     GlobalVariable.obj
 0003:00000d50       ?anGoldPoorCol@@3PADA      1003cd50     GlobalVariable.obj
 0003:00000d54       ?anGoldGoodCol@@3PADA      1003cd54     GlobalVariable.obj
 0003:00000d58       ?tPermShowOrb@@3UToggleVar@@A 1003cd58     GlobalVariable.obj
 0003:00000d6c       ?tStateMonitorToggle@@3UToggleVar@@A 1003cd6c     GlobalVariable.obj
 0003:00000d80       ?tGetHitCount@@3UToggleVar@@A 1003cd80     GlobalVariable.obj
 0003:00000d94       ?tKillCount@@3UToggleVar@@A 1003cd94     GlobalVariable.obj
 0003:00000da8       ?tShowPartyLevel@@3UToggleVar@@A 1003cda8     GlobalVariable.obj
 0003:00000dbc       ?tShowPartyPosition@@3UToggleVar@@A 1003cdbc     GlobalVariable.obj
 0003:00000dd0       ?tQuickNextGame2@@3UToggleVar@@A 1003cdd0     GlobalVariable.obj
 0003:00000de4       ?tQuickNextGame@@3UToggleVar@@A 1003cde4     GlobalVariable.obj
 0003:00000df8       ?tExitGame@@3UToggleVar@@A 1003cdf8     GlobalVariable.obj
 0003:00000e0c       ?tMousePosition@@3UToggleVar@@A 1003ce0c     GlobalVariable.obj
 0003:00000e20       ?tAreaLevel@@3UToggleVar@@A 1003ce20     GlobalVariable.obj
 0003:00000e34       ?tLayerLevelNo@@3UToggleVar@@A 1003ce34     GlobalVariable.obj
 0003:00000e48       ?tClock@@3UToggleVar@@A    1003ce48     GlobalVariable.obj
 0003:00000e5c       ?tGameTime@@3UToggleVar@@A 1003ce5c     GlobalVariable.obj
 0003:00000e70       ?tServerIp@@3UToggleVar@@A 1003ce70     GlobalVariable.obj
 0003:00000e84       ?tULCMask@@3UToggleVar@@A  1003ce84     GlobalVariable.obj
 0003:00000e98       ?tQuickDropToggle@@3UToggleVar@@A 1003ce98     GlobalVariable.obj
 0003:00000eac       ?tCtrlClickSwap@@3UToggleVar@@A 1003ceac     GlobalVariable.obj
 0003:00000ec0       ?tRightClickSwap@@3UToggleVar@@A 1003cec0     GlobalVariable.obj
 0003:00000ed4       ?dwMessageFileSize@@3KA    1003ced4     GlobalVariable.obj
 0003:00000ed8       ?tLogMessage@@3UToggleVar@@A 1003ced8     GlobalVariable.obj
 0003:00000eec       ?tShowPing@@3UToggleVar@@A 1003ceec     GlobalVariable.obj
 0003:00000f00       ?tShowExp@@3UToggleVar@@A  1003cf00     GlobalVariable.obj
 0003:00000f14       ?tAutoEnchant@@3UToggleVar@@A 1003cf14     GlobalVariable.obj
 0003:00000f28       ?tOutTownSelect@@3UToggleVar@@A 1003cf28     GlobalVariable.obj
 0003:00000f3c       ?mAutoPartyDelays@@3KA     1003cf3c     GlobalVariable.obj
 0003:00000f40       ?tAutoPermit@@3UToggleVar@@A 1003cf40     GlobalVariable.obj
 0003:00000f54       ?tAutoInvite@@3UToggleVar@@A 1003cf54     GlobalVariable.obj
 0003:00000f68       ?tAutoParty@@3UToggleVar@@A 1003cf68     GlobalVariable.obj
 0003:00000f7c       ?nTownportalAlertNums@@3KA 1003cf7c     GlobalVariable.obj
 0003:00000f80       ?tBackToTown@@3UToggleVar@@A 1003cf80     GlobalVariable.obj
 0003:00000f94       ?nScrollMode@@3KA          1003cf94     GlobalVariable.obj
 0003:00000f98       ?nMapScrollSpeed@@3KA      1003cf98     GlobalVariable.obj
 0003:00000f9c       ?tCenterMap@@3UToggleVar@@A 1003cf9c     GlobalVariable.obj
 0003:00000fb0       ?tScrollMap@@3UToggleVar@@A 1003cfb0     GlobalVariable.obj
 0003:00000fc4       ?tDiagonalScroll@@3UToggleVar@@A 1003cfc4     GlobalVariable.obj
 0003:00000fd8       ?tHiddenCorpse@@3UToggleVar@@A 1003cfd8     GlobalVariable.obj
 0003:00000fec       ?tScreenshake@@3UToggleVar@@A 1003cfec     GlobalVariable.obj
 0003:00001000       ?tInfravision@@3UToggleVar@@A 1003d000     GlobalVariable.obj
 0003:00001014       ?tLightRadiu@@3UToggleVar@@A 1003d014     GlobalVariable.obj
 0003:00001028       ?tWeather@@3UToggleVar@@A  1003d028     GlobalVariable.obj
 0003:0000103c       ?tFullVisuals@@3UToggleVar@@A 1003d03c     GlobalVariable.obj
 0003:00001050       ?tBossNameToggle@@3UToggleVar@@A 1003d050     GlobalVariable.obj
 0003:00001064       ?nMonsterTextCol@@3EA      1003d064     GlobalVariable.obj
 0003:00001065       ?nHostileTextColour@@3EA   1003d065     GlobalVariable.obj
 0003:00001066       ?nNeutralTextColour@@3EA   1003d066     GlobalVariable.obj
 0003:00001067       ?nPartyTextColour@@3EA     1003d067     GlobalVariable.obj
 0003:00001068       ?nPlayerMinionColor@@3EA   1003d068     GlobalVariable.obj
 0003:00001069       ?nFriendMinionColor@@3EA   1003d069     GlobalVariable.obj
 0003:0000106a       ?nHostilePlayerColor@@3EA  1003d06a     GlobalVariable.obj
 0003:0000106b       ?nNeutralPlayerColor@@3EA  1003d06b     GlobalVariable.obj
 0003:0000106c       ?nSuperUniqueColor@@3EA    1003d06c     GlobalVariable.obj
 0003:0000106d       ?nMonsterChampColor@@3EA   1003d06d     GlobalVariable.obj
 0003:0000106e       ?nMonsterMinionColor@@3EA  1003d06e     GlobalVariable.obj
 0003:0000106f       ?nMonsterBossColor@@3EA    1003d06f     GlobalVariable.obj
 0003:00001070       ?nMonsterNormalColor@@3EA  1003d070     GlobalVariable.obj
 0003:00001071       ?nChampionCorpseColor@@3EA 1003d071     GlobalVariable.obj
 0003:00001072       ?nMinionCorpseColor@@3EA   1003d072     GlobalVariable.obj
 0003:00001073       ?nBossCorpseColor@@3EA     1003d073     GlobalVariable.obj
 0003:00001074       ?nNormalCorpseColor@@3EA   1003d074     GlobalVariable.obj
 0003:00001075       ?nLockedChestColor@@3EA    1003d075     GlobalVariable.obj
 0003:00001076       ?nClosedChestColor@@3EA    1003d076     GlobalVariable.obj
 0003:00001077       ?nOtherMissileColor@@3EA   1003d077     GlobalVariable.obj
 0003:00001078       ?nTracerMissileColor@@3EA  1003d078     GlobalVariable.obj
 0003:00001079       ?nGuidedMissileColor@@3EA  1003d079     GlobalVariable.obj
 0003:0000107a       ?nHostileMissileColor@@3EA 1003d07a     GlobalVariable.obj
 0003:0000107b       ?nMinimapCellCol@@3EA      1003d07b     GlobalVariable.obj
 0003:0000107c       ?tAutomapItems@@3UToggleVar@@A 1003d07c     GlobalVariable.obj
 0003:00001090       ?tAutomapMissiles@@3UToggleVar@@A 1003d090     GlobalVariable.obj
 0003:000010a4       ?tAutomapChests@@3UToggleVar@@A 1003d0a4     GlobalVariable.obj
 0003:000010b8       ?tAutomapMonsters@@3UToggleVar@@A 1003d0b8     GlobalVariable.obj
 0003:000010cc       ?tAutomapCorpse@@3UToggleVar@@A 1003d0cc     GlobalVariable.obj
 0003:000010e0       ?tMinimap@@3UToggleVar@@A  1003d0e0     GlobalVariable.obj
 0003:000010f4       ?nMinimapSize@@3EA         1003d0f4     GlobalVariable.obj
 0003:000010f5       ?nAutomapScreenColors@@3EA 1003d0f5     GlobalVariable.obj
 0003:000010f6       ?nAutomapReadyColors@@3EA  1003d0f6     GlobalVariable.obj
 0003:000010f7       ?nAutomapActiveRoomColors@@3EA 1003d0f7     GlobalVariable.obj
 0003:000010f8       ?tAutomapScreenArea@@3UToggleVar@@A 1003d0f8     GlobalVariable.obj
 0003:0000110c       ?tAutomapReadyRoom@@3UToggleVar@@A 1003d10c     GlobalVariable.obj
 0003:00001120       ?tAutomapActiveRoom@@3UToggleVar@@A 1003d120     GlobalVariable.obj
 0003:00001134       ?tMiniShrine@@3UToggleVar@@A 1003d134     GlobalVariable.obj
 0003:00001148       ?tAutomapLevelNames@@3UToggleVar@@A 1003d148     GlobalVariable.obj
 0003:0000115c       ?tAutoMap@@3UToggleVar@@A  1003d15c     GlobalVariable.obj
 0003:00001170       ?tRevealLevel@@3UToggleVar@@A 1003d170     GlobalVariable.obj
 0003:00001184       ?tRevealAct@@3UToggleVar@@A 1003d184     GlobalVariable.obj
 0003:00001198       ?fAutoSetCHISupport@@3HA   1003d198     GlobalVariable.obj
 0003:0000119c       ?fLanguageCheck@@3HA       1003d19c     GlobalVariable.obj
 0003:000011a0       ?fAutomapNamesDefault@@3EA 1003d1a0     GlobalVariable.obj
 0003:000011a1       ?fAutomapPartyDefault@@3EA 1003d1a1     GlobalVariable.obj
 0003:000011a4       ?fShowCheckInfo@@3KA       1003d1a4     GlobalVariable.obj
 0003:000011a8       ?tReloadConfig@@3UToggleVar@@A 1003d1a8     GlobalVariable.obj
 0003:000011bc       ?actlvls@@3PAKA            1003d1bc     GlobalVariable.obj
 0003:000011d4       ?dwGameLng@@3HA            1003d1d4     GlobalVariable.obj
 0003:000011d8       ?fDefault@@3HA             1003d1d8     GlobalVariable.obj
 0003:000011dc       ?dwCurrentLevel@@3KA       1003d1dc     GlobalVariable.obj
 0003:000011e0       ?fPlayerInTown@@3HA        1003d1e0     GlobalVariable.obj
 0003:000011e4       ?szOrbPattern@@3PADA       1003d1e4     ShowOrbs.obj
 0003:000011e8       ?viewEquUnit@@3UViewUnitInfo@@A 1003d1e8     ViewTargetUnitInfo.obj
 0003:000011f8       ?viewStatUnit@@3UViewUnitInfo@@A 1003d1f8     ViewTargetUnitInfo.obj
 0003:00003cc0       ??_R0?AVbad_alloc@std@@@8  1003fcc0     LIBCMT:throw_bad_alloc.obj
 0003:00003cdc       ??_R0?AVexception@std@@@8  1003fcdc     LIBCMT:throw_bad_alloc.obj
 0003:00003cf8       ??_R0?AVbad_array_new_length@std@@@8 1003fcf8     LIBCMT:throw_bad_alloc.obj
 0003:00003d20       ??_R0?AVtype_info@@@8      1003fd20     LIBCMT:std_type_info_static.obj
 0003:00003d38       ___scrt_current_native_startup_state 1003fd38     LIBCMT:utility.obj
 0003:00003d3c       ___scrt_native_startup_lock 1003fd3c     LIBCMT:utility.obj
 0003:000040a8       ___isa_available           100400a8     LIBCMT:cpu_disp.obj
 0003:000040ac       ___favor                   100400ac     LIBCMT:cpu_disp.obj
 0003:000040b0       ___scrt_debugger_hook_flag 100400b0     LIBCMT:utility_desktop.obj
 0003:000040b4       ___castguard_check_failure_os_handled_fptr 100400b4     LIBCMT:guard_support.obj
 0003:000040b8       __tls_index                100400b8     LIBCMT:tlssup.obj
 0003:000040c0       ?__type_info_root_node@@3U__type_info_node@@A 100400c0     LIBCMT:tncleanup.obj
 0003:000040c8       ?_OptionsStorage@?1??__local_stdio_scanf_options@@9@4_KA 100400c8     LIBCMT:default_local_stdio_options.obj
 0003:000040d0       ?__WinRTOutOfMemoryExceptionCallback@@3P6GPAXXZA 100400d0     libvcruntime:ehhelpers.obj
 0003:00004118       ?pArgList@UnDecorator@@0PAVReplicator@@A 10040118     libvcruntime:undname.obj
 0003:0000411c       ?pZNameList@UnDecorator@@0PAVReplicator@@A 1004011c     libvcruntime:undname.obj
 0003:00004120       ?pTemplateArgList@UnDecorator@@0PAVReplicator@@A 10040120     libvcruntime:undname.obj
 0003:00004124       ?gName@UnDecorator@@0PBDB  10040124     libvcruntime:undname.obj
 0003:00004128       ?name@UnDecorator@@0PBDB   10040128     libvcruntime:undname.obj
 0003:0000412c       ?disableFlags@UnDecorator@@0KA 1004012c     libvcruntime:undname.obj
 0003:00004130       ?fExplicitTemplateParams@UnDecorator@@0_NA 10040130     libvcruntime:undname.obj
 0003:00004131       ?fGetTemplateArgumentList@UnDecorator@@0_NA 10040131     libvcruntime:undname.obj
 0003:00004134       ?m_pGetParameter@UnDecorator@@0P6APADJ@ZA 10040134     libvcruntime:undname.obj
 0003:00004138       ?m_CHPENameOffset@UnDecorator@@0KA 10040138     libvcruntime:undname.obj
 0003:0000413c       ?m_recursionLevel@UnDecorator@@0KA 1004013c     libvcruntime:undname.obj
 0003:00004174       ___pPurecall               10040174     libvcruntime:purevirt_data.obj
 0003:00004180       ?c_exit_complete@?1???R<lambda_6e4b09c48022b2350581041d5f6b0c4c>@@QBE@XZ@4_NA 10040180     libucrt:exit.obj
 0003:00004290       __environ_table            10040290     libucrt:environment_initialization.obj
 0003:00004294       __wenviron_table           10040294     libucrt:environment_initialization.obj
 0003:00004298       ___dcrt_initial_wide_environment 10040298     libucrt:environment_initialization.obj
 0003:0000429c       ___dcrt_initial_narrow_environment 1004029c     libucrt:environment_initialization.obj
 0003:000042a0       ___acrt_atexit_table       100402a0     libucrt:onexit.obj
 0003:000042ac       ___acrt_at_quick_exit_table 100402ac     libucrt:onexit.obj
 0003:000042bc       ___acrt_locale_changed_data 100402bc     libucrt:wsetlocale.obj
 0003:000042c0       ___acrt_current_locale_data 100402c0     libucrt:nlsdata.obj
 0003:000042d0       __nstream                  100402d0     libucrt:_file.obj
 0003:000042d4       ___piob                    100402d4     libucrt:_file.obj
 0003:000042dc       ___acrt_stdout_buffer      100402dc     libucrt:_sftbuf.obj
 0003:000042e0       ___acrt_stderr_buffer      100402e0     libucrt:_sftbuf.obj
 0003:000042e8       ___pioinfo                 100402e8     libucrt:ioinit.obj
 0003:000044e8       __nhandle                  100404e8     libucrt:ioinit.obj
 0003:0000471c       __mbctype                  1004071c     libucrt:mbctype.obj
 0003:00004720       __mbcasemap                10040720     libucrt:mbctype.obj
 0003:00004724       ___acrt_current_multibyte_data 10040724     libucrt:mbctype.obj
 0003:00004730       __pgmptr                   10040730     libucrt:argv_data.obj
 0003:00004734       ___argc                    10040734     libucrt:argv_data.obj
 0003:00004738       ___argv                    10040738     libucrt:argv_data.obj
 0003:0000473c       ___wargv                   1004073c     libucrt:argv_data.obj
 0003:00004740       __acmdln                   10040740     libucrt:argv_data.obj
 0003:00004744       __wcmdln                   10040744     libucrt:argv_data.obj
 0003:00004748       ___acrt_heap               10040748     libucrt:heap_handle.obj
 0003:00004760       ___acrt_lconv_static_null  10040760     libucrt:localeconv.obj
 0003:00004764       ___acrt_lconv_static_W_null 10040764     libucrt:localeconv.obj
 0003:0000476c       ___fastflag                1004076c     libucrt:fp_flags.obj
 0003:00004780       ?szPluginPath@@3PADA       10040780     DllMain.obj
 0003:00004884       ?hInstDLL@@3PAUHINSTANCE__@@A 10040884     DllMain.obj
 0003:00004888       ?fFullWindows@@3HA         10040888     GlobalVariable.obj
 0003:0000488c       ?pD2WinEditBox@@3PAUD2EditBox@@A 1004088c     GlobalVariable.obj
 0003:00004890       ?anDangerousMonster@@3PAY01DA 10040890     GlobalVariable.obj
 0003:00005060       ?dwChickenHostileNearbyLifePercent@@3KA 10041060     GlobalVariable.obj
 0003:00005064       ?dwChickenHostileLifePercent@@3KA 10041064     GlobalVariable.obj
 0003:00005068       ?dwChickenLifePercent@@3KA 10041068     GlobalVariable.obj
 0003:0000506c       ?dwChickenHostileNearbyLife@@3KA 1004106c     GlobalVariable.obj
 0003:00005070       ?dwChickenHostileLife@@3KA 10041070     GlobalVariable.obj
 0003:00005074       ?dwChickenLife@@3KA        10041074     GlobalVariable.obj
 0003:00005078       ?fDangerousMonsterActive@@3HA 10041078     GlobalVariable.obj
 0003:0000507c       ?fLifeProtectOn@@3HA       1004107c     GlobalVariable.obj
 0003:00005080       ?szItemExtInfoCfgName@@3PAY0BAA@DA 10041080     GlobalVariable.obj
 0003:00005280       ?anItemPicks@@3PAY37163DA  10041280     GlobalVariable.obj
 0003:00295680       ?nSkillMonitors@@3HA       102d1680     GlobalVariable.obj
 0003:00295684       ?wszEtherealItemPostfix@@3PA_WA 102d1684     GlobalVariable.obj
 0003:002956c0       ?sItemSkillStr@@3PAUStatMonitor@@A 102d16c0     GlobalVariable.obj
 0003:002a6060       ?wszEtherealItemPrefix@@3PA_WA 102e2060     GlobalVariable.obj
 0003:002a609c       ?dwGoldGoodNum@@3KA        102e209c     GlobalVariable.obj
 0003:002a60a0       ?anItemHideLevel@@3PAY07DA 102e20a0     GlobalVariable.obj
 0003:002abe60       ?anItemColours@@3PAY37163DA 102e7e60     GlobalVariable.obj
 0003:003f4060       ?anRuneColours@@3PAY03DA   10430060     GlobalVariable.obj
 0003:003f41f0       ?nMonitors@@3HA            104301f0     GlobalVariable.obj
 0003:003f41f4       ?dwOrgMode@@3KA            104301f4     GlobalVariable.obj
 0003:003f41f8       ?sMonitorStr@@3PAUStatMonitor@@A 104301f8     GlobalVariable.obj
 0003:003fac38       ?dwGetHits@@3KA            10436c38     GlobalVariable.obj
 0003:003fac3c       ?dwGetHitSum@@3KA          10436c3c     GlobalVariable.obj
 0003:003fac40       ?dwLastKills@@3KA          10436c40     GlobalVariable.obj
 0003:003fac44       ?dwGameKills@@3KA          10436c44     GlobalVariable.obj
 0003:003fac48       ?dwKillSum@@3KA            10436c48     GlobalVariable.obj
 0003:003fac4c       ?fGameFilter@@3HA          10436c4c     GlobalVariable.obj
 0003:003fac50       ?fCanExitGame@@3HA         10436c50     GlobalVariable.obj
 0003:003fac54       ?fAutoNextGamePassword@@3HA 10436c54     GlobalVariable.obj
 0003:003fac58       ?fAutoNextGameName@@3HA    10436c58     GlobalVariable.obj
 0003:003fac5c       ?mSkipQuestMessage@@3KA    10436c5c     GlobalVariable.obj
 0003:003fac60       ?wszGamePassword@@3PA_WA   10436c60     GlobalVariable.obj
 0003:003faca0       ?wszGameName@@3PA_WA       10436ca0     GlobalVariable.obj
 0003:003face0       ?currentgameexp@@3HA       10436ce0     GlobalVariable.obj
 0003:003face4       ?fCanPermit@@3HA           10436ce4     GlobalVariable.obj
 0003:003face8       ?fCanInvite@@3HA           10436ce8     GlobalVariable.obj
 0003:003facec       ?fBackToTown@@3HA          10436cec     GlobalVariable.obj
 0003:003facf0       ?tMapScrollKey@@3PAUToggleVar@@A 10436cf0     GlobalVariable.obj
 0003:003fada4       ?nSuperUniqueDescFont@@3EA 10436da4     GlobalVariable.obj
 0003:003fada5       ?nCaveNameTextCol@@3EA     10436da5     GlobalVariable.obj
 0003:003fada8       ?nMapScrollOffset@@3PAY141DA 10436da8     GlobalVariable.obj
 0003:003fae04       ?fAutoRevealAct@@3HA       10436e04     GlobalVariable.obj
 0003:003fae08       ?afMonsterDeathAnims@@3PAEA 10436e08     GlobalVariable.obj
 0003:003fb1f0       ?afMissileCorpses@@3PAEA   104371f0     GlobalVariable.obj
 0003:003fb5d8       ?afMonsterCorpses@@3PAEA   104375d8     GlobalVariable.obj
 0003:003fb9c0       ?anMonsterColours@@3PAEA   104379c0     GlobalVariable.obj
 0003:003fc190       ?anMissileColours@@3PAEA   10438190     GlobalVariable.obj
 0003:003fc578       ?anMonsterCorpseColors@@3PAEA 10438578     GlobalVariable.obj
 0003:003fc960       ?awszImmuneDescs@@3PAY0BE@_WA 10438960     GlobalVariable.obj
 0003:003fca50       ?awszAuraDescs@@3PAY0BE@_WA 10438a50     GlobalVariable.obj
 0003:003fcb68       ?awszEnchantDescs@@3PAY0BE@_WA 10438b68     GlobalVariable.obj
 0003:003fd338       ?wszStaffTombLvlDesc@@3PA_WA 10439338     GlobalVariable.obj
 0003:003fd39c       ?fLocalizationSupport@@3HA 1043939c     GlobalVariable.obj
 0003:003fd3a0       ?pMinimapObjectCell@@3PAUCellFile@@A 104393a0     GlobalVariable.obj
 0003:003fd3a4       ?pWaypointCell@@3PAUCellFile@@A 104393a4     GlobalVariable.obj
 0003:003fd3a8       ?apMyShrineCells@@3PAY0BH@PAUCellFile@@A 104393a8     GlobalVariable.obj
 0003:003fd460       ?pUnitBlobCells@@3PAPAUCellFile@@A 10439460     GlobalVariable.obj
 0003:003fd5f8       ?aszUnitBlobFiles@@3PAY0DC@DA 104395f8     GlobalVariable.obj
 0003:003fe9e4       ?fEnterGameSound@@3HA      1043a9e4     GlobalVariable.obj
 0003:003fe9e8       ?wszCFGVersion@@3PAY0BAA@_WA 1043a9e8     GlobalVariable.obj
 0003:003fede8       ?szCFGVersion@@3PAY0BAA@DA 1043ade8     GlobalVariable.obj
 0003:003fefe8       ?dwPlayerId@@3KA           1043afe8     GlobalVariable.obj
 0003:003fefec       ?dwKeyDown@@3KA            1043afec     GlobalVariable.obj
 0003:003feff0       ?fKeyRepeat@@3HA           1043aff0     GlobalVariable.obj
 0003:003feff4       ?dwCurrentAct@@3KA         1043aff4     GlobalVariable.obj
 0003:003feff8       ?fInGame@@3HA              1043aff8     GlobalVariable.obj
 0003:003feffc       ?fInstallPatch2@@3HA       1043affc     Install.obj
 0003:003ff000       ?nKeyCount@@3HA            1043b000     LoadConfig.obj
 0003:003ff004       ?fViewSocketableOn@@3HA    1043b004     ItemDesc.obj
 0003:003ff008       ?tKeyEvent@@3PAPAUToggleVar@@A 1043b008     LoadConfig.obj
 0003:003ff198       ?aMinimapConfigs@@3PAUMinimapConfig@@A 1043b198     LoadConfig.obj
 0003:00403568       ?wszDescText@@3PA_WA       1043f568     ItemDesc.obj
 0003:00403d68       ?fViewSockFlag@@3HA        1043fd68     ItemDesc.obj
 0003:00403d6c       ?tempItem@@3PAUUnitAny@@A  1043fd6c     ItemInGround.obj
 0003:00403d70       ?aMinimapPoints@@3PAUMinimapPoint@@A 1043fd70     MinimapPoint.obj
 0003:0040b350       ?mimimapCells@@3PAHA       10447350     MinimapPoint.obj
 0003:0040b5e0       ?aMinimapCells@@3PAY0BO@UMinimapCell@@A 104475e0     MinimapPoint.obj
 0003:00412930       ?fMyChatOn@@3HA            1044e930     GameChat.obj
 0003:00412934       ?fAddlistProc@@3HA         1044e934     GameFilter.obj
 0003:00412938       ?fQuickRefresh@@3HA        1044e938     GameFilter.obj
 0003:0041293c       ?fKeepWindowPatch@@3HA     1044e93c     GameWindow.obj
 0003:00412944       ?vD2ERR@@3KC               1044e944     Install.obj
 0003:00412948       ?vD2StartOfPtr@@3KC        1044e948     Install.obj
 0003:0041294c       ?vD2VD2SendToServer3@@3KC  1044e94c     Install.obj
 0003:00412950       ?D2ShowGameMessage@@3P6GXPA_WH@ZA 1044e950     Install.obj
 0003:00412954       ?D2ShowPartyMessage@@3P6GXPA_WH@ZA 1044e954     Install.obj
 0003:00412958       ?D2ShowMap@@3P6IXXZA       1044e958     Install.obj
 0003:0041295c       ?D2RevealAutomapRoom@@3P6GXPAUDrlgRoom1@@KPAUAutomapLayer@@@ZA 1044e95c     Install.obj
 0003:00412960       ?D2RecvCommand07@@3P6IXPAE@ZA 1044e960     Install.obj
 0003:00412964       ?D2RecvCommand08@@3P6IXPAE@ZA 1044e964     Install.obj
 0003:00412968       ?D2NewAutomapCell@@3P6IPAUAutomapCell@@XZA 1044e968     Install.obj
 0003:0041296c       ?D2AddAutomapCell@@3P6IXPAUAutomapCell@@PAPAU1@@ZA 1044e96c     Install.obj
 0003:00412970       ?D2GetPlayerXOffset@@3P6GJXZA 1044e970     Install.obj
 0003:00412974       ?D2GetPlayerYOffset@@3P6GJXZA 1044e974     Install.obj
 0003:00412978       ?D2SetUiStatus@@3P6IKKKK@ZA 1044e978     Install.obj
 0003:0041297c       ?D2CalcShake@@3P6GXPAK0@ZA 1044e97c     Install.obj
 0003:00412980       ?D2GetMonsterOwner@@3P6IKK@ZA 1044e980     Install.obj
 0003:00412984       ?D2GetUnitFromId@@3P6IPAUUnitAny@@KK@ZA 1044e984     Install.obj
 0003:00412988       ?D2GetSelectedUnit@@3P6GPAUUnitAny@@XZA 1044e988     Install.obj
 0003:0041298c       ?D2InitAutomapLayerStub@@3P6IPAUAutomapLayer@@K@ZA 1044e98c     Install.obj
 0003:00412990       ?D2CheckUiStatusStub@@3P6IKK@ZA 1044e990     Install.obj
 0003:00412994       ?D2SetAutomapPartyStub@@3P6IXK@ZA 1044e994     Install.obj
 0003:00412998       ?D2SetAutomapNamesStub@@3P6IXK@ZA 1044e998     Install.obj
 0003:0041299c       ?D2ChatInputStub@@3P6GXPAUD2MSG@@@ZA 1044e99c     Install.obj
 0003:004129a0       ?D2ItemProtect@@3P6GXPAUUnitAny@@K@ZA 1044e9a0     Install.obj
 0003:004129a4       ?D2DrawClient@@3P6IXXZA    1044e9a4     Install.obj
 0003:004129a8       ?D2Storm511@@3P6GXPAUD2MSG@@@ZA 1044e9a8     Install.obj
 0003:004129ac       ?p_D2AutomapLayerList@@3PAPAUAutomapLayer@@A 1044e9ac     Install.obj
 0003:004129b0       ?p_D2AutomapLayer@@3PAPAUAutomapLayer@@A 1044e9b0     Install.obj
 0003:004129b4       ?p_D2PlayerUnit@@3PAPAUUnitAny@@A 1044e9b4     Install.obj
 0003:004129b8       ?p_D2RosterUnitList@@3PAPAURosterUnit@@A 1044e9b8     Install.obj
 0003:004129bc       ?p_D2PetUnitList@@3PAPAUPetUnit@@A 1044e9bc     Install.obj
 0003:004129c0       ?p_D2DrlgAct@@3PAPAUDrlgAct@@A 1044e9c0     Install.obj
 0003:004129c4       ?p_D2Expansion@@3PAKA      1044e9c4     Install.obj
 0003:004129c8       ?p_D2Difficulty@@3PAEA     1044e9c8     Install.obj
 0003:004129cc       ?p_D2GameInfo@@3PAPAUGameStructInfo@@A 1044e9cc     Install.obj
 0003:004129d0       ?p_D2Fps@@3PAKA            1044e9d0     Install.obj
 0003:004129d4       ?p_D2Ping@@3PAKA           1044e9d4     Install.obj
 0003:004129d8       ?p_D2ExitAppFlag@@3PAKA    1044e9d8     Install.obj
 0003:004129dc       ?p_D2InGame@@3PAHA         1044e9dc     Install.obj
 0003:004129e0       ?p_D2AutomapOn@@3PAKA      1044e9e0     Install.obj
 0003:004129e4       ?p_D2Divisor@@3PAJA        1044e9e4     Install.obj
 0003:004129e8       ?p_D2Offset@@3PAUtagPOINT@@A 1044e9e8     Install.obj
 0003:004129ec       ?p_D2AutomapPos@@3PAUtagPOINT@@A 1044e9ec     Install.obj
 0003:004129f0       ?p_D2AutoMapSize@@3PAUtagPOINT@@A 1044e9f0     Install.obj
 0003:004129f4       ?p_D2MinmapType@@3PAKA     1044e9f4     Install.obj
 0003:004129f8       ?p_D2MinimapOffset@@3PAUtagPOINT@@A 1044e9f8     Install.obj
 0003:004129fc       ?p_D2IsMapShakeOn@@3PAHA   1044e9fc     Install.obj
 0003:00412a00       ?p_D2MapShakeY@@3PAJA      1044ea00     Install.obj
 0003:00412a04       ?p_D2MapShakeX@@3PAJA      1044ea04     Install.obj
 0003:00412a08       ?p_D2ScreenSizeX@@3PAHA    1044ea08     Install.obj
 0003:00412a0c       ?p_D2ScreenSizeY@@3PAHA    1044ea0c     Install.obj
 0003:00412a10       ?p_D2ScreenSize@@3PAUtagPOINT@@A 1044ea10     Install.obj
 0003:00412a14       ?p_D2DrawOffset@@3PAUtagPOINT@@A 1044ea14     Install.obj
 0003:00412a18       ?p_D2InfoPositionX@@3PAHA  1044ea18     Install.obj
 0003:00412a1c       ?p_D2InfoPositionY@@3PAHA  1044ea1c     Install.obj
 0003:00412a20       ?p_D2QuestData@@3PAPAXA    1044ea20     Install.obj
 0003:00412a24       ?p_D2GameQuestData@@3PAPAXA 1044ea24     Install.obj
 0003:00412a28       ?p_D2QuestPage@@3PAHA      1044ea28     Install.obj
 0003:00412a2c       ?p_D2MButton@@3PAHA        1044ea2c     Install.obj
 0003:00412a30       ?p_D2LastChatMessage@@3PA_WA 1044ea30     Install.obj
 0003:00412a34       ?p_D2ChatTextLength@@3PAHA 1044ea34     Install.obj
 0003:00412a38       ?p_D2MousePos@@3PAUD2_POINT_REV@@A 1044ea38     Install.obj
 0003:00412a3c       ?p_D2LastMousePos@@3PAUD2_POINT_REV@@A 1044ea3c     Install.obj
 0003:00412a40       ?p_D2CursorInvGridX@@3PAKA 1044ea40     Install.obj
 0003:00412a44       ?p_D2CursorInvGridY@@3PAKA 1044ea44     Install.obj
 0003:00412a48       ?p_D2CurrentViewItem@@3PAPAUUnitAny@@A 1044ea48     Install.obj
 0003:00412a4c       ?p_D2GoldInTranBox@@3PAHA  1044ea4c     Install.obj
 0003:00412a50       ?p_D2ShowLifeStr@@3PAHA    1044ea50     Install.obj
 0003:00412a54       ?p_D2ShowManaStr@@3PAHA    1044ea54     Install.obj
 0003:00412a58       ?vD2AutomapCellListBaseAddr@@3KA 1044ea58     Install.obj
 0003:00412a5c       ?vD2LoadUiImageFunc@@3KA   1044ea5c     Install.obj
 0003:00412a60       ?D2GetObjectTxt@@3P6GPAUObjectTxt@@K@ZA 1044ea60     Install.obj
 0003:00412a64       ?D2GetLevelDefTxt@@3P6IPAULevelDefTxt@@K@ZA 1044ea64     Install.obj
 0003:00412a68       ?D2GetLevelTxt@@3P6GPAULevelTxt@@K@ZA 1044ea68     Install.obj
 0003:00412a6c       ?D2GetItemTxt@@3P6GPAUItemTxt@@K@ZA 1044ea6c     Install.obj
 0003:00412a70       ?D2GetItemTxt2@@3P6GPAUItemTxt3@@K@ZA 1044ea70     Install.obj
 0003:00412a74       ?D2GetItemTxt3@@3P6GPAUItemTxt2@@K@ZA 1044ea74     Install.obj
 0003:00412a78       ?D2GetTreasureClasses@@3P6GPAUTreasureClass@@GK@ZA 1044ea78     Install.obj
 0003:00412a7c       ?D2GetSuperUniqueTxt@@3P6GPAUSuperUniqueTxt@@K@ZA 1044ea7c     Install.obj
 0003:00412a80       ?D2CheckItemType@@3P6GHPAUUnitAny@@K@ZA 1044ea80     Install.obj
 0003:00412a84       ?D2GetItemFileIndex@@3P6GKPAUUnitAny@@@ZA 1044ea84     Install.obj
 0003:00412a88       ?D2GetItemType@@3P6GHPAUUnitAny@@@ZA 1044ea88     Install.obj
 0003:00412a8c       ?D2GetMagicAffixRecord@@3P6GPAUAffixTxt@@H@ZA 1044ea8c     Install.obj
 0003:00412a90       ?D2GetSkillById@@3P6IPAUSkill@@PAUUnitAny@@HH@ZA 1044ea90     Install.obj
 0003:00412a94       ?D2GetListFromItem@@3P6GPAUStatList@@PAUUnitAny@@K@ZA 1044ea94     Install.obj
 0003:00412a98       ?D2GetListFromItem2@@3P6GPAUStatList2@@PAUUnitAny@@K@ZA 1044ea98     Install.obj
 0003:00412a9c       ?D2GetInvItemCount@@3P6GHPAUUnitInventory@@@ZA 1044ea9c     Install.obj
 0003:00412aa0       ?D2GetStatFromStatList@@3P6GHPAUStatList@@KPAUStatEx@@K@ZA 1044eaa0     Install.obj
 0003:00412aa4       ?D2GetStatListWithFlag@@3P6GPAUStatList@@PAUUnitAny@@KK@ZA 1044eaa4     Install.obj
 0003:00412aa8       ?D2GetUnitStat@@3P6GHPAUUnitAny@@KG@ZA 1044eaa8     Install.obj
 0003:00412aac       ?D2GetUnitBaseStat@@3P6GHPAUUnitAny@@KG@ZA 1044eaac     Install.obj
 0003:00412ab0       ?D2GetMonsterHpPercent@@3P6GHPAUUnitAny@@@ZA 1044eab0     Install.obj
 0003:00412ab4       ?D2EvalItemCalc@@3P6GHPAUUnitAny@@0K@ZA 1044eab4     Install.obj
 0003:00412ab8       ?D2CheckUnitState@@3P6GHPAUUnitAny@@K@ZA 1044eab8     Install.obj
 0003:00412abc       ?D2CheckQuestFlag@@3P6GHPAXKK@ZA 1044eabc     Install.obj
 0003:00412ac0       ?D2CheckItemFlag@@3P6GHPAUUnitAny@@KKPAD@ZA 1044eac0     Install.obj
 0003:00412ac4       ?D2CheckCorpseCanUse@@3P6GHPAUUnitAny@@K@ZA 1044eac4     Install.obj
 0003:00412ac8       ?D2GetItemValue@@3P6GHPAUUnitAny@@0KPAXHK@ZA 1044eac8     Install.obj
 0003:00412acc       ?D2GetCursorItem@@3P6GPAUUnitAny@@PAUUnitInventory@@@ZA 1044eacc     Install.obj
 0003:00412ad0       ?D2GetFirstItemInInv@@3P6GPAUUnitAny@@PAUUnitInventory@@@ZA 1044ead0     Install.obj
 0003:00412ad4       ?D2GetNextItemInInv@@3P6GPAUUnitAny@@PAU1@@ZA 1044ead4     Install.obj
 0003:00412ad8       ?D2GetBoxType@@3P6GKPAUUnitAny@@EK@ZA 1044ead8     Install.obj
 0003:00412adc       ?D2CheckInvLocation@@3P6GHPAUUnitInventory@@PAUUnitAny@@KKKPAH2E@ZA 1044eadc     Install.obj
 0003:00412ae0       ?D2GetDrlgLevel@@3P6IPAUDrlgLevel@@PAUDrlgMisc@@K@ZA 1044eae0     Install.obj
 0003:00412ae4       ?D2InitDrlgLevel@@3P6GXPAUDrlgLevel@@@ZA 1044eae4     Install.obj
 0003:00412ae8       ?D2GetLevelIdFromRoom@@3P6GKPAUDrlgRoom1@@@ZA 1044eae8     Install.obj
 0003:00412aec       ?D2GetUnitPosX@@3P6GKPAUDynamicPath@@@ZA 1044eaec     Install.obj
 0003:00412af0       ?D2GetUnitPosY@@3P6GKPAUDynamicPath@@@ZA 1044eaf0     Install.obj
 0003:00412af4       ?D2GetMinExpToLevel@@3P6GHKK@ZA 1044eaf4     Install.obj
 0003:00412af8       ?p_D2WeaponsTxts@@3PAHA    1044eaf8     Install.obj
 0003:00412afc       ?p_D2ArmorTxts@@3PAHA      1044eafc     Install.obj
 0003:00412b00       ?p_D2DataTables@@3PAKA     1044eb00     Install.obj
 0003:00412b04       ?p_D2RuneWords@@3PAKA      1044eb04     Install.obj
 0003:00412b08       ?p_D2RuneWordTxt@@3PAKA    1044eb08     Install.obj
 0003:00412b0c       ?D2GetHwnd@@3P6GPAUHWND__@@XZA 1044eb0c     Install.obj
 0003:00412b10       ?D2DrawRectangle@@3P6GXJJJJKK@ZA 1044eb10     Install.obj
 0003:00412b14       ?D2DrawLine@@3P6GXJJJJKK@ZA 1044eb14     Install.obj
 0003:00412b18       ?D2DrawCellFile@@3P6GXPAUCellContext@@KKKKPAE@ZA 1044eb18     Install.obj
 0003:00412b1c       ?D2DrawAutomapCell@@3P6GXPAUCellContext@@KKPAUtagRECT@@K@ZA 1044eb1c     Install.obj
 0003:00412b20       ?D2MinimizeWindows@@3P6GXK@ZA 1044eb20     Install.obj
 0003:00412b24       ?p_D2WinState@@3PAKA       1044eb24     Install.obj
 0003:00412b28       ?D2DrawText@@3P6IXPA_WJJKK@ZA 1044eb28     Install.obj
 0003:00412b2c       ?D2DrawHoverText@@3P6IXPA_WJJKK@ZA 1044eb2c     Install.obj
 0003:00412b30       ?D2DrawUnitLifeBar@@3P6IKPA_WJJKKK@ZA 1044eb30     Install.obj
 0003:00412b34       ?D2DrawHover@@3P6IXXZA     1044eb34     Install.obj
 0003:00412b38       ?D2GetTextAreaSize@@3P6IKPA_WPAK1@ZA 1044eb38     Install.obj
 0003:00412b3c       ?D2SetTextFont@@3P6IKK@ZA  1044eb3c     Install.obj
 0003:00412b40       ?D2GetTextPixelLen@@3P6IKPA_W@ZA 1044eb40     Install.obj
 0003:00412b44       ?D2GetEditBoxText@@3P6IPA_WPAUD2EditBox@@@ZA 1044eb44     Install.obj
 0003:00412b48       ?D2SelectEditBoxText@@3P6IXPAUD2EditBox@@@ZA 1044eb48     Install.obj
 0003:00412b4c       ?D2AddEditBoxChar@@3P6IKPAUD2EditBox@@E@ZA 1044eb4c     Install.obj
 0003:00412b50       ?D2DestroyEditBox@@3P6IKPAUD2EditBox@@@ZA 1044eb50     Install.obj
 0003:00412b54       ?D2DestroyListBox@@3P6GXPAUD2EditBox@@@ZA 1044eb54     Install.obj
 0003:00412b58       ?D2CreateEditBox@@3P6IPAUD2EditBox@@KKKKKKPAUCellFile@@KKKPAX@ZA 1044eb58     Install.obj
 0003:00412b5c       ?D2SetEditBoxText@@3P6IPAXPAUD2EditBox@@PA_W@ZA 1044eb5c     Install.obj
 0003:00412b60       ?D2SetEditBoxProc@@3P6IXPAUD2EditBox@@P6GH0KPAD@Z@ZA 1044eb60     Install.obj
 0003:00412b64       ?vD2ToggleSound@@3KA       1044eb64     Install.obj
 0003:00412b68       ?p_D2FocusedControl@@3PAPAUD2EditBox@@A 1044eb68     Install.obj
 0003:00412b6c       ?D2DeleteCellFile@@3P6GXPAUCellFile@@@ZA 1044eb6c     Install.obj
 0003:00412b70       ?D2InitCellFile@@3P6GXPAXPAPAUCellFile@@PADKK2@ZA 1044eb70     Install.obj
 0003:00412b74       ?D2GetLocaleText@@3P6IPA_WK@ZA 1044eb74     Install.obj
 0003:00412b78       ?p_D2UnkNetFlag@@3PAKA     1044eb78     Install.obj
 0003:00412b7c       ?D2SendPacket@@3P6GXIKPAE@ZA 1044eb7c     Install.obj
 0003:00412b80       ?p_D2BnChatMessage@@3PAPAKA 1044eb80     Install.obj
 0003:00412b84       ?vD2EndOfPtr@@3KC          1044eb84     Install.obj
 0003:00412b88       ?vD2StartOfPtr2@@3KC       1044eb88     Install.obj
 0003:00412b8c       ?p_D2GameListControl@@3PAPAUD2EditBox@@A 1044eb8c     Install.obj
 0003:00412b90       ?p_D2EditboxPreferences@@3PAPAXA 1044eb90     Install.obj
 0003:00412b94       ?vD2GetUnitName_I@@3KC     1044eb94     Install.obj
 0003:00412b98       ?vD2EndOfPtr2@@3KC         1044eb98     Install.obj
 0003:0a8a2850       ?_OptionsStorage@?1??__local_stdio_printf_options@@9@4_KA 1a8de850     Install.obj
 0003:0a8a2858       ___@@_PchSym_@00@UKlqKpyKoqKlsKqoKplKlvKooKpwKlsKpzKryUxQQUwCszxpnzkPwvevolkSorlmTUwCszxpnzkUKluKqkKopKlsKpyKrzKluKonKrzKluKrkKqyKlsKpoKpkUhgwzucOlyq@4B2008FD98C1DD4 1a8de858     stdafx.obj
 0003:0a8a4810       ?id@?$num_put@DV?$ostreambuf_iterator@DU?$char_traits@D@std@@@std@@@std@@2V0locale@2@A 1a8e0810     DllMain.obj
 0003:0a8a4814       ?id@?$collate@D@std@@2V0locale@2@A 1a8e0814     DllMain.obj
 0003:0a8a4818       ?id@?$codecvt@DDU_Mbstatet@@@std@@2V0locale@2@A 1a8e0818     DllMain.obj
 0003:0a8a481c       ?id@?$numpunct@D@std@@2V0locale@2@A 1a8e081c     DllMain.obj
 0003:0a8a4a24       ___dyn_tls_init_callback   1a8e0a24     <common>
 0003:0a8a4a28       ___scrt_ucrt_dll_is_in_use 1a8e0a28     <common>
 0003:0a8a4a2c       __pmatherr                 1a8e0a2c     <common>
 0003:0a8a4a30       ___use_sse2_mathfcns       1a8e0a30     <common>

 entry point at        0001:0001f1b9

 Static symbols

 0000:f5707000       .debug$S                   10000000     d2hackmap.exp
 0000:f5707000       .debug$S                   10000000     Version:VERSION.dll
 0000:f5707000       .debug$S                   10000000     Version:VERSION.dll
 0000:f5707000       .debug$S                   10000000     Version:VERSION.dll
 0000:f5707000       .debug$S                   10000000     imm32:IMM32.dll
 0000:f5707000       .debug$S                   10000000     kernel32:KERNEL32.dll
 0000:f5707000       .debug$S                   10000000     kernel32:KERNEL32.dll
 0000:f5707000       .debug$S                   10000000     kernel32:KERNEL32.dll
 0000:f5707000       .debug$S                   10000000     kernel32:KERNEL32.dll
 0000:f5707000       .debug$S                   10000000     kernel32:KERNEL32.dll
 0000:f5707000       .debug$S                   10000000     kernel32:KERNEL32.dll
 0000:f5707000       .debug$S                   10000000     kernel32:KERNEL32.dll
 0000:f5707000       .debug$S                   10000000     kernel32:KERNEL32.dll
 0000:f5707000       .debug$S                   10000000     kernel32:KERNEL32.dll
 0000:f5707000       .debug$S                   10000000     kernel32:KERNEL32.dll
 0000:f5707000       .debug$S                   10000000     kernel32:KERNEL32.dll
 0000:f5707000       .debug$S                   10000000     kernel32:KERNEL32.dll
 0000:f5707000       .debug$S                   10000000     kernel32:KERNEL32.dll
 0000:f5707000       .debug$S                   10000000     kernel32:KERNEL32.dll
 0000:f5707000       .debug$S                   10000000     kernel32:KERNEL32.dll
 0000:f5707000       .debug$S                   10000000     kernel32:KERNEL32.dll
 0000:f5707000       .debug$S                   10000000     kernel32:KERNEL32.dll
 0000:f5707000       .debug$S                   10000000     kernel32:KERNEL32.dll
 0000:f5707000       .debug$S                   10000000     kernel32:KERNEL32.dll
 0000:f5707000       .debug$S                   10000000     kernel32:KERNEL32.dll
 0000:f5707000       .debug$S                   10000000     kernel32:KERNEL32.dll
 0000:f5707000       .debug$S                   10000000     kernel32:KERNEL32.dll
 0000:f5707000       .debug$S                   10000000     kernel32:KERNEL32.dll
 0000:f5707000       .debug$S                   10000000     kernel32:KERNEL32.dll
 0000:f5707000       .debug$S                   10000000     kernel32:KERNEL32.dll
 0000:f5707000       .debug$S                   10000000     kernel32:KERNEL32.dll
 0000:f5707000       .debug$S                   10000000     kernel32:KERNEL32.dll
 0000:f5707000       .debug$S                   10000000     kernel32:KERNEL32.dll
 0000:f5707000       .debug$S                   10000000     kernel32:KERNEL32.dll
 0000:f5707000       .debug$S                   10000000     kernel32:KERNEL32.dll
 0000:f5707000       .debug$S                   10000000     kernel32:KERNEL32.dll
 0000:f5707000       .debug$S                   10000000     kernel32:KERNEL32.dll
 0000:f5707000       .debug$S                   10000000     kernel32:KERNEL32.dll
 0000:f5707000       .debug$S                   10000000     kernel32:KERNEL32.dll
 0000:f5707000       .debug$S                   10000000     kernel32:KERNEL32.dll
 0000:f5707000       .debug$S                   10000000     kernel32:KERNEL32.dll
 0000:f5707000       .debug$S                   10000000     kernel32:KERNEL32.dll
 0000:f5707000       .debug$S                   10000000     kernel32:KERNEL32.dll
 0000:f5707000       .debug$S                   10000000     kernel32:KERNEL32.dll
 0000:f5707000       .debug$S                   10000000     kernel32:KERNEL32.dll
 0000:f5707000       .debug$S                   10000000     kernel32:KERNEL32.dll
 0000:f5707000       .debug$S                   10000000     kernel32:KERNEL32.dll
 0000:f5707000       .debug$S                   10000000     kernel32:KERNEL32.dll
 0000:f5707000       .debug$S                   10000000     kernel32:KERNEL32.dll
 0000:f5707000       .debug$S                   10000000     kernel32:KERNEL32.dll
 0000:f5707000       .debug$S                   10000000     kernel32:KERNEL32.dll
 0000:f5707000       .debug$S                   10000000     kernel32:KERNEL32.dll
 0000:f5707000       .debug$S                   10000000     kernel32:KERNEL32.dll
 0000:f5707000       .debug$S                   10000000     kernel32:KERNEL32.dll
 0000:f5707000       .debug$S                   10000000     kernel32:KERNEL32.dll
 0000:f5707000       .debug$S                   10000000     kernel32:KERNEL32.dll
 0000:f5707000       .debug$S                   10000000     kernel32:KERNEL32.dll
 0000:f5707000       .debug$S                   10000000     kernel32:KERNEL32.dll
 0000:f5707000       .debug$S                   10000000     kernel32:KERNEL32.dll
 0000:f5707000       .debug$S                   10000000     kernel32:KERNEL32.dll
 0000:f5707000       .debug$S                   10000000     kernel32:KERNEL32.dll
 0000:f5707000       .debug$S                   10000000     kernel32:KERNEL32.dll
 0000:f5707000       .debug$S                   10000000     kernel32:KERNEL32.dll
 0000:f5707000       .debug$S                   10000000     kernel32:KERNEL32.dll
 0000:f5707000       .debug$S                   10000000     kernel32:KERNEL32.dll
 0000:f5707000       .debug$S                   10000000     kernel32:KERNEL32.dll
 0000:f5707000       .debug$S                   10000000     kernel32:KERNEL32.dll
 0000:f5707000       .debug$S                   10000000     kernel32:KERNEL32.dll
 0000:f5707000       .debug$S                   10000000     kernel32:KERNEL32.dll
 0000:f5707000       .debug$S                   10000000     kernel32:KERNEL32.dll
 0000:f5707000       .debug$S                   10000000     kernel32:KERNEL32.dll
 0000:f5707000       .debug$S                   10000000     kernel32:KERNEL32.dll
 0000:f5707000       .debug$S                   10000000     kernel32:KERNEL32.dll
 0000:f5707000       .debug$S                   10000000     kernel32:KERNEL32.dll
 0000:f5707000       .debug$S                   10000000     kernel32:KERNEL32.dll
 0000:f5707000       .debug$S                   10000000     kernel32:KERNEL32.dll
 0000:f5707000       .debug$S                   10000000     kernel32:KERNEL32.dll
 0000:f5707000       .debug$S                   10000000     kernel32:KERNEL32.dll
 0000:f5707000       .debug$S                   10000000     kernel32:KERNEL32.dll
 0000:f5707000       .debug$S                   10000000     kernel32:KERNEL32.dll
 0000:f5707000       .debug$S                   10000000     kernel32:KERNEL32.dll
 0000:f5707000       .debug$S                   10000000     kernel32:KERNEL32.dll
 0000:f5707000       .debug$S                   10000000     kernel32:KERNEL32.dll
 0000:f5707000       .debug$S                   10000000     kernel32:KERNEL32.dll
 0000:f5707000       .debug$S                   10000000     kernel32:KERNEL32.dll
 0000:f5707000       .debug$S                   10000000     kernel32:KERNEL32.dll
 0000:f5707000       .debug$S                   10000000     kernel32:KERNEL32.dll
 0000:f5707000       .debug$S                   10000000     kernel32:KERNEL32.dll
 0000:f5707000       .debug$S                   10000000     kernel32:KERNEL32.dll
 0000:f5707000       .debug$S                   10000000     kernel32:KERNEL32.dll
 0000:f5707000       .debug$S                   10000000     kernel32:KERNEL32.dll
 0000:f5707000       .debug$S                   10000000     kernel32:KERNEL32.dll
 0000:f5707000       .debug$S                   10000000     kernel32:KERNEL32.dll
 0000:f5707000       .debug$S                   10000000     kernel32:KERNEL32.dll
 0000:f5707000       .debug$S                   10000000     kernel32:KERNEL32.dll
 0000:f5707000       .debug$S                   10000000     kernel32:KERNEL32.dll
 0000:f5707000       .debug$S                   10000000     kernel32:KERNEL32.dll
 0000:f5707000       .debug$S                   10000000     kernel32:KERNEL32.dll
 0000:f5707000       .debug$S                   10000000     kernel32:KERNEL32.dll
 0000:f5707000       .debug$S                   10000000     kernel32:KERNEL32.dll
 0000:f5707000       .debug$S                   10000000     kernel32:KERNEL32.dll
 0000:f5707000       .debug$S                   10000000     kernel32:KERNEL32.dll
 0000:f5707000       .debug$S                   10000000     kernel32:KERNEL32.dll
 0000:f5707000       .debug$S                   10000000     kernel32:KERNEL32.dll
 0000:f5707000       .debug$S                   10000000     kernel32:KERNEL32.dll
 0000:f5707000       .debug$S                   10000000     kernel32:KERNEL32.dll
 0000:f5707000       .debug$S                   10000000     kernel32:KERNEL32.dll
 0000:f5707000       .debug$S                   10000000     user32:USER32.dll
 0000:f5707000       .debug$S                   10000000     user32:USER32.dll
 0000:f5707000       .debug$S                   10000000     user32:USER32.dll
 0000:f5707000       .debug$S                   10000000     user32:USER32.dll
 0000:f5707000       .debug$S                   10000000     user32:USER32.dll
 0000:f5707000       .debug$S                   10000000     user32:USER32.dll
 0000:f5707000       .debug$S                   10000000     user32:USER32.dll
 0000:f5707000       .debug$S                   10000000     user32:USER32.dll
 0000:f5707000       .debug$S                   10000000     user32:USER32.dll
 0000:f5707000       .debug$S                   10000000     ws2_32:WS2_32.dll
 0000:f5707000       .debug$S                   10000000     ws2_32:WS2_32.dll
 0001:00000000       ??__Ewsinit_@detail@httplib@@YAXXZ 10001000 f   DllMain.obj
 0001:00000020       ??__E?id@?$collate@D@std@@2V0locale@2@A@@YAXXZ 10001020 f   DllMain.obj
 0001:00000040       ??__E?id@?$num_put@DV?$ostreambuf_iterator@DU?$char_traits@D@std@@@std@@@std@@2V0locale@2@A@@YAXXZ 10001040 f   DllMain.obj
 0001:00000060       ??__E?id@?$codecvt@DDU_Mbstatet@@@std@@2V0locale@2@A@@YAXXZ 10001060 f   DllMain.obj
 0001:00000080       ??__E?id@?$numpunct@D@std@@2V0locale@2@A@@YAXXZ 10001080 f   DllMain.obj
 0001:000000a0       ??__EvD2ERR@@YAXXZ         100010a0 f   Install.obj
 0001:000000c0       ??__EvD2StartOfPtr@@YAXXZ  100010c0 f   Install.obj
 0001:000000e0       ??__EvD2VD2SendToServer3@@YAXXZ 100010e0 f   Install.obj
 0001:00000100       ??__ED2ShowGameMessage@@YAXXZ 10001100 f   Install.obj
 0001:00000150       ??__ED2ShowPartyMessage@@YAXXZ 10001150 f   Install.obj
 0001:000001a0       ??__ED2ShowMap@@YAXXZ      100011a0 f   Install.obj
 0001:000001f0       ??__ED2RevealAutomapRoom@@YAXXZ 100011f0 f   Install.obj
 0001:00000240       ??__ED2RecvCommand07@@YAXXZ 10001240 f   Install.obj
 0001:00000290       ??__ED2RecvCommand08@@YAXXZ 10001290 f   Install.obj
 0001:000002e0       ??__ED2NewAutomapCell@@YAXXZ 100012e0 f   Install.obj
 0001:00000330       ??__ED2AddAutomapCell@@YAXXZ 10001330 f   Install.obj
 0001:00000380       ??__ED2GetPlayerXOffset@@YAXXZ 10001380 f   Install.obj
 0001:000003d0       ??__ED2GetPlayerYOffset@@YAXXZ 100013d0 f   Install.obj
 0001:00000420       ??__ED2SetUiStatus@@YAXXZ  10001420 f   Install.obj
 0001:00000470       ??__ED2CalcShake@@YAXXZ    10001470 f   Install.obj
 0001:000004c0       ??__ED2GetMonsterOwner@@YAXXZ 100014c0 f   Install.obj
 0001:00000510       ??__ED2GetUnitFromId@@YAXXZ 10001510 f   Install.obj
 0001:00000560       ??__ED2GetSelectedUnit@@YAXXZ 10001560 f   Install.obj
 0001:000005b0       ??__ED2InitAutomapLayerStub@@YAXXZ 100015b0 f   Install.obj
 0001:00000600       ??__ED2CheckUiStatusStub@@YAXXZ 10001600 f   Install.obj
 0001:00000650       ??__ED2SetAutomapPartyStub@@YAXXZ 10001650 f   Install.obj
 0001:000006a0       ??__ED2SetAutomapNamesStub@@YAXXZ 100016a0 f   Install.obj
 0001:000006f0       ??__ED2ChatInputStub@@YAXXZ 100016f0 f   Install.obj
 0001:00000740       ??__ED2ItemProtect@@YAXXZ  10001740 f   Install.obj
 0001:00000790       ??__ED2DrawClient@@YAXXZ   10001790 f   Install.obj
 0001:000007e0       ??__ED2Storm511@@YAXXZ     100017e0 f   Install.obj
 0001:00000830       ??__Ep_D2AutomapLayerList@@YAXXZ 10001830 f   Install.obj
 0001:00000880       ??__Ep_D2AutomapLayer@@YAXXZ 10001880 f   Install.obj
 0001:000008d0       ??__Ep_D2PlayerUnit@@YAXXZ 100018d0 f   Install.obj
 0001:00000920       ??__Ep_D2RosterUnitList@@YAXXZ 10001920 f   Install.obj
 0001:00000970       ??__Ep_D2PetUnitList@@YAXXZ 10001970 f   Install.obj
 0001:000009c0       ??__Ep_D2DrlgAct@@YAXXZ    100019c0 f   Install.obj
 0001:00000a10       ??__Ep_D2Expansion@@YAXXZ  10001a10 f   Install.obj
 0001:00000a60       ??__Ep_D2Difficulty@@YAXXZ 10001a60 f   Install.obj
 0001:00000ab0       ??__Ep_D2GameInfo@@YAXXZ   10001ab0 f   Install.obj
 0001:00000b00       ??__Ep_D2Fps@@YAXXZ        10001b00 f   Install.obj
 0001:00000b50       ??__Ep_D2Ping@@YAXXZ       10001b50 f   Install.obj
 0001:00000ba0       ??__Ep_D2ExitAppFlag@@YAXXZ 10001ba0 f   Install.obj
 0001:00000bf0       ??__Ep_D2InGame@@YAXXZ     10001bf0 f   Install.obj
 0001:00000c40       ??__Ep_D2AutomapOn@@YAXXZ  10001c40 f   Install.obj
 0001:00000c90       ??__Ep_D2Divisor@@YAXXZ    10001c90 f   Install.obj
 0001:00000ce0       ??__Ep_D2Offset@@YAXXZ     10001ce0 f   Install.obj
 0001:00000d30       ??__Ep_D2AutomapPos@@YAXXZ 10001d30 f   Install.obj
 0001:00000d80       ??__Ep_D2AutoMapSize@@YAXXZ 10001d80 f   Install.obj
 0001:00000dd0       ??__Ep_D2MinmapType@@YAXXZ 10001dd0 f   Install.obj
 0001:00000e20       ??__Ep_D2MinimapOffset@@YAXXZ 10001e20 f   Install.obj
 0001:00000e70       ??__Ep_D2IsMapShakeOn@@YAXXZ 10001e70 f   Install.obj
 0001:00000ec0       ??__Ep_D2MapShakeY@@YAXXZ  10001ec0 f   Install.obj
 0001:00000f10       ??__Ep_D2MapShakeX@@YAXXZ  10001f10 f   Install.obj
 0001:00000f60       ??__Ep_D2ScreenSizeX@@YAXXZ 10001f60 f   Install.obj
 0001:00000fb0       ??__Ep_D2ScreenSizeY@@YAXXZ 10001fb0 f   Install.obj
 0001:00001000       ??__Ep_D2ScreenSize@@YAXXZ 10002000 f   Install.obj
 0001:00001050       ??__Ep_D2DrawOffset@@YAXXZ 10002050 f   Install.obj
 0001:000010a0       ??__Ep_D2InfoPositionX@@YAXXZ 100020a0 f   Install.obj
 0001:000010f0       ??__Ep_D2InfoPositionY@@YAXXZ 100020f0 f   Install.obj
 0001:00001140       ??__Ep_D2QuestData@@YAXXZ  10002140 f   Install.obj
 0001:00001190       ??__Ep_D2GameQuestData@@YAXXZ 10002190 f   Install.obj
 0001:000011e0       ??__Ep_D2QuestPage@@YAXXZ  100021e0 f   Install.obj
 0001:00001230       ??__Ep_D2MButton@@YAXXZ    10002230 f   Install.obj
 0001:00001280       ??__Ep_D2LastChatMessage@@YAXXZ 10002280 f   Install.obj
 0001:000012d0       ??__Ep_D2ChatTextLength@@YAXXZ 100022d0 f   Install.obj
 0001:00001320       ??__Ep_D2MousePos@@YAXXZ   10002320 f   Install.obj
 0001:00001370       ??__Ep_D2LastMousePos@@YAXXZ 10002370 f   Install.obj
 0001:000013c0       ??__Ep_D2CursorInvGridX@@YAXXZ 100023c0 f   Install.obj
 0001:00001410       ??__Ep_D2CursorInvGridY@@YAXXZ 10002410 f   Install.obj
 0001:00001460       ??__Ep_D2CurrentViewItem@@YAXXZ 10002460 f   Install.obj
 0001:000014b0       ??__Ep_D2GoldInTranBox@@YAXXZ 100024b0 f   Install.obj
 0001:00001500       ??__Ep_D2ShowLifeStr@@YAXXZ 10002500 f   Install.obj
 0001:00001550       ??__Ep_D2ShowManaStr@@YAXXZ 10002550 f   Install.obj
 0001:000015a0       ??__EvD2AutomapCellListBaseAddr@@YAXXZ 100025a0 f   Install.obj
 0001:000015f0       ??__EvD2LoadUiImageFunc@@YAXXZ 100025f0 f   Install.obj
 0001:00001640       ??__ED2GetObjectTxt@@YAXXZ 10002640 f   Install.obj
 0001:00001690       ??__ED2GetLevelDefTxt@@YAXXZ 10002690 f   Install.obj
 0001:000016e0       ??__ED2GetLevelTxt@@YAXXZ  100026e0 f   Install.obj
 0001:00001730       ??__ED2GetItemTxt@@YAXXZ   10002730 f   Install.obj
 0001:00001780       ??__ED2GetItemTxt2@@YAXXZ  10002780 f   Install.obj
 0001:000017d0       ??__ED2GetItemTxt3@@YAXXZ  100027d0 f   Install.obj
 0001:00001820       ??__ED2GetTreasureClasses@@YAXXZ 10002820 f   Install.obj
 0001:00001870       ??__ED2GetSuperUniqueTxt@@YAXXZ 10002870 f   Install.obj
 0001:000018c0       ??__ED2CheckItemType@@YAXXZ 100028c0 f   Install.obj
 0001:00001910       ??__ED2GetItemFileIndex@@YAXXZ 10002910 f   Install.obj
 0001:00001960       ??__ED2GetItemType@@YAXXZ  10002960 f   Install.obj
 0001:000019b0       ??__ED2GetMagicAffixRecord@@YAXXZ 100029b0 f   Install.obj
 0001:00001a00       ??__ED2GetSkillById@@YAXXZ 10002a00 f   Install.obj
 0001:00001a50       ??__ED2GetListFromItem@@YAXXZ 10002a50 f   Install.obj
 0001:00001aa0       ??__ED2GetListFromItem2@@YAXXZ 10002aa0 f   Install.obj
 0001:00001af0       ??__ED2GetInvItemCount@@YAXXZ 10002af0 f   Install.obj
 0001:00001b40       ??__ED2GetStatFromStatList@@YAXXZ 10002b40 f   Install.obj
 0001:00001b90       ??__ED2GetStatListWithFlag@@YAXXZ 10002b90 f   Install.obj
 0001:00001be0       ??__ED2GetUnitStat@@YAXXZ  10002be0 f   Install.obj
 0001:00001c30       ??__ED2GetUnitBaseStat@@YAXXZ 10002c30 f   Install.obj
 0001:00001c80       ??__ED2GetMonsterHpPercent@@YAXXZ 10002c80 f   Install.obj
 0001:00001cd0       ??__ED2EvalItemCalc@@YAXXZ 10002cd0 f   Install.obj
 0001:00001d20       ??__ED2CheckUnitState@@YAXXZ 10002d20 f   Install.obj
 0001:00001d70       ??__ED2CheckQuestFlag@@YAXXZ 10002d70 f   Install.obj
 0001:00001dc0       ??__ED2CheckItemFlag@@YAXXZ 10002dc0 f   Install.obj
 0001:00001e10       ??__ED2CheckCorpseCanUse@@YAXXZ 10002e10 f   Install.obj
 0001:00001e60       ??__ED2GetItemValue@@YAXXZ 10002e60 f   Install.obj
 0001:00001eb0       ??__ED2GetCursorItem@@YAXXZ 10002eb0 f   Install.obj
 0001:00001f00       ??__ED2GetFirstItemInInv@@YAXXZ 10002f00 f   Install.obj
 0001:00001f50       ??__ED2GetNextItemInInv@@YAXXZ 10002f50 f   Install.obj
 0001:00001fa0       ??__ED2GetBoxType@@YAXXZ   10002fa0 f   Install.obj
 0001:00001ff0       ??__ED2CheckInvLocation@@YAXXZ 10002ff0 f   Install.obj
 0001:00002040       ??__ED2GetDrlgLevel@@YAXXZ 10003040 f   Install.obj
 0001:00002090       ??__ED2InitDrlgLevel@@YAXXZ 10003090 f   Install.obj
 0001:000020e0       ??__ED2GetLevelIdFromRoom@@YAXXZ 100030e0 f   Install.obj
 0001:00002130       ??__ED2GetUnitPosX@@YAXXZ  10003130 f   Install.obj
 0001:00002180       ??__ED2GetUnitPosY@@YAXXZ  10003180 f   Install.obj
 0001:000021d0       ??__ED2GetMinExpToLevel@@YAXXZ 100031d0 f   Install.obj
 0001:00002220       ??__Ep_D2WeaponsTxts@@YAXXZ 10003220 f   Install.obj
 0001:00002270       ??__Ep_D2ArmorTxts@@YAXXZ  10003270 f   Install.obj
 0001:000022c0       ??__Ep_D2DataTables@@YAXXZ 100032c0 f   Install.obj
 0001:00002310       ??__Ep_D2RuneWords@@YAXXZ  10003310 f   Install.obj
 0001:00002360       ??__Ep_D2RuneWordTxt@@YAXXZ 10003360 f   Install.obj
 0001:000023b0       ??__ED2GetHwnd@@YAXXZ      100033b0 f   Install.obj
 0001:00002400       ??__ED2DrawRectangle@@YAXXZ 10003400 f   Install.obj
 0001:00002450       ??__ED2DrawLine@@YAXXZ     10003450 f   Install.obj
 0001:000024a0       ??__ED2DrawCellFile@@YAXXZ 100034a0 f   Install.obj
 0001:000024f0       ??__ED2DrawAutomapCell@@YAXXZ 100034f0 f   Install.obj
 0001:00002540       ??__ED2MinimizeWindows@@YAXXZ 10003540 f   Install.obj
 0001:00002590       ??__Ep_D2WinState@@YAXXZ   10003590 f   Install.obj
 0001:000025e0       ??__ED2DrawText@@YAXXZ     100035e0 f   Install.obj
 0001:00002630       ??__ED2DrawHoverText@@YAXXZ 10003630 f   Install.obj
 0001:00002680       ??__ED2DrawUnitLifeBar@@YAXXZ 10003680 f   Install.obj
 0001:000026d0       ??__ED2DrawHover@@YAXXZ    100036d0 f   Install.obj
 0001:00002720       ??__ED2GetTextAreaSize@@YAXXZ 10003720 f   Install.obj
 0001:00002770       ??__ED2SetTextFont@@YAXXZ  10003770 f   Install.obj
 0001:000027c0       ??__ED2GetTextPixelLen@@YAXXZ 100037c0 f   Install.obj
 0001:00002810       ??__ED2GetEditBoxText@@YAXXZ 10003810 f   Install.obj
 0001:00002860       ??__ED2SelectEditBoxText@@YAXXZ 10003860 f   Install.obj
 0001:000028b0       ??__ED2AddEditBoxChar@@YAXXZ 100038b0 f   Install.obj
 0001:00002900       ??__ED2DestroyEditBox@@YAXXZ 10003900 f   Install.obj
 0001:00002950       ??__ED2DestroyListBox@@YAXXZ 10003950 f   Install.obj
 0001:000029a0       ??__ED2CreateEditBox@@YAXXZ 100039a0 f   Install.obj
 0001:000029f0       ??__ED2SetEditBoxText@@YAXXZ 100039f0 f   Install.obj
 0001:00002a40       ??__ED2SetEditBoxProc@@YAXXZ 10003a40 f   Install.obj
 0001:00002a90       ??__EvD2ToggleSound@@YAXXZ 10003a90 f   Install.obj
 0001:00002ae0       ??__Ep_D2FocusedControl@@YAXXZ 10003ae0 f   Install.obj
 0001:00002b30       ??__ED2DeleteCellFile@@YAXXZ 10003b30 f   Install.obj
 0001:00002b80       ??__ED2InitCellFile@@YAXXZ 10003b80 f   Install.obj
 0001:00002bd0       ??__ED2GetLocaleText@@YAXXZ 10003bd0 f   Install.obj
 0001:00002c20       ??__Ep_D2UnkNetFlag@@YAXXZ 10003c20 f   Install.obj
 0001:00002c70       ??__ED2SendPacket@@YAXXZ   10003c70 f   Install.obj
 0001:00002cc0       ??__Ep_D2BnChatMessage@@YAXXZ 10003cc0 f   Install.obj
 0001:00002d10       ??__EvD2EndOfPtr@@YAXXZ    10003d10 f   Install.obj
 0001:00002d30       ??__EvD2StartOfPtr2@@YAXXZ 10003d30 f   Install.obj
 0001:00002d50       ??__Ep_D2GameListControl@@YAXXZ 10003d50 f   Install.obj
 0001:00002da0       ??__Ep_D2EditboxPreferences@@YAXXZ 10003da0 f   Install.obj
 0001:00002df0       ??__EvD2GetUnitName_I@@YAXXZ 10003df0 f   Install.obj
 0001:00002e10       ??__EvD2EndOfPtr2@@YAXXZ   10003e10 f   Install.obj
 0001:00002e40       ??__EaD2Patchs@@YAXXZ      10003e40 f   Install.obj
 0001:00006e30       ??__EaD2Patch2s@@YAXXZ     10007e30 f   Install.obj
 0001:00007270       ??__Ewsinit_@detail@httplib@@YAXXZ 10008270 f   stdafx.obj
 0001:00007290       ??__EaKeepGameWindowPatchs@@YAXXZ 10008290 f   GameWindow.obj
 0001:0000acec       $LN88                      1000bcec     LoadConfig.obj
 0001:0000ad10       $LN87                      1000bd10     LoadConfig.obj
 0001:0000b840       $LN17                      1000c840     D2HelpFunc.obj
 0001:0000b848       $LN16                      1000c848     D2HelpFunc.obj
 0001:0000cb50       $LN15                      1000db50     Environment.obj
 0001:0000f764       $LN104                     10010764     ItemExtInfo.obj
 0001:0000fd80       $LN35                      10010d80     ItemExtInfo.obj
 0001:0000fff0       ?FindClosestItemGround@@YAPAUUnitAny@@K@Z 10010ff0 f   ItemInGround.obj
 0001:00012d98       $LN13                      10013d98     ItemVariableProp.obj
 0001:00012da4       $LN12                      10013da4     ItemVariableProp.obj
 0001:0001b030       $LN13                      1001c030     AutoMapBlob.obj
 0001:0001b484       $LN38                      1001c484     AutoMapCell.obj
 0001:0001b498       $LN37                      1001c498     AutoMapCell.obj
 0001:0001e731       ?find_pe_section@@YAPAU_IMAGE_SECTION_HEADER@@QAEI@Z 1001f731 f   LIBCMT:utility.obj
 0001:0001ec94       ?__scrt_initialize_thread_safe_statics@@YAHXZ 1001fc94 f   LIBCMT:thread_safe_statics.obj
 0001:0001ecbb       ?__scrt_initialize_thread_safe_statics_platform_specific@@YAXXZ 1001fcbb f   LIBCMT:thread_safe_statics.obj
 0001:0001ed3d       ?__scrt_uninitialize_thread_safe_statics@@YAXXZ 1001fd3d f   LIBCMT:thread_safe_statics.obj
 0001:0001ee79       ?dllmain_crt_dispatch@@YGHQAUHINSTANCE__@@KQAX@Z 1001fe79 f   LIBCMT:dll_dllmain.obj
 0001:0001eecc       ?dllmain_crt_process_attach@@YAHQAUHINSTANCE__@@QAX@Z 1001fecc f   LIBCMT:dll_dllmain.obj
 0001:0001efd3       ?dllmain_crt_process_detach@@YAH_N@Z 1001ffd3 f   LIBCMT:dll_dllmain.obj
 0001:0001f083       ?dllmain_dispatch@@YAHQAUHINSTANCE__@@KQAX@Z 10020083 f   LIBCMT:dll_dllmain.obj
 0001:0001f18e       ?dllmain_raw@@YGHQAUHINSTANCE__@@KQAX@Z 1002018e f   LIBCMT:dll_dllmain.obj
 0001:0001f4e0       $$000000                   100204e0     LIBCMT:sehprolg4.obj
 0001:0001f645       ___get_entropy             10020645 f   LIBCMT:gs_support.obj
 0001:0001f847       ?_FilterSetCurrentException@@YAKPAU_EXCEPTION_POINTERS@@E@Z 10020847 f   libvcruntime:ehhelpers.obj
 0001:0001f8a0       $$000000                   100208a0     libvcruntime:strrchr.obj
 0001:0001f8dd       strrchr_sse_loop           100208dd     libvcruntime:strrchr.obj
 0001:0001f90d       strrchr_sse_break          1002090d     libvcruntime:strrchr.obj
 0001:0001f92d       strrchr_sttni              1002092d     libvcruntime:strrchr.obj
 0001:0001f93f       strrchr_sttni_chars        1002093f     libvcruntime:strrchr.obj
 0001:0001f954       strrchr_sttni_aligned      10020954     libvcruntime:strrchr.obj
 0001:0001f958       strrchr_sttni_xmm          10020958     libvcruntime:strrchr.obj
 0001:0001f96b       exit                       1002096b     libvcruntime:strrchr.obj
 0001:0001f96e       strrchr_zero               1002096e     libvcruntime:strrchr.obj
 0001:0001f993       strchr_zero_loop           10020993     libvcruntime:strrchr.obj
 0001:0001f9a7       strchr_zero_result         100209a7     libvcruntime:strrchr.obj
 0001:0001f9ae       strrchr_no_sse             100209ae     libvcruntime:strrchr.obj
 0001:0001f9d1       returndi                   100209d1     libvcruntime:strrchr.obj
 0001:0001f9d3       toend                      100209d3     libvcruntime:strrchr.obj
 0001:0001f9e0       _ValidateLocalCookies      100209e0 f   libvcruntime:chandler4.obj
 0001:0001fb80       $$000000                   10020b80     libvcruntime:strstr.obj
 0001:0001fbc3       strstr_sse_safeloop        10020bc3     libvcruntime:strstr.obj
 0001:0001fbea       strstr_sse_search          10020bea     libvcruntime:strstr.obj
 0001:0001fbea       strstr_sse_unsafe          10020bea     libvcruntime:strstr.obj
 0001:0001fbee       strstr_sse_srchloop        10020bee     libvcruntime:strstr.obj
 0001:0001fc24       strstr_sse_srchchar        10020c24     libvcruntime:strstr.obj
 0001:0001fc3b       strstr_sse_cmploop         10020c3b     libvcruntime:strstr.obj
 0001:0001fc76       strstr_sse_cmpchars        10020c76     libvcruntime:strstr.obj
 0001:0001fc7d       strstr_sse_cmpunsafe       10020c7d     libvcruntime:strstr.obj
 0001:0001fc94       strstr_sse_match           10020c94     libvcruntime:strstr.obj
 0001:0001fc99       strstr_sse_not_found       10020c99     libvcruntime:strstr.obj
 0001:0001fc9b       strstr_sse_exit            10020c9b     libvcruntime:strstr.obj
 0001:0001fc9f       strstr_sttni               10020c9f     libvcruntime:strstr.obj
 0001:0001fcbb       strstr_sttni_setchars      10020cbb     libvcruntime:strstr.obj
 0001:0001fcc0       strstr_sttni_setloopchar   10020cc0     libvcruntime:strstr.obj
 0001:0001fcc6       strstr_sttni_setloopnochar 10020cc6     libvcruntime:strstr.obj
 0001:0001fcda       strstr_sttni_srchnext      10020cda     libvcruntime:strstr.obj
 0001:0001fcdd       strstr_sttni_srch          10020cdd     libvcruntime:strstr.obj
 0001:0001fce1       strstr_sttni_srchloop      10020ce1     libvcruntime:strstr.obj
 0001:0001fd00       strstr_sttni_srchxmm       10020d00     libvcruntime:strstr.obj
 0001:0001fd13       strstr_sttni_srchcheck     10020d13     libvcruntime:strstr.obj
 0001:0001fd17       strstr_sttni_cmploop       10020d17     libvcruntime:strstr.obj
 0001:0001fd4f       strstr_sttni_cmpchar       10020d4f     libvcruntime:strstr.obj
 0001:0001fd6a       strstr_no_sse              10020d6a     libvcruntime:strstr.obj
 0001:0001fd7d       findnext                   10020d7d     libvcruntime:strstr.obj
 0001:0001fd90       loop_start                 10020d90     libvcruntime:strstr.obj
 0001:0001fd95       in_loop                    10020d95     libvcruntime:strstr.obj
 0001:0001fd9d       not_found                  10020d9d     libvcruntime:strstr.obj
 0001:0001fda3       first_char_found           10020da3     libvcruntime:strstr.obj
 0001:0001fdac       two_first_chars_equal      10020dac     libvcruntime:strstr.obj
 0001:0001fdaf       compare_loop               10020daf     libvcruntime:strstr.obj
 0001:0001fdd2       strchr_call                10020dd2     libvcruntime:strstr.obj
 0001:0001fdde       match                      10020dde     libvcruntime:strstr.obj
 0001:0001fde5       empty_str2                 10020de5     libvcruntime:strstr.obj
 0001:0001fdf0       $$000000                   10020df0     libvcruntime:strchr.obj
 0001:0001fe23       strchr_sse_loop            10020e23     libvcruntime:strchr.obj
 0001:0001fe47       strchr_sse_break           10020e47     libvcruntime:strchr.obj
 0001:0001fe58       strchr_no_sse2             10020e58     libvcruntime:strchr.obj
 0001:0001fe70       str_misaligned             10020e70     libvcruntime:strchr.obj
 0001:0001fe85       main_loop_start            10020e85     libvcruntime:strchr.obj
 0001:0001fe90       main_loop                  10020e90     libvcruntime:strchr.obj
 0001:0001fecc       retnull                    10020ecc     libvcruntime:strchr.obj
 0001:0001fece       retnull_bx                 10020ece     libvcruntime:strchr.obj
 0001:0001fed2       found_bx                   10020ed2     libvcruntime:strchr.obj
 0001:0001fed7       chr_is_found               10020ed7     libvcruntime:strchr.obj
 0001:0001feff       byte_3                     10020eff     libvcruntime:strchr.obj
 0001:0001ff06       byte_2                     10020f06     libvcruntime:strchr.obj
 0001:0001ff0d       byte_1                     10020f0d     libvcruntime:strchr.obj
 0001:0001ff14       byte_0                     10020f14     libvcruntime:strchr.obj
 0001:0001ff70       $$000000                   10020f70     libvcruntime:memset.obj
 0001:0001ffb5       XMMMov                     10020fb5     libvcruntime:memset.obj
 0001:0001fff0       LargeRangeBytes            10020ff0     libvcruntime:memset.obj
 0001:0002002d       XmmMovSmall                1002102d     libvcruntime:memset.obj
 0001:00020040       XmmSmallLoop               10021040     libvcruntime:memset.obj
 0001:00020045       MidRangeBytes              10021045     libvcruntime:memset.obj
 0001:00020061       XMMTrailingBytes           10021061     libvcruntime:memset.obj
 0001:00020075       SmallMov                   10021075     libvcruntime:memset.obj
 0001:0002007d       ByteLoop                   1002107d     libvcruntime:memset.obj
 0001:0002008b       DwordTest                  1002108b     libvcruntime:memset.obj
 0001:0002009b       QwordTest                  1002109b     libvcruntime:memset.obj
 0001:000200b0       QwordLoop                  100210b0     libvcruntime:memset.obj
 0001:000200c3       toend                      100210c3     libvcruntime:memset.obj
 0001:00020350       $$000000                   10021350     libvcruntime:exsup4.obj
 0001:00020382       _lu_top                    10021382     libvcruntime:exsup4.obj
 0001:000203e1       _lu_done                   100213e1     libvcruntime:exsup4.obj
 0001:000203f0       $$000000                   100213f0     libvcruntime:exsup4.obj
 0001:000203f0       __unwind_handler4          100213f0 f   libvcruntime:exsup4.obj
 0001:00020440       $$000000                   10021440     libvcruntime:exsup4.obj
 0001:00020460       $$000000                   10021460     libvcruntime:exsup4.obj
 0001:00020480       $$000000                   10021480     libvcruntime:exsup4.obj
 0001:00020495       ReturnPoint                10021495     libvcruntime:exsup4.obj
 0001:000204a0       $$000000                   100214a0     libvcruntime:exsup4.obj
 0001:00020522       ?try_get_first_available_module@@YAPAUHINSTANCE__@@QBW4module_id@?A0xeb687146@@0@Z 10021522 f   libvcruntime:winapi_downlevel.obj
 0001:000205bc       ?try_get_function@@YAPAXW4function_id@?A0xeb687146@@QBDQBW4module_id@2@2@Z 100215bc f   libvcruntime:winapi_downlevel.obj
 0001:00020740       $$000000                   10021740     libvcruntime:memcpy.obj
 0001:00020740       $$000000                   10021740     libvcruntime:memmove.obj
 0001:00020760       CopyUp                     10021760     libvcruntime:memcpy.obj
 0001:00020760       CopyUp                     10021760     libvcruntime:memmove.obj
 0001:00020784       CopyUpLargeMov             10021784     libvcruntime:memcpy.obj
 0001:00020784       CopyUpLargeMov             10021784     libvcruntime:memmove.obj
 0001:00020797       CopyUpSSE2Check            10021797     libvcruntime:memcpy.obj
 0001:00020797       CopyUpSSE2Check            10021797     libvcruntime:memmove.obj
 0001:000207b0       AtomChk                    100217b0     libvcruntime:memcpy.obj
 0001:000207b0       AtomChk                    100217b0     libvcruntime:memmove.obj
 0001:000207d6       PalignHead4                100217d6     libvcruntime:memcpy.obj
 0001:000207d6       PalignHead4                100217d6     libvcruntime:memmove.obj
 0001:000207e9       PalignHead8                100217e9     libvcruntime:memcpy.obj
 0001:000207e9       PalignHead8                100217e9     libvcruntime:memmove.obj
 0001:00020800       PalignLoop                 10021800     libvcruntime:memcpy.obj
 0001:00020800       PalignLoop                 10021800     libvcruntime:memmove.obj
 0001:00020812       MovPalign12                10021812     libvcruntime:memcpy.obj
 0001:00020812       MovPalign12                10021812     libvcruntime:memmove.obj
 0001:0002081c       PalignLoop12               1002181c     libvcruntime:memcpy.obj
 0001:0002081c       PalignLoop12               1002181c     libvcruntime:memmove.obj
 0001:0002086d       MovPalign8                 1002186d     libvcruntime:memcpy.obj
 0001:0002086d       MovPalign8                 1002186d     libvcruntime:memmove.obj
 0001:00020878       PalignLoop8                10021878     libvcruntime:memcpy.obj
 0001:00020878       PalignLoop8                10021878     libvcruntime:memmove.obj
 0001:000208c6       MovPalign4                 100218c6     libvcruntime:memcpy.obj
 0001:000208c6       MovPalign4                 100218c6     libvcruntime:memmove.obj
 0001:000208d0       PalignLoop4                100218d0     libvcruntime:memcpy.obj
 0001:000208d0       PalignLoop4                100218d0     libvcruntime:memmove.obj
 0001:0002091c       PalignTail                 1002191c     libvcruntime:memcpy.obj
 0001:0002091c       PalignTail                 1002191c     libvcruntime:memmove.obj
 0001:00020934       PalignTail4                10021934     libvcruntime:memcpy.obj
 0001:00020934       PalignTail4                10021934     libvcruntime:memmove.obj
 0001:00020947       PalignTail8                10021947     libvcruntime:memcpy.obj
 0001:00020947       PalignTail8                10021947     libvcruntime:memmove.obj
 0001:0002095e       PalignTailLE3              1002195e     libvcruntime:memcpy.obj
 0001:0002095e       PalignTailLE3              1002195e     libvcruntime:memmove.obj
 0001:00020967       Dword_align                10021967     libvcruntime:memcpy.obj
 0001:00020967       Dword_align                10021967     libvcruntime:memmove.obj
 0001:0002096f       Dword_up_align_loop        1002196f     libvcruntime:memcpy.obj
 0001:0002096f       Dword_up_align_loop        1002196f     libvcruntime:memmove.obj
 0001:00020982       Dword_align_Ok             10021982     libvcruntime:memcpy.obj
 0001:00020982       Dword_align_Ok             10021982     libvcruntime:memmove.obj
 0001:0002099c       ByteCopyUp                 1002199c     libvcruntime:memcpy.obj
 0001:0002099c       ByteCopyUp                 1002199c     libvcruntime:memmove.obj
 0001:000209a4       TrailingUpVec              100219a4     libvcruntime:memcpy.obj
 0001:000209a4       TrailingUpVec              100219a4     libvcruntime:memmove.obj
 0001:000209b4       TrailingUp0                100219b4     libvcruntime:memcpy.obj
 0001:000209b4       TrailingUp0                100219b4     libvcruntime:memmove.obj
 0001:000209bc       TrailingUp1                100219bc     libvcruntime:memcpy.obj
 0001:000209bc       TrailingUp1                100219bc     libvcruntime:memmove.obj
 0001:000209c8       TrailingUp2                100219c8     libvcruntime:memcpy.obj
 0001:000209c8       TrailingUp2                100219c8     libvcruntime:memmove.obj
 0001:000209dc       TrailingUp3                100219dc     libvcruntime:memcpy.obj
 0001:000209dc       TrailingUp3                100219dc     libvcruntime:memmove.obj
 0001:000209f4       CopyDown                   100219f4     libvcruntime:memcpy.obj
 0001:000209f4       CopyDown                   100219f4     libvcruntime:memmove.obj
 0001:00020a19       CopyDownNotAligned         10021a19     libvcruntime:memcpy.obj
 0001:00020a19       CopyDownNotAligned         10021a19     libvcruntime:memmove.obj
 0001:00020a20       CopyDownAlignLoop          10021a20     libvcruntime:memcpy.obj
 0001:00020a20       CopyDownAlignLoop          10021a20     libvcruntime:memmove.obj
 0001:00020a2d       CopyDownAligned            10021a2d     libvcruntime:memcpy.obj
 0001:00020a2d       CopyDownAligned            10021a2d     libvcruntime:memmove.obj
 0001:00020a50       TrailingDownVec            10021a50     libvcruntime:memcpy.obj
 0001:00020a50       TrailingDownVec            10021a50     libvcruntime:memmove.obj
 0001:00020a60       TrailingDown0              10021a60     libvcruntime:memcpy.obj
 0001:00020a60       TrailingDown0              10021a60     libvcruntime:memmove.obj
 0001:00020a68       TrailingDown1              10021a68     libvcruntime:memcpy.obj
 0001:00020a68       TrailingDown1              10021a68     libvcruntime:memmove.obj
 0001:00020a78       TrailingDown2              10021a78     libvcruntime:memcpy.obj
 0001:00020a78       TrailingDown2              10021a78     libvcruntime:memmove.obj
 0001:00020a8c       TrailingDown3              10021a8c     libvcruntime:memcpy.obj
 0001:00020a8c       TrailingDown3              10021a8c     libvcruntime:memmove.obj
 0001:00020aa5       XmmMovLargeAlignTest       10021aa5     libvcruntime:memcpy.obj
 0001:00020aa5       XmmMovLargeAlignTest       10021aa5     libvcruntime:memmove.obj
 0001:00020aad       XmmMovAlignLoop            10021aad     libvcruntime:memcpy.obj
 0001:00020aad       XmmMovAlignLoop            10021aad     libvcruntime:memmove.obj
 0001:00020abc       XmmMovLargeLoop            10021abc     libvcruntime:memcpy.obj
 0001:00020abc       XmmMovLargeLoop            10021abc     libvcruntime:memmove.obj
 0001:00020b2c       XmmMovSmallTest            10021b2c     libvcruntime:memcpy.obj
 0001:00020b2c       XmmMovSmallTest            10021b2c     libvcruntime:memmove.obj
 0001:00020b31       XmmMovSmallLoop            10021b31     libvcruntime:memcpy.obj
 0001:00020b31       XmmMovSmallLoop            10021b31     libvcruntime:memmove.obj
 0001:00020b54       CopyDownSmall              10021b54     libvcruntime:memcpy.obj
 0001:00020b54       CopyDownSmall              10021b54     libvcruntime:memmove.obj
 0001:00020b5c       CopyDownDwordLoop          10021b5c     libvcruntime:memcpy.obj
 0001:00020b5c       CopyDownDwordLoop          10021b5c     libvcruntime:memmove.obj
 0001:00020b71       CopyDownByteTest           10021b71     libvcruntime:memcpy.obj
 0001:00020b71       CopyDownByteTest           10021b71     libvcruntime:memmove.obj
 0001:00020b75       CopyDownByteLoop           10021b75     libvcruntime:memcpy.obj
 0001:00020b75       CopyDownByteLoop           10021b75     libvcruntime:memmove.obj
 0001:00020b84       CopyDownReturn             10021b84     libvcruntime:memcpy.obj
 0001:00020b84       CopyDownReturn             10021b84     libvcruntime:memmove.obj
 0001:00020b90       XmmCopy                    10021b90     libvcruntime:memcpy.obj
 0001:00020b90       XmmCopy                    10021b90     libvcruntime:memmove.obj
 0001:00020b9d       XmmCopyAligned             10021b9d     libvcruntime:memcpy.obj
 0001:00020b9d       XmmCopyAligned             10021b9d     libvcruntime:memmove.obj
 0001:00020bb0       XmmCopyLargeLoop           10021bb0     libvcruntime:memcpy.obj
 0001:00020bb0       XmmCopyLargeLoop           10021bb0     libvcruntime:memmove.obj
 0001:00020c0d       XmmCopySmallTest           10021c0d     libvcruntime:memcpy.obj
 0001:00020c0d       XmmCopySmallTest           10021c0d     libvcruntime:memmove.obj
 0001:00020c20       XmmCopySmallLoop           10021c20     libvcruntime:memcpy.obj
 0001:00020c20       XmmCopySmallLoop           10021c20     libvcruntime:memmove.obj
 0001:00020c3b       CopyUpDwordMov             10021c3b     libvcruntime:memcpy.obj
 0001:00020c3b       CopyUpDwordMov             10021c3b     libvcruntime:memmove.obj
 0001:00020c40       CopyUpDwordTest            10021c40     libvcruntime:memcpy.obj
 0001:00020c40       CopyUpDwordTest            10021c40     libvcruntime:memmove.obj
 0001:00020c47       CopyUpDwordLoop            10021c47     libvcruntime:memcpy.obj
 0001:00020c47       CopyUpDwordLoop            10021c47     libvcruntime:memmove.obj
 0001:00020c56       CopyUpByteTest             10021c56     libvcruntime:memcpy.obj
 0001:00020c56       CopyUpByteTest             10021c56     libvcruntime:memmove.obj
 0001:00020c5d       CopyUpByteLoop             10021c5d     libvcruntime:memcpy.obj
 0001:00020c5d       CopyUpByteLoop             10021c5d     libvcruntime:memmove.obj
 0001:00020c70       CopyUpReturn               10021c70     libvcruntime:memcpy.obj
 0001:00020c70       CopyUpReturn               10021c70     libvcruntime:memmove.obj
 0001:00020c80       XmmCopyUnaligned           10021c80     libvcruntime:memcpy.obj
 0001:00020c80       XmmCopyUnaligned           10021c80     libvcruntime:memmove.obj
 0001:00020c93       XmmAlignByte               10021c93     libvcruntime:memcpy.obj
 0001:00020c93       XmmAlignByte               10021c93     libvcruntime:memmove.obj
 0001:00020c9c       XmmAlignDwordTest          10021c9c     libvcruntime:memcpy.obj
 0001:00020c9c       XmmAlignDwordTest          10021c9c     libvcruntime:memmove.obj
 0001:00020ca1       XmmAlignDwordLoop          10021ca1     libvcruntime:memcpy.obj
 0001:00020ca1       XmmAlignDwordLoop          10021ca1     libvcruntime:memmove.obj
 0001:00020cae       XmmAlignAdjustCnt          10021cae     libvcruntime:memcpy.obj
 0001:00020cae       XmmAlignAdjustCnt          10021cae     libvcruntime:memmove.obj
 0001:00020cc0       $$000000                   10021cc0     libvcruntime:exsup.obj
 0001:00020ccb       __NLG_Go                   10021ccb     libvcruntime:exsup.obj
 0001:00020ce0       $$000000                   10021ce0     libvcruntime:exsup.obj
 0001:00021037       ?internal_to_string@@YAHQADIQAU_strflt@@HQAH2@Z 10022037 f   libucrt:fcvt.obj
 0001:000210b2       ?try_get_ptd_buffer@@YAPADXZ 100220b2 f   libucrt:fcvt.obj
 0001:00021d00       $$000000                   10022d00     libucrt:strncpy.obj
 0001:00021e24       ??$common_vsprintf@Vstandard_base@__crt_stdio_output@@D@@YAH_KQADIQBDQAU__crt_locale_pointers@@1@Z 10022e24 f   libucrt:output.obj
 0001:0002250d       $LN50                      1002350d     libucrt:output.obj
 0001:00022a2c       $LN18                      10023a2c     libucrt:output.obj
 0001:00022a40       $LN17                      10023a40     libucrt:output.obj
 0001:00023197       ??$__acrt_convert_wcs_mbs_cp@D_WV<lambda_62f6974d9771e494a5ea317cc32e971c>@@U__crt_win32_buffer_internal_dynamic_resizing@@@@YAHQBDAAV?$__crt_win32_buffer@_WU__crt_win32_buffer_internal_dynamic_resizing@@@@ABV<lambda_62f6974d9771e494a5ea317cc32e971c>@@I@Z 10024197 f   libucrt:rename.obj
 0001:000233cb       ?_strupr_s_l_stat@@YAHQADIQAU__crt_locale_pointers@@@Z 100243cb f   libucrt:strupr.obj
 0001:00023762       ??$?RV<lambda_03b1d95aef87969028cfba75ccab2455>@@AAV<lambda_6e4b09c48022b2350581041d5f6b0c4c>@@V<lambda_22bdf7517842c4b3e53723af5aa32b9e>@@@?$__crt_seh_guarded_call@X@@QAEX$$QAV<lambda_03b1d95aef87969028cfba75ccab2455>@@AAV<lambda_6e4b09c48022b2350581041d5f6b0c4c>@@$$QAV<lambda_22bdf7517842c4b3e53723af5aa32b9e>@@@Z 10024762 f   libucrt:exit.obj
 0001:000237af       ??R<lambda_6e4b09c48022b2350581041d5f6b0c4c>@@QBE@XZ 100247af f   libucrt:exit.obj
 0001:00023889       ?atexit_exception_filter@@YAHK@Z 10024889 f   libucrt:exit.obj
 0001:0002389c       ?common_exit@@YAXHW4_crt_exit_cleanup_mode@@W4_crt_exit_return_mode@@@Z 1002489c f   libucrt:exit.obj
 0001:00023900       ?exit_or_terminate_process@@YAXI@Z 10024900 f   libucrt:exit.obj
 0001:00023942       ?is_managed_app@@YA_NXZ    10024942 f   libucrt:exit.obj
 0001:00023985       ?try_cor_exit_process@@YAXI@Z 10024985 f   libucrt:exit.obj
 0001:00023a13       ??$common_configure_argv@D@@YAHW4_crt_argv_mode@@@Z 10024a13 f   libucrt:argv_parsing.obj
 0001:00023b49       ??$parse_command_line@D@@YAXPADPAPAD0PAI2@Z 10024b49 f   libucrt:argv_parsing.obj
 0001:00023d17       ??$common_initialize_environment_nolock@D@@YAHXZ 10024d17 f   libucrt:environment_initialization.obj
 0001:00023d6a       ??$create_environment@D@@YAQAPADQAD@Z 10024d6a f   libucrt:environment_initialization.obj
 0001:00023e3a       ??$free_environment@D@@YAXQAPAD@Z 10024e3a f   libucrt:environment_initialization.obj
 0001:00023e3a       ??$free_environment@_W@@YAXQAPA_W@Z 10024e3a f   libucrt:environment_initialization.obj
 0001:00023e92       ??$uninitialize_environment_internal@D@@YAXAAPAPAD@Z 10024e92 f   libucrt:environment_initialization.obj
 0001:00023ead       ??$uninitialize_environment_internal@_W@@YAXAAPAPA_W@Z 10024ead f   libucrt:environment_initialization.obj
 0001:00023f04       ??$?RV<lambda_69a2805e680e0e292e8ba93315fe43a8>@@AAV<lambda_f03950bc5685219e0bcd2087efbe011e>@@V<lambda_03fcd07e894ec930e3f35da366ca99d6>@@@?$__crt_seh_guarded_call@H@@QAEH$$QAV<lambda_69a2805e680e0e292e8ba93315fe43a8>@@AAV<lambda_f03950bc5685219e0bcd2087efbe011e>@@$$QAV<lambda_03fcd07e894ec930e3f35da366ca99d6>@@@Z 10024f04 f   libucrt:onexit.obj
 0001:00023f5f       ??$?RV<lambda_8e746cf0007f6ed984d6f78af1fec997>@@AAV<lambda_22ebabd17bc4fa466a2aca6d8deb888d>@@V<lambda_18ed0c0b38a6dc0daf1e7ac6d6adf05e>@@@?$__crt_seh_guarded_call@H@@QAEH$$QAV<lambda_8e746cf0007f6ed984d6f78af1fec997>@@AAV<lambda_22ebabd17bc4fa466a2aca6d8deb888d>@@$$QAV<lambda_18ed0c0b38a6dc0daf1e7ac6d6adf05e>@@@Z 10024f5f f   libucrt:onexit.obj
 0001:00023fd9       ??R<lambda_22ebabd17bc4fa466a2aca6d8deb888d>@@QBEHXZ 10024fd9 f   libucrt:onexit.obj
 0001:00024102       ??R<lambda_f03950bc5685219e0bcd2087efbe011e>@@QBEHXZ 10025102 f   libucrt:onexit.obj
 0001:0002427b       _initialize_global_variables 1002527b f   libucrt:initialization.obj
 0001:00024288       _initialize_c              10025288 f   libucrt:initialization.obj
 0001:000242a2       _initialize_environment    100252a2 f   libucrt:initialization.obj
 0001:000242a2       _initialize_global_state_isolation 100252a2 f   libucrt:initialization.obj
 0001:000242a2       _report_memory_leaks       100252a2 f   libucrt:initialization.obj
 0001:000242a2       _uninitialize_c            100252a2 f   libucrt:initialization.obj
 0001:000242a2       _uninitialize_global_state_isolation 100252a2 f   libucrt:initialization.obj
 0001:000242a5       _uninitialize_environment  100252a5 f   libucrt:initialization.obj
 0001:000242ad       _initialize_pointers       100252ad f   libucrt:initialization.obj
 0001:000242db       _uninitialize_vcruntime    100252db f   libucrt:initialization.obj
 0001:000242e4       _uninitialize_allocated_memory 100252e4 f   libucrt:initialization.obj
 0001:000242fb       _uninitialize_allocated_io_buffers 100252fb f   libucrt:initialization.obj
 0001:0002434b       ??R<lambda_af42a3ee9806e9a7305d451646e05244>@@QBEXAAPAU__crt_multibyte_data@@@Z 1002534b f   libucrt:initialization.obj
 0001:00024600       $$000000                   10025600     libucrt:strncmp.obj
 0001:0002477d       ??$?RV<lambda_15ade71b0218206bbe3333a0c9b79046>@@AAV<lambda_da44e0f8b0f19ba52fefafb335991732>@@V<lambda_207f2d024fc103971653565357d6cd41>@@@?$__crt_seh_guarded_call@X@@QAEX$$QAV<lambda_15ade71b0218206bbe3333a0c9b79046>@@AAV<lambda_da44e0f8b0f19ba52fefafb335991732>@@$$QAV<lambda_207f2d024fc103971653565357d6cd41>@@@Z 1002577d f   libucrt:per_thread_data.obj
 0001:000247cf       ??$?RV<lambda_38edbb1296d33220d7e4dd0ed76b244a>@@AAV<lambda_5ce1d447e08cb34b2473517608e21441>@@V<lambda_fb385d3da700c9147fc39e65dd577a8c>@@@?$__crt_seh_guarded_call@X@@QAEX$$QAV<lambda_38edbb1296d33220d7e4dd0ed76b244a>@@AAV<lambda_5ce1d447e08cb34b2473517608e21441>@@$$QAV<lambda_fb385d3da700c9147fc39e65dd577a8c>@@@Z 100257cf f   libucrt:per_thread_data.obj
 0001:0002483a       ??$?RV<lambda_6affb1475c98b40b75cdec977db92e3c>@@AAV<lambda_b8d4b9c228a6ecc3f80208dbb4b4a104>@@V<lambda_608742c3c92a14382c1684fc64f96c88>@@@?$__crt_seh_guarded_call@X@@QAEX$$QAV<lambda_6affb1475c98b40b75cdec977db92e3c>@@AAV<lambda_b8d4b9c228a6ecc3f80208dbb4b4a104>@@$$QAV<lambda_608742c3c92a14382c1684fc64f96c88>@@@Z 1002583a f   libucrt:per_thread_data.obj
 0001:0002488f       ??$?RV<lambda_a7e850c220f1c8d1e6efeecdedd162c6>@@AAV<lambda_46720907175c18b6c9d2717bc0d2d362>@@V<lambda_9048902d66e8d99359bc9897bbb930a8>@@@?$__crt_seh_guarded_call@X@@QAEX$$QAV<lambda_a7e850c220f1c8d1e6efeecdedd162c6>@@AAV<lambda_46720907175c18b6c9d2717bc0d2d362>@@$$QAV<lambda_9048902d66e8d99359bc9897bbb930a8>@@@Z 1002588f f   libucrt:per_thread_data.obj
 0001:000248e9       ?construct_ptd@@YAXQAU__acrt_ptd@@QAPAU__crt_locale_data@@@Z 100258e9 f   libucrt:per_thread_data.obj
 0001:00024982       ?destroy_fls@@YGXPAX@Z     10025982 f   libucrt:per_thread_data.obj
 0001:000249a3       ?destroy_ptd@@YAXQAU__acrt_ptd@@@Z 100259a3 f   libucrt:per_thread_data.obj
 0001:00024a70       ?replace_current_thread_locale_nolock@@YAXQAU__acrt_ptd@@QAU__crt_locale_data@@@Z 10025a70 f   libucrt:per_thread_data.obj
 0001:00024d93       ??$?RV<lambda_e5124f882df8998aaf41531e079ba474>@@AAV<lambda_3e16ef9562a7dcce91392c22ab16ea36>@@V<lambda_e25ca0880e6ef98be67edffd8c599615>@@@?$__crt_seh_guarded_call@X@@QAEX$$QAV<lambda_e5124f882df8998aaf41531e079ba474>@@AAV<lambda_3e16ef9562a7dcce91392c22ab16ea36>@@$$QAV<lambda_e25ca0880e6ef98be67edffd8c599615>@@@Z 10025d93 f   libucrt:wsetlocale.obj
 0001:000251a0       ?should_round_up@@YA_NQBDHW4__acrt_has_trailing_digits@@W4__acrt_rounding_mode@@@Z 100261a0 f   libucrt:_fptostr.obj
 0001:00026cff       _memcpy_s                  10027cff f   libucrt:cfout.obj
 0001:00026cff       _memcpy_s                  10027cff f   libucrt:mbctype.obj
 0001:00026d80       ?__acrt_LCMapStringA_stat@@YAHPAU__crt_locale_pointers@@PB_WKPBDHPADHHH@Z 10027d80 f   libucrt:lcmapstringa.obj
 0001:00027560       ?fe_to_nearest@@YA_NQBN_KF@Z 10028560 f   libucrt:cvt.obj
 0001:00027603       ?fp_format_a@@YAHQBNPADIQADIH_NIQAU__crt_locale_pointers@@W4__acrt_rounding_mode@@@Z 10028603 f   libucrt:cvt.obj
 0001:00027912       ?fp_format_e@@YAHQBNQADI1IH_NIQAU__crt_locale_pointers@@W4__acrt_rounding_mode@@@Z 10028912 f   libucrt:cvt.obj
 0001:000279ba       ?fp_format_e_internal@@YAHQADIH_NIQAU_strflt@@1QAU__crt_locale_pointers@@@Z 100289ba f   libucrt:cvt.obj
 0001:00027b02       ?fp_format_f@@YAHQBNQADI1IHQAU__crt_locale_pointers@@W4__acrt_rounding_mode@@@Z 10028b02 f   libucrt:cvt.obj
 0001:00027b93       ?fp_format_f_internal@@YAHQADIHQAU_strflt@@_NQAU__crt_locale_pointers@@@Z 10028b93 f   libucrt:cvt.obj
 0001:00027c8b       ?fp_format_g@@YAHQBNQADI1IH_NIW4__acrt_rounding_mode@@QAU__crt_locale_pointers@@@Z 10028c8b f   libucrt:cvt.obj
 0001:00027d55       ?fp_format_nan_or_infinity@@YAHW4__acrt_fp_class@@_NPADI1@Z 10028d55 f   libucrt:cvt.obj
 0001:00027dea       ?shift_bytes@@YAXQADI0H@Z  10028dea f   libucrt:cvt.obj
 0001:00027e1e       ?should_round_up@@YA_NQBN_KFW4__acrt_rounding_mode@@@Z 10028e1e f   libucrt:cvt.obj
 0001:00028185       ?initialize_inherited_file_handles_nolock@@YAXXZ 10029185 f   libucrt:ioinit.obj
 0001:0002823b       ?initialize_stdio_handles_nolock@@YAXXZ 1002923b f   libucrt:ioinit.obj
 0001:000284e3       ?try_get_AreFileApisANSI@@YAP6GHXZXZ 100294e3 f   libucrt:winapi_thunks.obj
 0001:000284fd       ?try_get_LCMapStringEx@@YAP6GHPB_WK0HPA_WHPAU_nlsversioninfo@@PAXJ@ZXZ 100294fd f   libucrt:winapi_thunks.obj
 0001:00028517       ?try_get_LocaleNameToLCID@@YAP6GKPB_WK@ZXZ 10029517 f   libucrt:winapi_thunks.obj
 0001:00028531       ?try_get_first_available_module@@YAPAUHINSTANCE__@@QBW4module_id@?A0x391cf84c@@0@Z 10029531 f   libucrt:winapi_thunks.obj
 0001:000285f8       ?try_get_function@@YAPAXW4function_id@?A0x391cf84c@@QBDQBW4module_id@2@2@Z 100295f8 f   libucrt:winapi_thunks.obj
 0001:00028a6e       ?<lambda_invoker_cdecl>@<lambda_838c7f62c73c983481e27c09e84b0b5d>@@CAHPBX0@Z 10029a6e f   libucrt:argv_wildcards.obj
 0001:00028a86       ??$__acrt_convert_wcs_mbs_cp@_WDV<lambda_28bda7af82a03b66c1cb3803a755f95d>@@U__crt_win32_buffer_internal_dynamic_resizing@@@@YAHQB_WAAV?$__crt_win32_buffer@DU__crt_win32_buffer_internal_dynamic_resizing@@@@ABV<lambda_28bda7af82a03b66c1cb3803a755f95d>@@I@Z 10029a86 f   libucrt:argv_wildcards.obj
 0001:00028b55       ??$common_expand_argv_wildcards@D@@YAHQAPADQAPAPAD@Z 10029b55 f   libucrt:argv_wildcards.obj
 0001:00028d44       ??$copy_and_add_argument_to_buffer@D@@YAHQBD0IAAV?$argument_list@D@?A0x5f5c8891@@@Z 10029d44 f   libucrt:argv_wildcards.obj
 0001:00028df5       ??$expand_argument_wildcards@D@@YAHQAD0AAV?$argument_list@D@?A0x5f5c8891@@@Z 10029df5 f   libucrt:argv_wildcards.obj
 0001:00029088       ?expand_if_necessary@?$argument_list@D@?A0x5f5c8891@@AAEHXZ 1002a088 f   libucrt:argv_wildcards.obj
 0001:0002911a       ??$__acrt_convert_wcs_mbs_cp@_WDV<lambda_0fec1a7b3f42a53036604e18c2d5e07e>@@U__crt_win32_buffer_no_resizing@@@@YAHQB_WAAV?$__crt_win32_buffer@DU__crt_win32_buffer_no_resizing@@@@ABV<lambda_0fec1a7b3f42a53036604e18c2d5e07e>@@I@Z 1002a11a f   libucrt:getmodulefilenamea.obj
 0001:000292bd       ??$?RV<lambda_ceb1ee4838e85a9d631eb091e2fbe199>@@AAV<lambda_ae742caa10f662c28703da3d2ea5e57e>@@V<lambda_cd08b5d6af4937fe54fc07d0c9bf6b37>@@@?$__crt_seh_guarded_call@X@@QAEX$$QAV<lambda_ceb1ee4838e85a9d631eb091e2fbe199>@@AAV<lambda_ae742caa10f662c28703da3d2ea5e57e>@@$$QAV<lambda_cd08b5d6af4937fe54fc07d0c9bf6b37>@@@Z 1002a2bd f   libucrt:mbctype.obj
 0001:0002930a       ??R<lambda_ae742caa10f662c28703da3d2ea5e57e>@@QBEXXZ 1002a30a f   libucrt:mbctype.obj
 0001:0002938d       ?CPtoLocaleName@@YAPB_WH@Z 1002a38d f   libucrt:mbctype.obj
 0001:000293cb       ?getSystemCP@@YAHH@Z       1002a3cb f   libucrt:mbctype.obj
 0001:0002943c       ?setSBCS@@YAXPAU__crt_multibyte_data@@@Z 1002a43c f   libucrt:mbctype.obj
 0001:000294a1       ?setSBUpLow@@YAXPAU__crt_multibyte_data@@@Z 1002a4a1 f   libucrt:mbctype.obj
 0001:00029621       ?setmbcp_internal@@YAHH_NQAU__acrt_ptd@@QAPAU__crt_multibyte_data@@@Z 1002a621 f   libucrt:mbctype.obj
 0001:00029735       ?update_thread_multibyte_data_internal@@YAPAU__crt_multibyte_data@@QAU__acrt_ptd@@QAPAU1@@Z 1002a735 f   libucrt:mbctype.obj
 0001:00029a23       ?x_ismbbtype_l@@YAHPAU__crt_locale_pointers@@IHH@Z 1002aa23 f   libucrt:ismbbyte.obj
 0001:00029b62       ?find_end_of_double_null_terminated_sequence@@YAPB_WQB_W@Z 1002ab62 f   libucrt:get_environment_from_os.obj
 0001:00029d3e       ??$?RV<lambda_cbab9ec6f41b0180b23cc171c22676b0>@@AAV<lambda_44731a7d0e6d81c3e6aa82d741081786>@@V<lambda_4b292cb8dd18144e164572427af410ab>@@@?$__crt_seh_guarded_call@P6AXH@Z@@QAEP6AXH@Z$$QAV<lambda_cbab9ec6f41b0180b23cc171c22676b0>@@AAV<lambda_44731a7d0e6d81c3e6aa82d741081786>@@$$QAV<lambda_4b292cb8dd18144e164572427af410ab>@@@Z 1002ad3e f   libucrt:signal.obj
 0001:00029da2       ?get_global_action_nolock@@YAPAP6AXH@ZH@Z 1002ada2 f   libucrt:signal.obj
 0001:00029de4       ?siglookup@@YAPAU__crt_signal_action_t@@HQAU1@@Z 1002ade4 f   libucrt:signal.obj
 0001:0002a09d       ??$?RV<lambda_2866be3712abc81a800a822484c830d8>@@AAV<lambda_39ca0ed439415581b5b15c265174cece>@@V<lambda_2b24c74d71094a6cd0cb82e44167d71b>@@@?$__crt_seh_guarded_call@X@@QAEX$$QAV<lambda_2866be3712abc81a800a822484c830d8>@@AAV<lambda_39ca0ed439415581b5b15c265174cece>@@$$QAV<lambda_2b24c74d71094a6cd0cb82e44167d71b>@@@Z 1002b09d f   libucrt:fflush.obj
 0001:0002a129       ??$?RV<lambda_2cc53f568c5a2bb6f192f930a45d44ea>@@AAV<lambda_ab61a845afdef5b7c387490eaf3616ee>@@V<lambda_c2ffc0b7726aa6be21d5f0026187e748>@@@?$__crt_seh_guarded_call@X@@QAEX$$QAV<lambda_2cc53f568c5a2bb6f192f930a45d44ea>@@AAV<lambda_ab61a845afdef5b7c387490eaf3616ee>@@$$QAV<lambda_c2ffc0b7726aa6be21d5f0026187e748>@@@Z 1002b129 f   libucrt:fflush.obj
 0001:0002a1d5       ?common_flush_all@@YAH_N@Z 1002b1d5 f   libucrt:fflush.obj
 0001:0002a222       ?common_flush_all_should_try_to_flush_stream@@YA_NV__crt_stdio_stream@@QAH@Z 1002b222 f   libucrt:fflush.obj
 0001:0002a255       ?is_stream_flushable_or_commitable@@YA_NJ@Z 1002b255 f   libucrt:fflush.obj
 0001:0002a934       ?free_crt_array_internal@@YAXQAPBXI@Z 1002b934 f   libucrt:inittime.obj
 0001:0002aba0       $$000000                   1002bba0     libucrt:log10_impl.obj
 0001:0002acb0       $$000000                   1002bcb0     libucrt:ceil_pentium4.obj
 0001:0002ade9       ??R<lambda_3d301b9e52f5099be73030e1f0bf487e>@@QBEIPBD@Z 1002bde9 f   libucrt:mbrtowc.obj
 0001:0002b3ea       ?GetTableIndexFromLocaleName@@YAHPB_W@Z 1002c3ea f   libucrt:lcidtoname_downlevel.obj
 0001:0002b95e       ??$common_tcsncpy_s@D@@YAHQADIQBDI@Z 1002c95e f   libucrt:strncpy_s.obj
 0001:0002ba20       $$000000                   1002ca20     libucrt:strpbrk.obj
 0001:0002bb04       ?initialize_multibyte@@YAHXZ 1002cb04 f   libucrt:multibyte_initializer.obj
 0001:0002bbaf       ??$?RV<lambda_9e9de3de5fa147e2223d7db92bc10aa6>@@AAV<lambda_38ce7e780aa69e748d6df282ebc68efe>@@V<lambda_8ca6da459f0f6780f1cff60fdc3d00e5>@@@?$__crt_seh_guarded_call@H@@QAEH$$QAV<lambda_9e9de3de5fa147e2223d7db92bc10aa6>@@AAV<lambda_38ce7e780aa69e748d6df282ebc68efe>@@$$QAV<lambda_8ca6da459f0f6780f1cff60fdc3d00e5>@@@Z 1002cbaf f   libucrt:commit.obj
 0001:0002bcce       ?write_double_translated_ansi_nolock@@YA?AUwrite_result@?A0x17268360@@HQBDI@Z 1002ccce f   libucrt:write.obj
 0001:0002c07a       ?write_double_translated_unicode_nolock@@YA?AUwrite_result@?A0x17268360@@QBDI@Z 1002d07a f   libucrt:write.obj
 0001:0002c0e2       ?write_requires_double_translation_nolock@@YA_NH@Z 1002d0e2 f   libucrt:write.obj
 0001:0002c153       ?write_text_ansi_nolock@@YA?AUwrite_result@?A0x17268360@@HQBDI@Z 1002d153 f   libucrt:write.obj
 0001:0002c22e       ?write_text_utf16le_nolock@@YA?AUwrite_result@?A0x17268360@@HQBDI@Z 1002d22e f   libucrt:write.obj
 0001:0002c317       ?write_text_utf8_nolock@@YA?AUwrite_result@?A0x17268360@@HQBDI@Z 1002d317 f   libucrt:write.obj
 0001:0002c764       ?to_abstract_control@@YA?AW4__acrt_fenv_abstract_control@@W4__acrt_fenv_machine_sse_control@@@Z 1002d764 f   libucrt:_fenvutils.obj
 0001:0002c820       ?to_abstract_control@@YA?AW4__acrt_fenv_abstract_control@@W4__acrt_fenv_machine_x87_control@@@Z 1002d820 f   libucrt:_fenvutils.obj
 0001:0002c8d9       ?to_machine_sse_control@@YA?AW4__acrt_fenv_machine_sse_control@@W4__acrt_fenv_abstract_control@@@Z 1002d8d9 f   libucrt:_fenvutils.obj
 0001:0002c9a6       ?to_machine_x87_control@@YA?AW4__acrt_fenv_machine_x87_control@@W4__acrt_fenv_abstract_control@@@Z 1002d9a6 f   libucrt:_fenvutils.obj
 0001:0002cd3a       ___hw_cw_sse2              1002dd3a f   libucrt:ieee87.obj
 0001:0002d1c0       __hw_cw                    1002e1c0 f   libucrt:ieee87.obj
 0001:0002d270       $$000000                   1002e270     libucrt:log10_pentium4.obj
 0001:0002d500       $$000000                   1002e500     libucrt:87tran.obj
 0001:0002d710       $$000000                   1002e710     libucrt:87disp.obj
 0001:0002d970       $$000000                   1002e970     libucrt:common.obj
 0001:0002db00       $$000000                   1002eb00     libucrt:genexcep.obj
 0001:0002dfa3       ??$common_lseek_nolock@_J@@YA_JH_JH@Z 1002efa3 f   libucrt:lseek.obj
 0001:0002ed74       ??$?RV<lambda_218ce3db14220d0be481dae8ef3383b6>@@AAV<lambda_628dfdc04ba53c8bfc02c9951375f3f5>@@V<lambda_57dc472bd5c9d5f3b2cbca59b8a843ae>@@@?$__crt_seh_guarded_call@H@@QAEH$$QAV<lambda_218ce3db14220d0be481dae8ef3383b6>@@AAV<lambda_628dfdc04ba53c8bfc02c9951375f3f5>@@$$QAV<lambda_57dc472bd5c9d5f3b2cbca59b8a843ae>@@@Z 1002fd74 f   libucrt:close.obj
 0001:0002ef70       $$000000                   1002ff70     libucrt:_strnicm.obj
 0001:0002efd1       ?__dcrt_lowio_initialize_console_output@@YAXXZ 1002ffd1 f   libucrt:initcon.obj
 0001:0002f270       $$000000                   10030270     LIBCMT:ulldvrm.obj
 0001:0002f2a1       L1                         100302a1     LIBCMT:ulldvrm.obj
 0001:0002f2af       L3                         100302af     LIBCMT:ulldvrm.obj
 0001:0002f2dd       L4                         100302dd     LIBCMT:ulldvrm.obj
 0001:0002f2e6       L5                         100302e6     LIBCMT:ulldvrm.obj
 0001:0002f2e8       L2                         100302e8     LIBCMT:ulldvrm.obj
 0001:0002f310       $$000000                   10030310     LIBCMT:llmul.obj
 0001:0002f329       hard                       10030329     LIBCMT:llmul.obj
 0001:0002f350       $$000000                   10030350     LIBCMT:alloca16.obj
 0001:0002f366       alloca_8                   10030366     LIBCMT:alloca16.obj
 0001:0002f380       $$000000                   10030380     LIBCMT:llshl.obj
 0001:0002f390       MORE32                     10030390     LIBCMT:llshl.obj
 0001:0002f39a       RETZERO                    1003039a     LIBCMT:llshl.obj
 0001:0002f3a0       $$000000                   100303a0     LIBCMT:ftol2.obj
 0001:0002f3b0       $$000000                   100303b0     LIBCMT:ftol2.obj
 0001:0002f3c1       L3B                        100303c1     LIBCMT:ftol2.obj
 0001:0002f404       L3F                        10030404     LIBCMT:ftol2.obj
 0001:0002f40c       L40                        1003040c     LIBCMT:ftol2.obj
 0001:0002f41f       L41                        1003041f     LIBCMT:ftol2.obj
 0001:0002f430       $$000000                   10030430     LIBCMT:lldvrm.obj
 0001:0002f454       L1                         10030454     LIBCMT:lldvrm.obj
 0001:0002f470       L2                         10030470     LIBCMT:lldvrm.obj
 0001:0002f49c       L3                         1003049c     LIBCMT:lldvrm.obj
 0001:0002f4aa       L5                         100304aa     LIBCMT:lldvrm.obj
 0001:0002f4d8       L6                         100304d8     LIBCMT:lldvrm.obj
 0001:0002f4e1       L7                         100304e1     LIBCMT:lldvrm.obj
 0001:0002f4e3       L4                         100304e3     LIBCMT:lldvrm.obj
 0001:0002f4f5       L9                         100304f5     LIBCMT:lldvrm.obj
 0001:0002f509       L8                         10030509     LIBCMT:lldvrm.obj
 0001:0002f510       $$000000                   10030510     LIBCMT:ullshr.obj
 0001:0002f520       MORE32                     10030520     LIBCMT:ullshr.obj
 0001:0002f52a       RETZERO                    1003052a     LIBCMT:ullshr.obj
 0001:0002f530       $$000000                   10030530     LIBCMT:chkstk.obj
 0001:0002f544       cs10                       10030544     LIBCMT:chkstk.obj
 0001:0002f554       cs20                       10030554     LIBCMT:chkstk.obj
 0001:0002f5e0       $$000000                   100305e0     LIBCMT:ftol3.obj
 0001:0002f5f0       _dtoui3_default            100305f0     LIBCMT:ftol3.obj
 0001:0002f619       _dtoui3_notsafe            10030619     LIBCMT:ftol3.obj
 0001:0002f630       _dtoui3_exact              10030630     LIBCMT:ftol3.obj
 0001:0002f639       _dtoui3_neg                10030639     LIBCMT:ftol3.obj
 0001:0002f648       _dtoui3_NaN                10030648     LIBCMT:ftol3.obj
 0001:0002f660       $$000000                   10030660     libucrt:sqrt_sse2_precise.obj
 0001:0002f760       $$000000                   10030760     libucrt:sqrt.obj
 0001:0002f770       $$000000                   10030770     libucrt:sqrt_impl.obj
 0001:0002f830       ??__Fwsinit_@detail@httplib@@YAXXZ 10030830 f   DllMain.obj
 0001:0002f840       ??__Fwsinit_@detail@httplib@@YAXXZ 10030840 f   stdafx.obj
 0002:000001b4       ?wsinit_$initializer$@detail@httplib@@3P6AXXZA 100311b4     DllMain.obj
 0002:000001b8       ??id$initializer$@?$collate@D@std@@2P6AXXZA@@3P6AXXZA 100311b8     DllMain.obj
 0002:000001bc       ??id$initializer$@?$num_put@DV?$ostreambuf_iterator@DU?$char_traits@D@std@@@std@@@std@@2P6AXXZA@@3P6AXXZA 100311bc     DllMain.obj
 0002:000001c0       ??id$initializer$@?$codecvt@DDU_Mbstatet@@@std@@2P6AXXZA@@3P6AXXZA 100311c0     DllMain.obj
 0002:000001c4       ??id$initializer$@?$numpunct@D@std@@2P6AXXZA@@3P6AXXZA 100311c4     DllMain.obj
 0002:000001c8       ?vD2ERR$initializer$@@3P6AXXZA 100311c8     Install.obj
 0002:000001cc       ?vD2StartOfPtr$initializer$@@3P6AXXZA 100311cc     Install.obj
 0002:000001d0       ?vD2VD2SendToServer3$initializer$@@3P6AXXZA 100311d0     Install.obj
 0002:000001d4       ?D2ShowGameMessage$initializer$@@3P6AXXZA 100311d4     Install.obj
 0002:000001d8       ?D2ShowPartyMessage$initializer$@@3P6AXXZA 100311d8     Install.obj
 0002:000001dc       ?D2ShowMap$initializer$@@3P6AXXZA 100311dc     Install.obj
 0002:000001e0       ?D2RevealAutomapRoom$initializer$@@3P6AXXZA 100311e0     Install.obj
 0002:000001e4       ?D2RecvCommand07$initializer$@@3P6AXXZA 100311e4     Install.obj
 0002:000001e8       ?D2RecvCommand08$initializer$@@3P6AXXZA 100311e8     Install.obj
 0002:000001ec       ?D2NewAutomapCell$initializer$@@3P6AXXZA 100311ec     Install.obj
 0002:000001f0       ?D2AddAutomapCell$initializer$@@3P6AXXZA 100311f0     Install.obj
 0002:000001f4       ?D2GetPlayerXOffset$initializer$@@3P6AXXZA 100311f4     Install.obj
 0002:000001f8       ?D2GetPlayerYOffset$initializer$@@3P6AXXZA 100311f8     Install.obj
 0002:000001fc       ?D2SetUiStatus$initializer$@@3P6AXXZA 100311fc     Install.obj
 0002:00000200       ?D2CalcShake$initializer$@@3P6AXXZA 10031200     Install.obj
 0002:00000204       ?D2GetMonsterOwner$initializer$@@3P6AXXZA 10031204     Install.obj
 0002:00000208       ?D2GetUnitFromId$initializer$@@3P6AXXZA 10031208     Install.obj
 0002:0000020c       ?D2GetSelectedUnit$initializer$@@3P6AXXZA 1003120c     Install.obj
 0002:00000210       ?D2InitAutomapLayerStub$initializer$@@3P6AXXZA 10031210     Install.obj
 0002:00000214       ?D2CheckUiStatusStub$initializer$@@3P6AXXZA 10031214     Install.obj
 0002:00000218       ?D2SetAutomapPartyStub$initializer$@@3P6AXXZA 10031218     Install.obj
 0002:0000021c       ?D2SetAutomapNamesStub$initializer$@@3P6AXXZA 1003121c     Install.obj
 0002:00000220       ?D2ChatInputStub$initializer$@@3P6AXXZA 10031220     Install.obj
 0002:00000224       ?D2ItemProtect$initializer$@@3P6AXXZA 10031224     Install.obj
 0002:00000228       ?D2DrawClient$initializer$@@3P6AXXZA 10031228     Install.obj
 0002:0000022c       ?D2Storm511$initializer$@@3P6AXXZA 1003122c     Install.obj
 0002:00000230       ?p_D2AutomapLayerList$initializer$@@3P6AXXZA 10031230     Install.obj
 0002:00000234       ?p_D2AutomapLayer$initializer$@@3P6AXXZA 10031234     Install.obj
 0002:00000238       ?p_D2PlayerUnit$initializer$@@3P6AXXZA 10031238     Install.obj
 0002:0000023c       ?p_D2RosterUnitList$initializer$@@3P6AXXZA 1003123c     Install.obj
 0002:00000240       ?p_D2PetUnitList$initializer$@@3P6AXXZA 10031240     Install.obj
 0002:00000244       ?p_D2DrlgAct$initializer$@@3P6AXXZA 10031244     Install.obj
 0002:00000248       ?p_D2Expansion$initializer$@@3P6AXXZA 10031248     Install.obj
 0002:0000024c       ?p_D2Difficulty$initializer$@@3P6AXXZA 1003124c     Install.obj
 0002:00000250       ?p_D2GameInfo$initializer$@@3P6AXXZA 10031250     Install.obj
 0002:00000254       ?p_D2Fps$initializer$@@3P6AXXZA 10031254     Install.obj
 0002:00000258       ?p_D2Ping$initializer$@@3P6AXXZA 10031258     Install.obj
 0002:0000025c       ?p_D2ExitAppFlag$initializer$@@3P6AXXZA 1003125c     Install.obj
 0002:00000260       ?p_D2InGame$initializer$@@3P6AXXZA 10031260     Install.obj
 0002:00000264       ?p_D2AutomapOn$initializer$@@3P6AXXZA 10031264     Install.obj
 0002:00000268       ?p_D2Divisor$initializer$@@3P6AXXZA 10031268     Install.obj
 0002:0000026c       ?p_D2Offset$initializer$@@3P6AXXZA 1003126c     Install.obj
 0002:00000270       ?p_D2AutomapPos$initializer$@@3P6AXXZA 10031270     Install.obj
 0002:00000274       ?p_D2AutoMapSize$initializer$@@3P6AXXZA 10031274     Install.obj
 0002:00000278       ?p_D2MinmapType$initializer$@@3P6AXXZA 10031278     Install.obj
 0002:0000027c       ?p_D2MinimapOffset$initializer$@@3P6AXXZA 1003127c     Install.obj
 0002:00000280       ?p_D2IsMapShakeOn$initializer$@@3P6AXXZA 10031280     Install.obj
 0002:00000284       ?p_D2MapShakeY$initializer$@@3P6AXXZA 10031284     Install.obj
 0002:00000288       ?p_D2MapShakeX$initializer$@@3P6AXXZA 10031288     Install.obj
 0002:0000028c       ?p_D2ScreenSizeX$initializer$@@3P6AXXZA 1003128c     Install.obj
 0002:00000290       ?p_D2ScreenSizeY$initializer$@@3P6AXXZA 10031290     Install.obj
 0002:00000294       ?p_D2ScreenSize$initializer$@@3P6AXXZA 10031294     Install.obj
 0002:00000298       ?p_D2DrawOffset$initializer$@@3P6AXXZA 10031298     Install.obj
 0002:0000029c       ?p_D2InfoPositionX$initializer$@@3P6AXXZA 1003129c     Install.obj
 0002:000002a0       ?p_D2InfoPositionY$initializer$@@3P6AXXZA 100312a0     Install.obj
 0002:000002a4       ?p_D2QuestData$initializer$@@3P6AXXZA 100312a4     Install.obj
 0002:000002a8       ?p_D2GameQuestData$initializer$@@3P6AXXZA 100312a8     Install.obj
 0002:000002ac       ?p_D2QuestPage$initializer$@@3P6AXXZA 100312ac     Install.obj
 0002:000002b0       ?p_D2MButton$initializer$@@3P6AXXZA 100312b0     Install.obj
 0002:000002b4       ?p_D2LastChatMessage$initializer$@@3P6AXXZA 100312b4     Install.obj
 0002:000002b8       ?p_D2ChatTextLength$initializer$@@3P6AXXZA 100312b8     Install.obj
 0002:000002bc       ?p_D2MousePos$initializer$@@3P6AXXZA 100312bc     Install.obj
 0002:000002c0       ?p_D2LastMousePos$initializer$@@3P6AXXZA 100312c0     Install.obj
 0002:000002c4       ?p_D2CursorInvGridX$initializer$@@3P6AXXZA 100312c4     Install.obj
 0002:000002c8       ?p_D2CursorInvGridY$initializer$@@3P6AXXZA 100312c8     Install.obj
 0002:000002cc       ?p_D2CurrentViewItem$initializer$@@3P6AXXZA 100312cc     Install.obj
 0002:000002d0       ?p_D2GoldInTranBox$initializer$@@3P6AXXZA 100312d0     Install.obj
 0002:000002d4       ?p_D2ShowLifeStr$initializer$@@3P6AXXZA 100312d4     Install.obj
 0002:000002d8       ?p_D2ShowManaStr$initializer$@@3P6AXXZA 100312d8     Install.obj
 0002:000002dc       ?vD2AutomapCellListBaseAddr$initializer$@@3P6AXXZA 100312dc     Install.obj
 0002:000002e0       ?vD2LoadUiImageFunc$initializer$@@3P6AXXZA 100312e0     Install.obj
 0002:000002e4       ?D2GetObjectTxt$initializer$@@3P6AXXZA 100312e4     Install.obj
 0002:000002e8       ?D2GetLevelDefTxt$initializer$@@3P6AXXZA 100312e8     Install.obj
 0002:000002ec       ?D2GetLevelTxt$initializer$@@3P6AXXZA 100312ec     Install.obj
 0002:000002f0       ?D2GetItemTxt$initializer$@@3P6AXXZA 100312f0     Install.obj
 0002:000002f4       ?D2GetItemTxt2$initializer$@@3P6AXXZA 100312f4     Install.obj
 0002:000002f8       ?D2GetItemTxt3$initializer$@@3P6AXXZA 100312f8     Install.obj
 0002:000002fc       ?D2GetTreasureClasses$initializer$@@3P6AXXZA 100312fc     Install.obj
 0002:00000300       ?D2GetSuperUniqueTxt$initializer$@@3P6AXXZA 10031300     Install.obj
 0002:00000304       ?D2CheckItemType$initializer$@@3P6AXXZA 10031304     Install.obj
 0002:00000308       ?D2GetItemFileIndex$initializer$@@3P6AXXZA 10031308     Install.obj
 0002:0000030c       ?D2GetItemType$initializer$@@3P6AXXZA 1003130c     Install.obj
 0002:00000310       ?D2GetMagicAffixRecord$initializer$@@3P6AXXZA 10031310     Install.obj
 0002:00000314       ?D2GetSkillById$initializer$@@3P6AXXZA 10031314     Install.obj
 0002:00000318       ?D2GetListFromItem$initializer$@@3P6AXXZA 10031318     Install.obj
 0002:0000031c       ?D2GetListFromItem2$initializer$@@3P6AXXZA 1003131c     Install.obj
 0002:00000320       ?D2GetInvItemCount$initializer$@@3P6AXXZA 10031320     Install.obj
 0002:00000324       ?D2GetStatFromStatList$initializer$@@3P6AXXZA 10031324     Install.obj
 0002:00000328       ?D2GetStatListWithFlag$initializer$@@3P6AXXZA 10031328     Install.obj
 0002:0000032c       ?D2GetUnitStat$initializer$@@3P6AXXZA 1003132c     Install.obj
 0002:00000330       ?D2GetUnitBaseStat$initializer$@@3P6AXXZA 10031330     Install.obj
 0002:00000334       ?D2GetMonsterHpPercent$initializer$@@3P6AXXZA 10031334     Install.obj
 0002:00000338       ?D2EvalItemCalc$initializer$@@3P6AXXZA 10031338     Install.obj
 0002:0000033c       ?D2CheckUnitState$initializer$@@3P6AXXZA 1003133c     Install.obj
 0002:00000340       ?D2CheckQuestFlag$initializer$@@3P6AXXZA 10031340     Install.obj
 0002:00000344       ?D2CheckItemFlag$initializer$@@3P6AXXZA 10031344     Install.obj
 0002:00000348       ?D2CheckCorpseCanUse$initializer$@@3P6AXXZA 10031348     Install.obj
 0002:0000034c       ?D2GetItemValue$initializer$@@3P6AXXZA 1003134c     Install.obj
 0002:00000350       ?D2GetCursorItem$initializer$@@3P6AXXZA 10031350     Install.obj
 0002:00000354       ?D2GetFirstItemInInv$initializer$@@3P6AXXZA 10031354     Install.obj
 0002:00000358       ?D2GetNextItemInInv$initializer$@@3P6AXXZA 10031358     Install.obj
 0002:0000035c       ?D2GetBoxType$initializer$@@3P6AXXZA 1003135c     Install.obj
 0002:00000360       ?D2CheckInvLocation$initializer$@@3P6AXXZA 10031360     Install.obj
 0002:00000364       ?D2GetDrlgLevel$initializer$@@3P6AXXZA 10031364     Install.obj
 0002:00000368       ?D2InitDrlgLevel$initializer$@@3P6AXXZA 10031368     Install.obj
 0002:0000036c       ?D2GetLevelIdFromRoom$initializer$@@3P6AXXZA 1003136c     Install.obj
 0002:00000370       ?D2GetUnitPosX$initializer$@@3P6AXXZA 10031370     Install.obj
 0002:00000374       ?D2GetUnitPosY$initializer$@@3P6AXXZA 10031374     Install.obj
 0002:00000378       ?D2GetMinExpToLevel$initializer$@@3P6AXXZA 10031378     Install.obj
 0002:0000037c       ?p_D2WeaponsTxts$initializer$@@3P6AXXZA 1003137c     Install.obj
 0002:00000380       ?p_D2ArmorTxts$initializer$@@3P6AXXZA 10031380     Install.obj
 0002:00000384       ?p_D2DataTables$initializer$@@3P6AXXZA 10031384     Install.obj
 0002:00000388       ?p_D2RuneWords$initializer$@@3P6AXXZA 10031388     Install.obj
 0002:0000038c       ?p_D2RuneWordTxt$initializer$@@3P6AXXZA 1003138c     Install.obj
 0002:00000390       ?D2GetHwnd$initializer$@@3P6AXXZA 10031390     Install.obj
 0002:00000394       ?D2DrawRectangle$initializer$@@3P6AXXZA 10031394     Install.obj
 0002:00000398       ?D2DrawLine$initializer$@@3P6AXXZA 10031398     Install.obj
 0002:0000039c       ?D2DrawCellFile$initializer$@@3P6AXXZA 1003139c     Install.obj
 0002:000003a0       ?D2DrawAutomapCell$initializer$@@3P6AXXZA 100313a0     Install.obj
 0002:000003a4       ?D2MinimizeWindows$initializer$@@3P6AXXZA 100313a4     Install.obj
 0002:000003a8       ?p_D2WinState$initializer$@@3P6AXXZA 100313a8     Install.obj
 0002:000003ac       ?D2DrawText$initializer$@@3P6AXXZA 100313ac     Install.obj
 0002:000003b0       ?D2DrawHoverText$initializer$@@3P6AXXZA 100313b0     Install.obj
 0002:000003b4       ?D2DrawUnitLifeBar$initializer$@@3P6AXXZA 100313b4     Install.obj
 0002:000003b8       ?D2DrawHover$initializer$@@3P6AXXZA 100313b8     Install.obj
 0002:000003bc       ?D2GetTextAreaSize$initializer$@@3P6AXXZA 100313bc     Install.obj
 0002:000003c0       ?D2SetTextFont$initializer$@@3P6AXXZA 100313c0     Install.obj
 0002:000003c4       ?D2GetTextPixelLen$initializer$@@3P6AXXZA 100313c4     Install.obj
 0002:000003c8       ?D2GetEditBoxText$initializer$@@3P6AXXZA 100313c8     Install.obj
 0002:000003cc       ?D2SelectEditBoxText$initializer$@@3P6AXXZA 100313cc     Install.obj
 0002:000003d0       ?D2AddEditBoxChar$initializer$@@3P6AXXZA 100313d0     Install.obj
 0002:000003d4       ?D2DestroyEditBox$initializer$@@3P6AXXZA 100313d4     Install.obj
 0002:000003d8       ?D2DestroyListBox$initializer$@@3P6AXXZA 100313d8     Install.obj
 0002:000003dc       ?D2CreateEditBox$initializer$@@3P6AXXZA 100313dc     Install.obj
 0002:000003e0       ?D2SetEditBoxText$initializer$@@3P6AXXZA 100313e0     Install.obj
 0002:000003e4       ?D2SetEditBoxProc$initializer$@@3P6AXXZA 100313e4     Install.obj
 0002:000003e8       ?vD2ToggleSound$initializer$@@3P6AXXZA 100313e8     Install.obj
 0002:000003ec       ?p_D2FocusedControl$initializer$@@3P6AXXZA 100313ec     Install.obj
 0002:000003f0       ?D2DeleteCellFile$initializer$@@3P6AXXZA 100313f0     Install.obj
 0002:000003f4       ?D2InitCellFile$initializer$@@3P6AXXZA 100313f4     Install.obj
 0002:000003f8       ?D2GetLocaleText$initializer$@@3P6AXXZA 100313f8     Install.obj
 0002:000003fc       ?p_D2UnkNetFlag$initializer$@@3P6AXXZA 100313fc     Install.obj
 0002:00000400       ?D2SendPacket$initializer$@@3P6AXXZA 10031400     Install.obj
 0002:00000404       ?p_D2BnChatMessage$initializer$@@3P6AXXZA 10031404     Install.obj
 0002:00000408       ?vD2EndOfPtr$initializer$@@3P6AXXZA 10031408     Install.obj
 0002:0000040c       ?vD2StartOfPtr2$initializer$@@3P6AXXZA 1003140c     Install.obj
 0002:00000410       ?p_D2GameListControl$initializer$@@3P6AXXZA 10031410     Install.obj
 0002:00000414       ?p_D2EditboxPreferences$initializer$@@3P6AXXZA 10031414     Install.obj
 0002:00000418       ?vD2GetUnitName_I$initializer$@@3P6AXXZA 10031418     Install.obj
 0002:0000041c       ?vD2EndOfPtr2$initializer$@@3P6AXXZA 1003141c     Install.obj
 0002:00000420       ?aD2Patchs$initializer$@@3P6AXXZA 10031420     Install.obj
 0002:00000424       ?aD2Patch2s$initializer$@@3P6AXXZA 10031424     Install.obj
 0002:00000428       ?wsinit_$initializer$@detail@httplib@@3P6AXXZA 10031428     stdafx.obj
 0002:0000042c       ?aKeepGameWindowPatchs$initializer$@@3P6AXXZA 1003142c     GameWindow.obj
 0002:00000438       ?__scrt_initialize_tss_var@@3P6AHXZA 10031438     LIBCMT:thread_safe_statics.obj
 0002:00000470       _GS_ExceptionPointers      10031470     LIBCMT:gs_report.obj
 0002:00000580       ?tokenTable@@3QBUStringLiteral@@B 10031580     libvcruntime:undname.obj
 0002:00000600       ?nameTable@@3QBUStringLiteral@@B 10031600     libvcruntime:undname.obj
 0002:00000898       ?rttiTable@@3QBUStringLiteral@@B 10031898     libvcruntime:undname.obj
 0002:000008c0       ?IndirectionName@@3QBUStringLiteral@@B 100318c0     libvcruntime:undname.obj
 0002:000008f0       ?PrefixName@@3QBUStringLiteral@@B 100318f0     libvcruntime:undname.obj
 0002:00000f20       ?module_names@?A0xeb687146@@3QBQB_WB 10031f20     libvcruntime:winapi_downlevel.obj
 0002:00000fc8       ?candidate_modules@?1??try_get_FlsAlloc@@YAP6GKP6GXPAX@Z@ZXZ@4QBW4module_id@?A0xeb687146@@B 10031fc8     libvcruntime:winapi_downlevel.obj
 0002:00000fdc       ?candidate_modules@?1??try_get_FlsFree@@YAP6GHK@ZXZ@4QBW4module_id@?A0xeb687146@@B 10031fdc     libvcruntime:winapi_downlevel.obj
 0002:00000fec       ?candidate_modules@?1??try_get_FlsGetValue@@YAP6GPAXK@ZXZ@4QBW4module_id@?A0xeb687146@@B 10031fec     libvcruntime:winapi_downlevel.obj
 0002:00001000       ?candidate_modules@?1??try_get_FlsSetValue@@YAP6GHKPAX@ZXZ@4QBW4module_id@?A0xeb687146@@B 10032000     libvcruntime:winapi_downlevel.obj
 0002:00001014       ?candidate_modules@?1??try_get_InitializeCriticalSectionEx@@YAP6GHPAU_RTL_CRITICAL_SECTION@@KK@ZXZ@4QBW4module_id@?A0xeb687146@@B 10032014     libvcruntime:winapi_downlevel.obj
 0002:00001518       ___acrt_initializers       10032518     libucrt:initialization.obj
 0002:00001a58       ?errtable@@3QBUerrentry@?A0x31fdb9ec@@B 10032a58     libucrt:errno.obj
 0002:00002db0       ?strings@?1??fp_format_nan_or_infinity@@YAHW4__acrt_fp_class@@_NPADI1@Z@4QAY03QBDA 10033db0     libucrt:cvt.obj
 0002:00002e38       ?module_names@?A0x391cf84c@@3QBQB_WB 10033e38     libucrt:winapi_thunks.obj
 0002:000032b0       ?candidate_modules@?1??try_get_AreFileApisANSI@@YAP6GHXZXZ@4QBW4module_id@?A0x391cf84c@@B 100342b0     libucrt:winapi_thunks.obj
 0002:000032c4       ?candidate_modules@?1??try_get_FlsAlloc@@YAP6GKP6GXPAX@Z@ZXZ@4QBW4module_id@?A0x391cf84c@@B 100342c4     libucrt:winapi_thunks.obj
 0002:000032cc       ?candidate_modules@?1??try_get_FlsFree@@YAP6GHK@ZXZ@4QBW4module_id@?A0x391cf84c@@B 100342cc     libucrt:winapi_thunks.obj
 0002:000032d4       ?candidate_modules@?1??try_get_FlsGetValue@@YAP6GPAXK@ZXZ@4QBW4module_id@?A0x391cf84c@@B 100342d4     libucrt:winapi_thunks.obj
 0002:000032dc       ?candidate_modules@?1??try_get_FlsSetValue@@YAP6GHKPAX@ZXZ@4QBW4module_id@?A0x391cf84c@@B 100342dc     libucrt:winapi_thunks.obj
 0002:000032e4       ?candidate_modules@?1??try_get_InitializeCriticalSectionEx@@YAP6GHPAU_RTL_CRITICAL_SECTION@@KK@ZXZ@4QBW4module_id@?A0x391cf84c@@B 100342e4     libucrt:winapi_thunks.obj
 0002:000032ec       ?candidate_modules@?1??try_get_LCMapStringEx@@YAP6GHPB_WK0HPA_WHPAU_nlsversioninfo@@PAXJ@ZXZ@4QBW4module_id@?A0x391cf84c@@B 100342ec     libucrt:winapi_thunks.obj
 0002:00003304       ?candidate_modules@?1??try_get_LocaleNameToLCID@@YAP6GKPB_WK@ZXZ@4QBW4module_id@?A0x391cf84c@@B 10034304     libucrt:winapi_thunks.obj
 0002:00003320       ?candidate_modules@?1??try_get_AppPolicyGetProcessTerminationMethod@@YAP6GJPAXPAW4AppPolicyProcessTerminationMethod@@@ZXZ@4QBW4module_id@?A0x391cf84c@@B 10034320     libucrt:winapi_thunks.obj
 0002:0000334c       ?_mb_locale_names@@3QBQB_WB 1003434c     libucrt:mbctype.obj
 0002:000033a0       LOG_name                   100343a0     libucrt:log10_impl.obj
 0002:000033b0       _One                       100343b0     libucrt:ceil_pentium4.obj
 0002:000033c0       _Bns                       100343c0     libucrt:ceil_pentium4.obj
 0002:000033d0       _Zero                      100343d0     libucrt:ceil_pentium4.obj
 0002:000033e0       _S                         100343e0     libucrt:ceil_pentium4.obj
 0002:000033f0       _NegZero                   100343f0     libucrt:ceil_pentium4.obj
 0002:000033f8       ?LcidToLocaleNameTable@?A0x881e4c05@@3QBULcidToLocaleName@1@B 100343f8     libucrt:lcidtoname_downlevel.obj
 0002:00004518       ?LocaleNameToIndexTable@?A0x881e4c05@@3QBULocaleNameIndex@1@B 10035518     libucrt:lcidtoname_downlevel.obj
 0002:00005470       emask                      10036470     libucrt:log10_pentium4.obj
 0002:00005480       CC                         10036480     libucrt:log10_pentium4.obj
 0002:00005490       Magic                      10036490     libucrt:log10_pentium4.obj
 0002:000054a0       hi_mask                    100364a0     libucrt:log10_pentium4.obj
 0002:000054b0       LOG10_2                    100364b0     libucrt:log10_pentium4.obj
 0002:000054c0       place_L                    100364c0     libucrt:log10_pentium4.obj
 0002:000054e0       One                        100364e0     libucrt:log10_pentium4.obj
 0002:000054f0       Zero                       100364f0     libucrt:log10_pentium4.obj
 0002:00005500       Two52                      10036500     libucrt:log10_pentium4.obj
 0002:00005510       Infs                       10036510     libucrt:log10_pentium4.obj
 0002:00005520       NaN                        10036520     libucrt:log10_pentium4.obj
 0002:00005530       coeff                      10036530     libucrt:log10_pentium4.obj
 0002:0000558e       _log2max                   1003658e     libucrt:87tran.obj
 0002:00005598       _smallarg                  10036598     libucrt:87tran.obj
 0002:000055a2       _half                      100365a2     libucrt:87tran.obj
 0002:000055ee       One                        100365ee     libucrt:87disp.obj
 0002:000055f6       Three                      100365f6     libucrt:87disp.obj
 0002:000055fe       XAMtoTagTab                100365fe     libucrt:87disp.obj
 0002:00005610       One                        10036610     libucrt:common.obj
 0002:00005624       DblMax                     10036624     libucrt:common.obj
 0002:0000562c       DblMin                     1003662c     libucrt:common.obj
 0002:00005634       IeeeAdjO                   10036634     libucrt:common.obj
 0002:0000563c       IeeeAdjU                   1003663c     libucrt:common.obj
 0002:00005644       _infinity                  10036644     libucrt:common.obj
 0002:0000564c       _zero                      1003664c     libucrt:common.obj
 0002:00005688       _over                      10036688     libucrt:fpctrl.obj
 0002:00005694       _under                     10036694     libucrt:fpctrl.obj
 0002:00005ec8       ?_names@?1??_get_fname@@9@9 10036ec8     libucrt:fpexcept.obj
 0002:00006080       two32                      10037080     LIBCMT:ftol2.obj
 0002:00006084       two63                      10037084     LIBCMT:ftol2.obj
 0002:00006088       _NaN                       10037088     LIBCMT:ftol2.obj
 0002:00006090       $SG4294966717              10037090     DllMain.obj
 0002:00006092       ?piecewise_construct@std@@3Upiecewise_construct_t@1@B 10037092     DllMain.obj
 0002:00006093       $SG4294951477              10037093     HelpFunc.obj
 0002:00006094       $SG4294966682              10037094     DllMain.obj
 0002:00006097       ?piecewise_construct@std@@3Upiecewise_construct_t@1@B 10037097     stdafx.obj
 0002:00006098       $SG4294966681              10037098     DllMain.obj
 0002:0000609b       $SG4294934227              1003709b     ViewUnitStat.obj
 0002:0000609c       $SG4294966680              1003709c     DllMain.obj
 0002:000060ab       $SG4294934225              100370ab     ViewUnitStat.obj
 0002:000060ac       $SG4294966679              100370ac     DllMain.obj
 0002:000060af       $SG4294934223              100370af     ViewUnitStat.obj
 0002:000060b0       $SG4294966678              100370b0     DllMain.obj
 0002:000060c0       $SG4294966677              100370c0     DllMain.obj
 0002:000060c3       $SG4294934221              100370c3     ViewUnitStat.obj
 0002:000060c4       $SG4294966676              100370c4     DllMain.obj
 0002:000060c7       $SG4294934219              100370c7     ViewUnitStat.obj
 0002:000060c8       $SG4294966675              100370c8     DllMain.obj
 0002:000060cb       $SG4294934217              100370cb     ViewUnitStat.obj
 0002:000060cc       $SG4294966674              100370cc     DllMain.obj
 0002:000060cf       $SG4294934215              100370cf     ViewUnitStat.obj
 0002:000060d0       $SG4294966673              100370d0     DllMain.obj
 0002:000060d5       $SG4294934213              100370d5     ViewUnitStat.obj
 0002:000060d6       $SG4294934211              100370d6     ViewUnitStat.obj
 0002:000060d7       $SG4294934209              100370d7     ViewUnitStat.obj
 0002:000060d8       $SG4294966672              100370d8     DllMain.obj
 0002:000060db       $SG4294934207              100370db     ViewUnitStat.obj
 0002:000060dc       $SG4294966671              100370dc     DllMain.obj
 0002:000060df       $SG4294934205              100370df     ViewUnitStat.obj
 0002:000060e0       $SG4294966670              100370e0     DllMain.obj
 0002:000060ef       $SG4294934203              100370ef     ViewUnitStat.obj
 0002:000060f0       $SG4294966669              100370f0     DllMain.obj
 0002:000060f3       $SG4294934201              100370f3     ViewUnitStat.obj
 0002:000060f4       $SG4294966668              100370f4     DllMain.obj
 0002:00006104       $SG4294966667              10037104     DllMain.obj
 0002:00006107       $SG4294934199              10037107     ViewUnitStat.obj
 0002:00006108       $SG4294966666              10037108     DllMain.obj
 0002:0000610b       $SG4294934197              1003710b     ViewUnitStat.obj
 0002:0000610c       $SG4294966665              1003710c     DllMain.obj
 0002:0000610f       $SG4294934195              1003710f     ViewUnitStat.obj
 0002:00006110       $SG4294966664              10037110     DllMain.obj
 0002:00006113       $SG4294934193              10037113     ViewUnitStat.obj
 0002:00006114       $SG4294966663              10037114     DllMain.obj
 0002:00006119       $SG4294934192              10037119     ViewUnitStat.obj
 0002:0000611a       $SG4294934191              1003711a     ViewUnitStat.obj
 0002:0000611b       $SG4294934190              1003711b     ViewUnitStat.obj
 0002:0000611c       $SG4294966656              1003711c     DllMain.obj
 0002:0000611f       $SG4294934189              1003711f     ViewUnitStat.obj
 0002:00006120       $SG4294966655              10037120     DllMain.obj
 0002:00006123       $SG4294934188              10037123     ViewUnitStat.obj
 0002:00006124       $SG4294966654              10037124     DllMain.obj
 0002:00006133       $SG4294934153              10037133     ViewUnitStat.obj
 0002:00006134       $SG4294966653              10037134     DllMain.obj
 0002:00006137       $SG4294934150              10037137     ViewUnitStat.obj
 0002:00006138       $SG4294966652              10037138     DllMain.obj
 0002:00006148       $SG4294966651              10037148     DllMain.obj
 0002:0000614b       $SG4294934147              1003714b     ViewUnitStat.obj
 0002:0000614c       $SG4294966650              1003714c     DllMain.obj
 0002:0000614f       $SG4294934144              1003714f     ViewUnitStat.obj
 0002:00006150       $SG4294966649              10037150     DllMain.obj
 0002:00006153       $SG4294934141              10037153     ViewUnitStat.obj
 0002:00006154       $SG4294966648              10037154     DllMain.obj
 0002:00006157       $SG4294934138              10037157     ViewUnitStat.obj
 0002:00006158       $SG4294966647              10037158     DllMain.obj
 0002:0000615d       $SG4294934135              1003715d     ViewUnitStat.obj
 0002:0000615e       $SG4294934132              1003715e     ViewUnitStat.obj
 0002:0000615f       $SG4294934129              1003715f     ViewUnitStat.obj
 0002:00006160       $SG4294966646              10037160     DllMain.obj
 0002:00006171       $SG4294934126              10037171     ViewUnitStat.obj
 0002:00006172       $SG4294934123              10037172     ViewUnitStat.obj
 0002:00006173       $SG4294934120              10037173     ViewUnitStat.obj
 0002:00006174       $SG4294966645              10037174     DllMain.obj
 0002:00006179       $SG4294934117              10037179     ViewUnitStat.obj
 0002:0000617a       $SG4294934114              1003717a     ViewUnitStat.obj
 0002:0000617b       $SG4294934111              1003717b     ViewUnitStat.obj
 0002:0000617c       $SG4294966644              1003717c     DllMain.obj
 0002:00006184       $SG4294966643              10037184     DllMain.obj
 0002:00006187       $SG4294934108              10037187     ViewUnitStat.obj
 0002:00006188       $SG4294966642              10037188     DllMain.obj
 0002:00006199       $SG4294934105              10037199     ViewUnitStat.obj
 0002:0000619a       $SG4294934102              1003719a     ViewUnitStat.obj
 0002:0000619b       $SG4294934099              1003719b     ViewUnitStat.obj
 0002:0000619c       $SG4294966641              1003719c     DllMain.obj
 0002:000061a1       $SG4294934096              100371a1     ViewUnitStat.obj
 0002:000061a2       $SG4294934093              100371a2     ViewUnitStat.obj
 0002:000061a3       $SG4294934090              100371a3     ViewUnitStat.obj
 0002:000061a4       $SG4294966640              100371a4     DllMain.obj
 0002:000061ac       $SG4294966639              100371ac     DllMain.obj
 0002:000061af       $SG4294934087              100371af     ViewUnitStat.obj
 0002:000061b0       $SG4294951806              100371b0     GlobalVariable.obj
 0002:000061c0       $SG4294951805              100371c0     GlobalVariable.obj
 0002:000061db       $SG4294934084              100371db     ViewUnitStat.obj
 0002:000061dc       $SG4294951804              100371dc     GlobalVariable.obj
 0002:000061ef       $SG4294934081              100371ef     ViewUnitStat.obj
 0002:000061f0       $SG4294951803              100371f0     GlobalVariable.obj
 0002:00006201       $SG4294934078              10037201     ViewUnitStat.obj
 0002:00006202       $SG4294934075              10037202     ViewUnitStat.obj
 0002:00006203       $SG4294934072              10037203     ViewUnitStat.obj
 0002:00006204       $SG4294951802              10037204     GlobalVariable.obj
 0002:00006217       $SG4294934070              10037217     ViewUnitStat.obj
 0002:00006218       $SG4294951801              10037218     GlobalVariable.obj
 0002:0000622f       $SG4294934069              1003722f     ViewUnitStat.obj
 0002:00006230       $SG4294951800              10037230     GlobalVariable.obj
 0002:00006242       $SG4294934067              10037242     ViewUnitStat.obj
 0002:00006243       $SG4294934066              10037243     ViewUnitStat.obj
 0002:00006244       $SG4294951799              10037244     GlobalVariable.obj
 0002:00006257       $SG4294934064              10037257     ViewUnitStat.obj
 0002:00006258       $SG4294951798              10037258     GlobalVariable.obj
 0002:00006270       $SG4294951797              10037270     GlobalVariable.obj
 0002:00006283       $SG4294934063              10037283     ViewUnitStat.obj
 0002:00006284       $SG4294951796              10037284     GlobalVariable.obj
 0002:00006291       $SG4294934061              10037291     ViewUnitStat.obj
 0002:00006292       $SG4294934060              10037292     ViewUnitStat.obj
 0002:00006293       $SG4294934058              10037293     ViewUnitStat.obj
 0002:00006294       $SG4294951795              10037294     GlobalVariable.obj
 0002:000062a4       $SG4294951794              100372a4     GlobalVariable.obj
 0002:000062b5       $SG4294934055              100372b5     ViewUnitStat.obj
 0002:000062b6       $SG4294934052              100372b6     ViewUnitStat.obj
 0002:000062b7       $SG4294934049              100372b7     ViewUnitStat.obj
 0002:000062b8       $SG4294951793              100372b8     GlobalVariable.obj
 0002:000062c9       $SG4294934046              100372c9     ViewUnitStat.obj
 0002:000062ca       $SG4294934043              100372ca     ViewUnitStat.obj
 0002:000062cb       $SG4294934040              100372cb     ViewUnitStat.obj
 0002:000062cc       $SG4294951792              100372cc     GlobalVariable.obj
 0002:000062dc       $SG4294951791              100372dc     GlobalVariable.obj
 0002:000062e7       $SG4294934037              100372e7     ViewUnitStat.obj
 0002:000062e8       $SG4294951790              100372e8     GlobalVariable.obj
 0002:000062f8       $SG4294951789              100372f8     GlobalVariable.obj
 0002:00006302       $SG4294934034              10037302     ViewUnitStat.obj
 0002:00006303       $SG4294934028              10037303     ViewUnitStat.obj
 0002:00006304       $SG4294951788              10037304     GlobalVariable.obj
 0002:0000630e       $SG4294934027              1003730e     ViewUnitStat.obj
 0002:0000630f       $SG4294934025              1003730f     ViewUnitStat.obj
 0002:00006310       $SG4294951787              10037310     GlobalVariable.obj
 0002:00006316       $SG4294934022              10037316     ViewUnitStat.obj
 0002:00006317       $SG4294934019              10037317     ViewUnitStat.obj
 0002:00006318       $SG4294951786              10037318     GlobalVariable.obj
 0002:00006326       $SG4294934016              10037326     ViewUnitStat.obj
 0002:00006327       $SG4294934013              10037327     ViewUnitStat.obj
 0002:00006328       $SG4294951785              10037328     GlobalVariable.obj
 0002:00006333       $SG4294934010              10037333     ViewUnitStat.obj
 0002:00006334       $SG4294951784              10037334     GlobalVariable.obj
 0002:00006342       $SG4294934007              10037342     ViewUnitStat.obj
 0002:00006343       $SG4294934004              10037343     ViewUnitStat.obj
 0002:00006344       $SG4294951783              10037344     GlobalVariable.obj
 0002:00006352       $SG4294934000              10037352     ViewUnitStat.obj
 0002:00006353       $SG4294933997              10037353     ViewUnitStat.obj
 0002:00006354       $SG4294951782              10037354     GlobalVariable.obj
 0002:00006368       $SG4294951781              10037368     GlobalVariable.obj
 0002:00006375       $SG4294933994              10037375     ViewUnitStat.obj
 0002:00006376       $SG4294933991              10037376     ViewUnitStat.obj
 0002:00006377       $SG4294933988              10037377     ViewUnitStat.obj
 0002:00006378       $SG4294951780              10037378     GlobalVariable.obj
 0002:00006387       $SG4294933985              10037387     ViewUnitStat.obj
 0002:00006388       $SG4294951779              10037388     GlobalVariable.obj
 0002:00006395       $SG4294933982              10037395     ViewUnitStat.obj
 0002:00006396       $SG4294933979              10037396     ViewUnitStat.obj
 0002:00006398       $SG4294951778              10037398     GlobalVariable.obj
 0002:000063b0       $SG4294951777              100373b0     GlobalVariable.obj
 0002:000063c4       $SG4294951776              100373c4     GlobalVariable.obj
 0002:000063d4       $SG4294951775              100373d4     GlobalVariable.obj
 0002:000063e4       $SG4294951774              100373e4     GlobalVariable.obj
 0002:000063f0       $SG4294951773              100373f0     GlobalVariable.obj
 0002:00006400       $SG4294951772              10037400     GlobalVariable.obj
 0002:00006414       $SG4294951771              10037414     GlobalVariable.obj
 0002:00006428       $SG4294951770              10037428     GlobalVariable.obj
 0002:00006434       $SG4294951769              10037434     GlobalVariable.obj
 0002:00006448       $SG4294951768              10037448     GlobalVariable.obj
 0002:0000645c       $SG4294951767              1003745c     GlobalVariable.obj
 0002:00006470       $SG4294951766              10037470     GlobalVariable.obj
 0002:00006488       $SG4294951765              10037488     GlobalVariable.obj
 0002:00006498       $SG4294951764              10037498     GlobalVariable.obj
 0002:000064a8       $SG4294951763              100374a8     GlobalVariable.obj
 0002:000064b8       $SG4294951762              100374b8     GlobalVariable.obj
 0002:000064d0       $SG4294951761              100374d0     GlobalVariable.obj
 0002:000064ec       $SG4294951760              100374ec     GlobalVariable.obj
 0002:000064fc       $SG4294951759              100374fc     GlobalVariable.obj
 0002:0000650c       $SG4294951758              1003750c     GlobalVariable.obj
 0002:0000651c       $SG4294951757              1003751c     GlobalVariable.obj
 0002:00006534       $SG4294951756              10037534     GlobalVariable.obj
 0002:00006544       $SG4294951755              10037544     GlobalVariable.obj
 0002:00006554       $SG4294951754              10037554     GlobalVariable.obj
 0002:00006568       $SG4294951753              10037568     GlobalVariable.obj
 0002:00006578       $SG4294951752              10037578     GlobalVariable.obj
 0002:0000658c       $SG4294951751              1003758c     GlobalVariable.obj
 0002:00006594       $SG4294951491              10037594     HelpFunc.obj
 0002:000065a4       $SG4294951490              100375a4     HelpFunc.obj
 0002:000065b4       $SG4294951489              100375b4     HelpFunc.obj
 0002:000065c0       $SG4294951488              100375c0     HelpFunc.obj
 0002:000065cc       $SG4294951487              100375cc     HelpFunc.obj
 0002:000065d8       $SG4294951486              100375d8     HelpFunc.obj
 0002:000065e4       $SG4294951485              100375e4     HelpFunc.obj
 0002:000065f0       $SG4294951484              100375f0     HelpFunc.obj
 0002:00006600       $SG4294951483              10037600     HelpFunc.obj
 0002:0000660c       $SG4294951482              1003760c     HelpFunc.obj
 0002:00006618       $SG4294951481              10037618     HelpFunc.obj
 0002:00006620       $SG4294951480              10037620     HelpFunc.obj
 0002:0000662c       $SG4294951479              1003762c     HelpFunc.obj
 0002:0000663c       $SG4294951478              1003763c     HelpFunc.obj
 0002:0000664c       $SG4294951355              1003764c     Install.obj
 0002:00006658       $SG4294951354              10037658     Install.obj
 0002:00006668       $SG4294951353              10037668     Install.obj
 0002:00006678       $SG4294951352              10037678     Install.obj
 0002:00006680       $SG4294951351              10037680     Install.obj
 0002:00006690       $SG4294951350              10037690     Install.obj
 0002:00006698       $SG4294951349              10037698     Install.obj
 0002:000066a4       $SG4294951348              100376a4     Install.obj
 0002:000066ac       $SG4294951347              100376ac     Install.obj
 0002:000066b8       $SG4294951346              100376b8     Install.obj
 0002:000066d4       $SG4294951345              100376d4     Install.obj
 0002:000066d8       $SG4294951344              100376d8     Install.obj
 0002:000066e4       $SG4294951343              100376e4     Install.obj
 0002:000066ec       $SG4294951342              100376ec     Install.obj
 0002:000066f8       $SG4294950526              100376f8     LoadConfig.obj
 0002:00006704       $SG4294950525              10037704     LoadConfig.obj
 0002:00006714       $SG4294950524              10037714     LoadConfig.obj
 0002:00006724       $SG4294950523              10037724     LoadConfig.obj
 0002:00006738       $SG4294950522              10037738     LoadConfig.obj
 0002:00006748       $SG4294950521              10037748     LoadConfig.obj
 0002:00006758       $SG4294950520              10037758     LoadConfig.obj
 0002:0000676c       $SG4294950519              1003776c     LoadConfig.obj
 0002:00006780       $SG4294950518              10037780     LoadConfig.obj
 0002:00006794       $SG4294950517              10037794     LoadConfig.obj
 0002:000067a8       $SG4294950516              100377a8     LoadConfig.obj
 0002:000067c0       $SG4294950515              100377c0     LoadConfig.obj
 0002:000067d0       $SG4294950514              100377d0     LoadConfig.obj
 0002:000067e0       $SG4294950513              100377e0     LoadConfig.obj
 0002:000067f8       $SG4294950512              100377f8     LoadConfig.obj
 0002:0000680c       $SG4294950511              1003780c     LoadConfig.obj
 0002:0000681c       $SG4294950510              1003781c     LoadConfig.obj
 0002:00006830       $SG4294950509              10037830     LoadConfig.obj
 0002:0000684c       $SG4294950508              1003784c     LoadConfig.obj
 0002:00006864       $SG4294950507              10037864     LoadConfig.obj
 0002:0000687c       $SG4294950506              1003787c     LoadConfig.obj
 0002:00006898       $SG4294950505              10037898     LoadConfig.obj
 0002:000068b0       $SG4294950504              100378b0     LoadConfig.obj
 0002:000068c8       $SG4294950503              100378c8     LoadConfig.obj
 0002:000068d8       $SG4294950502              100378d8     LoadConfig.obj
 0002:000068e8       $SG4294950501              100378e8     LoadConfig.obj
 0002:000068fc       $SG4294950500              100378fc     LoadConfig.obj
 0002:00006908       $SG4294950499              10037908     LoadConfig.obj
 0002:0000691c       $SG4294950498              1003791c     LoadConfig.obj
 0002:00006930       $SG4294950497              10037930     LoadConfig.obj
 0002:00006940       $SG4294950496              10037940     LoadConfig.obj
 0002:00006950       $SG4294950495              10037950     LoadConfig.obj
 0002:00006960       $SG4294950494              10037960     LoadConfig.obj
 0002:00006970       $SG4294950493              10037970     LoadConfig.obj
 0002:00006980       $SG4294950492              10037980     LoadConfig.obj
 0002:00006990       $SG4294950491              10037990     LoadConfig.obj
 0002:000069a0       $SG4294950490              100379a0     LoadConfig.obj
 0002:000069b0       $SG4294950489              100379b0     LoadConfig.obj
 0002:000069bc       $SG4294950488              100379bc     LoadConfig.obj
 0002:000069c8       $SG4294950487              100379c8     LoadConfig.obj
 0002:000069d8       $SG4294950486              100379d8     LoadConfig.obj
 0002:000069e8       $SG4294950485              100379e8     LoadConfig.obj
 0002:000069f8       $SG4294950484              100379f8     LoadConfig.obj
 0002:00006a10       $SG4294950483              10037a10     LoadConfig.obj
 0002:00006a28       $SG4294950482              10037a28     LoadConfig.obj
 0002:00006a3c       $SG4294950481              10037a3c     LoadConfig.obj
 0002:00006a54       $SG4294950480              10037a54     LoadConfig.obj
 0002:00006a68       $SG4294950479              10037a68     LoadConfig.obj
 0002:00006a78       $SG4294950478              10037a78     LoadConfig.obj
 0002:00006a90       $SG4294950477              10037a90     LoadConfig.obj
 0002:00006aa0       $SG4294950476              10037aa0     LoadConfig.obj
 0002:00006ab8       $SG4294950475              10037ab8     LoadConfig.obj
 0002:00006acc       $SG4294950474              10037acc     LoadConfig.obj
 0002:00006ae0       $SG4294950473              10037ae0     LoadConfig.obj
 0002:00006af4       $SG4294950472              10037af4     LoadConfig.obj
 0002:00006b08       $SG4294950471              10037b08     LoadConfig.obj
 0002:00006b1c       $SG4294950470              10037b1c     LoadConfig.obj
 0002:00006b30       $SG4294950469              10037b30     LoadConfig.obj
 0002:00006b44       $SG4294950468              10037b44     LoadConfig.obj
 0002:00006b58       $SG4294950467              10037b58     LoadConfig.obj
 0002:00006b70       $SG4294950466              10037b70     LoadConfig.obj
 0002:00006b84       $SG4294950465              10037b84     LoadConfig.obj
 0002:00006b98       $SG4294950464              10037b98     LoadConfig.obj
 0002:00006bac       $SG4294950463              10037bac     LoadConfig.obj
 0002:00006bc4       $SG4294950462              10037bc4     LoadConfig.obj
 0002:00006bd8       $SG4294950461              10037bd8     LoadConfig.obj
 0002:00006bec       $SG4294950460              10037bec     LoadConfig.obj
 0002:00006c00       $SG4294950459              10037c00     LoadConfig.obj
 0002:00006c14       $SG4294950458              10037c14     LoadConfig.obj
 0002:00006c28       $SG4294950457              10037c28     LoadConfig.obj
 0002:00006c3c       $SG4294950456              10037c3c     LoadConfig.obj
 0002:00006c54       $SG4294950455              10037c54     LoadConfig.obj
 0002:00006c6c       $SG4294950454              10037c6c     LoadConfig.obj
 0002:00006c84       $SG4294950453              10037c84     LoadConfig.obj
 0002:00006c98       $SG4294950452              10037c98     LoadConfig.obj
 0002:00006cac       $SG4294950451              10037cac     LoadConfig.obj
 0002:00006cc0       $SG4294950450              10037cc0     LoadConfig.obj
 0002:00006ccc       $SG4294950449              10037ccc     LoadConfig.obj
 0002:00006cdc       $SG4294950448              10037cdc     LoadConfig.obj
 0002:00006cec       $SG4294950447              10037cec     LoadConfig.obj
 0002:00006cfc       $SG4294950446              10037cfc     LoadConfig.obj
 0002:00006d08       $SG4294950445              10037d08     LoadConfig.obj
 0002:00006d1c       $SG4294950444              10037d1c     LoadConfig.obj
 0002:00006d30       $SG4294950443              10037d30     LoadConfig.obj
 0002:00006d40       $SG4294950442              10037d40     LoadConfig.obj
 0002:00006d58       $SG4294950441              10037d58     LoadConfig.obj
 0002:00006d6c       $SG4294950440              10037d6c     LoadConfig.obj
 0002:00006d78       $SG4294950439              10037d78     LoadConfig.obj
 0002:00006d88       $SG4294950438              10037d88     LoadConfig.obj
 0002:00006d9c       $SG4294950437              10037d9c     LoadConfig.obj
 0002:00006dac       $SG4294950436              10037dac     LoadConfig.obj
 0002:00006dbc       $SG4294950435              10037dbc     LoadConfig.obj
 0002:00006dd0       $SG4294950434              10037dd0     LoadConfig.obj
 0002:00006ddc       $SG4294950433              10037ddc     LoadConfig.obj
 0002:00006de8       $SG4294950432              10037de8     LoadConfig.obj
 0002:00006df8       $SG4294950431              10037df8     LoadConfig.obj
 0002:00006e08       $SG4294950430              10037e08     LoadConfig.obj
 0002:00006e18       $SG4294950429              10037e18     LoadConfig.obj
 0002:00006e2c       $SG4294950428              10037e2c     LoadConfig.obj
 0002:00006e40       $SG4294950427              10037e40     LoadConfig.obj
 0002:00006e54       $SG4294950426              10037e54     LoadConfig.obj
 0002:00006e68       $SG4294950425              10037e68     LoadConfig.obj
 0002:00006e7c       $SG4294950424              10037e7c     LoadConfig.obj
 0002:00006e90       $SG4294950423              10037e90     LoadConfig.obj
 0002:00006ea8       $SG4294950422              10037ea8     LoadConfig.obj
 0002:00006ebc       $SG4294950421              10037ebc     LoadConfig.obj
 0002:00006ed0       $SG4294950420              10037ed0     LoadConfig.obj
 0002:00006ee8       $SG4294950419              10037ee8     LoadConfig.obj
 0002:00006efc       $SG4294950418              10037efc     LoadConfig.obj
 0002:00006f10       $SG4294950417              10037f10     LoadConfig.obj
 0002:00006f24       $SG4294950416              10037f24     LoadConfig.obj
 0002:00006f34       $SG4294950415              10037f34     LoadConfig.obj
 0002:00006f48       $SG4294950414              10037f48     LoadConfig.obj
 0002:00006f5c       $SG4294950413              10037f5c     LoadConfig.obj
 0002:00006f70       $SG4294950412              10037f70     LoadConfig.obj
 0002:00006f80       $SG4294950411              10037f80     LoadConfig.obj
 0002:00006f90       $SG4294950410              10037f90     LoadConfig.obj
 0002:00006fa4       $SG4294950409              10037fa4     LoadConfig.obj
 0002:00006fb8       $SG4294950408              10037fb8     LoadConfig.obj
 0002:00006fc8       $SG4294950407              10037fc8     LoadConfig.obj
 0002:00006fe0       $SG4294950406              10037fe0     LoadConfig.obj
 0002:00006ff4       $SG4294950405              10037ff4     LoadConfig.obj
 0002:00007000       $SG4294950404              10038000     LoadConfig.obj
 0002:00007014       $SG4294950403              10038014     LoadConfig.obj
 0002:00007028       $SG4294950402              10038028     LoadConfig.obj
 0002:0000703c       $SG4294950401              1003803c     LoadConfig.obj
 0002:00007050       $SG4294950400              10038050     LoadConfig.obj
 0002:00007064       $SG4294950399              10038064     LoadConfig.obj
 0002:00007078       $SG4294950398              10038078     LoadConfig.obj
 0002:0000708c       $SG4294950397              1003808c     LoadConfig.obj
 0002:000070a0       $SG4294950396              100380a0     LoadConfig.obj
 0002:000070b0       $SG4294950395              100380b0     LoadConfig.obj
 0002:000070c0       $SG4294950394              100380c0     LoadConfig.obj
 0002:000070d0       $SG4294950393              100380d0     LoadConfig.obj
 0002:000070e0       $SG4294950392              100380e0     LoadConfig.obj
 0002:000070f0       $SG4294950391              100380f0     LoadConfig.obj
 0002:00007100       $SG4294950390              10038100     LoadConfig.obj
 0002:00007110       $SG4294950389              10038110     LoadConfig.obj
 0002:00007120       $SG4294950388              10038120     LoadConfig.obj
 0002:00007134       $SG4294950387              10038134     LoadConfig.obj
 0002:00007148       $SG4294950386              10038148     LoadConfig.obj
 0002:00007158       $SG4294950385              10038158     LoadConfig.obj
 0002:0000716c       $SG4294950384              1003816c     LoadConfig.obj
 0002:0000717c       $SG4294950383              1003817c     LoadConfig.obj
 0002:0000718c       $SG4294950382              1003818c     LoadConfig.obj
 0002:000071a0       $SG4294950381              100381a0     LoadConfig.obj
 0002:000071b4       $SG4294950380              100381b4     LoadConfig.obj
 0002:000071c4       $SG4294950379              100381c4     LoadConfig.obj
 0002:000071d4       $SG4294950378              100381d4     LoadConfig.obj
 0002:000071e8       $SG4294950377              100381e8     LoadConfig.obj
 0002:000071fc       $SG4294950376              100381fc     LoadConfig.obj
 0002:00007214       $SG4294950375              10038214     LoadConfig.obj
 0002:00007228       $SG4294950374              10038228     LoadConfig.obj
 0002:00007238       $SG4294950373              10038238     LoadConfig.obj
 0002:0000724c       $SG4294950372              1003824c     LoadConfig.obj
 0002:0000725c       $SG4294950371              1003825c     LoadConfig.obj
 0002:0000726c       $SG4294950370              1003826c     LoadConfig.obj
 0002:0000727c       $SG4294950369              1003827c     LoadConfig.obj
 0002:00007288       $SG4294950368              10038288     LoadConfig.obj
 0002:0000729c       $SG4294950367              1003829c     LoadConfig.obj
 0002:000072ac       $SG4294950366              100382ac     LoadConfig.obj
 0002:000072c0       $SG4294950365              100382c0     LoadConfig.obj
 0002:000072d4       $SG4294950364              100382d4     LoadConfig.obj
 0002:000072e8       $SG4294950363              100382e8     LoadConfig.obj
 0002:000072fc       $SG4294950362              100382fc     LoadConfig.obj
 0002:00007310       $SG4294950361              10038310     LoadConfig.obj
 0002:00007328       $SG4294950360              10038328     LoadConfig.obj
 0002:00007338       $SG4294950359              10038338     LoadConfig.obj
 0002:0000734c       $SG4294950358              1003834c     LoadConfig.obj
 0002:00007360       $SG4294950357              10038360     LoadConfig.obj
 0002:00007378       $SG4294950356              10038378     LoadConfig.obj
 0002:00007390       $SG4294950355              10038390     LoadConfig.obj
 0002:000073a0       $SG4294950354              100383a0     LoadConfig.obj
 0002:000073b4       $SG4294950353              100383b4     LoadConfig.obj
 0002:000073c4       $SG4294950352              100383c4     LoadConfig.obj
 0002:000073d8       $SG4294950351              100383d8     LoadConfig.obj
 0002:000073ec       $SG4294950350              100383ec     LoadConfig.obj
 0002:000073f8       $SG4294950349              100383f8     LoadConfig.obj
 0002:00007408       $SG4294950348              10038408     LoadConfig.obj
 0002:00007418       $SG4294950347              10038418     LoadConfig.obj
 0002:00007428       $SG4294950346              10038428     LoadConfig.obj
 0002:00007434       $SG4294950345              10038434     LoadConfig.obj
 0002:00007444       $SG4294950344              10038444     LoadConfig.obj
 0002:00007454       $SG4294950343              10038454     LoadConfig.obj
 0002:00007468       $SG4294950342              10038468     LoadConfig.obj
 0002:00007478       $SG4294950341              10038478     LoadConfig.obj
 0002:00007488       $SG4294950340              10038488     LoadConfig.obj
 0002:00007498       $SG4294950339              10038498     LoadConfig.obj
 0002:000074a8       $SG4294950338              100384a8     LoadConfig.obj
 0002:000074b8       $SG4294950337              100384b8     LoadConfig.obj
 0002:000074c4       $SG4294950336              100384c4     LoadConfig.obj
 0002:000074d4       $SG4294950335              100384d4     LoadConfig.obj
 0002:000074e4       $SG4294950334              100384e4     LoadConfig.obj
 0002:000074f0       $SG4294950333              100384f0     LoadConfig.obj
 0002:00007500       $SG4294950332              10038500     LoadConfig.obj
 0002:00007510       $SG4294950331              10038510     LoadConfig.obj
 0002:00007520       $SG4294950330              10038520     LoadConfig.obj
 0002:00007534       $SG4294950329              10038534     LoadConfig.obj
 0002:00007548       $SG4294950328              10038548     LoadConfig.obj
 0002:00007558       $SG4294950327              10038558     LoadConfig.obj
 0002:00007568       $SG4294950326              10038568     LoadConfig.obj
 0002:0000757c       $SG4294950325              1003857c     LoadConfig.obj
 0002:00007590       $SG4294950324              10038590     LoadConfig.obj
 0002:000075a4       $SG4294950323              100385a4     LoadConfig.obj
 0002:000075b4       $SG4294950322              100385b4     LoadConfig.obj
 0002:000075c8       $SG4294950321              100385c8     LoadConfig.obj
 0002:000075dc       $SG4294950320              100385dc     LoadConfig.obj
 0002:000075f4       $SG4294950319              100385f4     LoadConfig.obj
 0002:00007608       $SG4294950318              10038608     LoadConfig.obj
 0002:0000761c       $SG4294950317              1003861c     LoadConfig.obj
 0002:00007630       $SG4294950316              10038630     LoadConfig.obj
 0002:00007644       $SG4294950315              10038644     LoadConfig.obj
 0002:00007658       $SG4294950314              10038658     LoadConfig.obj
 0002:0000766c       $SG4294950313              1003866c     LoadConfig.obj
 0002:00007680       $SG4294950312              10038680     LoadConfig.obj
 0002:00007698       $SG4294950311              10038698     LoadConfig.obj
 0002:000076ac       $SG4294950310              100386ac     LoadConfig.obj
 0002:000076c0       $SG4294950309              100386c0     LoadConfig.obj
 0002:000076d4       $SG4294950308              100386d4     LoadConfig.obj
 0002:000076e0       $SG4294950307              100386e0     LoadConfig.obj
 0002:000076f4       $SG4294950306              100386f4     LoadConfig.obj
 0002:00007708       $SG4294950305              10038708     LoadConfig.obj
 0002:00007718       $SG4294950304              10038718     LoadConfig.obj
 0002:00007730       $SG4294950303              10038730     LoadConfig.obj
 0002:00007748       $SG4294950302              10038748     LoadConfig.obj
 0002:00007764       $SG4294950301              10038764     LoadConfig.obj
 0002:00007774       $SG4294950300              10038774     LoadConfig.obj
 0002:00007790       $SG4294950299              10038790     LoadConfig.obj
 0002:000077ac       $SG4294950298              100387ac     LoadConfig.obj
 0002:000077c8       $SG4294950297              100387c8     LoadConfig.obj
 0002:000077dc       $SG4294950296              100387dc     LoadConfig.obj
 0002:000077f0       $SG4294950295              100387f0     LoadConfig.obj
 0002:00007804       $SG4294950294              10038804     LoadConfig.obj
 0002:0000781c       $SG4294950293              1003881c     LoadConfig.obj
 0002:00007830       $SG4294950292              10038830     LoadConfig.obj
 0002:00007844       $SG4294950291              10038844     LoadConfig.obj
 0002:0000785c       $SG4294950290              1003885c     LoadConfig.obj
 0002:0000786c       $SG4294950289              1003886c     LoadConfig.obj
 0002:00007880       $SG4294950288              10038880     LoadConfig.obj
 0002:00007894       $SG4294950287              10038894     LoadConfig.obj
 0002:000078a4       $SG4294950286              100388a4     LoadConfig.obj
 0002:000078b8       $SG4294950285              100388b8     LoadConfig.obj
 0002:000078cc       $SG4294950284              100388cc     LoadConfig.obj
 0002:000078e4       $SG4294950283              100388e4     LoadConfig.obj
 0002:000078fc       $SG4294950282              100388fc     LoadConfig.obj
 0002:00007914       $SG4294950281              10038914     LoadConfig.obj
 0002:00007924       $SG4294950280              10038924     LoadConfig.obj
 0002:00007938       $SG4294950279              10038938     LoadConfig.obj
 0002:00007948       $SG4294950278              10038948     LoadConfig.obj
 0002:0000795c       $SG4294950277              1003895c     LoadConfig.obj
 0002:00007974       $SG4294950276              10038974     LoadConfig.obj
 0002:0000798c       $SG4294950275              1003898c     LoadConfig.obj
 0002:000079a0       $SG4294950274              100389a0     LoadConfig.obj
 0002:000079b8       $SG4294950273              100389b8     LoadConfig.obj
 0002:000079d4       $SG4294950272              100389d4     LoadConfig.obj
 0002:000079e0       $SG4294950271              100389e0     LoadConfig.obj
 0002:000079f4       $SG4294950270              100389f4     LoadConfig.obj
 0002:00007a10       $SG4294950269              10038a10     LoadConfig.obj
 0002:00007a24       $SG4294950268              10038a24     LoadConfig.obj
 0002:00007a40       $SG4294950267              10038a40     LoadConfig.obj
 0002:00007a60       $SG4294950266              10038a60     LoadConfig.obj
 0002:00007a74       $SG4294950265              10038a74     LoadConfig.obj
 0002:00007a88       $SG4294950264              10038a88     LoadConfig.obj
 0002:00007aa8       $SG4294950263              10038aa8     LoadConfig.obj
 0002:00007ac0       $SG4294950262              10038ac0     LoadConfig.obj
 0002:00007acc       $SG4294950261              10038acc     LoadConfig.obj
 0002:00007ad8       $SG4294950260              10038ad8     LoadConfig.obj
 0002:00007ae4       $SG4294950259              10038ae4     LoadConfig.obj
 0002:00007af8       $SG4294950258              10038af8     LoadConfig.obj
 0002:00007b08       $SG4294950257              10038b08     LoadConfig.obj
 0002:00007b14       $SG4294950256              10038b14     LoadConfig.obj
 0002:00007b28       $SG4294950255              10038b28     LoadConfig.obj
 0002:00007b3c       $SG4294950254              10038b3c     LoadConfig.obj
 0002:00007b4c       $SG4294950253              10038b4c     LoadConfig.obj
 0002:00007b60       $SG4294950252              10038b60     LoadConfig.obj
 0002:00007b74       $SG4294950251              10038b74     LoadConfig.obj
 0002:00007b84       $SG4294950250              10038b84     LoadConfig.obj
 0002:00007b9c       $SG4294950249              10038b9c     LoadConfig.obj
 0002:00007bac       $SG4294950248              10038bac     LoadConfig.obj
 0002:00007bbc       $SG4294950247              10038bbc     LoadConfig.obj
 0002:00007bdc       $SG4294950246              10038bdc     LoadConfig.obj
 0002:00007bec       $SG4294950245              10038bec     LoadConfig.obj
 0002:00007bf0       $SG4294950244              10038bf0     LoadConfig.obj
 0002:00007c18       $SG4294950243              10038c18     LoadConfig.obj
 0002:00007c28       $SG4294950242              10038c28     LoadConfig.obj
 0002:00007c34       $SG4294950241              10038c34     LoadConfig.obj
 0002:00007c3c       $SG4294950240              10038c3c     LoadConfig.obj
 0002:00007c44       $SG4294950239              10038c44     LoadConfig.obj
 0002:00007c4c       $SG4294950238              10038c4c     LoadConfig.obj
 0002:00007c50       $SG4294950237              10038c50     LoadConfig.obj
 0002:00007c54       $SG4294950236              10038c54     LoadConfig.obj
 0002:00007c58       $SG4294950235              10038c58     LoadConfig.obj
 0002:00007c5c       $SG4294950234              10038c5c     LoadConfig.obj
 0002:00007c60       $SG4294950233              10038c60     LoadConfig.obj
 0002:00007c70       $SG4294950232              10038c70     LoadConfig.obj
 0002:00007c74       $SG4294950231              10038c74     LoadConfig.obj
 0002:00007c84       $SG4294950230              10038c84     LoadConfig.obj
 0002:00007c9c       $SG4294949595              10038c9c     stdafx.obj
 0002:00007ca0       $SG4294949560              10038ca0     stdafx.obj
 0002:00007ca4       $SG4294949559              10038ca4     stdafx.obj
 0002:00007ca8       $SG4294949558              10038ca8     stdafx.obj
 0002:00007cb8       $SG4294949557              10038cb8     stdafx.obj
 0002:00007cbc       $SG4294949556              10038cbc     stdafx.obj
 0002:00007ccc       $SG4294949555              10038ccc     stdafx.obj
 0002:00007cd0       $SG4294949554              10038cd0     stdafx.obj
 0002:00007cd4       $SG4294949553              10038cd4     stdafx.obj
 0002:00007cd8       $SG4294949552              10038cd8     stdafx.obj
 0002:00007cdc       $SG4294949551              10038cdc     stdafx.obj
 0002:00007ce4       $SG4294949550              10038ce4     stdafx.obj
 0002:00007ce8       $SG4294949549              10038ce8     stdafx.obj
 0002:00007cec       $SG4294949548              10038cec     stdafx.obj
 0002:00007cfc       $SG4294949547              10038cfc     stdafx.obj
 0002:00007d00       $SG4294949546              10038d00     stdafx.obj
 0002:00007d10       $SG4294949545              10038d10     stdafx.obj
 0002:00007d14       $SG4294949544              10038d14     stdafx.obj
 0002:00007d18       $SG4294949543              10038d18     stdafx.obj
 0002:00007d1c       $SG4294949542              10038d1c     stdafx.obj
 0002:00007d20       $SG4294949541              10038d20     stdafx.obj
 0002:00007d28       $SG4294949534              10038d28     stdafx.obj
 0002:00007d2c       $SG4294949533              10038d2c     stdafx.obj
 0002:00007d30       $SG4294949532              10038d30     stdafx.obj
 0002:00007d40       $SG4294949531              10038d40     stdafx.obj
 0002:00007d44       $SG4294949530              10038d44     stdafx.obj
 0002:00007d54       $SG4294949529              10038d54     stdafx.obj
 0002:00007d58       $SG4294949528              10038d58     stdafx.obj
 0002:00007d5c       $SG4294949527              10038d5c     stdafx.obj
 0002:00007d60       $SG4294949526              10038d60     stdafx.obj
 0002:00007d64       $SG4294949525              10038d64     stdafx.obj
 0002:00007d6c       $SG4294949524              10038d6c     stdafx.obj
 0002:00007d80       $SG4294949523              10038d80     stdafx.obj
 0002:00007d88       $SG4294949522              10038d88     stdafx.obj
 0002:00007d90       $SG4294949521              10038d90     stdafx.obj
 0002:00007d94       $SG4294949520              10038d94     stdafx.obj
 0002:00007da8       $SG4294949519              10038da8     stdafx.obj
 0002:00007db0       $SG4294949518              10038db0     stdafx.obj
 0002:00007db8       $SG4294949517              10038db8     stdafx.obj
 0002:00007dbc       $SG4294934955              10038dbc     D2HelpFunc.obj
 0002:00007dcc       $SG4294934954              10038dcc     D2HelpFunc.obj
 0002:00007dec       $SG4294934953              10038dec     D2HelpFunc.obj
 0002:00007df0       $SG4294934952              10038df0     D2HelpFunc.obj
 0002:00007df4       $SG4294934835              10038df4     KeyEventControl.obj
 0002:00007df8       $SG4294934875              10038df8     GameMainLoop.obj
 0002:00007ea0       $SG4294934874              10038ea0     GameMainLoop.obj
 0002:00007ec0       $SG4294934834              10038ec0     KeyEventControl.obj
 0002:00007ec4       $SG4294934833              10038ec4     KeyEventControl.obj
 0002:00007ed8       $SG4294934792              10038ed8     GameCount.obj
 0002:00007eec       $SG4294934791              10038eec     GameCount.obj
 0002:00007ef4       $SG4294934790              10038ef4     GameCount.obj
 0002:00007f08       $SG4294934789              10038f08     GameCount.obj
 0002:00007f18       $SG4294934788              10038f18     GameCount.obj
 0002:00007f20       $SG4294934787              10038f20     GameCount.obj
 0002:00007f34       $SG4294934775              10038f34     GameMonitor.obj
 0002:00007f5c       $SG4294934759              10038f5c     MessageLog.obj
 0002:00007f84       $SG4294934758              10038f84     MessageLog.obj
 0002:00007fa8       $SG4294934757              10038fa8     MessageLog.obj
 0002:00007fd0       $SG4294934756              10038fd0     MessageLog.obj
 0002:00007fe0       $SG4294934755              10038fe0     MessageLog.obj
 0002:00007ffc       $SG4294934754              10038ffc     MessageLog.obj
 0002:0000800c       $SG4294934753              1003900c     MessageLog.obj
 0002:0000801c       $SG4294934752              1003901c     MessageLog.obj
 0002:00008038       $SG4294934751              10039038     MessageLog.obj
 0002:00008048       $SG4294934750              10039048     MessageLog.obj
 0002:00008070       $SG4294934749              10039070     MessageLog.obj
 0002:00008088       $SG4294934728              10039088     PartyInfo.obj
 0002:00008090       $SG4294934727              10039090     PartyInfo.obj
 0002:00008098       $SG4294934726              10039098     PartyInfo.obj
 0002:000080a0       $SG4294934713              100390a0     RoomInfo.obj
 0002:000080a8       $SG4294934712              100390a8     RoomInfo.obj
 0002:000080b0       $SG4294934711              100390b0     RoomInfo.obj
 0002:000080d0       $SG4294934710              100390d0     RoomInfo.obj
 0002:000080ec       $SG4294934709              100390ec     RoomInfo.obj
 0002:00008108       $SG4294934708              10039108     RoomInfo.obj
 0002:00008128       $SG4294934707              10039128     RoomInfo.obj
 0002:00008148       $SG4294934706              10039148     RoomInfo.obj
 0002:00008154       $SG4294934705              10039154     RoomInfo.obj
 0002:00008158       $SG4294934704              10039158     RoomInfo.obj
 0002:00008160       $SG4294934703              10039160     RoomInfo.obj
 0002:00008168       $SG4294934690              10039168     ScreenHook.obj
 0002:0000817c       $SG4294934689              1003917c     ScreenHook.obj
 0002:00008194       $SG4294934688              10039194     ScreenHook.obj
 0002:000081b0       $SG4294934687              100391b0     ScreenHook.obj
 0002:000081d0       $SG4294934686              100391d0     ScreenHook.obj
 0002:000081d4       $SG4294934685              100391d4     ScreenHook.obj
 0002:000081d8       $SG4294934670              100391d8     ShowOrbs.obj
 0002:000081e8       $SG4294934656              100391e8     ItemDefine.obj
 0002:000081ec       $SG4294934655              100391ec     ItemDefine.obj
 0002:0000821c       $SG4294934641              1003921c     ItemDesc.obj
 0002:00008224       $SG4294934620              10039224     ItemExtInfo.obj
 0002:0000822c       $SG4294934619              1003922c     ItemExtInfo.obj
 0002:0000823c       $SG4294934618              1003923c     ItemExtInfo.obj
 0002:00008248       $SG4294934617              10039248     ItemExtInfo.obj
 0002:00008258       $SG4294934616              10039258     ItemExtInfo.obj
 0002:00008268       $SG4294934615              10039268     ItemExtInfo.obj
 0002:00008274       $SG4294934614              10039274     ItemExtInfo.obj
 0002:00008280       $SG4294934613              10039280     ItemExtInfo.obj
 0002:00008284       $SG4294934612              10039284     ItemExtInfo.obj
 0002:0000828c       $SG4294934611              1003928c     ItemExtInfo.obj
 0002:00008298       $SG4294934610              10039298     ItemExtInfo.obj
 0002:000082a4       $SG4294934609              100392a4     ItemExtInfo.obj
 0002:000082dc       $SG4294934606              100392dc     ItemExtInfo.obj
 0002:000082e0       $SG4294934608              100392e0     ItemExtInfo.obj
 0002:00008350       $SG4294934607              10039350     ItemExtInfo.obj
 0002:00008368       $SG4294934605              10039368     ItemExtInfo.obj
 0002:0000836c       $SG4294934581              1003936c     ItemInGround.obj
 0002:00008370       $SG4294934580              10039370     ItemInGround.obj
 0002:00008374       $SG4294934579              10039374     ItemInGround.obj
 0002:00008378       $SG4294934578              10039378     ItemInGround.obj
 0002:00008388       $SG4294934577              10039388     ItemInGround.obj
 0002:00008398       $SG4294934576              10039398     ItemInGround.obj
 0002:000083a8       $SG4294934575              100393a8     ItemInGround.obj
 0002:000083b8       $SG4294934527              100393b8     ItemName.obj
 0002:000083dc       $SG4294934526              100393dc     ItemName.obj
 0002:000083e0       $SG4294934525              100393e0     ItemName.obj
 0002:000083f4       $SG4294934524              100393f4     ItemName.obj
 0002:00008410       $SG4294934523              10039410     ItemName.obj
 0002:0000842c       $SG4294934522              1003942c     ItemName.obj
 0002:00008448       $SG4294934521              10039448     ItemName.obj
 0002:00008464       $SG4294934520              10039464     ItemName.obj
 0002:0000847c       $SG4294934541              1003947c     ItemName.obj
 0002:00008480       $SG4294934540              10039480     ItemName.obj
 0002:00008484       $SG4294934539              10039484     ItemName.obj
 0002:000084a0       $SG4294934538              100394a0     ItemName.obj
 0002:000084ac       $SG4294934537              100394ac     ItemName.obj
 0002:000084b0       $SG4294934536              100394b0     ItemName.obj
 0002:000084c0       $SG4294934535              100394c0     ItemName.obj
 0002:000084d0       $SG4294934534              100394d0     ItemName.obj
 0002:000084e0       $SG4294934533              100394e0     ItemName.obj
 0002:000084f0       $SG4294934532              100394f0     ItemName.obj
 0002:00008508       $SG4294934531              10039508     ItemName.obj
 0002:0000851c       $SG4294934530              1003951c     ItemName.obj
 0002:00008530       $SG4294934529              10039530     ItemName.obj
 0002:00008544       $SG4294934528              10039544     ItemName.obj
 0002:00008568       $SG4294934497              10039568     ItemVariableProp.obj
 0002:0000856c       $SG4294934496              1003956c     ItemVariableProp.obj
 0002:00008570       $SG4294934495              10039570     ItemVariableProp.obj
 0002:00008590       $SG4294934494              10039590     ItemVariableProp.obj
 0002:000085b0       $SG4294934493              100395b0     ItemVariableProp.obj
 0002:000085d0       $SG4294934492              100395d0     ItemVariableProp.obj
 0002:000085f0       $SG4294934491              100395f0     ItemVariableProp.obj
 0002:00008610       $SG4294934490              10039610     ItemVariableProp.obj
 0002:00008614       $SG4294934489              10039614     ItemVariableProp.obj
 0002:00008618       $SG4294934488              10039618     ItemVariableProp.obj
 0002:0000861c       $SG4294934487              1003961c     ItemVariableProp.obj
 0002:00008620       $SG4294934486              10039620     ItemVariableProp.obj
 0002:00008624       $SG4294934485              10039624     ItemVariableProp.obj
 0002:00008630       $SG4294934484              10039630     ItemVariableProp.obj
 0002:00008674       $SG4294934483              10039674     ItemVariableProp.obj
 0002:000086b4       $SG4294934482              100396b4     ItemVariableProp.obj
 0002:000086d4       $SG4294934481              100396d4     ItemVariableProp.obj
 0002:000086d8       $SG4294934480              100396d8     ItemVariableProp.obj
 0002:00008700       $SG4294934479              10039700     ItemVariableProp.obj
 0002:00008718       $SG4294934447              10039718     CheckDangerous.obj
 0002:00008730       $SG4294934446              10039730     CheckDangerous.obj
 0002:0000874c       $SG4294934445              1003974c     CheckDangerous.obj
 0002:00008764       $SG4294934411              10039764     ItemSocketProtect.obj
 0002:000087a0       $SG4294934444              100397a0     CheckDangerous.obj
 0002:000087f4       $SG4294934399              100397f4     QuestProtect.obj
 0002:000087f8       $SG4294934443              100397f8     CheckDangerous.obj
 0002:0000884c       $SG4294934395              1003984c     QuestProtect.obj
 0002:0000887c       $SG4294934394              1003987c     QuestProtect.obj
 0002:00008898       $SG4294934442              10039898     CheckDangerous.obj
 0002:000088fc       $SG4294934393              100398fc     QuestProtect.obj
 0002:00008920       $SG4294934441              10039920     CheckDangerous.obj
 0002:00008990       $SG4294934440              10039990     CheckDangerous.obj
 0002:00008a00       $SG4294934398              10039a00     QuestProtect.obj
 0002:00008a08       $SG4294934397              10039a08     QuestProtect.obj
 0002:00008a10       $SG4294934396              10039a10     QuestProtect.obj
 0002:00008a18       $SG4294934392              10039a18     QuestProtect.obj
 0002:00008a44       $SG4294934391              10039a44     QuestProtect.obj
 0002:00008a48       $SG4294934390              10039a48     QuestProtect.obj
 0002:00008a4c       $SG4294934318              10039a4c     MonsterLifeBar.obj
 0002:00008a5c       $SG4294934317              10039a5c     MonsterLifeBar.obj
 0002:00008a6c       $SG4294934316              10039a6c     MonsterLifeBar.obj
 0002:00008a78       $SG4294934315              10039a78     MonsterLifeBar.obj
 0002:00008a8c       $SG4294934314              10039a8c     MonsterLifeBar.obj
 0002:00008a98       $SG4294934313              10039a98     MonsterLifeBar.obj
 0002:00008aa0       $SG4294934312              10039aa0     MonsterLifeBar.obj
 0002:00008aa8       $SG4294934311              10039aa8     MonsterLifeBar.obj
 0002:00008ab0       $SG4294934310              10039ab0     MonsterLifeBar.obj
 0002:00008ab8       $SG4294934309              10039ab8     MonsterLifeBar.obj
 0002:00008ac0       $SG4294934308              10039ac0     MonsterLifeBar.obj
 0002:00008ac8       $SG4294934307              10039ac8     MonsterLifeBar.obj
 0002:00008acc       $SG4294934306              10039acc     MonsterLifeBar.obj
 0002:00008ad0       $SG4294934276              10039ad0     PlayerLifeBar.obj
 0002:00008ae0       $SG4294934275              10039ae0     PlayerLifeBar.obj
 0002:00008af0       $SG4294934274              10039af0     PlayerLifeBar.obj
 0002:00008afc       $SG4294934263              10039afc     ViewTargetUnitInfo.obj
 0002:00008b00       $SG4294934238              10039b00     ViewUnitStat.obj
 0002:00008b08       $SG4294934237              10039b08     ViewUnitStat.obj
 0002:00008b10       $SG4294934236              10039b10     ViewUnitStat.obj
 0002:00008b14       $SG4294934235              10039b14     ViewUnitStat.obj
 0002:00008b1c       $SG4294934234              10039b1c     ViewUnitStat.obj
 0002:00008b24       $SG4294934233              10039b24     ViewUnitStat.obj
 0002:00008b28       $SG4294934232              10039b28     ViewUnitStat.obj
 0002:00008b30       $SG4294934231              10039b30     ViewUnitStat.obj
 0002:00008b38       $SG4294934230              10039b38     ViewUnitStat.obj
 0002:00008b3c       $SG4294934229              10039b3c     ViewUnitStat.obj
 0002:00008b40       $SG4294934228              10039b40     ViewUnitStat.obj
 0002:00008b48       $SG4294934226              10039b48     ViewUnitStat.obj
 0002:00008b4c       $SG4294934224              10039b4c     ViewUnitStat.obj
 0002:00008b50       $SG4294934222              10039b50     ViewUnitStat.obj
 0002:00008b54       $SG4294934220              10039b54     ViewUnitStat.obj
 0002:00008b58       $SG4294934218              10039b58     ViewUnitStat.obj
 0002:00008b5c       $SG4294934216              10039b5c     ViewUnitStat.obj
 0002:00008b60       $SG4294934214              10039b60     ViewUnitStat.obj
 0002:00008b64       $SG4294934212              10039b64     ViewUnitStat.obj
 0002:00008b68       $SG4294934210              10039b68     ViewUnitStat.obj
 0002:00008b6c       $SG4294934208              10039b6c     ViewUnitStat.obj
 0002:00008b70       $SG4294934206              10039b70     ViewUnitStat.obj
 0002:00008b74       $SG4294934204              10039b74     ViewUnitStat.obj
 0002:00008b78       $SG4294934202              10039b78     ViewUnitStat.obj
 0002:00008b7c       $SG4294934200              10039b7c     ViewUnitStat.obj
 0002:00008b80       $SG4294934198              10039b80     ViewUnitStat.obj
 0002:00008b84       $SG4294934196              10039b84     ViewUnitStat.obj
 0002:00008b88       $SG4294934194              10039b88     ViewUnitStat.obj
 0002:00008b8c       $SG4294934187              10039b8c     ViewUnitStat.obj
 0002:00008b90       $SG4294934186              10039b90     ViewUnitStat.obj
 0002:00008b94       $SG4294934185              10039b94     ViewUnitStat.obj
 0002:00008b98       $SG4294934184              10039b98     ViewUnitStat.obj
 0002:00008b9c       $SG4294934183              10039b9c     ViewUnitStat.obj
 0002:00008ba0       $SG4294934182              10039ba0     ViewUnitStat.obj
 0002:00008ba4       $SG4294934181              10039ba4     ViewUnitStat.obj
 0002:00008ba8       $SG4294934180              10039ba8     ViewUnitStat.obj
 0002:00008bac       $SG4294934179              10039bac     ViewUnitStat.obj
 0002:00008bb0       $SG4294934178              10039bb0     ViewUnitStat.obj
 0002:00008bb4       $SG4294934177              10039bb4     ViewUnitStat.obj
 0002:00008bb8       $SG4294934176              10039bb8     ViewUnitStat.obj
 0002:00008bbc       $SG4294934175              10039bbc     ViewUnitStat.obj
 0002:00008bc0       $SG4294934174              10039bc0     ViewUnitStat.obj
 0002:00008bc4       $SG4294934173              10039bc4     ViewUnitStat.obj
 0002:00008bc8       $SG4294934172              10039bc8     ViewUnitStat.obj
 0002:00008bcc       $SG4294934171              10039bcc     ViewUnitStat.obj
 0002:00008bd0       $SG4294934170              10039bd0     ViewUnitStat.obj
 0002:00008bd4       $SG4294934169              10039bd4     ViewUnitStat.obj
 0002:00008bd8       $SG4294934168              10039bd8     ViewUnitStat.obj
 0002:00008bdc       $SG4294934167              10039bdc     ViewUnitStat.obj
 0002:00008be0       $SG4294934166              10039be0     ViewUnitStat.obj
 0002:00008be4       $SG4294934165              10039be4     ViewUnitStat.obj
 0002:00008be8       $SG4294934164              10039be8     ViewUnitStat.obj
 0002:00008bec       $SG4294934163              10039bec     ViewUnitStat.obj
 0002:00008bf0       $SG4294934162              10039bf0     ViewUnitStat.obj
 0002:00008bf4       $SG4294934161              10039bf4     ViewUnitStat.obj
 0002:00008bf8       $SG4294934160              10039bf8     ViewUnitStat.obj
 0002:00008bfc       $SG4294934159              10039bfc     ViewUnitStat.obj
 0002:00008c00       $SG4294934158              10039c00     ViewUnitStat.obj
 0002:00008c04       $SG4294934157              10039c04     ViewUnitStat.obj
 0002:00008c08       $SG4294934156              10039c08     ViewUnitStat.obj
 0002:00008c0c       $SG4294934155              10039c0c     ViewUnitStat.obj
 0002:00008c14       $SG4294934154              10039c14     ViewUnitStat.obj
 0002:00008c20       $SG4294934152              10039c20     ViewUnitStat.obj
 0002:00008c28       $SG4294934151              10039c28     ViewUnitStat.obj
 0002:00008c30       $SG4294934149              10039c30     ViewUnitStat.obj
 0002:00008c38       $SG4294934148              10039c38     ViewUnitStat.obj
 0002:00008c40       $SG4294934146              10039c40     ViewUnitStat.obj
 0002:00008c48       $SG4294934145              10039c48     ViewUnitStat.obj
 0002:00008c50       $SG4294934143              10039c50     ViewUnitStat.obj
 0002:00008c58       $SG4294934142              10039c58     ViewUnitStat.obj
 0002:00008c60       $SG4294934140              10039c60     ViewUnitStat.obj
 0002:00008c68       $SG4294934139              10039c68     ViewUnitStat.obj
 0002:00008c70       $SG4294934137              10039c70     ViewUnitStat.obj
 0002:00008c78       $SG4294934136              10039c78     ViewUnitStat.obj
 0002:00008c80       $SG4294934134              10039c80     ViewUnitStat.obj
 0002:00008c88       $SG4294934133              10039c88     ViewUnitStat.obj
 0002:00008c90       $SG4294934131              10039c90     ViewUnitStat.obj
 0002:00008c98       $SG4294934130              10039c98     ViewUnitStat.obj
 0002:00008ca0       $SG4294934128              10039ca0     ViewUnitStat.obj
 0002:00008ca8       $SG4294934127              10039ca8     ViewUnitStat.obj
 0002:00008cb0       $SG4294934125              10039cb0     ViewUnitStat.obj
 0002:00008cb8       $SG4294934124              10039cb8     ViewUnitStat.obj
 0002:00008cc0       $SG4294934122              10039cc0     ViewUnitStat.obj
 0002:00008cc8       $SG4294934121              10039cc8     ViewUnitStat.obj
 0002:00008cd0       $SG4294934119              10039cd0     ViewUnitStat.obj
 0002:00008cd8       $SG4294934118              10039cd8     ViewUnitStat.obj
 0002:00008ce0       $SG4294934116              10039ce0     ViewUnitStat.obj
 0002:00008ce8       $SG4294934115              10039ce8     ViewUnitStat.obj
 0002:00008cf0       $SG4294934113              10039cf0     ViewUnitStat.obj
 0002:00008cf8       $SG4294934112              10039cf8     ViewUnitStat.obj
 0002:00008d00       $SG4294934110              10039d00     ViewUnitStat.obj
 0002:00008d08       $SG4294934109              10039d08     ViewUnitStat.obj
 0002:00008d10       $SG4294934107              10039d10     ViewUnitStat.obj
 0002:00008d18       $SG4294934106              10039d18     ViewUnitStat.obj
 0002:00008d20       $SG4294934104              10039d20     ViewUnitStat.obj
 0002:00008d28       $SG4294934103              10039d28     ViewUnitStat.obj
 0002:00008d30       $SG4294934101              10039d30     ViewUnitStat.obj
 0002:00008d38       $SG4294934100              10039d38     ViewUnitStat.obj
 0002:00008d40       $SG4294934098              10039d40     ViewUnitStat.obj
 0002:00008d48       $SG4294934097              10039d48     ViewUnitStat.obj
 0002:00008d50       $SG4294934095              10039d50     ViewUnitStat.obj
 0002:00008d58       $SG4294934094              10039d58     ViewUnitStat.obj
 0002:00008d60       $SG4294934092              10039d60     ViewUnitStat.obj
 0002:00008d68       $SG4294934091              10039d68     ViewUnitStat.obj
 0002:00008d70       $SG4294934089              10039d70     ViewUnitStat.obj
 0002:00008d78       $SG4294934088              10039d78     ViewUnitStat.obj
 0002:00008d80       $SG4294934086              10039d80     ViewUnitStat.obj
 0002:00008d88       $SG4294934085              10039d88     ViewUnitStat.obj
 0002:00008d90       $SG4294934083              10039d90     ViewUnitStat.obj
 0002:00008d98       $SG4294934082              10039d98     ViewUnitStat.obj
 0002:00008da0       $SG4294934080              10039da0     ViewUnitStat.obj
 0002:00008da8       $SG4294934079              10039da8     ViewUnitStat.obj
 0002:00008db0       $SG4294934077              10039db0     ViewUnitStat.obj
 0002:00008db8       $SG4294934076              10039db8     ViewUnitStat.obj
 0002:00008dc0       $SG4294934074              10039dc0     ViewUnitStat.obj
 0002:00008dc8       $SG4294934073              10039dc8     ViewUnitStat.obj
 0002:00008dd0       $SG4294934071              10039dd0     ViewUnitStat.obj
 0002:00008dd8       $SG4294934068              10039dd8     ViewUnitStat.obj
 0002:00008de0       $SG4294934065              10039de0     ViewUnitStat.obj
 0002:00008de8       $SG4294934062              10039de8     ViewUnitStat.obj
 0002:00008df0       $SG4294934059              10039df0     ViewUnitStat.obj
 0002:00008df8       $SG4294934057              10039df8     ViewUnitStat.obj
 0002:00008dfc       $SG4294934056              10039dfc     ViewUnitStat.obj
 0002:00008e04       $SG4294934054              10039e04     ViewUnitStat.obj
 0002:00008e08       $SG4294934053              10039e08     ViewUnitStat.obj
 0002:00008e10       $SG4294934051              10039e10     ViewUnitStat.obj
 0002:00008e14       $SG4294934050              10039e14     ViewUnitStat.obj
 0002:00008e1c       $SG4294934048              10039e1c     ViewUnitStat.obj
 0002:00008e20       $SG4294934047              10039e20     ViewUnitStat.obj
 0002:00008e28       $SG4294934045              10039e28     ViewUnitStat.obj
 0002:00008e2c       $SG4294934044              10039e2c     ViewUnitStat.obj
 0002:00008e34       $SG4294934042              10039e34     ViewUnitStat.obj
 0002:00008e38       $SG4294934041              10039e38     ViewUnitStat.obj
 0002:00008e40       $SG4294934039              10039e40     ViewUnitStat.obj
 0002:00008e44       $SG4294934038              10039e44     ViewUnitStat.obj
 0002:00008e4c       $SG4294934036              10039e4c     ViewUnitStat.obj
 0002:00008e50       $SG4294934035              10039e50     ViewUnitStat.obj
 0002:00008e58       $SG4294934033              10039e58     ViewUnitStat.obj
 0002:00008e5c       $SG4294934032              10039e5c     ViewUnitStat.obj
 0002:00008e64       $SG4294934031              10039e64     ViewUnitStat.obj
 0002:00008e70       $SG4294934030              10039e70     ViewUnitStat.obj
 0002:00008e74       $SG4294934029              10039e74     ViewUnitStat.obj
 0002:00008e7c       $SG4294934026              10039e7c     ViewUnitStat.obj
 0002:00008e84       $SG4294934024              10039e84     ViewUnitStat.obj
 0002:00008e88       $SG4294934023              10039e88     ViewUnitStat.obj
 0002:00008e90       $SG4294934021              10039e90     ViewUnitStat.obj
 0002:00008e94       $SG4294934020              10039e94     ViewUnitStat.obj
 0002:00008e9c       $SG4294934018              10039e9c     ViewUnitStat.obj
 0002:00008ea0       $SG4294934017              10039ea0     ViewUnitStat.obj
 0002:00008ea8       $SG4294934015              10039ea8     ViewUnitStat.obj
 0002:00008eac       $SG4294934014              10039eac     ViewUnitStat.obj
 0002:00008eb4       $SG4294934012              10039eb4     ViewUnitStat.obj
 0002:00008eb8       $SG4294934011              10039eb8     ViewUnitStat.obj
 0002:00008ec0       $SG4294934009              10039ec0     ViewUnitStat.obj
 0002:00008ec4       $SG4294934008              10039ec4     ViewUnitStat.obj
 0002:00008ecc       $SG4294934006              10039ecc     ViewUnitStat.obj
 0002:00008ed4       $SG4294934005              10039ed4     ViewUnitStat.obj
 0002:00008edc       $SG4294934003              10039edc     ViewUnitStat.obj
 0002:00008ee4       $SG4294934002              10039ee4     ViewUnitStat.obj
 0002:00008eec       $SG4294934001              10039eec     ViewUnitStat.obj
 0002:00008ef4       $SG4294933999              10039ef4     ViewUnitStat.obj
 0002:00008efc       $SG4294933998              10039efc     ViewUnitStat.obj
 0002:00008f04       $SG4294933996              10039f04     ViewUnitStat.obj
 0002:00008f0c       $SG4294933995              10039f0c     ViewUnitStat.obj
 0002:00008f14       $SG4294933993              10039f14     ViewUnitStat.obj
 0002:00008f1c       $SG4294933992              10039f1c     ViewUnitStat.obj
 0002:00008f24       $SG4294933990              10039f24     ViewUnitStat.obj
 0002:00008f2c       $SG4294933989              10039f2c     ViewUnitStat.obj
 0002:00008f38       $SG4294933987              10039f38     ViewUnitStat.obj
 0002:00008f40       $SG4294933986              10039f40     ViewUnitStat.obj
 0002:00008f4c       $SG4294933984              10039f4c     ViewUnitStat.obj
 0002:00008f54       $SG4294933983              10039f54     ViewUnitStat.obj
 0002:00008f5c       $SG4294933981              10039f5c     ViewUnitStat.obj
 0002:00008f64       $SG4294933980              10039f64     ViewUnitStat.obj
 0002:00008f6c       $SG4294933978              10039f6c     ViewUnitStat.obj
 0002:00008f74       $SG4294933838              10039f74     AutoMapCell.obj
 0002:00008f9c       $SG4294933746              10039f9c     GameFilter.obj
 0002:00008fc0       $SG4294933745              10039fc0     GameFilter.obj
 0002:00008fd0       $SG4294933744              10039fd0     GameFilter.obj
 0002:00008fe4       $SG4294933743              10039fe4     GameFilter.obj
 0002:00008ff4       $SG4294933577              10039ff4     ScrollLock.obj
 0002:00009008       $SG4294933638              1003a008     QuickBackTown.obj
 0002:00009068       $SG4294933626              1003a068     QuickGame.obj
 0002:000090c0       _NaN                       1003a0c0     LIBCMT:ftol3.obj
 0002:000090c4       _onept5                    1003a0c4     LIBCMT:ftol3.obj
 0002:000090c8       _DP2to32                   1003a0c8     LIBCMT:ftol3.obj
 0002:000090c8       _Int32ToUInt32             1003a0c8     LIBCMT:ftol3.obj
 0002:000090e0       _NAME_                     1003a0e0     libucrt:sqrt_impl.obj
 0002:00009700       __sehtable$?GB2GBK@@YAXPAD@Z 1003a700     HelpFunc.obj
 0002:00009720       __sehtable$?LoadConfig@@YAHXZ 1003a720     LoadConfig.obj
 0002:00009758       __sehtable$?LogMessage@@YIXPA_W@Z 1003a758     MessageLog.obj
 0002:00009778       __sehtable$?LoadExtInfo@@YAXXZ 1003a778     ItemExtInfo.obj
 0002:00009798       __sehtable$___scrt_is_nonwritable_in_current_image 1003a798     LIBCMT:utility.obj
 0002:000097b8       __sehtable$?dllmain_crt_process_attach@@YAHQAUHINSTANCE__@@QAX@Z 1003a7b8     LIBCMT:dll_dllmain.obj
 0002:000097d8       __sehtable$?dllmain_crt_process_detach@@YAH_N@Z 1003a7d8     LIBCMT:dll_dllmain.obj
 0002:00009800       __sehtable$?dllmain_dispatch@@YAHQAUHINSTANCE__@@KQAX@Z 1003a800     LIBCMT:dll_dllmain.obj
 0002:000098b0       __sehtable$___DestructExceptionObject 1003a8b0     libvcruntime:ehhelpers.obj
 0002:000098d0       __sehtable$??R<lambda_6e4b09c48022b2350581041d5f6b0c4c>@@QBE@XZ 1003a8d0     libucrt:exit.obj
 0002:000098f0       __sehtable$??$?RV<lambda_03b1d95aef87969028cfba75ccab2455>@@AAV<lambda_6e4b09c48022b2350581041d5f6b0c4c>@@V<lambda_22bdf7517842c4b3e53723af5aa32b9e>@@@?$__crt_seh_guarded_call@X@@QAEX$$QAV<lambda_03b1d95aef87969028cfba75ccab2455>@@AAV<lambda_6e4b09c48022b2350581041d5f6b0c4c>@@$$QAV<lambda_22bdf7517842c4b3e53723af5aa32b9e>@@@Z 1003a8f0     libucrt:exit.obj
 0002:00009910       __sehtable$??$?RV<lambda_8e746cf0007f6ed984d6f78af1fec997>@@AAV<lambda_22ebabd17bc4fa466a2aca6d8deb888d>@@V<lambda_18ed0c0b38a6dc0daf1e7ac6d6adf05e>@@@?$__crt_seh_guarded_call@H@@QAEH$$QAV<lambda_8e746cf0007f6ed984d6f78af1fec997>@@AAV<lambda_22ebabd17bc4fa466a2aca6d8deb888d>@@$$QAV<lambda_18ed0c0b38a6dc0daf1e7ac6d6adf05e>@@@Z 1003a910     libucrt:onexit.obj
 0002:00009930       __sehtable$??$?RV<lambda_69a2805e680e0e292e8ba93315fe43a8>@@AAV<lambda_f03950bc5685219e0bcd2087efbe011e>@@V<lambda_03fcd07e894ec930e3f35da366ca99d6>@@@?$__crt_seh_guarded_call@H@@QAEH$$QAV<lambda_69a2805e680e0e292e8ba93315fe43a8>@@AAV<lambda_f03950bc5685219e0bcd2087efbe011e>@@$$QAV<lambda_03fcd07e894ec930e3f35da366ca99d6>@@@Z 1003a930     libucrt:onexit.obj
 0002:00009950       __sehtable$__query_new_handler 1003a950     libucrt:new_handler.obj
 0002:00009970       __sehtable$_terminate      1003a970     libucrt:terminate.obj
 0002:00009990       __sehtable$??$?RV<lambda_15ade71b0218206bbe3333a0c9b79046>@@AAV<lambda_da44e0f8b0f19ba52fefafb335991732>@@V<lambda_207f2d024fc103971653565357d6cd41>@@@?$__crt_seh_guarded_call@X@@QAEX$$QAV<lambda_15ade71b0218206bbe3333a0c9b79046>@@AAV<lambda_da44e0f8b0f19ba52fefafb335991732>@@$$QAV<lambda_207f2d024fc103971653565357d6cd41>@@@Z 1003a990     libucrt:per_thread_data.obj
 0002:000099b0       __sehtable$??$?RV<lambda_a7e850c220f1c8d1e6efeecdedd162c6>@@AAV<lambda_46720907175c18b6c9d2717bc0d2d362>@@V<lambda_9048902d66e8d99359bc9897bbb930a8>@@@?$__crt_seh_guarded_call@X@@QAEX$$QAV<lambda_a7e850c220f1c8d1e6efeecdedd162c6>@@AAV<lambda_46720907175c18b6c9d2717bc0d2d362>@@$$QAV<lambda_9048902d66e8d99359bc9897bbb930a8>@@@Z 1003a9b0     libucrt:per_thread_data.obj
 0002:000099d0       __sehtable$??$?RV<lambda_38edbb1296d33220d7e4dd0ed76b244a>@@AAV<lambda_5ce1d447e08cb34b2473517608e21441>@@V<lambda_fb385d3da700c9147fc39e65dd577a8c>@@@?$__crt_seh_guarded_call@X@@QAEX$$QAV<lambda_38edbb1296d33220d7e4dd0ed76b244a>@@AAV<lambda_5ce1d447e08cb34b2473517608e21441>@@$$QAV<lambda_fb385d3da700c9147fc39e65dd577a8c>@@@Z 1003a9d0     libucrt:per_thread_data.obj
 0002:000099f0       __sehtable$??$?RV<lambda_6affb1475c98b40b75cdec977db92e3c>@@AAV<lambda_b8d4b9c228a6ecc3f80208dbb4b4a104>@@V<lambda_608742c3c92a14382c1684fc64f96c88>@@@?$__crt_seh_guarded_call@X@@QAEX$$QAV<lambda_6affb1475c98b40b75cdec977db92e3c>@@AAV<lambda_b8d4b9c228a6ecc3f80208dbb4b4a104>@@$$QAV<lambda_608742c3c92a14382c1684fc64f96c88>@@@Z 1003a9f0     libucrt:per_thread_data.obj
 0002:00009a10       __sehtable$??$?RV<lambda_e5124f882df8998aaf41531e079ba474>@@AAV<lambda_3e16ef9562a7dcce91392c22ab16ea36>@@V<lambda_e25ca0880e6ef98be67edffd8c599615>@@@?$__crt_seh_guarded_call@X@@QAEX$$QAV<lambda_e5124f882df8998aaf41531e079ba474>@@AAV<lambda_3e16ef9562a7dcce91392c22ab16ea36>@@$$QAV<lambda_e25ca0880e6ef98be67edffd8c599615>@@@Z 1003aa10     libucrt:wsetlocale.obj
 0002:00009a30       __sehtable$___acrt_initialize_lowio 1003aa30     libucrt:ioinit.obj
 0002:00009a50       __sehtable$?update_thread_multibyte_data_internal@@YAPAU__crt_multibyte_data@@QAU__acrt_ptd@@QAPAU1@@Z 1003aa50     libucrt:mbctype.obj
 0002:00009a70       __sehtable$??$?RV<lambda_ceb1ee4838e85a9d631eb091e2fbe199>@@AAV<lambda_ae742caa10f662c28703da3d2ea5e57e>@@V<lambda_cd08b5d6af4937fe54fc07d0c9bf6b37>@@@?$__crt_seh_guarded_call@X@@QAEX$$QAV<lambda_ceb1ee4838e85a9d631eb091e2fbe199>@@AAV<lambda_ae742caa10f662c28703da3d2ea5e57e>@@$$QAV<lambda_cd08b5d6af4937fe54fc07d0c9bf6b37>@@@Z 1003aa70     libucrt:mbctype.obj
 0002:00009a90       __sehtable$_raise          1003aa90     libucrt:signal.obj
 0002:00009ab0       __sehtable$??$?RV<lambda_cbab9ec6f41b0180b23cc171c22676b0>@@AAV<lambda_44731a7d0e6d81c3e6aa82d741081786>@@V<lambda_4b292cb8dd18144e164572427af410ab>@@@?$__crt_seh_guarded_call@P6AXH@Z@@QAEP6AXH@Z$$QAV<lambda_cbab9ec6f41b0180b23cc171c22676b0>@@AAV<lambda_44731a7d0e6d81c3e6aa82d741081786>@@$$QAV<lambda_4b292cb8dd18144e164572427af410ab>@@@Z 1003aab0     libucrt:signal.obj
 0002:00009ad0       __sehtable$??$?RV<lambda_2866be3712abc81a800a822484c830d8>@@AAV<lambda_39ca0ed439415581b5b15c265174cece>@@V<lambda_2b24c74d71094a6cd0cb82e44167d71b>@@@?$__crt_seh_guarded_call@X@@QAEX$$QAV<lambda_2866be3712abc81a800a822484c830d8>@@AAV<lambda_39ca0ed439415581b5b15c265174cece>@@$$QAV<lambda_2b24c74d71094a6cd0cb82e44167d71b>@@@Z 1003aad0     libucrt:fflush.obj
 0002:00009af0       __sehtable$??$?RV<lambda_2cc53f568c5a2bb6f192f930a45d44ea>@@AAV<lambda_ab61a845afdef5b7c387490eaf3616ee>@@V<lambda_c2ffc0b7726aa6be21d5f0026187e748>@@@?$__crt_seh_guarded_call@X@@QAEX$$QAV<lambda_2cc53f568c5a2bb6f192f930a45d44ea>@@AAV<lambda_ab61a845afdef5b7c387490eaf3616ee>@@$$QAV<lambda_c2ffc0b7726aa6be21d5f0026187e748>@@@Z 1003aaf0     libucrt:fflush.obj
 0002:00009b10       __sehtable$___acrt_update_thread_locale_data 1003ab10     libucrt:locale_refcounting.obj
 0002:00009b30       __sehtable$__fcloseall     1003ab30     libucrt:closeall.obj
 0002:00009b50       __sehtable$___acrt_lowio_ensure_fh_exists 1003ab50     libucrt:osfinfo.obj
 0002:00009b70       __sehtable$??$?RV<lambda_9e9de3de5fa147e2223d7db92bc10aa6>@@AAV<lambda_38ce7e780aa69e748d6df282ebc68efe>@@V<lambda_8ca6da459f0f6780f1cff60fdc3d00e5>@@@?$__crt_seh_guarded_call@H@@QAEH$$QAV<lambda_9e9de3de5fa147e2223d7db92bc10aa6>@@AAV<lambda_38ce7e780aa69e748d6df282ebc68efe>@@$$QAV<lambda_8ca6da459f0f6780f1cff60fdc3d00e5>@@@Z 1003ab70     libucrt:commit.obj
 0002:00009b90       __sehtable$__write         1003ab90     libucrt:write.obj
 0002:00009bb0       __sehtable$_fclose         1003abb0     libucrt:fclose.obj
 0002:00009bd0       __sehtable$___set_fpsr_sse2 1003abd0     libucrt:fpctrl.obj
 0002:00009bf0       __sehtable$??$?RV<lambda_218ce3db14220d0be481dae8ef3383b6>@@AAV<lambda_628dfdc04ba53c8bfc02c9951375f3f5>@@V<lambda_57dc472bd5c9d5f3b2cbca59b8a843ae>@@@?$__crt_seh_guarded_call@H@@QAEH$$QAV<lambda_218ce3db14220d0be481dae8ef3383b6>@@AAV<lambda_628dfdc04ba53c8bfc02c9951375f3f5>@@$$QAV<lambda_57dc472bd5c9d5f3b2cbca59b8a843ae>@@@Z 1003abf0     libucrt:close.obj
 0002:00009c10       __sehtable$__IsNonwritableInCurrentImage 1003ac10     LIBCMT:pesect.obj
 0002:00009c30       .edata                     1003ac30     d2hackmap.exp
 0002:00009c58       rgpv                       1003ac58     d2hackmap.exp
 0002:00009c5c       rgszName                   1003ac5c     d2hackmap.exp
 0002:00009c60       rgwOrd                     1003ac60     d2hackmap.exp
 0002:00009c62       szName                     1003ac62     d2hackmap.exp
 0002:00009c70       $N00001                    1003ac70     d2hackmap.exp
 0002:0000a06e       .idata$6                   1003b06e     kernel32:KERNEL32.dll
 0002:0000a10c       .idata$6                   1003b10c     user32:USER32.dll
 0002:0000a118       .idata$6                   1003b118     ws2_32:WS2_32.dll
 0002:0000a166       .idata$6                   1003b166     Version:VERSION.dll
 0002:0000a188       .idata$6                   1003b188     imm32:IMM32.dll
 0003:00000020       ?__vcrt_flsindex@@3KA      1003c020     libvcruntime:per_thread_data.obj
 0003:00000050       ?__acrt_flsindex@@3KA      1003c050     libucrt:per_thread_data.obj
 0003:0000011c       ?errno_no_memory@@3HA      1003c11c     libucrt:errno.obj
 0003:00000120       ?doserrno_no_memory@@3KA   1003c120     libucrt:errno.obj
 0003:000003f0       __mbctypes                 1003c3f0     libucrt:mbctype.obj
 0003:000004f8       __mbcasemaps               1003c4f8     libucrt:mbctype.obj
 0003:000005f8       ?__rgctypeflag@@3PADA      1003c5f8     libucrt:mbctype.obj
 0003:00000600       ?__rgcode_page_info@@3PAUcode_page_info@@A 1003c600     libucrt:mbctype.obj
 0003:00000850       ?__DAZ_ENABLED@?1??__set_fpsr_sse2@@9@9 1003c850     libucrt:fpctrl.obj
 0003:00000860       ?__dcrt_lowio_console_output_handle@@3PAXA 1003c860     libucrt:initcon.obj
 0003:00001208       ?aD2Patchs@@3PAUPatch_t@@A 1003d208     Install.obj
 0003:0000205c       ?afRevealedActs@@3PAHA     1003e05c     AutoMap.obj
 0003:00002070       ?aD2Patch2s@@3PAUPatch_t@@A 1003e070     Install.obj
 0003:00002170       ?aConfigVars@@3PAUConfigVar@@A 1003e170     LoadConfig.obj
 0003:00003b80       ?szMonsterDescComma@@3PA_WA 1003fb80     MonsterLifeBar.obj
 0003:00003b88       ?aKeepGameWindowPatchs@@3PAUPatch_t@@A 1003fb88     GameWindow.obj
 0003:00003bc0       ?dlls@?1??GetDllOffset@@YAKH@Z@4PAPADA 1003fbc0     HelpFunc.obj
 0003:00003bf8       ?version@?1??Map_D2Version@@YAKXZ@4KA 1003fbf8     Install.obj
 0003:00003bfc       ?version@?1??GetD2Version@@YAKPAD@Z@4KA 1003fbfc     Install.obj
 0003:00003c00       ?dc6head@?1??LoadBmpCellFile@@YAPAUCellFile@@PAEHH@Z@4PAKA 1003fc00     D2HelpFunc.obj
 0003:00003c3c       ?resistoffset@?1??GetUnitResist@@YAHPAUUnitAny@@K@Z@4PAY02HA 1003fc3c     D2HelpFunc.obj
 0003:00003c54       ?wszProgTitle@?1??GameLoopPatch@@YAXXZ@4PA_WA 1003fc54     GameMainLoop.obj
 0003:00003c58       ?statindexs@?1??CheckDangerousMonster@@YAXPAUUnitAny@@@Z@4PAKA 1003fc58     CheckDangerous.obj
 0003:00003c68       ?stats@?4??MonsterBlobDesc@@YIXPAUUnitAny@@@Z@4PAEA 1003fc68     AutoMapBlob.obj
 0003:00003c70       ?states@?BE@??MonsterBlobDesc@@YIXPAUUnitAny@@@Z@4PAEA 1003fc70     AutoMapBlob.obj
 0003:00003c78       ?blines@?CM@??DrawAutomapBlob@@YIXHHKPAUUnitAny@@@Z@4PAY01DA 1003fc78     AutoMapBlob.obj
 0003:00003c94       ?parm0cells@?BM@??AddAutoMapCell@@YAXPAUDrlgRoom2@@@Z@4PAGA 1003fc94     AutoMapCell.obj
 0003:00003c9c       ?dws@?6??InitD2EditBox@@YAHXZ@4PAKA 1003fc9c     GameChat.obj
 0003:00003ca4       ?NoticeMsg@?4??WisperPatch@@YAXXZ@4PADA 1003fca4     GameChat.obj
 0003:00003cb8       ?loading@?N@??DrawGameListPatch@@YAXXZ@4HA 1003fcb8     GameFilter.obj
 0003:00003d40       ?is_initialized_as_dll@@3_NA 1003fd40     LIBCMT:utility.obj
 0003:00003d41       ?module_local_atexit_table_initialized@@3_NA 1003fd41     LIBCMT:utility.obj
 0003:00003d44       ?module_local_atexit_table@@3U_onexit_table_t@@A 1003fd44     LIBCMT:utility.obj
 0003:00003d50       ?module_local_at_quick_exit_table@@3U_onexit_table_t@@A 1003fd50     LIBCMT:utility.obj
 0003:00003d60       _GS_ExceptionRecord        1003fd60     LIBCMT:gs_report.obj
 0003:00003db0       _GS_ContextRecord          1003fdb0     LIBCMT:gs_report.obj
 0003:0000407c       ?g_tss_cv@@3U_RTL_CONDITION_VARIABLE@@A 1004007c     LIBCMT:thread_safe_statics.obj
 0003:00004080       ?g_tss_event@@3PAXA        10040080     LIBCMT:thread_safe_statics.obj
 0003:00004084       ?g_tss_mutex@@3U_RTL_CRITICAL_SECTION@@A 10040084     LIBCMT:thread_safe_statics.obj
 0003:0000409c       ?g_sleep_condition_variable_cs@@3P6GHPAU_RTL_CONDITION_VARIABLE@@PAU_RTL_CRITICAL_SECTION@@K@ZA 1004009c     LIBCMT:thread_safe_statics.obj
 0003:000040a0       ?g_wake_all_condition_variable@@3P6GXPAU_RTL_CONDITION_VARIABLE@@@ZA 100400a0     LIBCMT:thread_safe_statics.obj
 0003:000040a4       ?__proc_attached@@3HA      100400a4     LIBCMT:dll_dllmain.obj
 0003:000040d4       ?__vcrt_startup_thread_ptd@@3U__vcrt_ptd@@A 100400d4     libvcruntime:per_thread_data.obj
 0003:000040fc       ___vcrt_lock_table         100400fc     libvcruntime:locks.obj
 0003:00004114       ___vcrt_locks_initialized  10040114     libvcruntime:locks.obj
 0003:00004140       ?heap@@3V_HeapManager@@A   10040140     libvcruntime:undname.obj
 0003:00004154       ?module_handles@@3PAPAUHINSTANCE__@@A 10040154     libvcruntime:winapi_downlevel.obj
 0003:00004160       ?function_pointers@@3PAPAXA 10040160     libvcruntime:winapi_downlevel.obj
 0003:00004178       ?c_termination_complete@@3JA 10040178     libucrt:exit.obj
 0003:0000417c       ?thread_local_exit_callback_func@@3P6GXPAXK0@ZA 1004017c     libucrt:exit.obj
 0003:00004188       ?program_name@?1???$common_configure_argv@D@@YAHW4_crt_argv_mode@@@Z@4PADA 10040188     libucrt:argv_parsing.obj
 0003:000042b8       ?__acrt_new_handler@@3V?$dual_state_global@P6AHI@Z@__crt_state_management@@A 100402b8     libucrt:new_handler.obj
 0003:000042c4       ?__acrt_invalid_parameter_handler@@3V?$dual_state_global@P6AXPB_W00II@Z@__crt_state_management@@A 100402c4     libucrt:invalid_parameter.obj
 0003:000042c8       ?internal_state@?1??_mbtowc_l@@9@4U_Mbstatet@@A 100402c8     libucrt:mbtowc.obj
 0003:000042d8       ?enable_percent_n@@3IA     100402d8     libucrt:printf_count_output.obj
 0003:000044f0       ?module_handles@@3PAPAUHINSTANCE__@@A 100404f0     libucrt:winapi_thunks.obj
 0003:00004540       ?encoded_function_pointers@@3PAPAXA 10040540     libucrt:winapi_thunks.obj
 0003:000045c8       ?__acrt_lock_table@@3PAU_RTL_CRITICAL_SECTION@@A 100405c8     libucrt:locks.obj
 0003:00004718       ?__acrt_locks_initialized@@3IA 10040718     libucrt:locks.obj
 0003:00004728       ?fSystemSet@@3HA           10040728     libucrt:mbctype.obj
 0003:0000472c       ?initialized@?1??__acrt_initialize_multibyte@@9@4_NA 1004072c     libucrt:mbctype.obj
 0003:0000474c       ?ctrlc_action@@3V?$dual_state_global@P6AXH@Z@__crt_state_management@@A 1004074c     libucrt:signal.obj
 0003:00004750       ?ctrlbreak_action@@3V?$dual_state_global@P6AXH@Z@__crt_state_management@@A 10040750     libucrt:signal.obj
 0003:00004754       ?abort_action@@3V?$dual_state_global@P6AXH@Z@__crt_state_management@@A 10040754     libucrt:signal.obj
 0003:00004758       ?term_action@@3V?$dual_state_global@P6AXH@Z@__crt_state_management@@A 10040758     libucrt:signal.obj
 0003:0000475c       ?user_matherr@@3V?$dual_state_global@P6AHPAU_exception@@@Z@__crt_state_management@@A 1004075c     libucrt:matherr.obj
 0003:00004768       ?__acrt_global_new_mode@@3V?$dual_state_global@J@__crt_state_management@@A 10040768     libucrt:new_mode.obj
 0003:00004770       __pmatherr_set             10040770     libucrt:libm_error.obj
 0003:00004774       ?internal_pst@?1??__mbrtoc32_utf8@__crt_mbstring@@YAIPA_UPBDIPAU_Mbstatet@@@Z@4U3@A 10040774     libucrt:mbrtoc32.obj
 0003:0000477c       ?__acrt_app_type@@3W4_crt_app_type@@A 1004077c     libucrt:report_runtime_error.obj
 0003:00412940       ?wsinit_@detail@httplib@@3VWSInit@12@A 1044e940     DllMain.obj
 0003:00412941       ?wsinit_@detail@httplib@@3VWSInit@12@A 1044e941     stdafx.obj
 0003:00412b9c       ?nMsgCount@@3HA            1044eb9c     LoadConfig.obj
 0003:00412ba0       ?WarningMsg@@3PAY0GE@DA    1044eba0     LoadConfig.obj
 0003:004179c0       ?pTreeRoot@@3PAUTreeNode@@A 104539c0     LoadConfig.obj
 0003:004179c4       ?blnDraw@@3HA              104539c4     D2HelpFunc.obj
 0003:004179c8       ?wszAlertMsg@@3PA_WA       104539c8     D2HelpFunc.obj
 0003:00417dc8       ?nTickCount@@3KA           10453dc8     RoomInfo.obj
 0003:00417dcc       ?xShowPos@@3HA             10453dcc     ItemExtInfo.obj
 0003:00417dd0       ?D2ScreenHook@@3PAUD2ScreenHookStruct@@A 10453dd0     ScreenHook.obj
 0003:0041a670       ?yShowPos@@3HA             10456670     ItemExtInfo.obj
 0003:0041a674       ?fLeft@@3HA                10456674     ItemExtInfo.obj
 0003:0041a678       ?pwszNormalInfo@@3PAY04PA_WA 10456678     ItemExtInfo.obj
 0003:00432d18       ?pwszUniqueInfo@@3PAPA_WA  1046ed18     ItemExtInfo.obj
 0003:0043c958       ?pwszSetInfo@@3PAPA_WA     10478958     ItemExtInfo.obj
 0003:00441778       ?pwszRuneWordInfo@@3PAPA_WA 1047d778     ItemExtInfo.obj
 0003:004466b0       ?wszRuneInfo@@3PAPA_WA     104826b0     ItemExtInfo.obj
 0003:00446778       ?wszCubeMain@@3PAPA_WA     10482778     ItemExtInfo.obj
 0003:00446840       ?fExtInfoLoad@@3HA         10482840     ItemExtInfo.obj
 0003:00446844       ?nStatCount@@3HA           10482844     ItemVariableProp.obj
 0003:00446848       ?aItemPropInfo@@3PAY2CHBA@BGH@3HA 10482848     ItemVariableProp.obj
 0003:0a89cd48       ?fDisabled@@3HA            1a8d8d48     IMEProtect.obj
 0003:0a89cd4c       ?BugTimer@@3KA             1a8d8d4c     QuestProtect.obj
 0003:0a89cd50       ?aBugInfo@@3PAUBugQuestInfo@@A 1a8d8d50     QuestProtect.obj
 0003:0a89cddc       ?BugTimerSet@@3PAEA        1a8d8ddc     QuestProtect.obj
 0003:0a89cde8       ?dwLastAct@@3KA            1a8d8de8     QuestProtect.obj
 0003:0a89cdec       ?fIsTcInit@@3HA            1a8d8dec     MonsterTC.obj
 0003:0a89cdf0       ?anMonsterTCs@@3PAUMonTC@@A 1a8d8df0     MonsterTC.obj
 0003:0a8a0d50       ?nCurrentPage@@3HA         1a8dcd50     ViewUnitStat.obj
 0003:0a8a0d54       ?pD2FilterBox@@3PAUD2EditBox@@A 1a8dcd54     GameFilter.obj
 0003:0a8a0d58       ?aLevelInfo@@3PAULevelInfo@@A 1a8dcd58     AutoMap.obj
 0003:0a8a167c       ?mGames@@3HA               1a8dd67c     GameFilter.obj
 0003:0a8a1680       ?pdwGamelist@@3PAKA        1a8dd680     GameFilter.obj
 0003:0a8a2620       ?szFilter@@3PADA           1a8de620     GameFilter.obj
 0003:0a8a2640       ?mGameShows@@3HA           1a8de640     GameFilter.obj
 0003:0a8a2644       ?nClickStatus@@3HA         1a8de644     QuickSwapItem.obj
 0003:0a8a2648       ?stTimer@@3PAUMyTimer@@A   1a8de648     PartyHelp.obj
 0003:0a8a26a8       ?fSwapProc@@3HA            1a8de6a8     QuickSwapItem.obj
 0003:0a8a26ac       ?fSwapProcLoop@@3HA        1a8de6ac     QuickSwapItem.obj
 0003:0a8a26b0       ?unDealMsg@@3UD2MSG@@A     1a8de6b0     QuickSwapItem.obj
 0003:0a8a26d0       ?dwSwapTimer@@3KA          1a8de6d0     QuickSwapItem.obj
 0003:0a8a26d4       ?pMapOffsetX@@3PAHA        1a8de6d4     ScrollLock.obj
 0003:0a8a26d8       ?xMapOffset@@3PAY04HA      1a8de6d8     ScrollLock.obj
 0003:0a8a278c       ?pMapOffsetY@@3PAHA        1a8de78c     ScrollLock.obj
 0003:0a8a2790       ?yMapOffset@@3PAY04HA      1a8de790     ScrollLock.obj
 0003:0a8a2844       ?nSrollIdx@@3HA            1a8de844     ScrollLock.obj
 0003:0a8a2848       ?fSkipMessageReq@@3HA      1a8de848     SkipNpcMessage.obj
 0003:0a8a284c       ?mSkipMessageTimer@@3KA    1a8de84c     SkipNpcMessage.obj
 0003:0a8a285c       ?wAreaLevel@?1??GetAreaLevel@@YAGXZ@4GA 1a8de85c     D2HelpFunc.obj
 0003:0a8a2860       ?dwLastLevelNo@?1??GetAreaLevel@@YAGXZ@4KA 1a8de860     D2HelpFunc.obj
 0003:0a8a2864       ?yPosition@?1??ItemDescPath@@YIXPA_WHHHH@Z@4HA 1a8de864     ItemDesc.obj
 0003:0a8a2868       ?fItemStatInit@?1??GetStatRange@@YAPA_WPA_WKK@Z@4HA 1a8de868     ItemVariableProp.obj
 0003:0a8a286c       ?hIMC@?1??ToggleIMEInput@@YAXH@Z@4PAUHIMC__@@A 1a8de86c     IMEProtect.obj
 0003:0a8a2870       ?lastcode@?1??ChannelEnterCharPatch@@YIKPAUD2EditBox@@E@Z@4EA 1a8de870     UnicodeSupport.obj
 0003:0a8a2874       ?lock@?1??AutoEnchant@@YAXPAUUnitAny@@@Z@4HA 1a8de874     AutoEnchant.obj
 0003:0a8a2878       ?unitCount@?1??AutoEnchantLoop@@YAXPAUUnitAny@@@Z@4PAY0DOI@HA 1a8de878     AutoEnchant.obj
 0003:0a8a47b8       ?delays@?1??AutoEnchantLoop@@YAXPAUUnitAny@@@Z@4HA 1a8e07b8     AutoEnchant.obj
 0003:0a8a47c0       ?invTypes@?1??MoveItem@@YAXPAUD2MSG@@@Z@4PAUInventoryType@@A 1a8e07c0     QuickSwapItem.obj
 0003:0a8a4820       ?coltab@?1??DrawAutomapCell@@YAXPAUCellFile@@HHE@Z@4PAY0BAA@EA 1a8e0820     D2HelpFunc.obj
 0003:0a8a4a20       ?$TSS0@?1??MoveItem@@YAXPAUD2MSG@@@Z@4HA 1a8e0a20     QuickSwapItem.obj
 0004:00000060       $R000000                   1a8e1060     * linker generated manifest res *
